; 8000 - 81ff : VIA1 (6522)
; 8400 - 85ff : VIA2 (6522)
; 8c00 - 8dff : RTC (RTC 72421A)
; 8200 - 82ff : Partition_Typ
; 8300 - 83ff : Partition_SizeHi
; 8600 - 86ff : Partition_SizeLo
; 8700 - 87ff : Partition_StartHi
; 8800 - 89ff : PIO (8255)
; 8a00 - 8aff : Partition_StartMi
; 8b00 - 8bff : Partition_StartLo
; 8f00 - 8fff : LED

              L0 = $0
              L1 = $1
              L2 = $2
              L3 = $3
              L4 = $4
              L5 = $5
              L6 = $6
              L7 = $7
              L8 = $8
              L9 = $9
              LA = $A
              LB = $B
              LC = $C
              LD = $D
              LE = $E
              LF = $F
              L10 = $10
              L11 = $11
              L13 = $13
              L14 = $14
              L16 = $16
              L17 = $17
              L18 = $18
              L1A = $1A
              L1C = $1C
              L1E = $1E
              L1F = $1F
              L20 = $20
              L21 = $21
              L22 = $22
              L23 = $23
              L24 = $24
              L25 = $25
              L26 = $26
              L27 = $27
              L2A = $2A
              L2B = $2B
              L30 = $30
              L35 = $35
              L38 = $38
              L40 = $40
              L41 = $41
              L42 = $42
              L44 = $44
              L45 = $45
              L46 = $46
              L48 = $48
              L49 = $49
              L4A = $4A
              L4B = $4B
              L4C = $4C
              L4F = $4F
              L50 = $50
              L51 = $51
              L52 = $52
              L53 = $53
              L54 = $54
              L55 = $55
              L56 = $56
              L57 = $57
              L58 = $58
              L59 = $59
              L5A = $5A
              L5B = $5B
              L5C = $5C
              L5D = $5D
              L5E = $5E
              L60 = $60
              L61 = $61
              L62 = $62
              L63 = $63
              L64 = $64
              L65 = $65
              L66 = $66
              L67 = $67
              L68 = $68
              L69 = $69
              L6A = $6A
              L6B = $6B
              L6C = $6C
              L6E = $6E
              L6F = $6F
              L70 = $70
              L71 = $71
              L77 = $77
              L78 = $78
              L80 = $80
              L81 = $81
              L82 = $82
              L83 = $83
              L84 = $84
              L85 = $85
              L86 = $86
              L87 = $87
              L88 = $88
              L89 = $89
              L8A = $8A
              L8B = $8B
              L8C = $8C
              L8D = $8D
              L8E = $8E
              L90 = $90
              L91 = $91
              L92 = $92
              L93 = $93
              L94 = $94
              L95 = $95
              L96 = $96
              L97 = $97
              L98 = $98
              L99 = $99
              L9A = $9A
              L9B = $9B
              L9C = $9C
              L9D = $9D
              L9F = $9F
              LA0 = $A0
              LA1 = $A1
              LA2 = $A2
              LA4 = $A4
              LA5 = $A5
              LA7 = $A7
              LA9 = $A9
              LAA = $AA
              LAB = $AB
              LAD = $AD
              LAE = $AE
              LB5 = $B5
              LBC = $BC
              LBD = $BD
              LC4 = $C4
              LC8 = $C8
              LCA = $CA
              LCD = $CD
              LD1 = $D1
              LD5 = $D5
              LD6 = $D6
              LD7 = $D7
              LDC = $DC
              LDD = $DD
              LDE = $DE
              LDF = $DF
              LE0 = $E0
              LE1 = $E1
              LE2 = $E2
              LE3 = $E3
              LE4 = $E4
              LE5 = $E5
              LE6 = $E6
              LE7 = $E7
              LE8 = $E8
              LE9 = $E9
              LEA = $EA
              LEB = $EB
              LEC = $EC
              LED = $ED
              LEF = $EF
              LF0 = $F0
              LF1 = $F1
              LF2 = $F2
              LF3 = $F3
              LF4 = $F4
              LF6 = $F6
              LF7 = $F7
              LF8 = $F8
              LF9 = $F9
              LFA = $FA
              LFB = $FB
              LFD = $FD
              L100 = $100
              L104 = $104
              L1A9 = $1A9
              L200 = $200
              L201 = $201
              L202 = $202
              L203 = $203
              L204 = $204
              L205 = $205
              L206 = $206
              L207 = $207
              L208 = $208
              L21B = $21B
              L2A2 = $2A2
              L2A9 = $2A9
              L38D = $38D
              L608 = $608
              L6A9 = $6A9
              L8A0 = $8A0
              L8A9 = $8A9
              LBA9 = $BA9
              LF29 = $F29
              L1BE4 = $1BE4
              L202F = $202F
              L2043 = $2043
              L2044 = $2044
              L2045 = $2045
              L20A5 = $20A5
              L20A9 = $20A9
              L2200 = $2200
              L2201 = $2201
              L2202 = $2202
              L2204 = $2204
              L2216 = $2216
              L2217 = $2217
              L2219 = $2219
              L221A = $221A
              L221B = $221B
              L221C = $221C
              L221D = $221D
              L2220 = $2220
              L2221 = $2221
              L2222 = $2222
              L2223 = $2223
              L2224 = $2224
              L2225 = $2225
              L2226 = $2226
              L22AB = $22AB
              L22AC = $22AC
              L2300 = $2300
              L2301 = $2301
              L2302 = $2302
              L2303 = $2303
              L2438 = $2438
              L2800 = $2800
              L2801 = $2801
              L283C = $283C
              L283D = $283D
              L283E = $283E
              L283F = $283F
              L2840 = $2840
              L2860 = $2860
              L287E = $287E
              L2880 = $2880
              L289E = $289E
              L28A0 = $28A0
              L28BE = $28BE
              L28C0 = $28C0
              L28E0 = $28E0
              L2900 = $2900
              L2920 = $2920
              L2940 = $2940
              L2960 = $2960
              L2A00 = $2A00
              L2A01 = $2A01
              L2A02 = $2A02
              L2A03 = $2A03
              L2A04 = $2A04
              L2A05 = $2A05
              L2A07 = $2A07
              L2A08 = $2A08
              L2A10 = $2A10
              L2A11 = $2A11
              L2A13 = $2A13
              L2A1D = $2A1D
              L2A30 = $2A30
              L2A50 = $2A50
              L2A51 = $2A51
              L2A52 = $2A52
              L2A53 = $2A53
              L2A54 = $2A54
              L2A55 = $2A55
              L2A56 = $2A56
              L2A57 = $2A57
              L2A58 = $2A58
              L2A59 = $2A59
              L2A5A = $2A5A
              L2A5B = $2A5B
              L2A5C = $2A5C
              L2A5D = $2A5D
              L2A5E = $2A5E
              L2A5F = $2A5F
              L2A60 = $2A60
              L2A61 = $2A61
              L2A62 = $2A62
              L2A63 = $2A63
              L2A64 = $2A64
              L2A65 = $2A65
              L2A66 = $2A66
              L2A67 = $2A67
              L2B00 = $2B00
              L2B07 = $2B07
              L2B08 = $2B08
              L2B0D = $2B0D
              L2B30 = $2B30
              L2B40 = $2B40
              L2B50 = $2B50
              L2B60 = $2B60
              L2B70 = $2B70
              L2B80 = $2B80
              L2B90 = $2B90
              L2BA0 = $2BA0
              L2BA1 = $2BA1
              L2BA2 = $2BA2
              L2BA3 = $2BA3
              L2BA4 = $2BA4
              L2BA5 = $2BA5
              L2BA6 = $2BA6
              L2BA7 = $2BA7
              L2BA8 = $2BA8
              L2BA9 = $2BA9
              L2BAA = $2BAA
              L2BAD = $2BAD
              L2BAF = $2BAF
              L2BB0 = $2BB0
              L2BB1 = $2BB1
              L2BB2 = $2BB2
              L2BB3 = $2BB3
              L2BB4 = $2BB4
              L2BB5 = $2BB5
              L2BB6 = $2BB6
              L2BB7 = $2BB7
              L2BB8 = $2BB8
              L2BB9 = $2BB9
              L2BBA = $2BBA
              L2BBB = $2BBB
              L2BBC = $2BBC
              L2BBD = $2BBD
              L2BBE = $2BBE
              L2BBF = $2BBF
              L2BC0 = $2BC0
              L2BC1 = $2BC1
              L2BC2 = $2BC2
              L2BC3 = $2BC3
              L2BC4 = $2BC4
              L2BC5 = $2BC5
              L2BC6 = $2BC6
              L2BC7 = $2BC7
              L2BC8 = $2BC8
              L2BC9 = $2BC9
              L2BCA = $2BCA
              L2BCB = $2BCB
              L2BCC = $2BCC
              L2BCD = $2BCD
              L2BCE = $2BCE
              L2BCF = $2BCF
              L2BD0 = $2BD0
              L2BD1 = $2BD1
              L2BD2 = $2BD2
              L2BD3 = $2BD3
              L2BD4 = $2BD4
              L2BD5 = $2BD5
              L2BD6 = $2BD6
              L2BD7 = $2BD7
              L2BD8 = $2BD8
              L2BDA = $2BDA
              L2BDB = $2BDB
              L2BDC = $2BDC
              L2BDD = $2BDD
              L2BDE = $2BDE
              L2BDF = $2BDF
              L2BE0 = $2BE0
              L2BE1 = $2BE1
              L2BE2 = $2BE2
              L2BE3 = $2BE3
              L2BE4 = $2BE4
              L2BE5 = $2BE5
              L2BE6 = $2BE6
              L2BE7 = $2BE7
              L2BE8 = $2BE8
              L2BE9 = $2BE9
              L2BEA = $2BEA
              L2BEB = $2BEB
              L2BEC = $2BEC
              L2BED = $2BED
              L2BEE = $2BEE
              L2BEF = $2BEF
              L2BF0 = $2BF0
              L2BF3 = $2BF3
              L2BF4 = $2BF4
              L2BF5 = $2BF5
              L2BF6 = $2BF6
              L2BF7 = $2BF7
              L2BF8 = $2BF8
              L2BF9 = $2BF9
              L2BFA = $2BFA
              L2BFB = $2BFB
              L2BFC = $2BFC
              L2BFD = $2BFD
              L2BFE = $2BFE
              L2BFF = $2BFF
              L2C00 = $2C00
              L2C01 = $2C01
              L2C08 = $2C08
              L2C09 = $2C09
              L2C0F = $2C0F
              L2C10 = $2C10
              L2C11 = $2C11
              L2C17 = $2C17
              L2C18 = $2C18
              L2C19 = $2C19
              L2C1F = $2C1F
              L2C20 = $2C20
              L2C27 = $2C27
              L2C28 = $2C28
              L2C29 = $2C29
              L2C2A = $2C2A
              L2C2F = $2C2F
              L2C30 = $2C30
              L2C31 = $2C31
              L2C37 = $2C37
              L2C38 = $2C38
              L2C39 = $2C39
              L2C3F = $2C3F
              L2C40 = $2C40
              L2C41 = $2C41
              L2C48 = $2C48
              L2C57 = $2C57
              L2C58 = $2C58
              L2C59 = $2C59
              L2C5A = $2C5A
              L2C68 = $2C68
              L2C86 = $2C86
              L2C87 = $2C87
              L2C88 = $2C88
              L2CA8 = $2CA8
              L2CC8 = $2CC8
              L2CE8 = $2CE8
              L2D08 = $2D08
              L2D28 = $2D28
              L2D48 = $2D48
              L2D68 = $2D68
              L2D88 = $2D88
              L2DA8 = $2DA8
              L2DC6 = $2DC6
              L2DC7 = $2DC7
              L2DC8 = $2DC8
              L2DE7 = $2DE7
              L2DE8 = $2DE8
              L2E07 = $2E07
              L2E08 = $2E08
              L2E28 = $2E28
              L2E43 = $2E43
              L2E48 = $2E48
              L2E68 = $2E68
              L2E88 = $2E88
              L2EA8 = $2EA8
              L2FC0 = $2FC0
              L2FD0 = $2FD0
              L2FDF = $2FDF
              L2FE0 = $2FE0
              L2FE1 = $2FE1
              L2FE2 = $2FE2
              L2FF2 = $2FF2
              L2FF3 = $2FF3
              L30A9 = $30A9
              L31A9 = $31A9
              L32A9 = $32A9
              L33A9 = $33A9
              L34A9 = $34A9
              L40A9 = $40A9
              L4220 = $4220
              L4300 = $4300
              L4345 = $4345
              L434F = $434F
              L4400 = $4400
              L454C = $454C
              L454E = $454E
              L4553 = $4553
              L4620 = $4620
              L4745 = $4745
              L4751 = $4751
              L4754 = $4754
              L47A0 = $47A0
              L47A9 = $47A9
              L488A = $488A
              L4920 = $4920
              L4946 = $4946
              L4A20 = $4A20
              L4C41 = $4C41
              L4D20 = $4D20
              L4E4F = $4E4F
              L4FA9 = $4FA9
              L5000 = $5000
              L5001 = $5001
              L5002 = $5002
              L5003 = $5003
              L5004 = $5004
              L5005 = $5005
              L50A9 = $50A9
              L5100 = $5100
              L51A9 = $51A9
              L51F0 = $51F0
              L5200 = $5200
              L5201 = $5201
              L5202 = $5202
              L5203 = $5203
              L5204 = $5204
              L5205 = $5205
              L5220 = $5220
              L5246 = $5246
              L524D = $524D
              L5300 = $5300
              L5344 = $5344
              L5345 = $5345
              L5542 = $5542
              L574F = $574F
              L5EA6 = $5EA6
              L62A9 = $62A9
              L7461 = $7461
              L74A9 = $74A9
              L77A9 = $77A9
              L7848 = $7848
              L78A9 = $78A9
              L8000 = $8000
              L8002 = $8002
              L8003 = $8003
              L8005 = $8005
              L8006 = $8006
              L8007 = $8007
              L8008 = $8008
              L8009 = $8009
              L800A = $800A
              L800B = $800B
              L800C = $800C
              L800D = $800D
              L800E = $800E
              L800F = $800F
              L80A9 = $80A9
              L8200 = $8200
              L8300 = $8300
              L8400 = $8400
              L8401 = $8401
              L8402 = $8402
              L8403 = $8403
              L840A = $840A
              L840C = $840C
              L840D = $840D
              L840E = $840E
              L8600 = $8600
              L86A9 = $86A9
              L8700 = $8700
              L8785 = $8785
              L8800 = $8800
              L8801 = $8801
              L8802 = $8802
              L8803 = $8803
              L8A00 = $8A00
              L8B00 = $8B00
              L8C00 = $8C00
              L8C05 = $8C05
              L8C0C = $8C0C
              L8C0D = $8C0D
              L8F00 = $8F00
              L9000 = $9000
              L9038 = $9038
              L9070 = $9070
              L90A0 = $90A0
              L90A8 = $90A8
              L90A9 = $90A9
              L90E0 = $90E0
              L90E1 = $90E1
              L90E2 = $90E2
              L90E3 = $90E3
              L90E4 = $90E4
              L90E5 = $90E5
              L90E6 = $90E6
              L90E7 = $90E7
              L90E8 = $90E8
              L90F8 = $90F8
              L9100 = $9100
              L9200 = $9200
              L9300 = $9300
              .ORG $9400
9400 43 4D 44   .BYTE $43,$4D,$44
9403 20 48 44   .BYTE $20,$48,$44
9406 20 44 4F   .BYTE $20,$44,$4F
9409 53 20 43   .BYTE $53,$20,$43
940C 4F 50 59   .BYTE $4F,$50,$59
940F 52 49 47   .BYTE $52,$49,$47
9412 48 54 20   .BYTE $48,$54,$20
9415 31 39 39   .BYTE $31,$39,$39
9418 30 20 43   .BYTE $30,$20,$43
941B 52 45 41   .BYTE $52,$45,$41
941E 54 49 56   .BYTE $54,$49,$56
9421 45 20 4D   .BYTE $45,$20,$4D
9424 49 43 52   .BYTE $49,$43,$52
9427 4F 20 44   .BYTE $4F,$20,$44
942A 45 53 49   .BYTE $45,$53,$49
942D 47 4E 53   .BYTE $47,$4E,$53
9430          L9430:
9430 2C 20 49   BIT L4920
9433 4E 43 2E   LSR L2E43
9436 20 41 4C   JSR L4C41
9439 4C 20 52   JMP L5220
943C 49 47 48   .BYTE $49,$47,$48
943F 54 53 20   .BYTE $54,$53,$20
9442 52 45 53   .BYTE $52,$45,$53
9445 45 52 56   .BYTE $45,$52,$56
9448          L9448:
9448 45 44      EOR L44
944A          L944A:
944A 78         SEI
944B D8         CLD
944C A6 5E      LDX L5E
944E 9A         TXS
944F A9 80      LDA #$80
9451 85 81      STA L81
9453 8D D7 2B   STA L2BD7
9456 2D D8 2B   AND L2BD8
9459 8D D8 2B   STA L2BD8
945C A9 00      LDA #$0
945E 8D FB 2B   STA L2BFB
9461 A5 46      LDA L46
9463 29 3F      AND #$3F
9465 85 46      STA L46
9467 A9 02      LDA #$2
9469 8D 0D 80   STA VIA1+$0D
946C 20 9B 97   JSR L979B
946F 2C 01 88   BIT PIO+$01
9472 10 03      BPL L9477
9474          L9474:
9474 4C 69 95   JMP L9569
9477          L9477:
9477 2C 00 80   BIT VIA1+$00
947A 10 77      BPL L94F3
947C          L947C:
947C A9 02      LDA #$2
947E 8D 00 80   STA VIA1+$00
9481          L9481:
9481 AD 00 80   LDA VIA1+$00
9484 10 6D      BPL L94F3
9486          L9486:
9486 29 04      AND #$4
9488 D0 F7      BNE L9481
948A          L948A:
948A 20 2E 96   JSR L962E
948D          L948D:
948D C9 3F      CMP #$3F
948F D0 04      BNE L9495
9491          L9491:
9491 A9 BF      LDA #$BF
9493 D0 06      BNE L949B
9495          L9495:
9495 C9 5F      CMP #$5F
9497 D0 0E      BNE L94A7
9499          L9499:
9499 A9 7F      LDA #$7F
949B          L949B:
949B 25 46      AND L46
949D 85 46      STA L46
949F A9 00      LDA #$0
94A1 8D D8 2B   STA L2BD8
94A4 4C 4E 95   JMP L954E
94A7          L94A7:
94A7 C5 78      CMP L78
94A9 D0 04      BNE L94AF
94AB          L94AB:
94AB A9 80      LDA #$80
94AD D0 06      BNE L94B5
94AF          L94AF:
94AF C5 77      CMP L77
94B1          L94B1:
              ; Instruction opcode accessed.
94B1 D0 15      BNE L94C8
94B3          L94B3:
94B3 A9 40      LDA #$40
94B5          L94B5:
94B5 05 46      ORA L46
94B7 85 46      STA L46
94B9 09 3F      ORA #$3F
94BB 25 46      AND L46
94BD 85 46      STA L46
94BF AD E3 90   LDA L90E3
94C2 8D D6 2B   STA L2BD6
94C5 4C E2 94   JMP L94E2
94C8          L94C8:
94C8 AA         TAX
94C9 29 60      AND #$60
94CB C9 60      CMP #$60
94CD D0 6A      BNE L9539
94CF          L94CF:
94CF 86 83      STX L83
94D1 8A         TXA
94D2 29 0F      AND #$F
94D4 85 82      STA L82
94D6 8A         TXA
94D7 29 F0      AND #$F0
94D9 C9 E0      CMP #$E0
94DB D0 71      BNE L954E
94DD          L94DD:
94DD 58         CLI
94DE 20 E3 CC   JSR LCCE3
94E1 78         SEI
94E2          L94E2:
94E2 2C FB 2B   BIT L2BFB
94E5 50 07      BVC L94EE
94E7          L94E7:
94E7 2C 01 88   BIT PIO+$01
94EA 30 9E      BMI L948A
94EC          L94EC:
94EC 10 05      BPL L94F3
94EE          L94EE:
94EE 2C 00 80   BIT VIA1+$00
94F1 30 97      BMI L948A
94F3          L94F3:
94F3 A2 00      LDX #$0
94F5 8E D7 2B   STX L2BD7
94F8 AD 00 80   LDA VIA1+$00
94FB 09 10      ORA #$10
94FD 8D 00 80   STA VIA1+$00
9500 24 46      BIT L46
9502 50 0E      BVC L9512
9504          L9504:
9504 2C D8 2B   BIT L2BD8
9507 10 03      BPL L950C
9509          L9509:
9509 20 87 97   JSR L9787
950C          L950C:
950C 20 3F FF   JSR LFF3F
950F 4C 30 95   JMP L9530
9512          L9512:
9512 24 46      BIT L46
9514 10 1A      BPL L9530
9516          L9516:
9516 2C FB 2B   BIT L2BFB
9519 50 06      BVC L9521
951B          L951B:
951B 20 22 96   JSR L9622
951E 4C 2A 95   JMP L952A
9521          L9521:
9521 20 5A 97   JSR L975A
9524 20 75 97   JSR L9775
9527 20 D2 97   JSR L97D2
952A          L952A:
952A 20 42 FF   JSR LFF42
952D 20 D2 97   JSR L97D2
9530          L9530:
9530 20 F9 95   JSR L95F9
9533 20 9B 97   JSR L979B
9536 4C 30 FF   JMP LFF30
9539          L9539:
9539 2C FB 2B   BIT L2BFB
953C 70 1C      BVS L955A
953E          L953E:
953E 2C D8 2B   BIT L2BD8
9541 50 06      BVC L9549
9543          L9543:
9543 A5 46      LDA L46
9545 29 C0      AND #$C0
9547 D0 05      BNE L954E
9549          L9549:
9549 A9 00      LDA #$0
954B 8D 00 80   STA VIA1+$00
954E          L954E:
954E 2C FB 2B   BIT L2BFB
9551 70 0F      BVS L9562
9553          L9553:
9553 2C 00 80   BIT VIA1+$00
9556 10 9B      BPL L94F3
9558          L9558:
9558 30 F9      BMI L9553
955A          L955A:
955A AD 02 88   LDA PIO+$02
955D 09 E0      ORA #$E0
955F 8D 02 88   STA PIO+$02
9562          L9562:
9562 2C 01 88   BIT PIO+$01
9565 10 8C      BPL L94F3
9567          L9567:
9567 30 F9      BMI L9562
9569          L9569:
9569 A2 0A      LDX #$A
956B          L956B:
956B CA         DEX
956C D0 FD      BNE L956B
956E          L956E:
956E A9 40      LDA #$40
9570 8D FB 2B   STA L2BFB
9573 AD 02 88   LDA PIO+$02
9576 29 7F      AND #$7F
9578 09 60      ORA #$60
957A 8D 02 88   STA PIO+$02
957D AA         TAX
957E A9 92      LDA #$92
9580 8D 03 88   STA PIO+$03
9583 8E 02 88   STX PIO+$02
9586 20 33 96   JSR L9633
9589 4C 8D 94   JMP L948D
958C          L958C:
958C 2C 01 88   BIT PIO+$01
958F 30 36      BMI L95C7
9591          L9591:
9591 70 F9      BVS L958C
9593          L9593:
9593 BD C8 2D   LDA L2DC8,X
9596 8D 00 88   STA PIO+$00
9599 BD A8 2D   LDA L2DA8,X
959C 29 08      AND #$8
959E D0 12      BNE L95B2
95A0          L95A0:
95A0 AD 02 88   LDA PIO+$02
95A3 29 BF      AND #$BF
95A5 8D 02 88   STA PIO+$02
95A8 09 80      ORA #$80
95AA 8D 02 88   STA PIO+$02
95AD A0 28      LDY #$28
95AF          L95AF:
95AF 88         DEY
95B0 D0 FD      BNE L95AF
95B2          L95B2:
95B2 AD 02 88   LDA PIO+$02
95B5 09 C0      ORA #$C0
95B7 8D 02 88   STA PIO+$02
95BA 29 7F      AND #$7F
95BC          L95BC:
95BC 2C 01 88   BIT PIO+$01
95BF 30 06      BMI L95C7
95C1          L95C1:
95C1 50 F9      BVC L95BC
95C3          L95C3:
95C3 8D 02 88   STA PIO+$02
95C6 60         RTS
95C7          L95C7:
95C7 4C 4A 94   JMP L944A
95CA          L95CA:
95CA 2C 01 88   BIT PIO+$01
95CD 30 F8      BMI L95C7
95CF          L95CF:
95CF 70 F9      BVS L95CA
95D1          L95D1:
95D1 AC 00 88   LDY PIO+$00
95D4 84 84      STY L84
95D6 AD 02 88   LDA PIO+$02
95D9 09 80      ORA #$80
95DB 8D 02 88   STA PIO+$02
95DE A9 01      LDA #$1
95E0          L95E0:
95E0 2C 01 88   BIT PIO+$01
95E3 30 E2      BMI L95C7
95E5          L95E5:
95E5 D0 0C      BNE L95F3
95E7          L95E7:
95E7 50 F7      BVC L95E0
95E9          L95E9:
95E9 AD 02 88   LDA PIO+$02
95EC 29 7F      AND #$7F
95EE 8D 02 88   STA PIO+$02
95F1 98         TYA
95F2 60         RTS
95F3          L95F3:
95F3 A9 00      LDA #$0
95F5 85 81      STA L81
95F7 F0 E7      BEQ L95E0
95F9          L95F9:
95F9 08         PHP
95FA 78         SEI
95FB AD 02 88   LDA PIO+$02
95FE 09 E0      ORA #$E0
9600 29 7F      AND #$7F
9602 A8         TAY
9603 A2 92      LDX #$92
9605 8E 03 88   STX PIO+$03
9608 8D 02 88   STA PIO+$02
960B 09 80      ORA #$80
960D 2C 01 88   BIT PIO+$01
9610 30 08      BMI L961A
9612          L9612:
9612 8D 02 88   STA PIO+$02
9615 2C 01 88   BIT PIO+$01
9618 10 06      BPL L9620
961A          L961A:
961A 8C 02 88   STY PIO+$02
961D 4C 4A 94   JMP L944A
9620          L9620:
9620 28         PLP
9621 60         RTS
9622          L9622:
9622 AD 02 88   LDA PIO+$02
9625 A2 82      LDX #$82
9627 8E 03 88   STX PIO+$03
962A 8D 02 88   STA PIO+$02
962D 60         RTS
962E          L962E:
962E 2C FB 2B   BIT L2BFB
9631 50 4B      BVC L967E
9633          L9633:
9633 AD 02 88   LDA PIO+$02
9636 09 80      ORA #$80
9638 8D 02 88   STA PIO+$02
963B          L963B:
963B 2C 01 88   BIT PIO+$01
963E 10 3B      BPL L967B
9640          L9640:
9640 70 F9      BVS L963B
9642          L9642:
9642 AC 00 88   LDY PIO+$00
9645 84 84      STY L84
9647 A9 01      LDA #$1
9649 2C 01 88   BIT PIO+$01
964C F0 0B      BEQ L9659
964E          L964E:
964E C4 78      CPY L78
9650 F0 07      BEQ L9659
9652          L9652:
9652 C4 77      CPY L77
9654 F0 03      BEQ L9659
9656          L9656:
9656 4C 5A 95   JMP L955A
9659          L9659:
9659 AD 02 88   LDA PIO+$02
965C 29 7F      AND #$7F
965E 8D 02 88   STA PIO+$02
9661          L9661:
9661 2C 01 88   BIT PIO+$01
9664 10 15      BPL L967B
9666          L9666:
9666 50 F9      BVC L9661
9668          L9668:
9668 98         TYA
9669 24 46      BIT L46
966B 50 0B      BVC L9678
966D          L966D:
966D C9 60      CMP #$60
966F D0 07      BNE L9678
9671          L9671:
9671 8D FB 2B   STA L2BFB
9674 A9 61      LDA #$61
9676 85 84      STA L84
9678          L9678:
9678 4C 1B 97   JMP L971B
967B          L967B:
967B 4C F3 94   JMP L94F3
967E          L967E:
967E A9 08      LDA #$8
9680 85 96      STA L96
9682          L9682:
9682 20 30 97   JSR L9730
9685 D0 FB      BNE L9682
9687          L9687:
9687 20 5A 97   JSR L975A
968A A9 01      LDA #$1
968C          L968C:
968C 2C 00 80   BIT VIA1+$00
968F D0 FB      BNE L968C
9691          L9691:
9691 A2 0A      LDX #$A
9693          L9693:
9693 20 44 97   JSR L9744
9696 CA         DEX
9697 F0 09      BEQ L96A2
9699          L9699:
9699 20 7E 97   JSR L977E
969C 29 04      AND #$4
969E F0 F3      BEQ L9693
96A0          L96A0:
96A0 D0 14      BNE L96B6
96A2          L96A2:
96A2 20 63 97   JSR L9763
96A5 A2 18      LDX #$18
96A7          L96A7:
96A7 CA         DEX
96A8 D0 FD      BNE L96A7
96AA          L96AA:
96AA 20 5A 97   JSR L975A
96AD          L96AD:
96AD 20 30 97   JSR L9730
96B0 F0 FB      BEQ L96AD
96B2          L96B2:
96B2 A9 00      LDA #$0
96B4 85 81      STA L81
96B6          L96B6:
96B6 A2 1A      LDX #$1A
96B8          L96B8:
96B8 AD 00 80   LDA VIA1+$00
96BB A8         TAY
96BC 29 04      AND #$4
96BE F0 3B      BEQ L96FB
96C0          L96C0:
96C0 CA         DEX
96C1 D0 F5      BNE L96B8
96C3          L96C3:
96C3 A9 3F      LDA #$3F
96C5 2C D8 2B   BIT L2BD8
96C8 30 2D      BMI L96F7
96CA          L96CA:
96CA 70 10      BVS L96DC
96CC          L96CC:
96CC D0 29      BNE L96F7
96CE          L96CE:
96CE A6 96      LDX L96
96D0 E0 01      CPX #$1
96D2 F0 08      BEQ L96DC
96D4          L96D4:
96D4 A2 01      LDX #$1
96D6 8E D8 2B   STX L2BD8
96D9 CA         DEX
96DA F0 DC      BEQ L96B8
96DC          L96DC:
96DC A5 84      LDA L84
96DE 4A         LSR A
96DF C5 77      CMP L77
96E1 F0 04      BEQ L96E7
96E3          L96E3:
96E3 C5 78      CMP L78
96E5 D0 10      BNE L96F7
96E7          L96E7:
96E7 A9 40      LDA #$40
96E9 8D D8 2B   STA L2BD8
96EC A2 1E      LDX #$1E
96EE 20 63 97   JSR L9763
96F1          L96F1:
96F1 CA         DEX
96F2 D0 FD      BNE L96F1
96F4          L96F4:
96F4 20 5A 97   JSR L975A
96F7          L96F7:
96F7 A2 00      LDX #$0
96F9 F0 BD      BEQ L96B8
96FB          L96FB:
96FB 98         TYA
96FC 49 01      EOR #$1
96FE 4A         LSR A
96FF 66 84      ROR L84
9701          L9701:
9701 20 30 97   JSR L9730
9704 F0 FB      BEQ L9701
9706          L9706:
9706 C6 96      DEC L96
9708 D0 AC      BNE L96B6
970A          L970A:
970A 20 63 97   JSR L9763
970D A5 84      LDA L84
970F D0 0A      BNE L971B
9711          L9711:
9711 A9 80      LDA #$80
9713 2D D8 2B   AND L2BD8
9716 8D D8 2B   STA L2BD8
9719 A9 00      LDA #$0
971B          L971B:
971B 2C D8 2B   BIT L2BD8
971E 30 0F      BMI L972F
9720          L9720:
9720 C9 61      CMP #$61
9722 D0 0B      BNE L972F
9724          L9724:
9724 24 46      BIT L46
9726 10 07      BPL L972F
9728          L9728:
9728 8D D8 2B   STA L2BD8
972B A9 60      LDA #$60
972D 85 84      STA L84
972F          L972F:
972F 60         RTS
9730          L9730:
9730 20 44 97   JSR L9744
9733 29 04      AND #$4
9735 60         RTS
9736          L9736:
9736 20 44 97   JSR L9744
9739 6A         ROR A
973A 90 FA      BCC L9736
973C          L973C:
973C 60         RTS
973D          L973D:
973D 20 44 97   JSR L9744
9740 6A         ROR A
9741 B0 FA      BCS L973D
9743          L9743:
9743 60         RTS
9744          L9744:
9744 2C D7 2B   BIT L2BD7
9747 10 06      BPL L974F
9749          L9749:
9749 AD 00 80   LDA VIA1+$00
974C 10 09      BPL L9757
974E          L974E:
974E 60         RTS
974F          L974F:
974F AD 00 80   LDA VIA1+$00
9752 10 FA      BPL L974E
9754          L9754:
9754 4C 3C FF   JMP LFF3C
9757          L9757:
9757 4C F3 94   JMP L94F3
975A          L975A:
975A AD 00 80   LDA VIA1+$00
975D 29 FD      AND #$FD
975F 8D 00 80   STA VIA1+$00
9762 60         RTS
9763          L9763:
9763 AD 00 80   LDA VIA1+$00
9766 09 02      ORA #$2
9768 8D 00 80   STA VIA1+$00
976B 60         RTS
976C          L976C:
976C AD 00 80   LDA VIA1+$00
976F 29 F7      AND #$F7
9771 8D 00 80   STA VIA1+$00
9774 60         RTS
9775          L9775:
9775 AD 00 80   LDA VIA1+$00
9778 09 08      ORA #$8
977A 8D 00 80   STA VIA1+$00
977D 60         RTS
977E          L977E:
977E AD 00 80   LDA VIA1+$00
9781 CD 00 80   CMP VIA1+$00
9784 D0 F8      BNE L977E
9786          L9786:
9786 60         RTS
9787          L9787:
9787 20 30 97   JSR L9730
978A D0 FB      BNE L9787
978C          L978C:
978C 20 B9 97   JSR L97B9
978F A9 00      LDA #$0
9791 8D 0A 80   STA VIA1+$0A
9794 A9 04      LDA #$4
9796          L9796:
9796 2C 0D 80   BIT VIA1+$0D
9799 F0 FB      BEQ L9796
979B          L979B:
979B 08         PHP
979C 78         SEI
979D AD 0B 80   LDA VIA1+$0B
97A0 29 E3      AND #$E3
97A2 8D 0B 80   STA VIA1+$0B
97A5 09 0C      ORA #$C
97A7 8D 0B 80   STA VIA1+$0B
97AA AD 00 80   LDA VIA1+$00
97AD 29 DF      AND #$DF
97AF 8D 00 80   STA VIA1+$00
97B2 2C 0A 80   BIT VIA1+$0A
97B5 28         PLP
97B6 60         RTS
97B7          L97B7:
97B7 90 E2      BCC L979B
97B9          L97B9:
97B9 08         PHP
97BA 78         SEI
97BB AD 00 80   LDA VIA1+$00
97BE 09 20      ORA #$20
97C0 8D 00 80   STA VIA1+$00
97C3 AD 0B 80   LDA VIA1+$0B
97C6 29 E3      AND #$E3
97C8 8D 0B 80   STA VIA1+$0B
97CB 09 14      ORA #$14
97CD 8D 0B 80   STA VIA1+$0B
97D0 28         PLP
97D1 60         RTS
97D2          L97D2:
97D2 8A         TXA
97D3 EA         NOP
97D4 A2 0C      LDX #$C
97D6 D0 03      BNE L97DB
97D8          L97D8:
97D8 8A         TXA
97D9 A2 1D      LDX #$1D
97DB          L97DB:
97DB CA         DEX
97DC D0 FD      BNE L97DB
97DE          L97DE:
97DE AA         TAX
97DF 60         RTS
97E0          L97E0:
97E0 2C 00 80   BIT VIA1+$00
97E3 30 62      BMI L9847
97E5          L97E5:
97E5 20 6C 97   JSR L976C
97E8 20 3D 97   JSR L973D
97EB 20 36 97   JSR L9736
97EE A9 01      LDA #$1
97F0 D0 15      BNE L9807
97F2          L97F2:
97F2 BD A8 2D   LDA L2DA8,X
97F5 29 08      AND #$8
97F7 F0 E7      BEQ L97E0
97F9          L97F9:
97F9 AD 00 80   LDA VIA1+$00
97FC 29 01      AND #$1
97FE F0 E0      BEQ L97E0
9800          L9800:
9800 09 10      ORA #$10
9802 8D 00 80   STA VIA1+$00
9805 29 01      AND #$1
9807          L9807:
9807 2C 00 80   BIT VIA1+$00
980A 30 3B      BMI L9847
980C          L980C:
980C D0 F9      BNE L9807
980E          L980E:
980E A9 38      LDA #$38
9810 8D 00 80   STA VIA1+$00
9813 AD 0B 80   LDA VIA1+$0B
9816 29 E3      AND #$E3
9818 8D 0B 80   STA VIA1+$0B
981B 09 14      ORA #$14
981D 8D 0B 80   STA VIA1+$0B
9820 BD C8 2D   LDA L2DC8,X
9823 8D 09 80   STA VIA1+$09
9826 8D 0A 80   STA VIA1+$0A
9829 A9 04      LDA #$4
982B          L982B:
982B 2C 0D 80   BIT VIA1+$0D
982E F0 FB      BEQ L982B
9830          L9830:
9830 AD 0B 80   LDA VIA1+$0B
9833 49 18      EOR #$18
9835 8D 0B 80   STA VIA1+$0B
9838 A9 18      LDA #$18
983A 8D 00 80   STA VIA1+$00
983D A9 01      LDA #$1
983F          L983F:
983F 2C 00 80   BIT VIA1+$00
9842 30 03      BMI L9847
9844          L9844:
9844 F0 F9      BEQ L983F
9846          L9846:
9846 60         RTS
9847          L9847:
9847 4C 3C FF   JMP LFF3C
984A          L984A:
984A 20 59 98   JSR L9859
984D 29 02      AND #$2
984F F0 07      BEQ L9858
9851          L9851:
9851 A5 60      LDA L60
9853 09 0D      ORA #$D
9855 20 F4 98   JSR L98F4
9858          L9858:
9858 60         RTS
9859          L9859:
9859 AD 00 80   LDA VIA1+$00
985C 29 7D      AND #$7D
985E 85 6F      STA L6F
9860 29 71      AND #$71
9862 85 60      STA L60
9864 BD A8 2D   LDA L2DA8,X
9867 29 08      AND #$8
9869 D0 06      BNE L9871
986B          L986B:
986B A5 60      LDA L60
986D 09 03      ORA #$3
986F 85 6F      STA L6F
9871          L9871:
9871 BD C8 2D   LDA L2DC8,X
9874 A6 60      LDX L60
9876 2C 00 80   BIT VIA1+$00
9879 30 07      BMI L9882
987B          L987B:
987B 8E 00 80   STX VIA1+$00
987E A0 FF      LDY #$FF
9880 D0 1F      BNE L98A1
9882          L9882:
9882 4C 3C FF   JMP LFF3C
9885          L9885:
9885 AD 00 80   LDA VIA1+$00
9888 29 70      AND #$70
988A 85 60      STA L60
988C 09 0D      ORA #$D
988E 85 6F      STA L6F
9890 09 02      ORA #$2
9892 8D 00 80   STA VIA1+$00
9895 49 0D      EOR #$D
9897 8D 00 80   STA VIA1+$00
989A A2 0E      LDX #$E
989C          L989C:
989C CA         DEX
989D D0 FD      BNE L989C
989F          L989F:
989F B1 68      LDA (L68),Y
98A1          L98A1:
98A1 AA         TAX
98A2 4A         LSR A
98A3 4A         LSR A
98A4 4A         LSR A
98A5 4A         LSR A
98A6 85 6C      STA L6C
98A8 8A         TXA
98A9 29 0F      AND #$F
98AB AA         TAX
98AC BD 0C 99   LDA L990C,X
98AF A6 60      LDX L60
98B1 20 02 99   JSR L9902
98B4 8E 00 80   STX VIA1+$00
98B7 2C 00 80   BIT VIA1+$00
98BA          L98BA:
98BA EC 00 80   CPX VIA1+$00
98BD F0 FB      BEQ L98BA
98BF          L98BF:
98BF 48         PHA
98C0 68         PLA
98C1 EA         NOP
98C2 8D 00 80   STA VIA1+$00
98C5 0A         ASL A
98C6 09 10      ORA #$10
98C8 29 1F      AND #$1F
98CA 48         PHA
98CB 68         PLA
98CC 24 00      BIT L0
98CE 8D 00 80   STA VIA1+$00
98D1 A6 6C      LDX L6C
98D3 BD 0C 99   LDA L990C,X
98D6 48         PHA
98D7 68         PLA
98D8          L98D8:
98D8 2C 00 80   BIT VIA1+$00
98DB 8D 00 80   STA VIA1+$00
98DE 0A         ASL A
98DF 09 10      ORA #$10
98E1 29 1F      AND #$1F
98E3 EA         NOP
98E4 EA         NOP
98E5 EA         NOP
98E6 EA         NOP
98E7 A2 00      LDX #$0
98E9 C8         INY
98EA 8D 00 80   STA VIA1+$00
98ED D0 B0      BNE L989F
98EF          L98EF:
98EF B5 6F      LDA L6F,X
98F1 20 0B 99   JSR L990B
98F4          L98F4:
98F4 8D 00 80   STA VIA1+$00
98F7          L98F7:
98F7 2C 00 80   BIT VIA1+$00
98FA          L98FA:
98FA CD 00 80   CMP VIA1+$00
98FD 90 83      BCC L9882
98FF          L98FF:
98FF D0 F6      BNE L98F7
9901          L9901:
9901 60         RTS
9902          L9902:
9902 2C 00 E0   BIT LE000
9905          L9905:
9905 2C 00 E0   BIT LE000
9908 2C 00 E0   BIT LE000
990B          L990B:
990B 60         RTS
990C          L990C:
990C 1F 17 1D   .BYTE $1F,$17,$1D
990F 15 1B 13   .BYTE $15,$1B,$13
9912 19 11 1E   .BYTE $19,$11,$1E
9915 16 1C 14   .BYTE $16,$1C,$14
9918 1A 12 18   .BYTE $1A,$12,$18
991C          L991C = * + 1
991B 10 00 80   .BYTE $10,$0,$80
991E 20 A0 40   .BYTE $20,$A0,$40
9921 C0 60 E0   .BYTE $C0,$60,$E0
9924 10 90      .BYTE $10,$90
9926 30 B0      BMI L98D8
9928          L9928:
9928 50 D0      BVC L98FA
992A 70 F0      .BYTE $70,$F0
992C          L992C:
992C 2C 0A 80   BIT VIA1+$0A
992F A9 04      LDA #$4
9931          L9931:
9931 2C 00 80   BIT VIA1+$00
9934 30 2E      BMI L9964
9936          L9936:
9936 D0 F9      BNE L9931
9938          L9938:
9938 09 10      ORA #$10
993A 8D 00 80   STA VIA1+$00
993D A2 80      LDX #$80
993F A9 04      LDA #$4
9941          L9941:
9941 2C 00 80   BIT VIA1+$00
9944 30 1E      BMI L9964
9946          L9946:
9946 D0 0A      BNE L9952
9948          L9948:
9948 CA         DEX
9949 D0 F6      BNE L9941
994B          L994B:
994B A9 08      LDA #$8
994D 85 96      STA L96
994F 4C 3E 9A   JMP L9A3E
9952          L9952:
9952 A2 12      LDX #$12
9954 A9 04      LDA #$4
9956          L9956:
9956 2C 0D 80   BIT VIA1+$0D
9959          L9959:
9959 F0 FB      BEQ L9956
995B          L995B:
995B AD 0A 80   LDA VIA1+$0A
995E 8E 00 80   STX VIA1+$00
9961 85 84      STA L84
9963 60         RTS
9964          L9964:
9964 4C 3C FF   JMP LFF3C
9967          L9967:
9967 A9 14      LDA #$14
9969 8D 00 80   STA VIA1+$00
996C 29 04      AND #$4
996E          L996E:
996E 2C 00 80   BIT VIA1+$00
9971 D0 FB      BNE L996E
9973          L9973:
9973 20 02 99   JSR L9902
9976 AD 00 80   LDA VIA1+$00
9979 0A         ASL A
997A 20 05 99   JSR L9905
997D 0D 00 80   ORA VIA1+$00
9980 29 0F      AND #$F
9982 AA         TAX
9983 A0 00      LDY #$0
9985 20 0B 99   JSR L990B
9988 AD 00 80   LDA VIA1+$00
998B 0A         ASL A
998C 20 05 99   JSR L9905
998F 0D 00 80   ORA VIA1+$00
9992 29 0F      AND #$F
9994 1D 1C 99   ORA L991C,X
9997 85 84      STA L84
9999 20 0B 99   JSR L990B
999C AD 00 80   LDA VIA1+$00
999F 24 84      BIT L84
99A1 24 84      BIT L84
99A3 09 02      ORA #$2
99A5 8D 00 80   STA VIA1+$00
99A8 30 BA      BMI L9964
99AA          L99AA:
99AA 29 04      AND #$4
99AC D0 02      BNE L99B0
99AE          L99AE:
99AE 84 81      STY L81
99B0          L99B0:
99B0 A5 84      LDA L84
99B2 60         RTS
99B3          L99B3:
99B3 A9 08      LDA #$8
99B5 85 96      STA L96
99B7 AD 00 80   LDA VIA1+$00
99BA 29 F7      AND #$F7
99BC 8D 00 80   STA VIA1+$00
99BF 4A         LSR A
99C0 90 0A      BCC L99CC
99C2          L99C2:
99C2 20 3D 97   JSR L973D
99C5 BD A8 2D   LDA L2DA8,X
99C8 29 08      AND #$8
99CA D0 13      BNE L99DF
99CC          L99CC:
99CC 20 36 97   JSR L9736
99CF 20 DF 99   JSR L99DF
99D2 A2 32      LDX #$32
99D4          L99D4:
99D4 20 44 97   JSR L9744
99D7 29 01      AND #$1
99D9 F0 03      BEQ L99DE
99DB          L99DB:
99DB CA         DEX
99DC D0 F6      BNE L99D4
99DE          L99DE:
99DE 60         RTS
99DF          L99DF:
99DF 20 75 97   JSR L9775
99E2 20 D2 97   JSR L97D2
99E5 20 3D 97   JSR L973D
99E8 20 DE 99   JSR L99DE
99EB          L99EB:
99EB 20 D2 97   JSR L97D2
99EE 7E C8 2D   ROR L2DC8,X
99F1 20 DE 99   JSR L99DE
99F4 20 5A 97   JSR L975A
99F7 B0 02      BCS L99FB
99F9          L99F9:
99F9 09 02      ORA #$2
99FB          L99FB:
99FB 8D 00 80   STA VIA1+$00
99FE 20 6C 97   JSR L976C
9A01 20 D2 97   JSR L97D2
9A04 8A         TXA
9A05 A2 0B      LDX #$B
9A07          L9A07:
9A07 CA         DEX
9A08 D0 FD      BNE L9A07
9A0A          L9A0A:
9A0A AA         TAX
9A0B AD 00 80   LDA VIA1+$00
9A0E 09 08      ORA #$8
9A10 29 FD      AND #$FD
9A12 8D 00 80   STA VIA1+$00
9A15 C6 96      DEC L96
9A17 D0 D2      BNE L99EB
9A19          L9A19:
9A19 4C 36 97   JMP L9736
9A1C          L9A1C:
9A1C 2C 0A 80   BIT VIA1+$0A
9A1F A9 08      LDA #$8
9A21 85 96      STA L96
9A23          L9A23:
9A23 20 30 97   JSR L9730
9A26 D0 FB      BNE L9A23
9A28          L9A28:
9A28 20 5A 97   JSR L975A
9A2B A9 01      LDA #$1
9A2D          L9A2D:
9A2D 2C 00 80   BIT VIA1+$00
9A30 30 47      BMI L9A79
9A32          L9A32:
9A32 D0 F9      BNE L9A2D
9A34          L9A34:
9A34 A2 14      LDX #$14
9A36          L9A36:
9A36 20 30 97   JSR L9730
9A39 D0 15      BNE L9A50
9A3B          L9A3B:
9A3B CA         DEX
9A3C D0 F8      BNE L9A36
9A3E          L9A3E:
9A3E 20 63 97   JSR L9763
9A41 20 D8 97   JSR L97D8
9A44 20 5A 97   JSR L975A
9A47          L9A47:
9A47 20 30 97   JSR L9730
9A4A F0 FB      BEQ L9A47
9A4C          L9A4C:
9A4C A9 00      LDA #$0
9A4E 85 81      STA L81
9A50          L9A50:
9A50 AE 00 80   LDX VIA1+$00
9A53 A9 04      LDA #$4
9A55 2C 0D 80   BIT VIA1+$0D
9A58 F0 05      BEQ L9A5F
9A5A          L9A5A:
9A5A A2 12      LDX #$12
9A5C 4C 5B 99   JMP L995B
9A5F          L9A5F:
9A5F 8A         TXA
9A60 29 04      AND #$4
9A62 D0 EC      BNE L9A50
9A64          L9A64:
9A64 8A         TXA
9A65 49 01      EOR #$1
9A67 4A         LSR A
9A68 66 84      ROR L84
9A6A          L9A6A:
9A6A 20 30 97   JSR L9730
9A6D F0 FB      BEQ L9A6A
9A6F          L9A6F:
9A6F C6 96      DEC L96
9A71 D0 DD      BNE L9A50
9A73          L9A73:
9A73 20 63 97   JSR L9763
9A76 A5 84      LDA L84
9A78          L9A78:
9A78 60         RTS
9A79          L9A79:
9A79 4C 3C FF   JMP LFF3C
9A7C          L9A7C:
9A7C AD 02 02   LDA L202
9A7F C9 2B      CMP #$2B
9A81 F0 F5      BEQ L9A78
9A83          L9A83:
9A83 C9 2D      CMP #$2D
9A85 F0 F1      BEQ L9A78
9A87          L9A87:
9A87 4C 2A FF   JMP LFF2A
9A8A          L9A8A:
9A8A 20 3D 97   JSR L973D
9A8D A9 04      LDA #$4
9A8F          L9A8F:
9A8F AA         TAX
9A90 A5 69      LDA L69
9A92 48         PHA
9A93 8A         TXA
9A94 48         PHA
9A95 A0 01      LDY #$1
9A97 B1 68      LDA (L68),Y
9A99 85 5B      STA L5B
9A9B AA         TAX
9A9C 88         DEY
9A9D B1 68      LDA (L68),Y
9A9F 85 5A      STA L5A
9AA1 D0 0C      BNE L9AAF
9AA3          L9AA3:
9AA3 68         PLA
9AA4 18         CLC
9AA5 E5 5B      SBC L5B
9AA7 E8         INX
9AA8 86 68      STX L68
9AAA F0 02      BEQ L9AAE
9AAC          L9AAC:
9AAC C6 69      DEC L69
9AAE          L9AAE:
9AAE 48         PHA
9AAF          L9AAF:
9AAF 68         PLA
9AB0 A8         TAY
9AB1 20 85 98   JSR L9885
9AB4 68         PLA
9AB5 85 69      STA L69
9AB7 A5 5A      LDA L5A
9AB9 F0 07      BEQ L9AC2
9ABB          L9ABB:
9ABB 20 E2 9A   JSR L9AE2
9ABE A9 02      LDA #$2
9AC0 D0 CD      BNE L9A8F
9AC2          L9AC2:
9AC2 85 68      STA L68
9AC4 20 DA 9A   JSR L9ADA
9AC7 20 DA 9A   JSR L9ADA
9ACA 20 D7 9A   JSR L9AD7
9ACD A0 00      LDY #$0
9ACF          L9ACF:
9ACF B1 68      LDA (L68),Y
9AD1 91 66      STA (L66),Y
9AD3 C8         INY
9AD4 D0 F9      BNE L9ACF
9AD6          L9AD6:
9AD6 60         RTS
9AD7          L9AD7:
9AD7 20 75 97   JSR L9775
9ADA          L9ADA:
9ADA A2 28      LDX #$28
9ADC          L9ADC:
9ADC CA         DEX
9ADD D0 FD      BNE L9ADC
9ADF          L9ADF:
9ADF 4C 6C 97   JMP L976C
9AE2          L9AE2:
9AE2 20 73 D9   JSR LD973
9AE5 98         TYA
9AE6 4A         LSR A
9AE7 AA         TAX
9AE8 A9 AA      LDA #$AA
9AEA 4C 1C E8   JMP LE81C
9AED          L9AED:
9AED A9 04      LDA #$4
9AEF          L9AEF:
9AEF 48         PHA
9AF0 A0 01      LDY #$1
9AF2 B1 68      LDA (L68),Y
9AF4 85 5B      STA L5B
9AF6 AA         TAX
9AF7 88         DEY
9AF8 B1 68      LDA (L68),Y
9AFA 85 5A      STA L5A
9AFC F0 08      BEQ L9B06
9AFE          L9AFE:
9AFE 68         PLA
9AFF 48         PHA
9B00 49 FF      EOR #$FF
9B02 AA         TAX
9B03 E8         INX
9B04 D0 09      BNE L9B0F
9B06          L9B06:
9B06 CA         DEX
9B07 68         PLA
9B08 48         PHA
9B09 C9 02      CMP #$2
9B0B F0 02      BEQ L9B0F
9B0D          L9B0D:
9B0D CA         DEX
9B0E CA         DEX
9B0F          L9B0F:
9B0F 68         PLA
9B10 20 47 9B   JSR L9B47
9B13 A5 5A      LDA L5A
9B15 F0 07      BEQ L9B1E
9B17          L9B17:
9B17 20 98 9B   JSR L9B98
9B1A A9 02      LDA #$2
9B1C D0 D1      BNE L9AEF
9B1E          L9B1E:
9B1E A9 00      LDA #$0
9B20          L9B20:
9B20 2C 01 88   BIT PIO+$01
9B23 30 1F      BMI L9B44
9B25          L9B25:
9B25 70 F7      BVS L9B1E
9B27          L9B27:
9B27 8D 00 88   STA PIO+$00
9B2A AD 02 88   LDA PIO+$02
9B2D 09 80      ORA #$80
9B2F 8D 02 88   STA PIO+$02
9B32          L9B32:
9B32 2C 01 88   BIT PIO+$01
9B35 30 0D      BMI L9B44
9B37          L9B37:
9B37 50 F9      BVC L9B32
9B39          L9B39:
9B39 29 7F      AND #$7F
9B3B 8D 02 88   STA PIO+$02
9B3E A2 28      LDX #$28
9B40          L9B40:
9B40 CA         DEX
9B41 D0 FD      BNE L9B40
9B43          L9B43:
9B43 60         RTS
9B44          L9B44:
9B44 4C 4A 94   JMP L944A
9B47          L9B47:
9B47 A8         TAY
9B48          L9B48:
9B48 2C 01 88   BIT PIO+$01
9B4B 30 F7      BMI L9B44
9B4D          L9B4D:
9B4D 70 F9      BVS L9B48
9B4F          L9B4F:
9B4F 8E 00 88   STX PIO+$00
9B52 AD 02 88   LDA PIO+$02
9B55 09 80      ORA #$80
9B57 8D 02 88   STA PIO+$02
9B5A          L9B5A:
9B5A 2C 01 88   BIT PIO+$01
9B5D 30 E5      BMI L9B44
9B5F          L9B5F:
9B5F 50 F9      BVC L9B5A
9B61          L9B61:
9B61 B1 68      LDA (L68),Y
9B63 8D 00 88   STA PIO+$00
9B66 AD 02 88   LDA PIO+$02
9B69 29 7F      AND #$7F
9B6B 8D 02 88   STA PIO+$02
9B6E CA         DEX
9B6F F0 1C      BEQ L9B8D
9B71          L9B71:
9B71 C8         INY
9B72 B1 68      LDA (L68),Y
9B74          L9B74:
9B74 2C 01 88   BIT PIO+$01
9B77 70 FB      BVS L9B74
9B79          L9B79:
9B79 8D 00 88   STA PIO+$00
9B7C CA         DEX
9B7D F0 13      BEQ L9B92
9B7F          L9B7F:
9B7F C8         INY
9B80 B1 68      LDA (L68),Y
9B82          L9B82:
9B82 2C 01 88   BIT PIO+$01
9B85 50 FB      BVC L9B82
9B87          L9B87:
9B87 8D 00 88   STA PIO+$00
9B8A CA         DEX
9B8B D0 E4      BNE L9B71
9B8D          L9B8D:
9B8D 2C 01 88   BIT PIO+$01
9B90 70 FB      BVS L9B8D
9B92          L9B92:
9B92 2C 01 88   BIT PIO+$01
9B95 50 FB      BVC L9B92
9B97          L9B97:
9B97 60         RTS
9B98          L9B98:
9B98 20 73 D9   JSR LD973
9B9B 98         TYA
9B9C 4A         LSR A
9B9D AA         TAX
9B9E A9 AA      LDA #$AA
9BA0 20 25 E8   JSR LE825
9BA3 B0 01      BCS L9BA6
9BA5          L9BA5:
9BA5 60         RTS
9BA6          L9BA6:
9BA6 48         PHA
9BA7 8A         TXA
9BA8 48         PHA
9BA9 A9 FF      LDA #$FF
9BAB 20 20 9B   JSR L9B20
9BAE 68         PLA
9BAF AA         TAX
9BB0 68         PLA
9BB1 4C 36 FF   JMP LFF36
9BB4          L9BB4:
9BB4 4E 67 2A   LSR L2A67
9BB7 A0 00      LDY #$0
9BB9 20 13 9C   JSR L9C13
9BBC A9 04      LDA #$4
9BBF          L9BBF = * + 1
              ; Instruction parameter jumped to.
9BBE 2C A9 02   BIT L2A9
9BC1 48         PHA
9BC2 20 CA 95   JSR L95CA
9BC5 AA         TAX
9BC6 68         PLA
9BC7 A8         TAY
9BC8          L9BC8:
9BC8 2C 01 88   BIT PIO+$01
9BCB 70 FB      BVS L9BC8
9BCD          L9BCD:
9BCD AD 00 88   LDA PIO+$00
9BD0 91 66      STA (L66),Y
9BD2 C8         INY
9BD3 CA         DEX
9BD4 F0 0E      BEQ L9BE4
9BD6          L9BD6:
9BD6 2C 01 88   BIT PIO+$01
9BD9 50 FB      BVC L9BD6
9BDB          L9BDB:
9BDB AD 00 88   LDA PIO+$00
9BDE 91 66      STA (L66),Y
9BE0 C8         INY
9BE1 CA         DEX
9BE2 D0 E4      BNE L9BC8
9BE4          L9BE4:
9BE4 2C 01 88   BIT PIO+$01
9BE7 30 27      BMI L9C10
9BE9          L9BE9:
9BE9 50 F9      BVC L9BE4
9BEB          L9BEB:
9BEB 20 24 9C   JSR L9C24
9BEE          L9BEE:
9BEE 2C 01 88   BIT PIO+$01
9BF1 30 1D      BMI L9C10
9BF3          L9BF3:
9BF3 70 F9      BVS L9BEE
9BF5          L9BF5:
9BF5 20 F3 A3   JSR LA3F3
9BF8 20 13 9C   JSR L9C13
9BFB A0 00      LDY #$0
9BFD A5 5A      LDA L5A
9BFF 91 66      STA (L66),Y
9C01 C8         INY
9C02 A5 5B      LDA L5B
9C04 91 66      STA (L66),Y
9C06 C8         INY
9C07 20 24 9C   JSR L9C24
9C0A 20 2D 9C   JSR L9C2D
9C0D 4C BF 9B   JMP L9BBF
9C10          L9C10:
9C10 4C 4A 94   JMP L944A
9C13          L9C13:
9C13 A6 80      LDX L80
9C15 BD 68 2C   LDA L2C68,X
9C18 8D 57 2A   STA L2A57
9C1B 18         CLC
9C1C 69 03      ADC #$3
9C1E 85 67      STA L67
9C20 A9 00      LDA #$0
9C22 85 66      STA L66
9C24          L9C24:
9C24 AD 57 2A   LDA L2A57
9C27 0A         ASL A
9C28 AA         TAX
9C29 98         TYA
9C2A 95 A0      STA LA0,X
9C2C 60         RTS
9C2D          L9C2D:
9C2D 20 C7 E9   JSR LE9C7
9C30 90 03      BCC L9C35
9C32          L9C32:
9C32 4C 59 A1   JMP LA159
9C35          L9C35:
9C35 2C 5D 2A   BIT L2A5D
9C38 30 2D      BMI L9C67
9C3A          L9C3A:
9C3A AD 57 2A   LDA L2A57
9C3D 0A         ASL A
9C3E AA         TAX
9C3F A5 5A      LDA L5A
9C41 DD 00 28   CMP L2800,X
9C44 D0 3C      BNE L9C82
9C46          L9C46:
9C46 A5 5B      LDA L5B
9C48 E9 01      SBC #$1
9C4A DD 01 28   CMP L2801,X
9C4D D0 33      BNE L9C82
9C4F          L9C4F:
9C4F 6E 67 2A   ROR L2A67
9C52 20 AC EE   JSR LEEAC
9C55 20 68 EE   JSR LEE68
9C58 A0 00      LDY #$0
9C5A          L9C5A:
9C5A B1 66      LDA (L66),Y
9C5C 91 68      STA (L68),Y
9C5E 99 00 52   STA L5200,Y
9C61 C8         INY
9C62 D0 F6      BNE L9C5A
9C64          L9C64:
9C64 4C 3F A1   JMP LA13F
9C67          L9C67:
9C67 2C 67 2A   BIT L2A67
9C6A 10 16      BPL L9C82
9C6C          L9C6C:
9C6C 4E 67 2A   LSR L2A67
9C6F 20 78 EE   JSR LEE78
9C72 F0 0E      BEQ L9C82
9C74          L9C74:
9C74 A0 00      LDY #$0
9C76          L9C76:
9C76 B9 00 52   LDA L5200,Y
9C79 99 00 50   STA L5000,Y
9C7C C8         INY
9C7D D0 F7      BNE L9C76
9C7F          L9C7F:
9C7F 20 AC EE   JSR LEEAC
9C82          L9C82:
9C82 20 28 ED   JSR LED28
9C85 4C 3F A1   JMP LA13F
9C88          L9C88:
9C88 20 78 B6   JSR LB678
9C8B 20 03 AF   JSR LAF03
9C8E 20 8E B0   JSR LB08E
9C91 48         PHA
9C92 20 95 B0   JSR LB095
9C95 48         PHA
9C96 20 85 B0   JSR LB085
9C99 D0 06      BNE L9CA1
9C9B          L9C9B:
9C9B 20 10 B0   JSR LB010
9C9E 20 26 B0   JSR LB026
9CA1          L9CA1:
9CA1 20 C7 A2   JSR LA2C7
9CA4 A2 00      LDX #$0
9CA6 8E 00 2C   STX L2C00
9CA9 A0 90      LDY #$90
9CAB          L9CAB:
9CAB B1 58      LDA (L58),Y
9CAD 9D 00 02   STA L200,X
9CB0 C8         INY
9CB1 E8         INX
9CB2 E0 10      CPX #$10
9CB4 90 F5      BCC L9CAB
9CB6          L9CB6:
9CB6 86 56      STX L56
9CB8 20 E1 A7   JSR LA7E1
9CBB 20 7E A1   JSR LA17E
9CBE A2 AD      LDX #$AD
9CC0          L9CC0:
9CC0 BD 00 22   LDA L2200,X
9CC3 DD 9C 9D   CMP L9D9C,X
9CC6 D0 37      BNE L9CFF
9CC8          L9CC8:
9CC8 E8         INX
9CC9 E0 B8      CPX #$B8
9CCB 90 F3      BCC L9CC0
9CCD          L9CCD:
9CCD AD AB 22   LDA L22AB
9CD0 F0 2D      BEQ L9CFF
9CD2          L9CD2:
9CD2 85 5A      STA L5A
9CD4 8D A7 2B   STA L2BA7
9CD7 AD AC 22   LDA L22AC
9CDA 85 5B      STA L5B
9CDC 8D A9 2B   STA L2BA9
9CDF 20 85 B0   JSR LB085
9CE2 C9 02      CMP #$2
9CE4 F0 04      BEQ L9CEA
9CE6          L9CE6:
9CE6 C9 03      CMP #$3
9CE8 D0 0F      BNE L9CF9
9CEA          L9CEA:
9CEA 20 C7 A2   JSR LA2C7
9CED A0 AB      LDY #$AB
9CEF          L9CEF:
9CEF B9 00 22   LDA L2200,Y
9CF2 91 58      STA (L58),Y
9CF4 C8         INY
9CF5 C0 BD      CPY #$BD
9CF7 90 F6      BCC L9CEF
9CF9          L9CF9:
9CF9 20 2D 9E   JSR L9E2D
9CFC 20 1B 9D   JSR L9D1B
9CFF          L9CFF:
9CFF 20 1B 9D   JSR L9D1B
9D02 AD A7 2B   LDA L2BA7
9D05 85 5A      STA L5A
9D07 AD A8 2B   LDA L2BA8
9D0A 85 5B      STA L5B
9D0C 20 2D 9E   JSR L9E2D
9D0F 20 48 A3   JSR LA348
9D12 68         PLA
9D13 A8         TAY
9D14 68         PLA
9D15 20 13 B0   JSR LB013
9D18 4C 54 B6   JMP LB654
9D1B          L9D1B:
9D1B A9 00      LDA #$0
9D1D 8D BC 2B   STA L2BBC
9D20 20 7C C0   JSR LC07C
9D23 F0 03      BEQ L9D28
9D25          L9D25:
9D25 4C 0C 9E   JMP L9E0C
9D28          L9D28:
9D28 20 26 B0   JSR LB026
9D2B 20 85 B0   JSR LB085
9D2E D0 38      BNE L9D68
9D30          L9D30:
9D30 20 7E A1   JSR LA17E
9D33 AD 22 22   LDA L2222
9D36 F0 30      BEQ L9D68
9D38          L9D38:
9D38 AC 23 22   LDY L2223
9D3B 20 13 B0   JSR LB013
9D3E 20 26 B0   JSR LB026
9D41 AD 24 22   LDA L2224
9D44 8D B6 2B   STA L2BB6
9D47 AD 25 22   LDA L2225
9D4A 8D B7 2B   STA L2BB7
9D4D AD 26 22   LDA L2226
9D50 8D B8 2B   STA L2BB8
9D53 4A         LSR A
9D54 4A         LSR A
9D55 4A         LSR A
9D56 4A         LSR A
9D57 4A         LSR A
9D58 38         SEC
9D59 E9 07      SBC #$7
9D5B 49 FF      EOR #$FF
9D5D 8D C1 2B   STA L2BC1
9D60 A9 FF      LDA #$FF
9D62 8D C0 2B   STA L2BC0
9D65 4C 04 9E   JMP L9E04
9D68          L9D68:
9D68 60         RTS
9D69          L9D69:
9D69 A0 01      LDY #$1
9D6B B1 94      LDA (L94),Y
9D6D 48         PHA
9D6E C8         INY
9D6F B1 94      LDA (L94),Y
9D71 48         PHA
9D72 A0 13      LDY #$13
9D74 B1 94      LDA (L94),Y
9D76 F0 4F      BEQ L9DC7
9D78          L9D78:
9D78 85 5A      STA L5A
9D7A C8         INY
9D7B B1 94      LDA (L94),Y
9D7D 85 5B      STA L5B
9D7F C8         INY
9D80 B1 94      LDA (L94),Y
9D82 48         PHA
9D83 C8         INY
9D84 B1 94      LDA (L94),Y
9D86 48         PHA
9D87 AD ED 2B   LDA L2BED
9D8A 48         PHA
9D8B 20 2D 9E   JSR L9E2D
9D8E 68         PLA
9D8F 8D ED 2B   STA L2BED
9D92 A8         TAY
9D93 68         PLA
9D94 AA         TAX
9D95 68         PLA
9D96 C9 01      CMP #$1
9D98 D0 2D      BNE L9DC7
9D9A          L9D9A:
9D9A 8A         TXA
9D9C          L9D9C = * + 1
9D9B F0 2A      BEQ L9DC7
9D9D          L9D9D:
9D9D C0 03      CPY #$3
9D9F D0 26      BNE L9DC7
9DA1          L9DA1:
9DA1 68         PLA
9DA2 AA         TAX
9DA3 85 5B      STA L5B
9DA5 68         PLA
9DA6 85 5A      STA L5A
9DA8 48         PHA
9DA9 8A         TXA
9DAA 48         PHA
9DAB 20 A2 A1   JSR LA1A2
9DAE A0 02      LDY #$2
9DB0          L9DB0:
9DB0 84 9D      STY L9D
9DB2 B9 00 22   LDA L2200,Y
9DB5 F0 0C      BEQ L9DC3
9DB7          L9DB7:
9DB7 85 5A      STA L5A
9DB9 B9 01 22   LDA L2201,Y
9DBC 85 5B      STA L5B
9DBE 20 2D 9E   JSR L9E2D
9DC1 A4 9D      LDY L9D
9DC3          L9DC3:
9DC3 C8         INY
9DC4 C8         INY
9DC5 D0 E9      BNE L9DB0
9DC7          L9DC7:
9DC7 68         PLA
9DC8 85 5B      STA L5B
9DCA 68         PLA
9DCB 85 5A      STA L5A
9DCD 20 85 B0   JSR LB085
9DD0 D0 2F      BNE L9E01
9DD2          L9DD2:
9DD2 AD ED 2B   LDA L2BED
9DD5 C9 06      CMP #$6
9DD7 D0 28      BNE L9E01
9DD9          L9DD9:
9DD9 A5 5A      LDA L5A
9DDB A4 5B      LDY L5B
9DDD 20 13 B0   JSR LB013
9DE0 20 26 B0   JSR LB026
9DE3 20 7E A1   JSR LA17E
9DE6 AD B6 2B   LDA L2BB6
9DE9 8D 24 22   STA L2224
9DEC AD B7 2B   LDA L2BB7
9DEF 8D 25 22   STA L2225
9DF2 AD B8 2B   LDA L2BB8
9DF5 8D 26 22   STA L2226
9DF8 20 CF A1   JSR LA1CF
9DFB 20 2D 9E   JSR L9E2D
9DFE 4C 1B 9D   JMP L9D1B
9E01          L9E01:
9E01 20 2D 9E   JSR L9E2D
9E04          L9E04:
9E04 20 E0 C0   JSR LC0E0
9E07 D0 03      BNE L9E0C
9E09          L9E09:
9E09 4C 28 9D   JMP L9D28
9E0C          L9E0C:
9E0C A0 00      LDY #$0
9E0E B1 94      LDA (L94),Y
9E10 30 06      BMI L9E18
9E12          L9E12:
9E12 20 6D C3   JSR LC36D
9E15 4C 04 9E   JMP L9E04
9E18          L9E18:
9E18 29 07      AND #$7
9E1A 8D ED 2B   STA L2BED
9E1D C9 05      CMP #$5
9E1F F0 03      BEQ L9E24
9E21          L9E21:
9E21 4C 69 9D   JMP L9D69
9E24          L9E24:
9E24 20 AB BC   JSR LBCAB
9E27 20 C4 BC   JSR LBCC4
9E2A 4C 04 9E   JMP L9E04
9E2D          L9E2D:
9E2D 20 1C D9   JSR LD91C
9E30 20 5C A3   JSR LA35C
9E33 20 78 C3   JSR LC378
9E36          L9E36:
9E36 20 DB D9   JSR LD9DB
9E39 A5 5A      LDA L5A
9E3B D0 03      BNE L9E40
9E3D          L9E3D:
9E3D 4C 04 DB   JMP LDB04
9E40          L9E40:
9E40 20 5C A3   JSR LA35C
9E43 20 5E 9F   JSR L9F5E
9E46 4C 36 9E   JMP L9E36
9E49 47 45 4F   .BYTE $47,$45,$4F
9E4C 53 20 66   .BYTE $53,$20,$66
9E4F 6F 72      .BYTE $6F,$72
9E51          L9E51:
9E51 6D 61 74   ADC L7461
9E54          L9E54:
9E54 78         SEI
9E55 2C FB 2B   BIT L2BFB
9E58 70 05      BVS L9E5F
9E5A          L9E5A:
9E5A A2 64      LDX #$64
9E5C          L9E5C:
9E5C CA         DEX
9E5D D0 FD      BNE L9E5C
9E5F          L9E5F:
9E5F 20 60 DA   JSR LDA60
9E62 B0 07      BCS L9E6B
9E64          L9E64:
9E64 A6 80      LDX L80
9E66 BD A8 2D   LDA L2DA8,X
9E69 30 01      BMI L9E6C
9E6B          L9E6B:
9E6B 60         RTS
9E6C          L9E6C:
9E6C AD D8 2B   LDA L2BD8
9E6F C9 61      CMP #$61
9E71 D0 0B      BNE L9E7E
9E73          L9E73:
9E73 2C FB 2B   BIT L2BFB
9E76 50 03      BVC L9E7B
9E78          L9E78:
9E78 4C ED 9A   JMP L9AED
9E7B          L9E7B:
9E7B 4C 8A 9A   JMP L9A8A
9E7E          L9E7E:
9E7E 20 E0 9E   JSR L9EE0
9E81 A5 82      LDA L82
9E83 D0 07      BNE L9E8C
9E85          L9E85:
9E85 AD C5 2B   LDA L2BC5
9E88 F0 02      BEQ L9E8C
9E8A          L9E8A:
9E8A A2 0C      LDX #$C
9E8C          L9E8C:
9E8C BD CA 9E   LDA L9ECA,X
9E8F 8D FC 2B   STA L2BFC
9E92 BD CB 9E   LDA L9ECB,X
9E95 8D FD 2B   STA L2BFD
9E98 2C FB 2B   BIT L2BFB
9E9B 50 04      BVC L9EA1
9E9D          L9E9D:
9E9D A2 06      LDX #$6
9E9F D0 0A      BNE L9EAB
9EA1          L9EA1:
9EA1 AD D8 2B   LDA L2BD8
9EA4 29 C0      AND #$C0
9EA6 0A         ASL A
9EA7 2A         ROL A
9EA8 2A         ROL A
9EA9 2A         ROL A
9EAA AA         TAX
9EAB          L9EAB:
9EAB BD D8 9E   LDA L9ED8,X
9EAE 8D FE 2B   STA L2BFE
9EB1 BD D9 9E   LDA L9ED9,X
9EB4 8D FF 2B   STA L2BFF
9EB7          L9EB7:
9EB7 A6 80      LDX L80
9EB9 BD A8 2D   LDA L2DA8,X
9EBC 10 AD      BPL L9E6B
9EBE          L9EBE:
9EBE 20 96 A0   JSR LA096
9EC1 20 C7 9E   JSR L9EC7
9EC4 4C B7 9E   JMP L9EB7
9EC7          L9EC7:
9EC7 6C FC 2B   JMP (L2BFC)
9ECA          L9ECA:
9ECB          L9ECB = * + 1
9ECA F3 9E      .WORD L9EF3
9ECC 2B 9F      .WORD L9F2B
9ECE 2B 9F      .WORD L9F2B
9ED0 2B 9F      .WORD L9F2B
9ED2 A5 9F      .WORD L9FA5
9ED4 D6 9F      .WORD L9FD6
9ED6 A8 9F      .WORD L9FA8
9ED8          L9ED8:
9ED9          L9ED9 = * + 1
9ED8 B3 99      .WORD L99B3
9EDA 4A 98      .WORD L984A
9EDC F2 97      .WORD L97F2
9EDE 8C 95      .WORD L958C
9EE0          L9EE0:
9EE0 A5 82      LDA L82
9EE2 38         SEC
9EE3 E9 0F      SBC #$F
9EE5 F0 09      BEQ L9EF0
9EE7          L9EE7:
9EE7 20 AC DA   JSR LDAAC
9EEA C9 07      CMP #$7
9EEC D0 02      BNE L9EF0
9EEE          L9EEE:
9EEE A9 05      LDA #$5
9EF0          L9EF0:
9EF0 0A         ASL A
9EF1 AA         TAX
9EF2 60         RTS
9EF3          L9EF3:
9EF3 A5 DE      LDA LDE
9EF5 C9 FF      CMP #$FF
9EF7 D0 18      BNE L9F11
9EF9          L9EF9:
9EF9 A5 DF      LDA LDF
9EFB C9 22      CMP #$22
9EFD D0 12      BNE L9F11
9EFF          L9EFF:
9EFF A9 0D      LDA #$D
9F01 85 84      STA L84
9F03 20 42 EE   JSR LEE42
9F06 A9 00      LDA #$0
9F08 20 AD DF   JSR LDFAD
9F0B C6 DE      DEC LDE
9F0D A9 80      LDA #$80
9F0F D0 11      BNE L9F22
9F11          L9F11:
9F11 20 08 A0   JSR LA008
9F14 85 84      STA L84
9F16 D0 08      BNE L9F20
9F18          L9F18:
9F18 A9 FF      LDA #$FF
9F1A 85 DE      STA LDE
9F1C A9 22      LDA #$22
9F1E 85 DF      STA LDF
9F20          L9F20:
9F20 A9 88      LDA #$88
9F22          L9F22:
9F22 8D C7 2D   STA L2DC7
9F25 A5 84      LDA L84
9F27 8D E7 2D   STA L2DE7
9F2A 60         RTS
9F2B          L9F2B:
9F2B A4 80      LDY L80
9F2D B9 A8 2D   LDA L2DA8,Y
9F30 29 08      AND #$8
9F32 D0 04      BNE L9F38
9F34          L9F34:
9F34 99 A8 2D   STA L2DA8,Y
9F37 60         RTS
9F38          L9F38:
9F38 B9 68 2C   LDA L2C68,Y
9F3B 0A         ASL A
9F3C AA         TAX
9F3D A1 A0      LDA (LA0,X)
9F3F 48         PHA
9F40 B9 E8 2D   LDA L2DE8,Y
9F43 D5 A0      CMP LA0,X
9F45 D0 0B      BNE L9F52
9F47          L9F47:
9F47 A9 00      LDA #$0
9F49 95 A0      STA LA0,X
9F4B A9 80      LDA #$80
9F4D 99 A8 2D   STA L2DA8,Y
9F50 D0 07      BNE L9F59
9F52          L9F52:
9F52 F6 A0      INC LA0,X
9F54 D0 03      BNE L9F59
9F56          L9F56:
9F56 20 6E 9F   JSR L9F6E
9F59          L9F59:
9F59 68         PLA
9F5A 99 C8 2D   STA L2DC8,Y
9F5D 60         RTS
9F5E          L9F5E:
9F5E A4 80      LDY L80
9F60 B9 68 2C   LDA L2C68,Y
9F63 0A         ASL A
9F64 AA         TAX
9F65 A9 00      LDA #$0
9F67 95 A0      STA LA0,X
9F69 A1 A0      LDA (LA0,X)
9F6B D0 01      BNE L9F6E
9F6D          L9F6D:
9F6D 60         RTS
9F6E          L9F6E:
9F6E F6 A0      INC LA0,X
9F70 A1 A0      LDA (LA0,X)
9F72 9D 01 28   STA L2801,X
9F75 D6 A0      DEC LA0,X
9F77 A1 A0      LDA (LA0,X)
9F79 9D 00 28   STA L2800,X
9F7C 8A         TXA
9F7D 4A         LSR A
9F7E AA         TAX
9F7F A9 80      LDA #$80
9F81 20 1C E8   JSR LE81C
9F84 8A         TXA
9F85 0A         ASL A
9F86 AA         TAX
9F87 A1 A0      LDA (LA0,X)
9F89 85 5A      STA L5A
9F8B 08         PHP
9F8C F6 A0      INC LA0,X
9F8E A1 A0      LDA (LA0,X)
9F90 85 5B      STA L5B
9F92 F6 A0      INC LA0,X
9F94 28         PLP
9F95 D0 03      BNE L9F9A
9F97          L9F97:
9F97 99 E8 2D   STA L2DE8,Y
9F9A          L9F9A:
9F9A 98         TYA
9F9B AA         TAX
9F9C FE 48 2D   INC L2D48,X
9F9F D0 03      BNE L9FA4
9FA1          L9FA1:
9FA1 FE 68 2D   INC L2D68,X
9FA4          L9FA4:
9FA4 60         RTS
9FA5          L9FA5:
9FA5 4C F0 D2   JMP LD2F0
9FA8          L9FA8:
9FA8 A4 80      LDY L80
9FAA B9 A8 2D   LDA L2DA8,Y
9FAD 29 08      AND #$8
9FAF D0 04      BNE L9FB5
9FB1          L9FB1:
9FB1 99 A8 2D   STA L2DA8,Y
9FB4 60         RTS
9FB5          L9FB5:
9FB5 20 FE CE   JSR LCEFE
9FB8 48         PHA
9FB9 D0 16      BNE L9FD1
9FBB          L9FBB:
9FBB B9 E8 2D   LDA L2DE8,Y
9FBE F0 07      BEQ L9FC7
9FC0          L9FC0:
9FC0 A9 80      LDA #$80
9FC2 99 A8 2D   STA L2DA8,Y
9FC5 D0 0A      BNE L9FD1
9FC7          L9FC7:
9FC7 A9 00      LDA #$0
9FC9 8D B1 2B   STA L2BB1
9FCC 20 37 C5   JSR LC537
9FCF A4 80      LDY L80
9FD1          L9FD1:
9FD1 68         PLA
9FD2 99 C8 2D   STA L2DC8,Y
9FD5 60         RTS
9FD6          L9FD6:
9FD6 A4 80      LDY L80
9FD8 B9 A8 2D   LDA L2DA8,Y
9FDB 29 08      AND #$8
9FDD D0 05      BNE L9FE4
9FDF          L9FDF:
9FDF A9 89      LDA #$89
9FE1 99 A8 2D   STA L2DA8,Y
9FE4          L9FE4:
9FE4 B9 68 2C   LDA L2C68,Y
9FE7 0A         ASL A
9FE8 AA         TAX
9FE9 B5 A0      LDA LA0,X
9FEB DD E8 2D   CMP L2DE8,X
9FEE D0 04      BNE L9FF4
9FF0          L9FF0:
9FF0 A9 00      LDA #$0
9FF2 95 A0      STA LA0,X
9FF4          L9FF4:
9FF4 F6 A0      INC LA0,X
9FF6          L9FF6:
9FF6 A1 A0      LDA (LA0,X)
9FF8 99 C8 2D   STA L2DC8,Y
9FFB B5 A0      LDA LA0,X
9FFD D9 E8 2D   CMP L2DE8,Y
A000 D0 05      BNE LA007
A002          LA002:
A002 A9 81      LDA #$81
A004 99 A8 2D   STA L2DA8,Y
A007          LA007:
A007 60         RTS
A008          LA008:
A008 A4 80      LDY L80
A00A B9 68 2C   LDA L2C68,Y
A00D 0A         ASL A
A00E AA         TAX
A00F A1 A0      LDA (LA0,X)
A011 48         PHA
A012 B9 E8 2D   LDA L2DE8,Y
A015 D5 A0      CMP LA0,X
A017 D0 04      BNE LA01D
A019          LA019:
A019 A9 FF      LDA #$FF
A01B 95 A0      STA LA0,X
A01D          LA01D:
A01D 68         PLA
A01E F6 A0      INC LA0,X
A020          LA020:
A020 60         RTS
A021          LA021:
A021 78         SEI
A022 A5 83      LDA L83
A024 29 8F      AND #$8F
A026 C9 0F      CMP #$F
A028 B0 06      BCS LA030
A02A          LA02A:
A02A 20 92 DA   JSR LDA92
A02D 90 13      BCC LA042
A02F          LA02F:
A02F 60         RTS
A030          LA030:
A030 20 A9 F5   JSR LF5A9
A033 A9 1E      LDA #$1E
A035 85 80      STA L80
A037 A2 00      LDX #$0
A039 8A         TXA
A03A          LA03A:
A03A 9D 00 02   STA L200,X
A03D E8         INX
A03E D0 FA      BNE LA03A
A040          LA040:
A040 F0 0D      BEQ LA04F
A042          LA042:
A042 AD FB 2B   LDA L2BFB
A045 C9 60      CMP #$60
A047 D0 03      BNE LA04C
A049          LA049:
A049 4C B4 9B   JMP L9BB4
A04C          LA04C:
A04C 20 E0 9E   JSR L9EE0
A04F          LA04F:
A04F BD 99 A0   LDA LA099,X
A052 8D FC 2B   STA L2BFC
A055 BD 9A A0   LDA LA09A,X
A058 8D FD 2B   STA L2BFD
A05B 2C FB 2B   BIT L2BFB
A05E 50 04      BVC LA064
A060          LA060:
A060 A2 06      LDX #$6
A062 D0 0A      BNE LA06E
A064          LA064:
A064 AD D8 2B   LDA L2BD8
A067 29 C0      AND #$C0
A069 0A         ASL A
A06A 2A         ROL A
A06B 2A         ROL A
A06C 2A         ROL A
A06D AA         TAX
A06E          LA06E:
A06E BD A5 A0   LDA LA0A5,X
A071 8D FE 2B   STA L2BFE
A074 BD A6 A0   LDA LA0A6,X
A077 8D FF 2B   STA L2BFF
A07A          LA07A:
A07A A6 80      LDX L80
A07C BD A8 2D   LDA L2DA8,X
A07F 4A         LSR A
A080 B0 08      BCS LA08A
A082          LA082:
A082 A5 83      LDA L83
A084 29 F0      AND #$F0
A086 C9 F0      CMP #$F0
A088 D0 A5      BNE LA02F
A08A          LA08A:
A08A 20 96 A0   JSR LA096
A08D 20 93 A0   JSR LA093
A090 4C 7A A0   JMP LA07A
A093          LA093:
A093 6C FC 2B   JMP (L2BFC)
A096          LA096:
A096 6C FE 2B   JMP (L2BFE)
A099          LA099:
A09A          LA09A = * + 1
A099 AD A0      .WORD LA0AD
A09B C1 A0      .WORD LA0C1
A09D C1 A0      .WORD LA0C1
A09F C1 A0      .WORD LA0C1
A0A1 63 A1      .WORD LA163
A0A3 68 A1      .WORD LA168
A0A5          LA0A5:
A0A6          LA0A6 = * + 1
A0A5 1C 9A      .WORD L9A1C
A0A7 67 99      .WORD L9967
A0A9          LA0A9:
A0A9 2C         .BYTE $2C
A0AA          LA0AA:
A0AA 99 CA 95   STA L95CA,Y
A0AD          LA0AD:
A0AD A6 DC      LDX LDC
A0AF E0 FF      CPX #$FF
A0B1 F0 07      BEQ LA0BA
A0B3          LA0B3:
A0B3 A5 84      LDA L84
A0B5 9D 00 02   STA L200,X
A0B8 E6 DC      INC LDC
A0BA          LA0BA:
A0BA 24 81      BIT L81
A0BC 30 02      BMI LA0C0
A0BE          LA0BE:
A0BE E6 4B      INC L4B
A0C0          LA0C0:
A0C0 60         RTS
A0C1          LA0C1:
A0C1 A4 80      LDY L80
A0C3 B9 68 2C   LDA L2C68,Y
A0C6 0A         ASL A
A0C7 AA         TAX
A0C8 B5 A0      LDA LA0,X
A0CA D0 0A      BNE LA0D6
A0CC          LA0CC:
A0CC 20 DD A0   JSR LA0DD
A0CF A6 80      LDX L80
A0D1 BD 68 2C   LDA L2C68,X
A0D4 0A         ASL A
A0D5 AA         TAX
A0D6          LA0D6:
A0D6 A5 84      LDA L84
A0D8 81 A0      STA (LA0,X)
A0DA F6 A0      INC LA0,X
A0DC 60         RTS
A0DD          LA0DD:
A0DD 20 F3 A3   JSR LA3F3
A0E0 AE A1 2B   LDX L2BA1
A0E3 BD 70 2B   LDA L2B70,X
A0E6 F0 13      BEQ LA0FB
A0E8          LA0E8:
A0E8 AC E8 90   LDY L90E8
A0EB BE 00 82   LDX Partition_Typ+$00,Y
A0EE DD 79 AF   CMP LAF79,X
A0F1 F0 08      BEQ LA0FB
A0F3          LA0F3:
A0F3 20 0D D9   JSR LD90D
A0F6 A9 73      LDA #$73
A0F8 4C 33 FF   JMP LFF33
A0FB          LA0FB:
A0FB A4 80      LDY L80
A0FD B9 68 2C   LDA L2C68,Y
A100 8D 57 2A   STA L2A57
A103 0A         ASL A
A104 AA         TAX
A105 A5 5A      LDA L5A
A107 81 A0      STA (LA0,X)
A109 F6 A0      INC LA0,X
A10B A5 5B      LDA L5B
A10D 81 A0      STA (LA0,X)
A10F F6 A0      INC LA0,X
A111 08         PHP
A112 78         SEI
A113 20 C7 E9   JSR LE9C7
A116 B0 41      BCS LA159
A118          LA118:
A118 2C 5D 2A   BIT L2A5D
A11B 30 1E      BMI LA13B
A11D          LA11D:
A11D AD 57 2A   LDA L2A57
A120 0A         ASL A
A121 AA         TAX
A122 A5 5A      LDA L5A
A124 DD 00 28   CMP L2800,X
A127 D0 12      BNE LA13B
A129          LA129:
A129 A5 5B      LDA L5B
A12B E9 01      SBC #$1
A12D DD 01 28   CMP L2801,X
A130 D0 09      BNE LA13B
A132          LA132:
A132 20 AC EE   JSR LEEAC
A135 20 34 ED   JSR LED34
A138 4C 3E A1   JMP LA13E
A13B          LA13B:
A13B 20 28 ED   JSR LED28
A13E          LA13E:
A13E 28         PLP
A13F          LA13F:
A13F AD 57 2A   LDA L2A57
A142 0A         ASL A
A143 AA         TAX
A144 A5 5A      LDA L5A
A146 9D 00 28   STA L2800,X
A149 A5 5B      LDA L5B
A14B 9D 01 28   STA L2801,X
A14E A6 80      LDX L80
A150 FE 48 2D   INC L2D48,X
A153 D0 03      BNE LA158
A155          LA155:
A155 FE 68 2D   INC L2D68,X
A158          LA158:
A158 60         RTS
A159          LA159:
A159 A9 04      LDA #$4
A15B AE 57 2A   LDX L2A57
A15E 95 20      STA L20,X
A160 4C 36 FF   JMP LFF36
A163          LA163:
A163 4C 7B D2   JMP LD27B
A166 60 60      .BYTE $60,$60
A168          LA168:
A168 A5 84      LDA L84
A16A 20 70 A1   JSR LA170
A16D 4C F6 9F   JMP L9FF6
A170          LA170:
A170 48         PHA
A171 A4 80      LDY L80
A173 B9 68 2C   LDA L2C68,Y
A176 0A         ASL A
A177 AA         TAX
A178 68         PLA
A179 81 A0      STA (LA0,X)
A17B F6 A0      INC LA0,X
A17D 60         RTS
A17E          LA17E:
A17E A9 80      LDA #$80
A181          LA181 = * + 1
              ; Instruction parameter jumped to.
A180 2C A9 90   BIT L90A9
A183 48         PHA
A184 AD A8 2B   LDA L2BA8
A187          LA187:
A187 8D 3F 28   STA L283F
A18A AD A7 2B   LDA L2BA7
A18D          LA18D:
A18D 8D 3E 28   STA L283E
A190 A2 1F      LDX #$1F
A192 68         PLA
A193 4C 4B FF   JMP LFF4B
A196          LA196:
A196 A9 80      LDA #$80
A199          LA199 = * + 1
              ; Instruction parameter jumped to.
A198 2C A9 90   BIT L90A9
A19B 48         PHA
A19C AD A9 2B   LDA L2BA9
A19F 4C 87 A1   JMP LA187
A1A2          LA1A2:
A1A2 A9 80      LDA #$80
A1A5          LA1A5 = * + 1
              ; Instruction parameter jumped to.
A1A4 2C A9 90   BIT L90A9
A1A7 48         PHA
A1A8 A5 5B      LDA L5B
A1AA 8D 3F 28   STA L283F
A1AD A5 5A      LDA L5A
A1AF 4C 8D A1   JMP LA18D
A1B2          LA1B2:
A1B2 20 7E A1   JSR LA17E
A1B5 AD 24 22   LDA L2224
A1B8 8D 3E 28   STA L283E
A1BB AD 25 22   LDA L2225
A1BE 8D 3F 28   STA L283F
A1C1 AD 26 22   LDA L2226
A1C4 48         PHA
A1C5 A9 80      LDA #$80
A1C7 A2 1F      LDX #$1F
A1C9 20 4B FF   JSR LFF4B
A1CC 68         PLA
A1CD AA         TAX
A1CE 60         RTS
A1CF          LA1CF:
A1CF A9 90      LDA #$90
A1D1 A2 1F      LDX #$1F
A1D3 4C 4B FF   JMP LFF4B
A1D6          LA1D6:
A1D6 18         CLC
A1D8          LA1D8 = * + 1
              ; Instruction parameter jumped to.
A1D7 24 38      BIT L38
A1D9 6E A2 2B   ROR L2BA2
A1DC AE A1 2B   LDX L2BA1
A1DF A9 00      LDA #$0
A1E1 9D 40 2B   STA L2B40,X
A1E4 20 7E B0   JSR LB07E
A1E7 0A         ASL A
A1E8 AA         TAX
A1E9 BD F6 A1   LDA LA1F6,X
A1EC 8D DC 2B   STA L2BDC
A1EF BD F7 A1   LDA LA1F7,X
A1F2 8D DD 2B   STA L2BDD
A1F6          LA1F6 = * + 1
A1F7          LA1F7 = * + 2
A1F5 6C DC 2B   JMP (L2BDC)
A1F8 26 A2      .WORD LA226
A1FA 02 A2      .WORD LA202
A1FC 09 A2      .WORD LA209
A1FE 18 A2      .WORD LA218
A200 18 A2      .WORD LA218
A202          LA202:
A202 A9 12      LDA #$12
A204 A2 00      LDX #$0
A206 4C 41 A2   JMP LA241
A209          LA209:
A209 20 02 A2   JSR LA202
A20C A9 35      LDA #$35
A20E A2 00      LDX #$0
A210          LA210:
A210 E6 59      INC L59
A212 20 41 A2   JSR LA241
A215 C6 59      DEC L59
A217 60         RTS
A218          LA218:
A218 20 8E B0   JSR LB08E
A21B 48         PHA
A21C A2 01      LDX #$1
A21E 20 41 A2   JSR LA241
A221 68         PLA
A222 A2 02      LDX #$2
A224 D0 EA      BNE LA210
A226          LA226:
A226 AE A1 2B   LDX L2BA1
A229 BD 80 2B   LDA L2B80,X
A22C 0A         ASL A
A22D 18         CLC
A22E 69 02      ADC #$2
A230 29 FE      AND #$FE
A232 AA         TAX
A233 A9 01      LDA #$1
A235 20 41 A2   JSR LA241
A238 A9 01      LDA #$1
A23A AE 3D 28   LDX L283D
A23D E8         INX
A23E 4C 10 A2   JMP LA210
A241          LA241:
A241 8D 3C 28   STA L283C
A244 8E 3D 28   STX L283D
A247 A5 59      LDA L59
A249 8D 7E 28   STA L287E
A24C A9 00      LDA #$0
A24E 8D 9E 28   STA L289E
A251 A9 01      LDA #$1
A253 8D BE 28   STA L28BE
A256 A2 1E      LDX #$1E
A258 A9 CC      LDA #$CC
A25A 2C A2 2B   BIT L2BA2
A25D 10 02      BPL LA261
A25F          LA25F:
A25F A9 CE      LDA #$CE
A261          LA261:
A261 20 4B FF   JSR LFF4B
A264 AE A1 2B   LDX L2BA1
A267 60         RTS
A268          LA268:
A268 20 C7 A2   JSR LA2C7
A26B A5 5A      LDA L5A
A26D 4A         LSR A
A26E 4A         LSR A
A26F 4A         LSR A
A270 4A         LSR A
A271 DD 80 2B   CMP L2B80,X
A274 D0 01      BNE LA277
A276          LA276:
A276 60         RTS
A277          LA277:
A277 48         PHA
A278 BD 40 2B   LDA L2B40,X
A27B F0 03      BEQ LA280
A27D          LA27D:
A27D 20 D8 A1   JSR LA1D8
A280          LA280:
A280 68         PLA
A281 9D 80 2B   STA L2B80,X
A284 4C D6 A1   JMP LA1D6
A287          LA287:
A287 20 C7 A2   JSR LA2C7
A28A BD 80 2B   LDA L2B80,X
A28D 10 03      BPL LA292
A28F          LA28F:
A28F 20 AA A2   JSR LA2AA
A292          LA292:
A292 60         RTS
A293          LA293:
A293 20 C7 A2   JSR LA2C7
A296 BD 80 2B   LDA L2B80,X
A299 F0 0B      BEQ LA2A6
A29B          LA29B:
A29B BD 40 2B   LDA L2B40,X
A29E F0 03      BEQ LA2A3
A2A0          LA2A0:
              ; Instruction opcode accessed.
              ; Instruction opcode accessed.
A2A0 20 D8 A1   JSR LA1D8
A2A3          LA2A3:
A2A3 20 AA A2   JSR LA2AA
A2A6          LA2A6:
A2A6 60         RTS
A2A7          LA2A7:
A2A7 20 C7 A2   JSR LA2C7
A2AA          LA2AA:
A2AA A9 00      LDA #$0
A2AC 9D 80 2B   STA L2B80,X
A2AF 4C D6 A1   JMP LA1D6
A2B2          LA2B2:
A2B2 20 C7 A2   JSR LA2C7
A2B5 FE 80 2B   INC L2B80,X
A2B8 BD 80 2B   LDA L2B80,X
A2BB C9 10      CMP #$10
A2BD 90 05      BCC LA2C4
A2BF          LA2BF:
A2BF A9 00      LDA #$0
A2C1 9D 80 2B   STA L2B80,X
A2C4          LA2C4:
A2C4 4C D6 A1   JMP LA1D6
A2C7          LA2C7:
A2C7 AD E8 90   LDA L90E8
A2CA A2 0F      LDX #$F
A2CC          LA2CC:
A2CC 8E A1 2B   STX L2BA1
A2CF DD 30 2B   CMP L2B30,X
A2D2 F0 4D      BEQ LA321
A2D4          LA2D4:
A2D4 CA         DEX
A2D5 10 F5      BPL LA2CC
A2D7          LA2D7:
A2D7 48         PHA
A2D8 A2 00      LDX #$0
A2DA          LA2DA:
A2DA 8E A1 2B   STX L2BA1
A2DD BD 30 2B   LDA L2B30,X
A2E0 F0 1F      BEQ LA301
A2E2          LA2E2:
A2E2 E8         INX
A2E3 E0 10      CPX #$10
A2E5 90 F3      BCC LA2DA
A2E7          LA2E7:
A2E7 CA         DEX
A2E8          LA2E8:
A2E8 8E A1 2B   STX L2BA1
A2EB BD 30 2B   LDA L2B30,X
A2EE 8D FA 2B   STA L2BFA
A2F1 20 2D A3   JSR LA32D
A2F4 90 0B      BCC LA301
A2F6          LA2F6:
A2F6 AE A1 2B   LDX L2BA1
A2F9 CA         DEX
A2FA 10 EC      BPL LA2E8
A2FC          LA2FC:
A2FC A9 70      LDA #$70
A2FE 4C 33 FF   JMP LFF33
A301          LA301:
A301 AE A1 2B   LDX L2BA1
A304 68         PLA
A305 9D 30 2B   STA L2B30,X
A308 A9 00      LDA #$0
A30A 9D 40 2B   STA L2B40,X
A30D 9D 50 2B   STA L2B50,X
A310 9D 60 2B   STA L2B60,X
A313 9D 70 2B   STA L2B70,X
A316 9D C0 2F   STA L2FC0,X
A319 A9 FF      LDA #$FF
A31B 9D 80 2B   STA L2B80,X
A31E 9D 90 2B   STA L2B90,X
A321          LA321:
A321 8A         TXA
A322 0A         ASL A
A323 18         CLC
A324 69 60      ADC #$60
A326 85 59      STA L59
A328 A9 00      LDA #$0
A32A 85 58      STA L58
A32C 60         RTS
A32D          LA32D:
A32D A2 00      LDX #$0
A32F          LA32F:
A32F BD 48 2C   LDA L2C48,X
A332 C9 FF      CMP #$FF
A334 F0 0B      BEQ LA341
A336          LA336:
A336 29 1F      AND #$1F
A338 A8         TAY
A339 B9 C8 2C   LDA L2CC8,Y
A33C CD FA 2B   CMP L2BFA
A33F F0 06      BEQ LA347
A341          LA341:
A341 E8         INX
A342 E0 13      CPX #$13
A344 90 E9      BCC LA32F
A346          LA346:
A346 18         CLC
A347          LA347:
A347 60         RTS
A348          LA348:
A348 20 C7 A2   JSR LA2C7
A34B BD 40 2B   LDA L2B40,X
A34E F0 0B      BEQ LA35B
A350          LA350:
A350 4C D8 A1   JMP LA1D8
A353          LA353:
A353 20 C7 A2   JSR LA2C7
A356 BD 80 2B   LDA L2B80,X
A359 10 F5      BPL LA350
A35B          LA35B:
A35B 60         RTS
A35C          LA35C:
A35C 20 39 A5   JSR LA539
A35F F0 2F      BEQ LA390
A361          LA361:
A361 91 58      STA (L58),Y
A363 20 B4 A5   JSR LA5B4
A366 B0 05      BCS LA36D
A368          LA368:
A368 38         SEC
A369 E9 01      SBC #$1
A36B 91 58      STA (L58),Y
A36D          LA36D:
A36D 20 B1 A3   JSR LA3B1
A370 B0 0B      BCS LA37D
A372          LA372:
A372 BD 50 2B   LDA L2B50,X
A375 D0 03      BNE LA37A
A377          LA377:
A377 DE 60 2B   DEC L2B60,X
A37A          LA37A:
A37A DE 50 2B   DEC L2B50,X
A37D          LA37D:
A37D BD 60 2B   LDA L2B60,X
A380 D0 0C      BNE LA38E
A382          LA382:
A382 BD 50 2B   LDA L2B50,X
A385 C9 03      CMP #$3
A387 B0 05      BCS LA38E
A389          LA389:
A389 A9 72      LDA #$72
A38B 20 B5 DF   JSR LDFB5
A38E          LA38E:
A38E A9 01      LDA #$1
A390          LA390:
A390 60         RTS
A391          LA391:
A391 20 39 A5   JSR LA539
A394 D0 1A      BNE LA3B0
A396          LA396:
A396 91 58      STA (L58),Y
A398 20 B4 A5   JSR LA5B4
A39B B0 04      BCS LA3A1
A39D          LA39D:
A39D 69 01      ADC #$1
A39F 91 58      STA (L58),Y
A3A1          LA3A1:
A3A1 20 B1 A3   JSR LA3B1
A3A4 B0 08      BCS LA3AE
A3A6          LA3A6:
A3A6 FE 50 2B   INC L2B50,X
A3A9 D0 03      BNE LA3AE
A3AB          LA3AB:
A3AB FE 60 2B   INC L2B60,X
A3AE          LA3AE:
A3AE A9 01      LDA #$1
A3B0          LA3B0:
A3B0 60         RTS
A3B1          LA3B1:
A3B1 20 8E B0   JSR LB08E
A3B4 C5 5A      CMP L5A
A3B6 D0 15      BNE LA3CD
A3B8          LA3B8:
A3B8 BD 00 82   LDA Partition_Typ+$00,X
A3BB C9 01      CMP #$1
A3BD D0 0C      BNE LA3CB
A3BF          LA3BF:
A3BF A5 5A      LDA L5A
A3C1 C9 01      CMP #$1
A3C3 D0 08      BNE LA3CD
A3C5          LA3C5:
A3C5 A5 5B      LDA L5B
A3C7 C9 40      CMP #$40
A3C9 B0 02      BCS LA3CD
A3CB          LA3CB:
A3CB 38         SEC
A3CD          LA3CD = * + 1
              ; Instruction parameter jumped to.
A3CC 24 18      BIT L18
A3CE AE A1 2B   LDX L2BA1
A3D1 A9 01      LDA #$1
A3D3 9D 40 2B   STA L2B40,X
A3D6 60         RTS
A3D7          LA3D7:
A3D7 A6 5A      LDX L5A
A3D9 20 7F AF   JSR LAF7F
A3DC          LA3DC:
A3DC AD C9 2B   LDA L2BC9
A3DF F0 06      BEQ LA3E7
A3E1          LA3E1:
A3E1 C5 5B      CMP L5B
A3E3 90 0B      BCC LA3F0
A3E5          LA3E5:
A3E5 F0 09      BEQ LA3F0
A3E7          LA3E7:
A3E7 20 39 A5   JSR LA539
A3EA D0 06      BNE LA3F2
A3EC          LA3EC:
A3EC E6 5B      INC L5B
A3EE D0 EC      BNE LA3DC
A3F0          LA3F0:
A3F0 A9 00      LDA #$0
A3F2          LA3F2:
A3F2 60         RTS
A3F3          LA3F3:
A3F3 20 CF A4   JSR LA4CF
A3F6 D0 03      BNE LA3FB
A3F8          LA3F8:
A3F8 4C FF A4   JMP LA4FF
A3FB          LA3FB:
A3FB A9 03      LDA #$3
A3FE          LA3FE = * + 1
              ; Instruction parameter jumped to.
A3FD 2C A9 01   BIT L1A9
A400 8D A0 2B   STA L2BA0
A403          LA403:
A403 20 B4 A5   JSR LA5B4
A406 D0 2D      BNE LA435
A408          LA408:
A408 AE C6 2B   LDX L2BC6
A40B E4 5A      CPX L5A
A40D F0 21      BEQ LA430
A40F          LA40F:
A40F B0 13      BCS LA424
A411          LA411:
A411 E6 5A      INC L5A
A413 A5 5A      LDA L5A
A415 CD C8 2B   CMP L2BC8
A418 90 E9      BCC LA403
A41A          LA41A:
A41A CA         DEX
A41B          LA41B:
A41B 86 5A      STX L5A
A41D CE A0 2B   DEC L2BA0
A420 D0 E1      BNE LA403
A422          LA422:
A422 F0 0C      BEQ LA430
A424          LA424:
A424 C6 5A      DEC L5A
A426 A5 5A      LDA L5A
A428 CD C7 2B   CMP L2BC7
A42B B0 D6      BCS LA403
A42D          LA42D:
A42D E8         INX
A42E D0 EB      BNE LA41B
A430          LA430:
A430 A9 72      LDA #$72
A432 4C 6F B6   JMP LB66F
A435          LA435:
A435 A6 5A      LDX L5A
A437 20 7F AF   JSR LAF7F
A43A 20 6C A4   JSR LA46C
A43D 18         CLC
A43E 65 5B      ADC L5B
A440 85 5B      STA L5B
A442 A5 5B      LDA L5B
A444 CD C9 2B   CMP L2BC9
A447 90 05      BCC LA44E
A449          LA449:
A449 ED C9 2B   SBC L2BC9
A44C 85 5B      STA L5B
A44E          LA44E:
A44E 20 D7 A3   JSR LA3D7
A451 D0 09      BNE LA45C
A453          LA453:
A453 A9 00      LDA #$0
A455 85 5B      STA L5B
A457 20 D7 A3   JSR LA3D7
A45A F0 03      BEQ LA45F
A45C          LA45C:
A45C 4C 5C A3   JMP LA35C
A45F          LA45F:
A45F A9 71      LDA #$71
A461 4C 33 FF   JMP LFF33
A464          LA464:
A464 20 D2 A4   JSR LA4D2
A467 D0 95      BNE LA3FE
A469          LA469:
A469 4C DB A4   JMP LA4DB
A46C          LA46C:
A46C 20 7E B0   JSR LB07E
A46F C9 04      CMP #$4
A471 90 03      BCC LA476
A473          LA473:
A473 A9 01      LDA #$1
A475 60         RTS
A476          LA476:
A476 A9 01      LDA #$1
A478 A6 5A      LDX L5A
A47A E0 12      CPX #$12
A47C D0 02      BNE LA480
A47E          LA47E:
A47E A9 03      LDA #$3
A480          LA480:
A480 60         RTS
A481          LA481:
A481 20 D2 A4   JSR LA4D2
A484 D0 03      BNE LA489
A486          LA486:
A486 4C EC A4   JMP LA4EC
A489          LA489:
A489 A9 00      LDA #$0
A48B 8D A0 2B   STA L2BA0
A48E AD C6 2B   LDA L2BC6
A491 85 5A      STA L5A
A493          LA493:
A493 EE A0 2B   INC L2BA0
A496 A5 5A      LDA L5A
A498 CD C6 2B   CMP L2BC6
A49B 90 17      BCC LA4B4
A49D          LA49D:
A49D AD C6 2B   LDA L2BC6
A4A0 ED A0 2B   SBC L2BA0
A4A3 90 0F      BCC LA4B4
A4A5          LA4A5:
A4A5 85 5A      STA L5A
A4A7 CD C7 2B   CMP L2BC7
A4AA 90 08      BCC LA4B4
A4AC          LA4AC:
A4AC 20 B4 A5   JSR LA5B4
A4AF F0 03      BEQ LA4B4
A4B1          LA4B1:
A4B1 4C 53 A4   JMP LA453
A4B4          LA4B4:
A4B4 AD C6 2B   LDA L2BC6
A4B7 18         CLC
A4B8 6D A0 2B   ADC L2BA0
A4BB 85 5A      STA L5A
A4BD CD C8 2B   CMP L2BC8
A4C0 B0 08      BCS LA4CA
A4C2          LA4C2:
A4C2 20 B4 A5   JSR LA5B4
A4C5 F0 CC      BEQ LA493
A4C7          LA4C7:
A4C7 4C 53 A4   JMP LA453
A4CA          LA4CA:
A4CA A9 67      LDA #$67
A4CC 4C 33 FF   JMP LFF33
A4CF          LA4CF:
A4CF 20 89 D9   JSR LD989
A4D2          LA4D2:
A4D2 20 87 A2   JSR LA287
A4D5 20 7F AF   JSR LAF7F
A4D8 4C 85 B0   JMP LB085
A4DB          LA4DB:
A4DB A5 5A      LDA L5A
A4DD C9 01      CMP #$1
A4DF D0 1E      BNE LA4FF
A4E1          LA4E1:
A4E1 A5 5B      LDA L5B
A4E3 C9 40      CMP #$40
A4E5 B0 18      BCS LA4FF
A4E7          LA4E7:
A4E7 AD A7 2B   LDA L2BA7
A4EA D0 0C      BNE LA4F8
A4EC          LA4EC:
A4EC AD A7 2B   LDA L2BA7
A4EF C9 01      CMP #$1
A4F1 D0 05      BNE LA4F8
A4F3          LA4F3:
A4F3 CD A8 2B   CMP L2BA8
A4F6 F0 0E      BEQ LA506
A4F8          LA4F8:
A4F8 85 5A      STA L5A
A4FA AD A9 2B   LDA L2BA9
A4FD 85 5B      STA L5B
A4FF          LA4FF:
A4FF 20 19 A5   JSR LA519
A502 D0 12      BNE LA516
A504          LA504:
A504 A9 01      LDA #$1
A506          LA506:
A506 85 5A      STA L5A
A508 A9 40      LDA #$40
A50A 85 5B      STA L5B
A50C 20 19 A5   JSR LA519
A50F D0 05      BNE LA516
A511          LA511:
A511 A9 72      LDA #$72
A513 4C 6F B6   JMP LB66F
A516          LA516:
A516 4C 61 A3   JMP LA361
A519          LA519:
A519 20 44 A5   JSR LA544
A51C          LA51C:
A51C 20 50 A5   JSR LA550
A51F D0 17      BNE LA538
A521          LA521:
A521 E6 5B      INC L5B
A523 E8         INX
A524 E0 08      CPX #$8
A526 90 F4      BCC LA51C
A528          LA528:
A528 A2 00      LDX #$0
A52A C8         INY
A52B C0 20      CPY #$20
A52D 90 ED      BCC LA51C
A52F          LA52F:
A52F E6 5A      INC L5A
A531 A5 5A      LDA L5A
A533 CD C8 2B   CMP L2BC8
A536 D0 E1      BNE LA519
A538          LA538:
A538 60         RTS
A539          LA539:
A539 20 7E B0   JSR LB07E
A53C C9 04      CMP #$4
A53E B0 25      BCS LA565
A540          LA540:
A540 C9 01      CMP #$1
A542 D0 35      BNE LA579
A544          LA544:
A544 20 0B A6   JSR LA60B
A547 20 68 A2   JSR LA268
A54A 20 C5 A5   JSR LA5C5
A54D 20 A0 A5   JSR LA5A0
A550          LA550:
A550 B1 58      LDA (L58),Y
A552 3D 5D A5   AND LA55D,X
A555 08         PHP
A556 B1 58      LDA (L58),Y
A558 5D 5D A5   EOR LA55D,X
A55B 28         PLP
A55C 60         RTS
A55D          LA55D:
A55D 80 40 20   .BYTE $80,$40,$20
A560 10 08 04   .BYTE $10,$8,$4
A563 02         .BYTE $2
A564          LA564:
A565          LA565 = * + 1
              ; Instruction parameter jumped to.
A564 01 20      ORA (L20,X)
A566          LA566:
A568          LA568 = * + 2
              ; Instruction parameter jumped to.
A566 D9 A5 20   CMP L20A5,Y
A569          LA569:
A56A          LA56A = * + 1
              ; Instruction parameter jumped to.
A569 A0 A5      LDY #$A5
A56B          LA56B:
A56B C8         INY
A56C          LA56C:
A56C B1 58      LDA (L58),Y
A56E 3D AC A5   AND LA5AC,X
A571 08         PHP
A572 B1 58      LDA (L58),Y
A574 5D AC A5   EOR LA5AC,X
A577 28         PLP
A578 60         RTS
A579          LA579:
A579 20 0B A6   JSR LA60B
A57C A5 5A      LDA L5A
A57E C9 24      CMP #$24
A580 90 15      BCC LA597
A582          LA582:
A582 E6 59      INC L59
A584 A5 5A      LDA L5A
A586 38         SEC
A587 E9 24      SBC #$24
A589 85 58      STA L58
A58B 0A         ASL A
A58C 18         CLC
A58D 65 58      ADC L58
A58F 85 58      STA L58
A591 20 A0 A5   JSR LA5A0
A594 4C 6C A5   JMP LA56C
A597          LA597:
A597 A5 5A      LDA L5A
A599 0A         ASL A
A59A 0A         ASL A
A59B 85 58      STA L58
A59D 4C 68 A5   JMP LA568
A5A0          LA5A0:
A5A0 A5 5B      LDA L5B
A5A2 29 07      AND #$7
A5A4 AA         TAX
A5A5 A5 5B      LDA L5B
A5A7 4A         LSR A
A5A8 4A         LSR A
A5A9 4A         LSR A
A5AA A8         TAY
A5AB 60         RTS
A5AC          LA5AC:
A5AC 01 02 04   .BYTE $1,$2,$4
A5AF          LA5AF:
A5AF 08         PHP
A5B0 10 20      BPL LA5D2
A5B2          LA5B2:
A5B2 40         RTI
A5B3 80         .BYTE $80
A5B4          LA5B4:
A5B4 20 7E B0   JSR LB07E
A5B7 C9 04      CMP #$4
A5B9 B0 1E      BCS LA5D9
A5BB          LA5BB:
A5BB C9 01      CMP #$1
A5BD D0 38      BNE LA5F7
A5BF          LA5BF:
A5BF 20 0B A6   JSR LA60B
A5C2 20 68 A2   JSR LA268
A5C5          LA5C5:
A5C5 A5 5A      LDA L5A
A5C7 0A         ASL A
A5C8 0A         ASL A
A5C9 0A         ASL A
A5CA 0A         ASL A
A5CB 0A         ASL A
A5CC 90 02      BCC LA5D0
A5CE          LA5CE:
A5CE E6 59      INC L59
A5D0          LA5D0:
A5D0 18         CLC
A5D2          LA5D2 = * + 1
              ; Instruction parameter jumped to.
A5D1 65 58      ADC L58
A5D3 85 58      STA L58
A5D5 A0 00      LDY #$0
A5D7 38         SEC
A5D8 60         RTS
A5D9          LA5D9:
A5D9 20 0B A6   JSR LA60B
A5DC A5 5A      LDA L5A
A5DE C9 29      CMP #$29
A5E0 90 04      BCC LA5E6
A5E2          LA5E2:
A5E2 E6 59      INC L59
A5E4 E9 28      SBC #$28
A5E6          LA5E6:
A5E6 0A         ASL A
A5E7 85 58      STA L58
A5E9 0A         ASL A
A5EA 18         CLC
A5EB 65 58      ADC L58
A5ED 69 0A      ADC #$A
A5EF 85 58      STA L58
A5F1          LA5F1:
A5F1 A0 00      LDY #$0
A5F3 B1 58      LDA (L58),Y
A5F5 18         CLC
A5F6 60         RTS
A5F7          LA5F7:
A5F7 20 0B A6   JSR LA60B
A5FA A5 5A      LDA L5A
A5FC C9 24      CMP #$24
A5FE 90 04      BCC LA604
A600          LA600:
A600 69 B8      ADC #$B8
A602 D0 02      BNE LA606
A604          LA604:
A604 0A         ASL A
A605 0A         ASL A
A606          LA606:
A606 85 58      STA L58
A608 4C F1 A5   JMP LA5F1
A60B          LA60B:
A60B 20 C7 A2   JSR LA2C7
A60E BD 90 2B   LDA L2B90,X
A611 10 05      BPL LA618
A613          LA613:
A613 A9 74      LDA #$74
A615 4C 33 FF   JMP LFF33
A618          LA618:
A618 60         RTS
A619          LA619:
A619 20 C7 A2   JSR LA2C7
A61C A2 01      LDX #$1
A61E 20 7F AF   JSR LAF7F
A621 AE A1 2B   LDX L2BA1
A624 A9 00      LDA #$0
A626 9D 50 2B   STA L2B50,X
A629 9D 60 2B   STA L2B60,X
A62C 20 85 B0   JSR LB085
A62F F0 33      BEQ LA664
A631          LA631:
A631 A5 5A      LDA L5A
A633 48         PHA
A634 AE C7 2B   LDX L2BC7
A637 CA         DEX
A638 86 5A      STX L5A
A63A          LA63A:
A63A E6 5A      INC L5A
A63C A5 5A      LDA L5A
A63E CD C6 2B   CMP L2BC6
A641 F0 F7      BEQ LA63A
A643          LA643:
A643 CD C8 2B   CMP L2BC8
A646 B0 16      BCS LA65E
A648          LA648:
A648 20 B4 A5   JSR LA5B4
A64B B1 58      LDA (L58),Y
A64D 18         CLC
A64E AE A1 2B   LDX L2BA1
A651 7D 50 2B   ADC L2B50,X
A654 9D 50 2B   STA L2B50,X
A657 90 E1      BCC LA63A
A659          LA659:
A659 FE 60 2B   INC L2B60,X
A65C D0 DC      BNE LA63A
A65E          LA65E:
A65E 68         PLA
A65F 85 5A      STA L5A
A661 A2 00      LDX #$0
A663 60         RTS
A664          LA664:
A664 A5 5A      LDA L5A
A666 48         PHA
A667 20 93 A2   JSR LA293
A66A A9 01      LDA #$1
A66C 85 5A      STA L5A
A66E A9 20      LDA #$20
A670 85 58      STA L58
A672 A0 08      LDY #$8
A675          LA675 = * + 1
              ; Instruction parameter jumped to.
A674 2C A0 00   BIT LA0
A677 A9 00      LDA #$0
A679 8D A0 2B   STA L2BA0
A67C          LA67C:
A67C A2 08      LDX #$8
A67E B1 58      LDA (L58),Y
A680          LA680:
A680 0A         ASL A
A681 90 05      BCC LA688
A683          LA683:
A683 EE A0 2B   INC L2BA0
A686 F0 17      BEQ LA69F
A688          LA688:
A688 CA         DEX
A689 D0 F5      BNE LA680
A68B          LA68B:
A68B C8         INY
A68C C0 20      CPY #$20
A68E 90 EC      BCC LA67C
A690          LA690:
A690 AE A1 2B   LDX L2BA1
A693 BD 50 2B   LDA L2B50,X
A696 18         CLC
A697 6D A0 2B   ADC L2BA0
A69A 9D 50 2B   STA L2B50,X
A69D 90 06      BCC LA6A5
A69F          LA69F:
A69F AE A1 2B   LDX L2BA1
A6A2 FE 60 2B   INC L2B60,X
A6A5          LA6A5:
A6A5 E6 5A      INC L5A
A6A7 A5 5A      LDA L5A
A6A9 CD C8 2B   CMP L2BC8
A6AC F0 19      BEQ LA6C7
A6AE          LA6AE:
A6AE A5 58      LDA L58
A6B0 18         CLC
A6B1 69 20      ADC #$20
A6B3 85 58      STA L58
A6B5 D0 BE      BNE LA675
A6B7          LA6B7:
A6B7 E6 59      INC L59
A6B9 A5 59      LDA L59
A6BB 29 01      AND #$1
A6BD D0 B6      BNE LA675
A6BF          LA6BF:
A6BF 20 B2 A2   JSR LA2B2
A6C2 BD 80 2B   LDA L2B80,X
A6C5 D0 AE      BNE LA675
A6C7          LA6C7:
A6C7 68         PLA
A6C8 85 5A      STA L5A
A6CA A2 00      LDX #$0
A6CC 60         RTS
A6CD          LA6CD:
A6CD 20 E7 B6   JSR LB6E7
A6D0 20 33 B8   JSR LB833
A6D3 20 3C EE   JSR LEE3C
A6D6 20 7E B0   JSR LB07E
A6D9 F0 04      BEQ LA6DF
A6DB          LA6DB:
A6DB C9 06      CMP #$6
A6DD 90 05      BCC LA6E4
A6DF          LA6DF:
A6DF A9 77      LDA #$77
A6E1 4C 3B DF   JMP LDF3B
A6E4          LA6E4:
A6E4 20 C7 A2   JSR LA2C7
A6E7 A9 00      LDA #$0
A6E9 9D 90 2B   STA L2B90,X
A6EC 20 26 DB   JSR LDB26
A6EF AE 01 2C   LDX L2C01
A6F2 E4 56      CPX L56
A6F4 F0 18      BEQ LA70E
A6F6          LA6F6:
A6F6 BD 00 02   LDA L200,X
A6F9 8D A3 2B   STA L2BA3
A6FC BD 01 02   LDA L201,X
A6FF 8D A4 2B   STA L2BA4
A702 20 8E B0   JSR LB08E
A705 D0 14      BNE LA71B
A707          LA707:
A707 8A         TXA
A708 20 F4 AF   JSR LAFF4
A70B 4C 1B A7   JMP LA71B
A70E          LA70E:
A70E 20 03 AF   JSR LAF03
A711 20 8E B0   JSR LB08E
A714 D0 05      BNE LA71B
A716          LA716:
A716 A9 73      LDA #$73
A718 4C 6F B6   JMP LB66F
A71B          LA71B:
A71B A2 01      LDX #$1
A71D 20 7F AF   JSR LAF7F
A720 20 85 B0   JSR LB085
A723 D0 0D      BNE LA732
A725          LA725:
A725 A9 01      LDA #$1
A727 CD A7 2B   CMP L2BA7
A72A D0 05      BNE LA731
A72C          LA72C:
A72C CD A8 2B   CMP L2BA8
A72F F0 05      BEQ LA736
A731          LA731:
A731 60         RTS
A732          LA732:
A732 C9 04      CMP #$4
A734 90 06      BCC LA73C
A736          LA736:
A736 20 4B A7   JSR LA74B
A739 20 81 A1   JSR LA181
A73C          LA73C:
A73C 20 BF A7   JSR LA7BF
A73F 20 99 A1   JSR LA199
A742 20 E1 A7   JSR LA7E1
A745 20 48 A3   JSR LA348
A748 4C 03 AF   JMP LAF03
A74B          LA74B:
A74B 20 67 A7   JSR LA767
A74E 20 85 B0   JSR LB085
A751 D0 61      BNE LA7B4
A753          LA753:
A753 AD A7 2B   LDA L2BA7
A756 8D 20 22   STA L2220
A759 AD A8 2B   LDA L2BA8
A75C 8D 21 22   STA L2221
A75F A9 48      LDA #$48
A761 A2 31      LDX #$31
A763 A8         TAY
A764 4C AB A7   JMP LA7AB
A767          LA767:
A767 20 B5 A7   JSR LA7B5
A76A AD A7 2B   LDA L2BA7
A76D 8D 00 22   STA L2200
A770 AD A9 2B   LDA L2BA9
A773 8D 01 22   STA L2201
A776 A2 18      LDX #$18
A778 A9 A0      LDA #$A0
A77A          LA77A:
A77A 9D 04 22   STA L2204,X
A77D CA         DEX
A77E 10 FA      BPL LA77A
A780          LA780:
A780 AE 00 2C   LDX L2C00
A783 A0 00      LDY #$0
A785          LA785:
A785 BD 00 02   LDA L200,X
A788 C9 2C      CMP #$2C
A78A F0 0D      BEQ LA799
A78C          LA78C:
A78C 99 04 22   STA L2204,Y
A78F E8         INX
A790 E4 56      CPX L56
A792 B0 05      BCS LA799
A794          LA794:
A794 C8         INY
A795 C0 10      CPY #$10
A797 90 EC      BCC LA785
A799          LA799:
A799 AD A3 2B   LDA L2BA3
A79C 8D 16 22   STA L2216
A79F AD A4 2B   LDA L2BA4
A7A2 8D 17 22   STA L2217
A7A5 A9 44      LDA #$44
A7A7 A2 33      LDX #$33
A7A9 A0 44      LDY #$44
A7AB          LA7AB:
A7AB 8D 02 22   STA L2202
A7AE 8E 19 22   STX L2219
A7B1 8C 1A 22   STY L221A
A7B4          LA7B4:
A7B4 60         RTS
A7B5          LA7B5:
A7B5 A9 00      LDA #$0
A7B7 AA         TAX
A7B8          LA7B8:
A7B8 9D 00 22   STA L2200,X
A7BB E8         INX
A7BC D0 FA      BNE LA7B8
A7BE          LA7BE:
A7BE 60         RTS
A7BF          LA7BF:
A7BF 20 96 A1   JSR LA196
A7C2 A2 00      LDX #$0
A7C4          LA7C4:
A7C4 A9 00      LDA #$0
A7C6 9D 00 22   STA L2200,X
A7C9 9D 01 22   STA L2201,X
A7CC 9D 02 22   STA L2202,X
A7CF 8A         TXA
A7D0 18         CLC
A7D1 69 20      ADC #$20
A7D3 AA         TAX
A7D4 D0 EE      BNE LA7C4
A7D6          LA7D6:
A7D6 F0 03      BEQ LA7DB
A7D8          LA7D8:
A7D8 20 B5 A7   JSR LA7B5
A7DB          LA7DB:
A7DB A9 FF      LDA #$FF
A7DD 8D 01 22   STA L2201
A7E0 60         RTS
A7E1          LA7E1:
A7E1 20 C7 A2   JSR LA2C7
A7E4 20 A3 A9   JSR LA9A3
A7E7 AE A1 2B   LDX L2BA1
A7EA A9 01      LDA #$1
A7EC 9D 40 2B   STA L2B40,X
A7EF 20 7E B0   JSR LB07E
A7F2 0A         ASL A
A7F3 AA         TAX
A7F4 BD 01 A8   LDA LA801,X
A7F7 8D DC 2B   STA L2BDC
A7FA BD 02 A8   LDA LA802,X
A7FD 8D DD 2B   STA L2BDD
A801          LA801 = * + 1
A802          LA802 = * + 2
A800 6C DC 2B   JMP (L2BDC)
A803 0D A8      .BYTE $D,$A8
A805 BE A8      .WORD LA8BE
A807 17 A9      .WORD LA917
A809 5B A8      .WORD LA85B
A80B 5B         .BYTE $5B
A80C          LA80C:
A80C A8         TAY
A80D A0 02      LDY #$2
A80F A9 48      LDA #$48
A811 91 58      STA (L58),Y
A813 C8         INY
A814 49 FF      EOR #$FF
A816 91 58      STA (L58),Y
A818 C8         INY
A819 20 0A A9   JSR LA90A
A81C A9 C0      LDA #$C0
A81E 91 58      STA (L58),Y
A820 A0 08      LDY #$8
A822 AE C8 2B   LDX L2BC8
A825 CA         DEX
A826 8A         TXA
A827 91 58      STA (L58),Y
A829 A0 24      LDY #$24
A82B A9 1F      LDA #$1F
A82D 91 58      STA (L58),Y
A82F C8         INY
A830 A9 00      LDA #$0
A832 AE A1 2B   LDX L2BA1
A835 9D 80 2B   STA L2B80,X
A839          LA839 = * + 1
              ; Instruction parameter jumped to.
A838 2C A0 00   BIT LA0
A83B A9 FF      LDA #$FF
A83D 20 A6 A9   JSR LA9A6
A840 20 D8 A1   JSR LA1D8
A843 FE 80 2B   INC L2B80,X
A846 BD 80 2B   LDA L2B80,X
A849 C9 10      CMP #$10
A84B 90 EC      BCC LA839
A84D          LA84D:
A84D AD C8 2B   LDA L2BC8
A850 E9 02      SBC #$2
A852 9D 60 2B   STA L2B60,X
A855 A9 C0      LDA #$C0
A857 9D 50 2B   STA L2B50,X
A85A 60         RTS
A85B          LA85B:
A85B AD C7 2B   LDA L2BC7
A85E 85 5A      STA L5A
A860          LA860:
A860 20 D9 A5   JSR LA5D9
A863 A9 28      LDA #$28
A865 91 58      STA (L58),Y
A867 A9 FF      LDA #$FF
A869          LA869:
A869 C8         INY
A86A 91 58      STA (L58),Y
A86C C0 05      CPY #$5
A86E 90 F9      BCC LA869
A870          LA870:
A870 E6 5A      INC L5A
A872 A5 5A      LDA L5A
A874 CD C8 2B   CMP L2BC8
A877 90 E7      BCC LA860
A879          LA879:
A879 AD A7 2B   LDA L2BA7
A87C 85 5A      STA L5A
A87E 20 D9 A5   JSR LA5D9
A881 A9 24      LDA #$24
A883 91 58      STA (L58),Y
A885 C8         INY
A886 A9 F0      LDA #$F0
A888 91 58      STA (L58),Y
A88A 20 C7 A2   JSR LA2C7
A88D AD A7 2B   LDA L2BA7
A890 A2 02      LDX #$2
A892 20 A3 A8   JSR LA8A3
A895 E6 59      INC L59
A897 A9 00      LDA #$0
A899 A2 FF      LDX #$FF
A89B 20 A3 A8   JSR LA8A3
A89E C6 59      DEC L59
A8A0 4C 19 A6   JMP LA619
A8A3          LA8A3:
A8A3 A0 00      LDY #$0
A8A5 91 58      STA (L58),Y
A8A7 C8         INY
A8A8 8A         TXA
A8A9 91 58      STA (L58),Y
A8AB C8         INY
A8AC A9 44      LDA #$44
A8AE 91 58      STA (L58),Y
A8B0 C8         INY
A8B1 49 FF      EOR #$FF
A8B3 91 58      STA (L58),Y
A8B5 C8         INY
A8B6 20 0A A9   JSR LA90A
A8B9 A9 C0      LDA #$C0
A8BB 91 58      STA (L58),Y
A8BD 60         RTS
A8BE          LA8BE:
A8BE 20 C4 A8   JSR LA8C4
A8C1 4C 19 A6   JMP LA619
A8C4          LA8C4:
A8C4 A0 00      LDY #$0
A8C6 A2 00      LDX #$0
A8C8          LA8C8:
A8C8 BD 76 A9   LDA LA976,X
A8CB 8D A0 2B   STA L2BA0
A8CE          LA8CE:
A8CE BD 7F A9   LDA LA97F,X
A8D1 91 58      STA (L58),Y
A8D3 C8         INY
A8D4 BD 88 A9   LDA LA988,X
A8D7 91 58      STA (L58),Y
A8D9 C8         INY
A8DA BD 91 A9   LDA LA991,X
A8DD 91 58      STA (L58),Y
A8DF C8         INY
A8E0 BD 9A A9   LDA LA99A,X
A8E3 91 58      STA (L58),Y
A8E5 C8         INY
A8E6 CE A0 2B   DEC L2BA0
A8E9 D0 E3      BNE LA8CE
A8EB          LA8EB:
A8EB E8         INX
A8EC E0 09      CPX #$9
A8EE 90 D8      BCC LA8C8
A8F0          LA8F0:
A8F0 A0 90      LDY #$90
A8F2 AE 00 2C   LDX L2C00
A8F5          LA8F5:
A8F5 BD 00 02   LDA L200,X
A8F8 C9 2C      CMP #$2C
A8FA F0 0C      BEQ LA908
A8FC          LA8FC:
A8FC 91 58      STA (L58),Y
A8FE E8         INX
A8FF E4 56      CPX L56
A901 B0 05      BCS LA908
A903          LA903:
A903 C8         INY
A904 C0 A0      CPY #$A0
A906 90 ED      BCC LA8F5
A908          LA908:
A908 A0 A2      LDY #$A2
A90A          LA90A:
A90A AD A3 2B   LDA L2BA3
A90D 91 58      STA (L58),Y
A90F C8         INY
A910 AD A4 2B   LDA L2BA4
A913 91 58      STA (L58),Y
A915 C8         INY
A916 60         RTS
A917          LA917:
A917 20 C4 A8   JSR LA8C4
A91A A0 03      LDY #$3
A91C A9 80      LDA #$80
A91E 91 58      STA (L58),Y
A920 A2 01      LDX #$1
A922 A0 DD      LDY #$DD
A924          LA924:
A924 BD 76 A9   LDA LA976,X
A927 8D A0 2B   STA L2BA0
A92C          LA92C = * + 2
              ; Instruction parameter accessed.
A92A BD 7F A9   LDA LA97F,X
A92D          LA92D:
A92D 91 58      STA (L58),Y
A92F C8         INY
A930 CE A0 2B   DEC L2BA0
A933 D0 F8      BNE LA92D
A935          LA935:
A935 E8         INX
A936 E0 06      CPX #$6
A938 90 EA      BCC LA924
A93A          LA93A:
A93A A0 EE      LDY #$EE
A93C A9 00      LDA #$0
A93E 91 58      STA (L58),Y
A940 E6 59      INC L59
A942 A2 01      LDX #$1
A944 A0 00      LDY #$0
A946          LA946:
A946 BD 76 A9   LDA LA976,X
A949 8D A0 2B   STA L2BA0
A94C          LA94C:
A94C BD 88 A9   LDA LA988,X
A94F 91 58      STA (L58),Y
A951 C8         INY
A952 BD 91 A9   LDA LA991,X
A955 91 58      STA (L58),Y
A957 C8         INY
A958 BD 9A A9   LDA LA99A,X
A95B 91 58      STA (L58),Y
A95D C8         INY
A95E CE A0 2B   DEC L2BA0
A961 D0 E9      BNE LA94C
A963          LA963:
A963 E8         INX
A964 E0 06      CPX #$6
A966 90 DE      BCC LA946
A968          LA968:
A968 A0 33      LDY #$33
A96A A9 00      LDA #$0
A96C          LA96C:
A96C 91 58      STA (L58),Y
A96E C8         INY
A96F C0 36      CPY #$36
A971 90 F9      BCC LA96C
A973          LA973:
A973 4C 19 A6   JMP LA619
A976          LA976:
A976 01 11 01   .BYTE $1,$11,$1
A979 06 06 05   .BYTE $6,$6,$5
A97C 05 01 01   .BYTE $5,$1,$1
A97F          LA97F:
A97F 12 15 11   .BYTE $12,$15,$11
A982 13 12 11   .BYTE $13,$12,$11
A985 A0 A0 A0   .BYTE $A0,$A0,$A0
A988          LA988:
A988 01 FF FC   .BYTE $1,$FF,$FC
A98B FF FF FF   .BYTE $FF,$FF,$FF
A98E A0 32 A0   .BYTE $A0,$32,$A0
A991          LA991:
A991 41 FF FF   .BYTE $41,$FF,$FF
A994 FF FF FF   .BYTE $FF,$FF,$FF
A997 A0 41 A0   .BYTE $A0,$41,$A0
A99A          LA99A:
A99A 00 1F 07   .BYTE $0,$1F,$7
A99D 07 03      .BYTE $7,$3
A99F          LA99F:
A99F 01 A0      ORA (LA0,X)
A9A1 A0 00      LDY #$0
A9A3          LA9A3:
A9A3 A9 00      LDA #$0
A9A5 A8         TAY
A9A6          LA9A6:
A9A6 91 58      STA (L58),Y
A9A8 C8         INY
A9A9 D0 FB      BNE LA9A6
A9AB          LA9AB:
A9AB E6 59      INC L59
A9AD          LA9AD:
A9AD 91 58      STA (L58),Y
A9AF C8         INY
A9B0 D0 FB      BNE LA9AD
A9B2          LA9B2:
A9B2 C6 59      DEC L59
A9B4 60         RTS
A9B5          LA9B5:
A9B5 A0 00      LDY #$0
A9B7 A2 00      LDX #$0
A9B9 A9 2D      LDA #$2D
A9BB 20 61 B7   JSR LB761
A9BE D0 06      BNE LA9C6
A9C0          LA9C0:
A9C0 4C 97 DF   JMP LDF97
A9C3          LA9C3:
A9C3 4C 94 DF   JMP LDF94
A9C6          LA9C6:
A9C6 8A         TXA
A9C7 D0 FA      BNE LA9C3
A9C9          LA9C9:
A9C9 A2 07      LDX #$7
A9CB B9 00 02   LDA L200,Y
A9CE          LA9CE:
A9CE DD 09 AC   CMP LAC09,X
A9D1 F0 05      BEQ LA9D8
A9D3          LA9D3:
A9D3 CA         DEX
A9D4 10 F8      BPL LA9CE
A9D6          LA9D6:
A9D6 30 E8      BMI LA9C0
A9D8          LA9D8:
A9D8 8A         TXA
A9D9 09 80      ORA #$80
A9DB 8D E2 2B   STA L2BE2
A9DE 20 F3 A9   JSR LA9F3
A9E1 AD E2 2B   LDA L2BE2
A9E4 0A         ASL A
A9E5 AA         TAX
A9E6 BD 12 AC   LDA LAC12,X
A9E9 85 51      STA L51
A9ED          LA9ED = * + 2
              ; Instruction parameter accessed.
A9EB BD 11 AC   LDA LAC11,X
A9EE 85 50      STA L50
A9F0          LA9F0:
A9F0 6C 50 00   JMP (L50)
A9F3          LA9F3:
A9F3 A0 00      LDY #$0
A9F5 A2 00      LDX #$0
A9F7 A9 3A      LDA #$3A
A9F9 20 61 B7   JSR LB761
A9FC D0 02      BNE LAA00
A9FE          LA9FE:
A9FE A0 03      LDY #$3
AA00          LAA00:
AA00 B9 00 02   LDA L200,Y
AA03 C9 20      CMP #$20
AA05 F0 08      BEQ LAA0F
AA07          LAA07:
AA07 C9 1D      CMP #$1D
AA09 F0 04      BEQ LAA0F
AA0B          LAA0B:
AA0B C9 2C      CMP #$2C
AA0D D0 06      BNE LAA15
AA0F          LAA0F:
AA0F C8         INY
AA10 C4 56      CPY L56
AA12 90 EC      BCC LAA00
AA14          LAA14:
AA14 60         RTS
AA15          LAA15:
AA15 20 24 AA   JSR LAA24
AA18 EE EA 2B   INC L2BEA
AA1B AC EC 2B   LDY L2BEC
AA1E E0 04      CPX #$4
AA20 90 ED      BCC LAA0F
AA22          LAA22:
AA22 B0 9F      BCS LA9C3
AA24          LAA24:
AA24 A9 00      LDA #$0
AA26 85 50      STA L50
AA28 85 51      STA L51
AA2A 85 53      STA L53
AA2C A2 FF      LDX #$FF
AA2E          LAA2E:
AA2E B9 00 02   LDA L200,Y
AA31 C9 40      CMP #$40
AA33 B0 17      BCS LAA4C
AA35          LAA35:
AA35 C9 30      CMP #$30
AA37 90 13      BCC LAA4C
AA39          LAA39:
AA39 29 0F      AND #$F
AA3B 48         PHA
AA3C A5 51      LDA L51
AA3E 85 52      STA L52
AA40 A5 50      LDA L50
AA42 85 51      STA L51
AA44 68         PLA
AA45 85 50      STA L50
AA47 C8         INY
AA48 C4 56      CPY L56
AA4A 90 E2      BCC LAA2E
AA4C          LAA4C:
AA4C 8C EC 2B   STY L2BEC
AA4F 18         CLC
AA50 A9 00      LDA #$0
AA52          LAA52:
AA52 E8         INX
AA53 E0 03      CPX #$3
AA55 B0 0F      BCS LAA66
AA57          LAA57:
AA57 B4 50      LDY L50,X
AA59          LAA59:
AA59 88         DEY
AA5A 30 F6      BMI LAA52
AA5C          LAA5C:
AA5C 7D 74 AA   ADC LAA74,X
AA5F 90 F8      BCC LAA59
AA61          LAA61:
AA61 18         CLC
AA62 E6 53      INC L53
AA64 D0 F3      BNE LAA59
AA66          LAA66:
AA66 48         PHA
AA67 AE EA 2B   LDX L2BEA
AA6A A5 53      LDA L53
AA6C 9D 20 2C   STA L2C20,X
AA6F 68         PLA
AA70 9D 28 2C   STA L2C28,X
AA73 60         RTS
AA74          LAA74:
AA74 01 0A 64   .BYTE $1,$A,$64
AA77          LAA77:
AA77 20 E7 AB   JSR LABE7
AA7A 20 D0 AE   JSR LAED0
AA7D 20 91 A3   JSR LA391
AA80 4C 54 B6   JMP LB654
AA83          LAA83:
AA83 20 E7 AB   JSR LABE7
AA86 20 D0 AE   JSR LAED0
AA89 A5 5B      LDA L5B
AA8B 48         PHA
AA8C 20 D7 A3   JSR LA3D7
AA8F F0 0B      BEQ LAA9C
AA91          LAA91:
AA91 68         PLA
AA92 C5 5B      CMP L5B
AA94 D0 1F      BNE LAAB5
AA96          LAA96:
AA96 20 5C A3   JSR LA35C
AA99 4C 54 B6   JMP LB654
AA9C          LAA9C:
AA9C 68         PLA
AA9D          LAA9D:
AA9D A9 00      LDA #$0
AA9F 85 5B      STA L5B
AAA1 E6 5A      INC L5A
AAA3 F0 15      BEQ LAABA
AAA5          LAAA5:
AAA5 AD C8 2B   LDA L2BC8
AAA8 F0 06      BEQ LAAB0
AAAA          LAAAA:
AAAA C5 5A      CMP L5A
AAAC 90 0C      BCC LAABA
AAAE          LAAAE:
AAAE F0 0A      BEQ LAABA
AAB0          LAAB0:
AAB0 20 D7 A3   JSR LA3D7
AAB3 F0 E8      BEQ LAA9D
AAB5          LAAB5:
AAB5 A9 65      LDA #$65
AAB7 20 33 FF   JSR LFF33
AABA          LAABA:
AABA A9 65      LDA #$65
AABC 20 6F B6   JSR LB66F
AABF          LAABF:
AABF 20 E3 AB   JSR LABE3
AAC2 4C AA D8   JMP LD8AA
AAC5          LAAC5:
AAC5 20 B7 DA   JSR LDAB7
AAC8 A1 A0      LDA (LA0,X)
AACA 60         RTS
AACB          LAACB:
AACB 20 BF AA   JSR LAABF
AACE A9 00      LDA #$0
AAD0 20 C6 DC   JSR LDCC6
AAD3 20 C5 AA   JSR LAAC5
AAD6 99 E8 2D   STA L2DE8,Y
AAD9 A9 89      LDA #$89
AADB 99 A8 2D   STA L2DA8,Y
AADE 60         RTS
AADF          LAADF:
AADF 20 CB AA   JSR LAACB
AAE2 20 F4 9F   JSR L9FF4
AAE5 4C 54 B6   JMP LB654
AAE8          LAAE8:
AAE8 48         PHA
AAE9 48         PHA
AAEA 4C F0 AA   JMP LAAF0
AAED          LAAED:
AAED 20 F3 A9   JSR LA9F3
AAF0          LAAF0:
AAF0 20 CB AA   JSR LAACB
AAF3 B9 E8 2D   LDA L2DE8,Y
AAF6 99 C8 2D   STA L2DC8,Y
AAF9 A9 FF      LDA #$FF
AAFB 99 E8 2D   STA L2DE8,Y
AAFE 68         PLA
AAFF 68         PLA
AB00 4C 54 B6   JMP LB654
AB03          LAB03:
AB03 20 E3 AB   JSR LABE3
AB06 20 D4 DC   JSR LDCD4
AB09 A8         TAY
AB0A 88         DEY
AB0B C9 02      CMP #$2
AB0D B0 02      BCS LAB11
AB0F          LAB0F:
AB0F A0 01      LDY #$1
AB11          LAB11:
AB11 A9 00      LDA #$0
AB13 20 C6 DC   JSR LDCC6
AB16 98         TYA
AB17 20 EA CE   JSR LCEEA
AB1A 8A         TXA
AB1B 48         PHA
AB1C 20 39 AB   JSR LAB39
AB1F 68         PLA
AB20 AA         TAX
AB21 A4 80      LDY L80
AB23 4C C2 AB   JMP LABC2
AB26          LAB26:
AB26 48         PHA
AB27 48         PHA
AB28 4C 2E AB   JMP LAB2E
AB2B          LAB2B:
AB2B 20 F3 A9   JSR LA9F3
AB2E          LAB2E:
AB2E 20 E3 AB   JSR LABE3
AB31 20 39 AB   JSR LAB39
AB34 68         PLA
AB35 68         PLA
AB36 4C 54 B6   JMP LB654
AB39          LAB39:
AB39 20 AD D8   JSR LD8AD
AB3C 20 C7 A2   JSR LA2C7
AB3F A9 00      LDA #$0
AB41 20 C6 DC   JSR LDCC6
AB44 20 85 B0   JSR LB085
AB47 A6 5A      LDX L5A
AB49 A4 5B      LDY L5B
AB4B C9 06      CMP #$6
AB4D B0 28      BCS LAB77
AB4F          LAB4F:
AB4F C9 04      CMP #$4
AB51 B0 25      BCS LAB78
AB53          LAB53:
AB53 C9 02      CMP #$2
AB55 F0 34      BEQ LAB8B
AB57          LAB57:
AB57 B0 2A      BCS LAB83
AB59          LAB59:
AB59 E0 01      CPX #$1
AB5B D0 1A      BNE LAB77
AB5D          LAB5D:
AB5D C0 02      CPY #$2
AB5F 90 16      BCC LAB77
AB61          LAB61:
AB61 C0 22      CPY #$22
AB63 B0 12      BCS LAB77
AB65          LAB65:
AB65 88         DEY
AB66 88         DEY
AB67 98         TYA
AB68 4A         LSR A
AB69 AE A1 2B   LDX L2BA1
AB6C DD 80 2B   CMP L2B80,X
AB6F D0 06      BNE LAB77
AB71          LAB71:
AB71 98         TYA
AB72 4A         LSR A
AB73 90 20      BCC LAB95
AB75          LAB75:
AB75 B0 1C      BCS LAB93
AB77          LAB77:
AB77 60         RTS
AB78          LAB78:
AB78 E0 28      CPX #$28
AB7A D0 06      BNE LAB82
AB7C          LAB7C:
AB7C 88         DEY
AB7D F0 16      BEQ LAB95
AB7F          LAB7F:
AB7F 88         DEY
AB80 F0 11      BEQ LAB93
AB82          LAB82:
AB82 60         RTS
AB83          LAB83:
AB83 E0 35      CPX #$35
AB85 D0 04      BNE LAB8B
AB87          LAB87:
AB87 98         TYA
AB88 F0 09      BEQ LAB93
AB8A          LAB8A:
AB8A 60         RTS
AB8B          LAB8B:
AB8B E0 12      CPX #$12
AB8D D0 03      BNE LAB92
AB8F          LAB8F:
AB8F 98         TYA
AB90 F0 03      BEQ LAB95
AB92          LAB92:
AB92 60         RTS
AB93          LAB93:
AB93 E6 59      INC L59
AB95          LAB95:
AB95 A0 00      LDY #$0
AB97          LAB97:
AB97 B1 94      LDA (L94),Y
AB99 91 58      STA (L58),Y
AB9B C8         INY
AB9C D0 F9      BNE LAB97
AB9E          LAB9E:
AB9E 60         RTS
AB9F          LAB9F:
AB9F 20 BF AA   JSR LAABF
ABA2 A9 00      LDA #$0
ABA4 85 50      STA L50
ABA6 A5 9C      LDA L9C
ABA8 18         CLC
ABA9 69 03      ADC #$3
ABAB 85 51      STA L51
ABAD 20 F0 A9   JSR LA9F0
ABB0 4C 54 B6   JMP LB654
ABB3          LABB3:
ABB3 20 C8 AB   JSR LABC8
ABB6 A5 9C      LDA L9C
ABB8 0A         ASL A
ABB9 AA         TAX
ABBA AD 29 2C   LDA L2C29
ABBD 95 A0      STA LA0,X
ABBF 20 B7 DA   JSR LDAB7
ABC2          LABC2:
ABC2 20 F6 9F   JSR L9FF6
ABC5 4C 54 B6   JMP LB654
ABC8          LABC8:
ABC8 AD 28 2C   LDA L2C28
ABCB C9 0F      CMP #$F
ABCD 90 05      BCC LABD4
ABCF          LABCF:
ABCF A9 70      LDA #$70
ABD1 4C 6F B6   JMP LB66F
ABD4          LABD4:
ABD4 85 82      STA L82
ABD6 20 60 DA   JSR LDA60
ABD9 B0 F4      BCS LABCF
ABDB          LABDB:
ABDB 20 F2 DC   JSR LDCF2
ABDE 85 9C      STA L9C
ABE0 A2 01      LDX #$1
ABE2          LABE2:
ABE2 60         RTS
ABE3          LABE3:
ABE3 20 C8 AB   JSR LABC8
ABE7          LABE7 = * + 1
              ; Instruction parameter jumped to.
ABE6 2C A2 00   BIT LA2
ABE9 BD 29 2C   LDA L2C29,X
ABEC 85 5A      STA L5A
ABEE BD 2A 2C   LDA L2C2A,X
ABF1 85 5B      STA L5B
ABF3 BD 28 2C   LDA L2C28,X
ABF6 D0 0C      BNE LAC04
ABF8          LABF8:
ABF8 AD E8 90   LDA L90E8
ABFB 20 93 B6   JSR LB693
ABFE 20 1C D9   JSR LD91C
AC01 4C 3C EE   JMP LEE3C
AC04          LAC04:
AC04 A9 74      LDA #$74
AC06 4C 6F B6   JMP LB66F
AC09          LAC09:
AC09 41 46 52   .BYTE $41,$46,$52
AC0C 57 45 50   .BYTE $57,$45,$50
AC0F D2 D7      .BYTE $D2,$D7
AC11          LAC11:
AC12          LAC12 = * + 1
AC11 83 AA      .WORD LAA83
AC13 77 AA      .WORD LAA77
AC15 DF AA      .WORD LAADF
AC17 03 AB      .WORD LAB03
AC19 9F AB      .WORD LAB9F
AC1B B3 AB      .WORD LABB3
AC1D          LAC1D:
AC1D E8         INX
AC1E AA         TAX
AC1F 26 AB      ROL LAB
AC21          LAC21:
AC21 20 DE B6   JSR LB6DE
AC24 D0 03      BNE LAC29
AC26          LAC26:
AC26 4C 14 B1   JMP LB114
AC29          LAC29:
AC29 20 F1 B6   JSR LB6F1
AC2C 20 3D B8   JSR LB83D
AC2F AD E3 2B   LDA L2BE3
AC32 29 55      AND #$55
AC34 D0 0D      BNE LAC43
AC36          LAC36:
AC36 AE 00 2C   LDX L2C00
AC39 BD 00 02   LDA L200,X
AC3C C9 2A      CMP #$2A
AC3E D0 03      BNE LAC43
AC40          LAC40:
AC40 4C 94 DF   JMP LDF94
AC43          LAC43:
AC43 AD E3 2B   LDA L2BE3
AC46 29 D9      AND #$D9
AC48 D0 F6      BNE LAC40
AC4A          LAC4A:
AC4A 20 95 BE   JSR LBE95
AC4D 20 71 AD   JSR LAD71
AC50 AD EB 2B   LDA L2BEB
AC53 C9 03      CMP #$3
AC55 90 53      BCC LACAA
AC57          LAC57:
AC57 AD 10 2C   LDA L2C10
AC5A CD 11 2C   CMP L2C11
AC5D D0 4B      BNE LACAA
AC5F          LAC5F:
AC5F AD 40 2C   LDA L2C40
AC62 CD 41 2C   CMP L2C41
AC65 D0 43      BNE LACAA
AC67          LAC67:
AC67 AD 38 2C   LDA L2C38
AC6A CD 39 2C   CMP L2C39
AC6D D0 3B      BNE LACAA
AC6F          LAC6F:
AC6F AD 30 2C   LDA L2C30
AC72 CD 31 2C   CMP L2C31
AC75 D0 33      BNE LACAA
AC77          LAC77:
AC77 20 CE B1   JSR LB1CE
AC7A A9 01      LDA #$1
AC7C 8D EC 2B   STA L2BEC
AC7F 20 03 AD   JSR LAD03
AC82 20 AC DA   JSR LDAAC
AC85 B0 04      BCS LAC8B
AC87          LAC87:
AC87 C9 02      CMP #$2
AC89 D0 05      BNE LAC90
AC8B          LAC8B:
AC8B A9 64      LDA #$64
AC8D 20 6F B6   JSR LB66F
AC90          LAC90:
AC90 A9 12      LDA #$12
AC92 85 82      STA L82
AC94 AD 59 2C   LDA L2C59
AC97 8D 5A 2C   STA L2C5A
AC9A A9 FF      LDA #$FF
AC9C 8D 59 2C   STA L2C59
AC9F 20 29 C9   JSR LC929
ACA2 A2 02      LDX #$2
ACA4 20 C2 AC   JSR LACC2
ACA7 4C 54 B6   JMP LB654
ACAA          LACAA:
ACAA 20 B0 AC   JSR LACB0
ACAD 4C 54 B6   JMP LB654
ACB0          LACB0:
ACB0 20 EA B1   JSR LB1EA
ACB3 AD 10 2C   LDA L2C10
ACB6 20 23 B0   JSR LB023
ACB9 20 89 C3   JSR LC389
ACBC 20 BD C3   JSR LC3BD
ACBF AE EA 2B   LDX L2BEA
ACC2          LACC2:
ACC2 8E EC 2B   STX L2BEC
ACC5 20 03 AD   JSR LAD03
ACC8 A9 11      LDA #$11
ACCA 85 82      STA L82
ACCC 20 60 DA   JSR LDA60
ACCF 20 AC DA   JSR LDAAC
ACD2 D0 03      BNE LACD7
ACD4          LACD4:
ACD4 20 41 AD   JSR LAD41
ACD7          LACD7:
ACD7 A9 08      LDA #$8
ACD9 85 81      STA L81
ACDB 4C E1 AC   JMP LACE1
ACDE          LACDE:
ACDE 20 BD CE   JSR LCEBD
ACE1          LACE1:
ACE1 20 84 CE   JSR LCE84
ACE4 A9 80      LDA #$80
ACE6 20 FD D9   JSR LD9FD
ACE9 F0 F3      BEQ LACDE
ACEB          LACEB:
ACEB 20 AC DA   JSR LDAAC
ACEE F0 03      BEQ LACF3
ACF0          LACF0:
ACF0 20 BD CE   JSR LCEBD
ACF3          LACF3:
ACF3 AE EC 2B   LDX L2BEC
ACF6 E8         INX
ACF7 EC EB 2B   CPX L2BEB
ACFA 90 C6      BCC LACC2
ACFC          LACFC:
ACFC A9 12      LDA #$12
ACFE 85 82      STA L82
AD00 4C 1C CD   JMP LCD1C
AD03          LAD03:
AD03 AE EC 2B   LDX L2BEC
AD06 BD 30 2C   LDA L2C30,X
AD09 85 5A      STA L5A
AD0B BD 38 2C   LDA L2C38,X
AD0E 85 5B      STA L5B
AD10 BD 10 2C   LDA L2C10,X
AD13 20 23 B0   JSR LB023
AD16 20 78 C3   JSR LC378
AD19 AE EC 2B   LDX L2BEC
AD1C BD 40 2C   LDA L2C40,X
AD1F 20 C6 DC   JSR LDCC6
AD22 AE EC 2B   LDX L2BEC
AD25 BD 18 2C   LDA L2C18,X
AD28 29 07      AND #$7
AD2A 8D ED 2B   STA L2BED
AD2D A9 00      LDA #$0
AD2F 8D F3 2B   STA L2BF3
AD32 20 94 C8   JSR LC894
AD35 A0 01      LDY #$1
AD37 20 AC DA   JSR LDAAC
AD3A F0 01      BEQ LAD3D
AD3C          LAD3C:
AD3C C8         INY
AD3D          LAD3D:
AD3D 98         TYA
AD3E 4C C6 DC   JMP LDCC6
AD41          LAD41:
AD41 20 A6 D3   JSR LD3A6
AD44 20 BE D7   JSR LD7BE
AD47 D0 04      BNE LAD4D
AD49          LAD49:
AD49 AD F6 2B   LDA L2BF6
AD4C 48         PHA
AD4D          LAD4D:
AD4D A5 9A      LDA L9A
AD4F 48         PHA
AD50 A5 99      LDA L99
AD52 48         PHA
AD53 A9 12      LDA #$12
AD55 85 82      STA L82
AD57 20 92 DA   JSR LDA92
AD5A 20 87 D6   JSR LD687
AD5D 85 9B      STA L9B
AD5F 68         PLA
AD60 85 99      STA L99
AD62 68         PLA
AD63 85 9A      STA L9A
AD65 20 BE D7   JSR LD7BE
AD68 D0 04      BNE LAD6E
AD6A          LAD6A:
AD6A 68         PLA
AD6B 8D F6 2B   STA L2BF6
AD6E          LAD6E:
AD6E 4C 2B D5   JMP LD52B
AD71          LAD71:
AD71 A2 00      LDX #$0
AD73          LAD73:
AD73 BD 18 2C   LDA L2C18,X
AD76 29 07      AND #$7
AD78 C9 05      CMP #$5
AD7A B0 07      BCS LAD83
AD7C          LAD7C:
AD7C E8         INX
AD7D EC EB 2B   CPX L2BEB
AD80 90 F1      BCC LAD73
AD82          LAD82:
AD82 60         RTS
AD83          LAD83:
AD83 A9 64      LDA #$64
AD85 4C 6F B6   JMP LB66F
AD88          LAD88:
AD88 AD 01 02   LDA L201
AD8B C9 2D      CMP #$2D
AD8D D0 1F      BNE LADAE
AD8F          LAD8F:
AD8F AD 02 02   LDA L202
AD92 C9 43      CMP #$43
AD94 F0 1E      BEQ LADB4
AD96          LAD96:
AD96 C9 38      CMP #$38
AD98 F0 0E      BEQ LADA8
AD9A          LAD9A:
AD9A C9 39      CMP #$39
AD9C F0 0A      BEQ LADA8
AD9E          LAD9E:
AD9E C9 44      CMP #$44
ADA0 D0 0C      BNE LADAE
ADA2          LADA2:
ADA2 A9 80      LDA #$80
ADA4 8D E7 2B   STA L2BE7
ADA7 60         RTS
ADA8          LADA8:
ADA8 29 0F      AND #$F
ADAA 8D E6 2B   STA L2BE6
ADAD 60         RTS
ADAE          LADAE:
ADAE 4C 60 B2   JMP LB260
ADB1          LADB1:
ADB1 4C 97 DF   JMP LDF97
ADB4          LADB4:
ADB4 A5 56      LDA L56
ADB6 C9 0C      CMP #$C
ADB8 90 F7      BCC LADB1
ADBA          LADBA:
ADBA 78         SEI
ADBB 20 39 AE   JSR LAE39
ADBE AD 00 2A   LDA L2A00
ADC1 C9 2F      CMP #$2F
ADC3 F0 17      BEQ LADDC
ADC5          LADC5:
ADC5 20 57 AE   JSR LAE57
ADC8          LADC8:
ADC8 AD 10 2A   LDA L2A10
ADCB 8D E7 2D   STA L2DE7
ADCE A9 FF      LDA #$FF
ADD0 A2 23      LDX #$23
ADD2 85 DE      STA LDE
ADD4 86 DF      STX LDF
ADD6 A9 88      LDA #$88
ADD8 8D C7 2D   STA L2DC7
ADDB 60         RTS
ADDC          LADDC:
ADDC 20 28 AE   JSR LAE28
ADDF F0 E4      BEQ LADC5
ADE1          LADE1:
ADE1 A9 28      LDA #$28
ADE3 8D 00 2A   STA L2A00
ADE6 AD 08 2A   LDA L2A08
ADE9 85 DE      STA LDE
ADEB AD 07 2A   LDA L2A07
ADEE 85 DF      STA LDF
ADF0 A9 00      LDA #$0
ADF2 8D 07 2A   STA L2A07
ADF5 A9 01      LDA #$1
ADF7 8D 08 2A   STA L2A08
ADFA          LADFA:
ADFA 20 11 EF   JSR LEF11
ADFD A9 00      LDA #$0
ADFF 85 68      STA L68
AE01 A9 52      LDA #$52
AE03 85 69      STA L69
AE05 20 57 AE   JSR LAE57
AE08 D0 BE      BNE LADC8
AE0A          LAE0A:
AE0A EE 05 2A   INC L2A05
AE0D D0 08      BNE LAE17
AE0F          LAE0F:
AE0F EE 04 2A   INC L2A04
AE12 D0 03      BNE LAE17
AE14          LAE14:
AE14 EE 03 2A   INC L2A03
AE17          LAE17:
AE17 A6 DE      LDX LDE
AE19 D0 02      BNE LAE1D
AE1B          LAE1B:
AE1B C6 DF      DEC LDF
AE1D          LAE1D:
AE1D C6 DE      DEC LDE
AE1F D0 D9      BNE LADFA
AE21          LAE21:
AE21 A6 DF      LDX LDF
AE23 D0 D5      BNE LADFA
AE25          LAE25:
AE25 4C C8 AD   JMP LADC8
AE28          LAE28:
AE28 A9 00      LDA #$0
AE2A 8D 07 2A   STA L2A07
AE2D 8D 08 2A   STA L2A08
AE30 20 57 AE   JSR LAE57
AE33 48         PHA
AE34 20 39 AE   JSR LAE39
AE37 68         PLA
AE38 60         RTS
AE39          LAE39:
AE39 20 07 EF   JSR LEF07
AE3C AD 04 02   LDA L204
AE3F 85 68      STA L68
AE41 AD 05 02   LDA L205
AE44 85 69      STA L69
AE46 A2 06      LDX #$6
AE48 A0 00      LDY #$0
AE4A          LAE4A:
AE4A BD 00 02   LDA L200,X
AE4D 99 00 2A   STA L2A00,Y
AE50 C8         INY
AE51 E8         INX
AE52 E4 56      CPX L56
AE54 90 F4      BCC LAE4A
AE56          LAE56:
AE56 60         RTS
AE57          LAE57:
AE57 AD 03 02   LDA L203
AE5A 20 13 F1   JSR LF113
AE5D D0 06      BNE LAE65
AE5F          LAE5F:
AE5F A9 85      LDA #$85
AE61 8D 10 2A   STA L2A10
AE64 60         RTS
AE65          LAE65:
AE65 20 6C EF   JSR LEF6C
AE68 AD 10 2A   LDA L2A10
AE6B 60         RTS
AE6C          LAE6C:
AE6C A6 56      LDX L56
AE6E CA         DEX
AE6F D0 0D      BNE LAE7E
AE71          LAE71:
AE71 A9 01      LDA #$1
AE73 20 C2 DA   JSR LDAC2
AE76 4C A6 AE   JMP LAEA6
AE79          LAE79:
AE79 A9 70      LDA #$70
AE7B 4C 6F B6   JMP LB66F
AE7E          LAE7E:
AE7E A0 01      LDY #$1
AE80 20 00 AA   JSR LAA00
AE83 AD 28 2C   LDA L2C28
AE86 C9 1E      CMP #$1E
AE88 B0 EF      BCS LAE79
AE8A          LAE8A:
AE8A 85 41      STA L41
AE8C 20 A5 DC   JSR LDCA5
AE8F F0 E8      BEQ LAE79
AE91          LAE91:
AE91 A9 00      LDA #$0
AE93 20 C2 DA   JSR LDAC2
AE96 A6 80      LDX L80
AE98 AD 28 2C   LDA L2C28
AE9B 9D 68 2C   STA L2C68,X
AE9E AA         TAX
AE9F A9 00      LDA #$0
AEA1 95 20      STA L20,X
AEA3 9D 60 29   STA L2960,X
AEA6          LAEA6:
AEA6 A6 82      LDX L82
AEA8 BD 48 2C   LDA L2C48,X
AEAB 09 40      ORA #$40
AEAD 9D 48 2C   STA L2C48,X
AEB0 A4 80      LDY L80
AEB2 A9 FF      LDA #$FF
AEB4 99 E8 2D   STA L2DE8,Y
AEB7 A9 89      LDA #$89
AEB9 99 A8 2D   STA L2DA8,Y
AEBC B9 68 2C   LDA L2C68,Y
AEBF 99 C8 2D   STA L2DC8,Y
AEC2 0A         ASL A
AEC3 AA         TAX
AEC4 A9 01      LDA #$1
AEC6 95 A0      STA LA0,X
AEC8 A9 0E      LDA #$E
AECA 99 88 2D   STA L2D88,Y
AECD 4C 54 B6   JMP LB654
AED0          LAED0:
AED0 20 7E B0   JSR LB07E
AED3 C9 FF      CMP #$FF
AED5 D0 03      BNE LAEDA
AED7          LAED7:
AED7 A9 00      LDA #$0
AED9 60         RTS
AEDA          LAEDA:
AEDA 20 C7 A2   JSR LA2C7
AEDD BD 90 2B   LDA L2B90,X
AEE0 F0 09      BEQ LAEEB
AEE2          LAEE2:
AEE2 20 03 AF   JSR LAF03
AEE5 AE A1 2B   LDX L2BA1
AEE8 BD 90 2B   LDA L2B90,X
AEEB          LAEEB:
AEEB 60         RTS
AEEC          LAEEC:
AEEC 20 78 B6   JSR LB678
AEEF 20 7E B0   JSR LB07E
AEF2 C9 04      CMP #$4
AEF4 F0 04      BEQ LAEFA
AEF6          LAEF6:
AEF6 C9 05      CMP #$5
AEF8 D0 03      BNE LAEFD
AEFA          LAEFA:
AEFA 20 F4 AF   JSR LAFF4
AEFD          LAEFD:
AEFD 20 03 AF   JSR LAF03
AF00 4C 54 B6   JMP LB654
AF03          LAF03:
AF03 20 26 DB   JSR LDB26
AF06 A9 00      LDA #$0
AF08 8D F7 2B   STA L2BF7
AF0B 20 C7 A2   JSR LA2C7
AF0E A9 FF      LDA #$FF
AF10 9D 90 2B   STA L2B90,X
AF13 20 7E B0   JSR LB07E
AF16 F0 08      BEQ LAF20
AF18          LAF18:
AF18 C9 FF      CMP #$FF
AF1A F0 04      BEQ LAF20
AF1C          LAF1C:
AF1C C9 06      CMP #$6
AF1E 90 01      BCC LAF21
AF20          LAF20:
AF20 60         RTS
AF21          LAF21:
AF21 20 8E B0   JSR LB08E
AF24 D0 03      BNE LAF29
AF26          LAF26:
AF26 20 F4 AF   JSR LAFF4
AF29          LAF29:
AF29 20 A7 A2   JSR LA2A7
AF2C AE A1 2B   LDX L2BA1
AF2F A0 02      LDY #$2
AF31 B1 58      LDA (L58),Y
AF33 9D 70 2B   STA L2B70,X
AF36 20 85 B0   JSR LB085
AF39 F0 04      BEQ LAF3F
AF3B          LAF3B:
AF3B C9 04      CMP #$4
AF3D 90 11      BCC LAF50
AF3F          LAF3F:
AF3F A0 03      LDY #$3
AF41 B1 58      LDA (L58),Y
AF43 49 FF      EOR #$FF
AF45 AE A1 2B   LDX L2BA1
AF48 DD 70 2B   CMP L2B70,X
AF4B D0 D3      BNE LAF20
AF4D          LAF4D:
AF4D A0 04      LDY #$4
AF50          LAF50 = * + 1
              ; Instruction parameter jumped to.
AF4F 2C A0 A2   BIT LA2A0
AF52 B1 58      LDA (L58),Y
AF54 8D A3 2B   STA L2BA3
AF57 C8         INY
AF58 B1 58      LDA (L58),Y
AF5A 8D A4 2B   STA L2BA4
AF5D AE A1 2B   LDX L2BA1
AF60 A9 00      LDA #$0
AF62 9D 90 2B   STA L2B90,X
AF65 20 26 B0   JSR LB026
AF68 4C 19 A6   JMP LA619
AF6B          LAF6B:
AF6B C9 00      CMP #$0
AF6D F0 09      BEQ LAF78
AF6F          LAF6F:
AF6F 48         PHA
AF70 20 7E B0   JSR LB07E
AF73 AA         TAX
AF74 68         PLA
AF75 DD 79 AF   CMP LAF79,X
AF78          LAF78:
AF78 60         RTS
AF79          LAF79:
AF79 00 48 41   .BYTE $0,$48,$41
AF7C 41 44 44   .BYTE $41,$44,$44
AF7F          LAF7F:
AF7F 8E C9 2B   STX L2BC9
AF82 20 8E B0   JSR LB08E
AF85 8D C6 2B   STA L2BC6
AF88 20 85 B0   JSR LB085
AF8B F0 16      BEQ LAFA3
AF8D          LAF8D:
AF8D C9 03      CMP #$3
AF8F F0 2C      BEQ LAFBD
AF91          LAF91:
AF91 90 27      BCC LAFBA
AF93          LAF93:
AF93 C9 06      CMP #$6
AF95 90 45      BCC LAFDC
AF97          LAF97:
AF97 C9 FF      CMP #$FF
AF99 F0 01      BEQ LAF9C
AF9B          LAF9B:
AF9B 60         RTS
AF9C          LAF9C:
AF9C A9 01      LDA #$1
AF9E 8D C6 2B   STA L2BC6
AFA1 A2 00      LDX #$0
AFA3          LAFA3:
AFA3 BD 00 86   LDA Partition_SizeLo+$00,X
AFA6 0A         ASL A
AFA7 BD 00 83   LDA Partition_SizeHi+$00,X
AFAA 2A         ROL A
AFAB AA         TAX
AFAC E8         INX
AFAD 8E C8 2B   STX L2BC8
AFB0 A2 01      LDX #$1
AFB2 8E C7 2B   STX L2BC7
AFB5 CA         DEX
AFB6 8E C9 2B   STX L2BC9
AFB9 60         RTS
AFBA          LAFBA:
AFBA A9 24      LDA #$24
AFBD          LAFBD = * + 1
              ; Instruction parameter jumped to.
AFBC 2C A9 47   BIT L47A9
AFBF 8D C8 2B   STA L2BC8
AFC2 A9 01      LDA #$1
AFC4 8D C7 2B   STA L2BC7
AFC7 AD C9 2B   LDA L2BC9
AFCA A2 00      LDX #$0
AFCC          LAFCC:
AFCC DD C3 EA   CMP LEAC3,X
AFCF 90 03      BCC LAFD4
AFD1          LAFD1:
AFD1 E8         INX
AFD2 D0 F8      BNE LAFCC
AFD4          LAFD4:
AFD4 CA         DEX
AFD5 BD DC EA   LDA LEADC,X
AFD8 8D C9 2B   STA L2BC9
AFDB 60         RTS
AFDC          LAFDC:
AFDC BD 00 92   LDA L9200,X
AFDF 8D C8 2B   STA L2BC8
AFE2 AD C6 2B   LDA L2BC6
AFE5 C9 28      CMP #$28
AFE7 D0 02      BNE LAFEB
AFE9          LAFE9:
AFE9 A9 01      LDA #$1
AFEB          LAFEB:
AFEB 8D C7 2B   STA L2BC7
AFEE A9 28      LDA #$28
AFF0 8D C9 2B   STA L2BC9
AFF3 60         RTS
AFF4          LAFF4:
AFF4 20 85 B0   JSR LB085
AFF7 F0 17      BEQ LB010
AFF9          LAFF9:
AFF9 C9 04      CMP #$4
AFFB 90 06      BCC LB003
AFFD          LAFFD:
AFFD A9 28      LDA #$28
AFFF A0 51      LDY #$51
B001 D0 10      BNE LB013
B003          LB003:
B003 C9 02      CMP #$2
B005 D0 03      BNE LB00A
B007          LB007:
B007 A0 24      LDY #$24
B00A          LB00A = * + 1
              ; Instruction parameter jumped to.
B009 2C A0 47   BIT L47A0
B00C A9 12      LDA #$12
B00E D0 03      BNE LB013
B010          LB010:
B010 A9 01      LDA #$1
B012 A8         TAY
B013          LB013:
B013 20 00 F7   JSR LF700
B016 AE E8 90   LDX L90E8
B019 9D 00 91   STA L9100,X
B01C 98         TYA
B01D 9D 00 92   STA L9200,X
B020 4C F5 F6   JMP LF6F5
B023          LB023:
B023 20 63 F7   JSR LF763
B026          LB026:
B026 20 8E B0   JSR LB08E
B029 D0 06      BNE LB031
B02B          LB02B:
B02B 20 F4 AF   JSR LAFF4
B02E 20 8E B0   JSR LB08E
B031          LB031:
B031 8D A7 2B   STA L2BA7
B034 A9 00      LDA #$0
B036 8D A8 2B   STA L2BA8
B039 20 85 B0   JSR LB085
B03C F0 28      BEQ LB066
B03E          LB03E:
B03E C9 04      CMP #$4
B040 90 1E      BCC LB060
B042          LB042:
B042 C9 06      CMP #$6
B044 90 14      BCC LB05A
B046          LB046:
B046 C9 FF      CMP #$FF
B048 D0 0F      BNE LB059
B04A          LB04A:
B04A AD E6 90   LDA L90E6
B04D 8D A7 2B   STA L2BA7
B050 AD E7 90   LDA L90E7
B053 8D A8 2B   STA L2BA8
B056 8D A9 2B   STA L2BA9
B059          LB059:
B059 60         RTS
B05A          LB05A:
B05A A9 03      LDA #$3
B05C 8D A9 2B   STA L2BA9
B05F 60         RTS
B060          LB060:
B060 A9 01      LDA #$1
B062 8D A9 2B   STA L2BA9
B065 60         RTS
B066          LB066:
B066 20 95 B0   JSR LB095
B069 8D A8 2B   STA L2BA8
B06C C9 01      CMP #$1
B06E D0 07      BNE LB077
B070          LB070:
B070 CD A7 2B   CMP L2BA7
B073 D0 02      BNE LB077
B075          LB075:
B075 A9 21      LDA #$21
B077          LB077:
B077 18         CLC
B078 69 01      ADC #$1
B07A 8D A9 2B   STA L2BA9
B07D 60         RTS
B07E          LB07E:
B07E AE E8 90   LDX L90E8
B081 BD 00 82   LDA Partition_Typ+$00,X
B084 60         RTS
B085          LB085:
B085 AE E8 90   LDX L90E8
B088 BD 00 82   LDA Partition_Typ+$00,X
B08B C9 01      CMP #$1
B08D 60         RTS
B08E          LB08E:
B08E AE E8 90   LDX L90E8
B091 BD 00 91   LDA L9100,X
B094 60         RTS
B095          LB095:
B095 AE E8 90   LDX L90E8
B098 BD 00 92   LDA L9200,X
B09B 60         RTS
B09C          LB09C:
B09C AD 01 02   LDA L201
B09F C9 2D      CMP #$2D
B0A1 D0 71      BNE LB114
B0A3          LB0A3:
B0A3 AD 03 02   LDA L203
B0A6 85 50      STA L50
B0A8 AD 04 02   LDA L204
B0AB 85 51      STA L51
B0AD A0 00      LDY #$0
B0AF AD 02 02   LDA L202
B0B2 C9 52      CMP #$52
B0B4 F0 34      BEQ LB0EA
B0B6          LB0B6:
B0B6 C9 57      CMP #$57
B0B8 F0 5F      BEQ LB119
B0BA          LB0BA:
B0BA C9 45      CMP #$45
B0BC D0 56      BNE LB114
B0BE          LB0BE:
B0BE A5 51      LDA L51
B0C0 C9 80      CMP #$80
B0C2 90 05      BCC LB0C9
B0C4          LB0C4:
B0C4 C9 FF      CMP #$FF
B0C6 B0 01      BCS LB0C9
B0C8          LB0C8:
B0C8 60         RTS
B0C9          LB0C9:
B0C9 C9 06      CMP #$6
B0CB D0 14      BNE LB0E1
B0CD          LB0CD:
B0CD A5 50      LDA L50
B0CF D0 10      BNE LB0E1
B0D1          LB0D1:
B0D1 A0 07      LDY #$7
B0D3          LB0D3:
B0D3 B9 08 06   LDA L608,Y
B0D6 D9 25 B1   CMP LB125,Y
B0D9 D0 06      BNE LB0E1
B0DB          LB0DB:
B0DB 88         DEY
B0DC 10 F5      BPL LB0D3
B0DE          LB0DE:
B0DE 4C 09 B2   JMP LB209
B0E1          LB0E1:
B0E1 A0 00      LDY #$0
B0E3 A9 45      LDA #$45
B0E5 C9 45      CMP #$45
B0E7 6C 50 00   JMP (L50)
B0EA          LB0EA:
B0EA B1 50      LDA (L50),Y
B0EC 85 84      STA L84
B0EE A5 56      LDA L56
B0F0 C9 06      CMP #$6
B0F2 90 1A      BCC LB10E
B0F4          LB0F4:
B0F4 AE 05 02   LDX L205
B0F7 CA         DEX
B0F8 F0 14      BEQ LB10E
B0FA          LB0FA:
B0FA 8A         TXA
B0FB 18         CLC
B0FC 65 50      ADC L50
B0FE E6 50      INC L50
B100 8D 07 2E   STA L2E07
B103 A5 50      LDA L50
B105 85 DE      STA LDE
B107 A5 51      LDA L51
B109 85 DF      STA LDF
B10B 4C 20 9F   JMP L9F20
B10E          LB10E:
B10E 20 60 DA   JSR LDA60
B111 4C 18 9F   JMP L9F18
B114          LB114:
B114 A9 31      LDA #$31
B116 4C 6F B6   JMP LB66F
B119          LB119:
B119 B9 06 02   LDA L206,Y
B11C 91 50      STA (L50),Y
B11E C8         INY
B11F CC 05 02   CPY L205
B122 90 F5      BCC LB119
B124          LB124:
B124 60         RTS
B125          LB125:
B125 06         .BYTE $6
B126          LB126:
B126 A2 00      LDX #$0
B128 86 F9      STX LF9
B12A 20 86 D5   JSR LD586
B12D          LB12D:
B12D AD 01 02   LDA L201
B130 C9 2D      CMP #$2D
B132 D0 42      BNE LB176
B134          LB134:
B134 AD 02 02   LDA L202
B137 C9 48      CMP #$48
B139 D0 39      BNE LB174
B13B          LB13B:
B13B 20 F5 BD   JSR LBDF5
B13E A9 00      LDA #$0
B140 20 20 BA   JSR LBA20
B143 20 7E A1   JSR LA17E
B146 20 85 B0   JSR LB085
B149 F0 04      BEQ LB14F
B14B          LB14B:
B14B C9 04      CMP #$4
B14D 90 03      BCC LB152
B14F          LB14F:
B14F A0 04      LDY #$4
B152          LB152 = * + 1
              ; Instruction parameter jumped to.
B151 2C A0 90   BIT L90A0
B154 A9 10      LDA #$10
B156 85 50      STA L50
B158 AE 00 2C   LDX L2C00
B15B          LB15B:
B15B E4 56      CPX L56
B15D B0 04      BCS LB163
B15F          LB15F:
B15F BD 00 02   LDA L200,X
B163          LB163 = * + 1
              ; Instruction parameter jumped to.
B162 2C A9 A0   BIT LA0A9
B165 99 00 22   STA L2200,Y
B168 E8         INX
B169 C8         INY
B16A C6 50      DEC L50
B16C D0 ED      BNE LB15B
B16E          LB16E:
B16E 20 81 A1   JSR LA181
B171 4C 54 B6   JMP LB654
B174          LB174:
B174 C9 50      CMP #$50
B176          LB176:
B176 08         PHP
B177 20 E7 B6   JSR LB6E7
B17A 20 3D B8   JSR LB83D
B17D 28         PLP
B17E D0 0E      BNE LB18E
B180          LB180:
B180 A9 00      LDA #$0
B182 8D 10 2C   STA L2C10
B185 20 23 B0   JSR LB023
B188 AD 00 2C   LDA L2C00
B18B 8D 08 2C   STA L2C08
B18E          LB18E:
B18E AD 10 2C   LDA L2C10
B191 8D 11 2C   STA L2C11
B194 AD 01 2C   LDA L2C01
B197 8D 09 2C   STA L2C09
B19A 20 CF BE   JSR LBECF
B19D 20 EA B1   JSR LB1EA
B1A0 AD 31 2C   LDA L2C31
B1A3 85 5A      STA L5A
B1A5 AD 39 2C   LDA L2C39
B1A8 85 5B      STA L5B
B1AA 20 A1 D9   JSR LD9A1
B1AD 20 65 D9   JSR LD965
B1B0 AD 41 2C   LDA L2C41
B1B3 18         CLC
B1B4 69 03      ADC #$3
B1B6 20 C6 DC   JSR LDCC6
B1B9 20 F2 DC   JSR LDCF2
B1BC A8         TAY
B1BD AE 00 2C   LDX L2C00
B1C0 A9 10      LDA #$10
B1C2 20 1E C1   JSR LC11E
B1C5 20 A7 D9   JSR LD9A7
B1C8 20 65 D9   JSR LD965
B1CB 4C 54 B6   JMP LB654
B1CE          LB1CE:
B1CE AD 19 2C   LDA L2C19
B1D1 29 07      AND #$7
B1D3 8D ED 2B   STA L2BED
B1D6 AE EB 2B   LDX L2BEB
B1D9          LB1D9:
B1D9 CA         DEX
B1DA EC EA 2B   CPX L2BEA
B1DD 90 0A      BCC LB1E9
B1DF          LB1DF:
B1DF BD 20 2C   LDA L2C20,X
B1E2 D0 F5      BNE LB1D9
B1E4          LB1E4:
B1E4 A9 62      LDA #$62
B1E6 4C 6F B6   JMP LB66F
B1E9          LB1E9:
B1E9 60         RTS
B1EA          LB1EA:
B1EA 20 CE B1   JSR LB1CE
B1ED          LB1ED:
B1ED BD 20 2C   LDA L2C20,X
B1F0 F0 05      BEQ LB1F7
B1F2          LB1F2:
B1F2 A9 63      LDA #$63
B1F4 4C 6F B6   JMP LB66F
B1F7          LB1F7:
B1F7 CA         DEX
B1F8 10 F3      BPL LB1ED
B1FA          LB1FA:
B1FA 60         RTS
B1FB          LB1FB:
B1FB 20 F5 BD   JSR LBDF5
B1FE 20 D0 AE   JSR LAED0
B201 20 CF BE   JSR LBECF
B204 AD 20 2C   LDA L2C20
B207 F0 1E      BEQ LB227
B209          LB209:
B209 AE B6 2B   LDX L2BB6
B20C AC B7 2B   LDY L2BB7
B20F AD B8 2B   LDA L2BB8
B212 48         PHA
B213 86 5A      STX L5A
B215 84 5B      STY L5B
B217 20 A2 A1   JSR LA1A2
B21A 68         PLA
B21B AA         TAX
B21C BD 00 22   LDA L2200,X
B21F 49 40      EOR #$40
B221 9D 00 22   STA L2200,X
B224 20 A5 A1   JSR LA1A5
B227          LB227:
B227 4C 6B DB   JMP LDB6B
B22A          LB22A:
B22A AD 01 02   LDA L201
B22D C9 2D      CMP #$2D
B22F D0 0B      BNE LB23C
B231          LB231:
B231 AD 02 02   LDA L202
B234 C9 30      CMP #$30
B236 F0 07      BEQ LB23F
B238          LB238:
B238 C9 31      CMP #$31
B23A F0 16      BEQ LB252
B23C          LB23C:
B23C 4C 97 DF   JMP LDF97
B23F          LB23F:
B23F A9 80      LDA #$80
B241 2C F9 2B   BIT L2BF9
B244 F0 0B      BEQ LB251
B246          LB246:
B246 A9 7F      LDA #$7F
B248 25 49      AND L49
B24A 85 49      STA L49
B24C A9 00      LDA #$0
B24E 8D F9 2B   STA L2BF9
B251          LB251:
B251 60         RTS
B252          LB252:
B252 A9 80      LDA #$80
B254 24 49      BIT L49
B256 D0 07      BNE LB25F
B258          LB258:
B258 8D F9 2B   STA L2BF9
B25B 05 49      ORA L49
B25D 85 49      STA L49
B25F          LB25F:
B25F 60         RTS
B260          LB260:
B260 20 E7 B6   JSR LB6E7
B263 20 F8 B8   JSR LB8F8
B266 20 3D B8   JSR LB83D
B269          LB269:
B269 A2 00      LDX #$0
B26B 86 85      STX L85
B26D          LB26D:
B26D 8E BD 2B   STX L2BBD
B270 BD 10 2C   LDA L2C10,X
B273 D0 03      BNE LB278
B275          LB275:
B275 4C 20 B3   JMP LB320
B278          LB278:
B278 20 B4 BE   JSR LBEB4
B27B 20 23 B0   JSR LB023
B27E 20 84 BE   JSR LBE84
B281 AD BD 2B   LDA L2BBD
B284 20 0B BF   JSR LBF0B
B287 10 03      BPL LB28C
B289          LB289:
B289 4C 11 B3   JMP LB311
B28C          LB28C:
B28C 20 0F DA   JSR LDA0F
B28F 90 78      BCC LB309
B291          LB291:
B291 A0 00      LDY #$0
B293 B1 94      LDA (L94),Y
B295 8D A6 2B   STA L2BA6
B298 29 40      AND #$40
B29A D0 6D      BNE LB309
B29C          LB29C:
B29C AD A6 2B   LDA L2BA6
B29F 29 07      AND #$7
B2A1 C9 06      CMP #$6
B2A3 D0 07      BNE LB2AC
B2A5          LB2A5:
B2A5 AD E2 2B   LDA L2BE2
B2A8 C9 03      CMP #$3
B2AA D0 5D      BNE LB309
B2AC          LB2AC:
B2AC 20 6D C3   JSR LC36D
B2AF AD A6 2B   LDA L2BA6
B2B2 29 07      AND #$7
B2B4 C9 05      CMP #$5
B2B6 D0 28      BNE LB2E0
B2B8          LB2B8:
B2B8 C8         INY
B2B9 B1 94      LDA (L94),Y
B2BB 85 5A      STA L5A
B2BD C8         INY
B2BE B1 94      LDA (L94),Y
B2C0 85 5B      STA L5B
B2C2 A0 1C      LDY #$1C
B2C4 B1 94      LDA (L94),Y
B2C6 8D A6 2B   STA L2BA6
B2C9 C8         INY
B2CA B1 94      LDA (L94),Y
B2CC 8D A5 2B   STA L2BA5
B2CF          LB2CF:
B2CF 20 1C D9   JSR LD91C
B2D2 20 91 A3   JSR LA391
B2D5 20 76 BC   JSR LBC76
B2D8 D0 F5      BNE LB2CF
B2DA          LB2DA:
B2DA 20 48 A3   JSR LA348
B2DD 4C 07 B3   JMP LB307
B2E0          LB2E0:
B2E0 A0 13      LDY #$13
B2E2 B1 94      LDA (L94),Y
B2E4 F0 0A      BEQ LB2F0
B2E6          LB2E6:
B2E6 85 5A      STA L5A
B2E8 C8         INY
B2E9 B1 94      LDA (L94),Y
B2EB 85 5B      STA L5B
B2ED 20 2B B3   JSR LB32B
B2F0          LB2F0:
B2F0 AE BF 2B   LDX L2BBF
B2F3 A9 20      LDA #$20
B2F5 3D 18 2C   AND L2C18,X
B2F8 D0 0D      BNE LB307
B2FA          LB2FA:
B2FA BD 20 2C   LDA L2C20,X
B2FD 85 5A      STA L5A
B2FF BD 28 2C   LDA L2C28,X
B302 85 5B      STA L5B
B304 20 2B B3   JSR LB32B
B307          LB307:
B307 E6 85      INC L85
B309          LB309:
B309 20 02 BF   JSR LBF02
B30C 30 03      BMI LB311
B30E          LB30E:
B30E 4C 8C B2   JMP LB28C
B311          LB311:
B311 20 B4 BE   JSR LBEB4
B314 AE BD 2B   LDX L2BBD
B317 E8         INX
B318 EC EB 2B   CPX L2BEB
B31B B0 03      BCS LB320
B31D          LB31D:
B31D 4C 6D B2   JMP LB26D
B320          LB320:
B320 A5 85      LDA L85
B322 85 5A      STA L5A
B324 A0 00      LDY #$0
B326 A9 01      LDA #$1
B328 4C 61 B6   JMP LB661
B32B          LB32B:
B32B 20 91 A3   JSR LA391
B32E A5 5A      LDA L5A
B330 8D 3E 28   STA L283E
B333 A5 5B      LDA L5B
B335 8D 3F 28   STA L283F
B338 A2 1F      LDX #$1F
B33A A9 AA      LDA #$AA
B33C 20 1C E8   JSR LE81C
B33F A0 01      LDY #$1
B341 B1 68      LDA (L68),Y
B343 85 5B      STA L5B
B345 88         DEY
B346 B1 68      LDA (L68),Y
B348 85 5A      STA L5A
B34A D0 DF      BNE LB32B
B34C          LB34C:
B34C 20 48 A3   JSR LA348
B34F 4C 04 DB   JMP LDB04
B352          LB352:
B352 78         SEI
B353 AD 01 02   LDA L201
B356 C9 2D      CMP #$2D
B358 D0 0E      BNE LB368
B35A          LB35A:
B35A AD 02 02   LDA L202
B35D C9 52      CMP #$52
B35F F0 4B      BEQ LB3AC
B361          LB361:
B361 C9 57      CMP #$57
B363 D0 03      BNE LB368
B365          LB365:
B365 4C 8B B4   JMP LB48B
B368          LB368:
B368 4C 97 DF   JMP LDF97
B36B          LB36B:
B36B 15 14 12   .BYTE $15,$14,$12
B36E 11 0F 0E   .BYTE $11,$F,$E
B371 09 08 06   .BYTE $9,$8,$6
B374 05 0C 0B   .BYTE $5,$C,$B
B377          LB377:
B377 53 4D 54   .BYTE $53,$4D,$54
B37A 57 54 46   .BYTE $57,$54,$46
B37E          LB37E = * + 1
B37D 53 55 4F   .BYTE $53,$55,$4F
B380 55 45 48   .BYTE $55,$45,$48
B385          LB385 = * + 2
B383 52 41 4E   .BYTE $52,$41,$4E
B386 4E 45 44   .BYTE $4E,$45,$44
B389 55 49 54   .BYTE $55,$49,$54
B38C          LB38C:
B38C 2E 2E 53   .BYTE $2E,$2E,$53
B38F 2E 52 2E   .BYTE $2E,$52,$2E
B393          LB393 = * + 1
B392 2E 20 20   .BYTE $2E,$20,$20
B395 20 20 20   .BYTE $20,$20,$20
B398 20 20 2F   .BYTE $20,$20,$2F
B39B 20 20 2F   .BYTE $20,$20,$2F
B39E 20 20 20   .BYTE $20,$20,$20
B3A1 20 20 3A   .BYTE $20,$20,$3A
B3A4 20 20 3A   .BYTE $20,$20,$3A
B3A7 20 20      .BYTE $20,$20
B3A9          LB3A9:
B3A9 20 20 4D   JSR L4D20
B3AC          LB3AC:
B3AC AD 03 02   LDA L203
B3AF C9 41      CMP #$41
B3B1 F0 0E      BEQ LB3C1
B3B3          LB3B3:
B3B3 C9 42      CMP #$42
B3B5 D0 03      BNE LB3BA
B3B7          LB3B7:
B3B7 4C 2C B4   JMP LB42C
B3BA          LB3BA:
B3BA C9 44      CMP #$44
B3BC D0 AA      BNE LB368
B3BE          LB3BE:
B3BE 4C 40 B4   JMP LB440
B3C1          LB3C1:
B3C1 A2 18      LDX #$18
B3C3          LB3C3:
B3C3 BD 93 B3   LDA LB393,X
B3C6 9D 00 23   STA L2300,X
B3C9 CA         DEX
B3CA 10 F7      BPL LB3C3
B3CC          LB3CC:
B3CC 20 A5 B5   JSR LB5A5
B3CF AD 0C 8C   LDA RTC+$0C
B3D2 29 07      AND #$7
B3D4 AA         TAX
B3D5 BD 77 B3   LDA LB377,X
B3D8 8D E7 2D   STA L2DE7
B3DB 8D 00 23   STA L2300
B3DE BD 7E B3   LDA LB37E,X
B3E1 8D 01 23   STA L2301
B3E4 BD 85 B3   LDA LB385,X
B3E7 8D 02 23   STA L2302
B3EA BD 8C B3   LDA LB38C,X
B3ED 8D 03 23   STA L2303
B3F0 A2 0B      LDX #$B
B3F2          LB3F2:
B3F2 BD 00 8C   LDA RTC+$00,X
B3F5 3D 50 B5   AND LB550,X
B3F8 09 30      ORA #$30
B3FA BC 6B B3   LDY LB36B,X
B3FD 99 00 23   STA L2300,Y
B400 CA         DEX
B401 10 EF      BPL LB3F2
B403          LB403:
B403 A0 17      LDY #$17
B405 AD 05 8C   LDA RTC+$05
B408 29 04      AND #$4
B40A D0 03      BNE LB40F
B40C          LB40C:
B40C A9 41      LDA #$41
B40F          LB40F = * + 1
              ; Instruction parameter jumped to.
B40E 2C A9 50   BIT L50A9
B411 99 00 23   STA L2300,Y
B414 C8         INY
B415          LB415:
B415 98         TYA
B416 18         CLC
B417 69 00      ADC #$0
B419 8D 07 2E   STA L2E07
B41C 20 B2 F5   JSR LF5B2
B41F E6 DE      INC LDE
B421 A9 88      LDA #$88
B423 8D C7 2D   STA L2DC7
B426          LB426:
B426 A9 00      LDA #$0
B428 8D 0D 8C   STA RTC+$0D
B42B 60         RTS
B42C          LB42C:
B42C 20 57 B4   JSR LB457
B42F A0 01      LDY #$1
B431          LB431:
B431 B9 00 2B   LDA L2B00,Y
B434 99 00 23   STA L2300,Y
B437 C8         INY
B438 C0 08      CPY #$8
B43A 90 F5      BCC LB431
B43C          LB43C:
B43C 88         DEY
B43D 4C 15 B4   JMP LB415
B440          LB440:
B440 20 57 B4   JSR LB457
B443 A0 01      LDY #$1
B445          LB445:
B445 B9 00 2B   LDA L2B00,Y
B448 20 64 B4   JSR LB464
B44B 99 00 23   STA L2300,Y
B44E C8         INY
B44F C0 08      CPY #$8
B451 90 F2      BCC LB445
B453          LB453:
B453 88         DEY
B454 4C 15 B4   JMP LB415
B457          LB457:
B457 20 5D B5   JSR LB55D
B45A AD 00 2B   LDA L2B00
B45D 8D E7 2D   STA L2DE7
B460 8D 00 23   STA L2300
B463 60         RTS
B464          LB464:
B464 48         PHA
B465 29 0F      AND #$F
B467 85 50      STA L50
B469 68         PLA
B46A 29 F0      AND #$F0
B46C 4A         LSR A
B46D 48         PHA
B46E 18         CLC
B46F 65 50      ADC L50
B471 85 50      STA L50
B473 68         PLA
B474 4A         LSR A
B475 4A         LSR A
B476 18         CLC
B477 65 50      ADC L50
B479 60         RTS
B47A          LB47A:
B47A 48         PHA
B47B A9 00      LDA #$0
B47D 85 50      STA L50
B47F 68         PLA
B480          LB480:
B480 C9 0A      CMP #$A
B482 90 06      BCC LB48A
B484          LB484:
B484 E9 0A      SBC #$A
B486 E6 50      INC L50
B488 D0 F6      BNE LB480
B48A          LB48A:
B48A 60         RTS
B48B          LB48B:
B48B AD 03 02   LDA L203
B48E C9 41      CMP #$41
B490 F0 11      BEQ LB4A3
B492          LB492:
B492 C9 42      CMP #$42
B494 D0 03      BNE LB499
B496          LB496:
B496 4C E1 B4   JMP LB4E1
B499          LB499:
B499 C9 44      CMP #$44
B49B D0 03      BNE LB4A0
B49D          LB49D:
B49D 4C 12 B5   JMP LB512
B4A0          LB4A0:
B4A0 4C 97 DF   JMP LDF97
B4A3          LB4A3:
B4A3 A5 56      LDA L56
B4A5 C9 1D      CMP #$1D
B4A7 90 15      BCC LB4BE
B4A9          LB4A9:
B4A9 A2 06      LDX #$6
B4AB          LB4AB:
B4AB AD 04 02   LDA L204
B4AE DD 77 B3   CMP LB377,X
B4B1 D0 08      BNE LB4BB
B4B3          LB4B3:
B4B3 AD 05 02   LDA L205
B4B6 DD 7E B3   CMP LB37E,X
B4B9 F0 06      BEQ LB4C1
B4BB          LB4BB:
B4BB CA         DEX
B4BC 10 ED      BPL LB4AB
B4BE          LB4BE:
B4BE 4C 97 DF   JMP LDF97
B4C1          LB4C1:
B4C1 8A         TXA
B4C2 20 A5 B5   JSR LB5A5
B4C5 8D 0C 8C   STA RTC+$0C
B4C8 A2 0B      LDX #$B
B4CA          LB4CA:
B4CA BC 6B B3   LDY LB36B,X
B4CD B9 04 02   LDA L204,Y
B4D0 3D 50 B5   AND LB550,X
B4D3 9D 00 8C   STA RTC+$00,X
B4D6 CA         DEX
B4D7 10 F1      BPL LB4CA
B4D9          LB4D9:
B4D9 AD 1B 02   LDA L21B
B4DC 29 10      AND #$10
B4DE 4C 05 B5   JMP LB505
B4E1          LB4E1:
B4E1 20 39 B5   JSR LB539
B4E4 A0 05      LDY #$5
B4E6 A2 0B      LDX #$B
B4E8          LB4E8:
B4E8 B9 00 02   LDA L200,Y
B4EB 48         PHA
B4EC 4A         LSR A
B4ED 4A         LSR A
B4EE 4A         LSR A
B4EF 4A         LSR A
B4F0 3D 50 B5   AND LB550,X
B4F3 9D 00 8C   STA RTC+$00,X
B4F6 68         PLA
B4F7 CA         DEX
B4F8 3D 50 B5   AND LB550,X
B4FB 9D 00 8C   STA RTC+$00,X
B4FE C8         INY
B4FF CA         DEX
B500 10 E6      BPL LB4E8
B502          LB502:
B502 B9 00 02   LDA L200,Y
B505          LB505:
B505 F0 02      BEQ LB509
B507          LB507:
B507 A9 04      LDA #$4
B509          LB509:
B509 0D 05 8C   ORA RTC+$05
B50C 8D 05 8C   STA RTC+$05
B50F 4C 26 B4   JMP LB426
B512          LB512:
B512 20 39 B5   JSR LB539
B515 A2 0B      LDX #$B
B517 A0 05      LDY #$5
B519          LB519:
B519 B9 00 02   LDA L200,Y
B51C 20 7A B4   JSR LB47A
B51F 48         PHA
B520 A5 50      LDA L50
B522 3D 50 B5   AND LB550,X
B525 9D 00 8C   STA RTC+$00,X
B528 68         PLA
B529 CA         DEX
B52A 3D 50 B5   AND LB550,X
B52D 9D 00 8C   STA RTC+$00,X
B530 CA         DEX
B531 C8         INY
B532 C0 0B      CPY #$B
B534 90 E3      BCC LB519
B536          LB536:
B536 4C 02 B5   JMP LB502
B539          LB539:
B539 A5 56      LDA L56
B53B C9 0C      CMP #$C
B53D 90 07      BCC LB546
B53F          LB53F:
B53F AD 04 02   LDA L204
B542 C9 07      CMP #$7
B544 90 03      BCC LB549
B546          LB546:
B546 4C 97 DF   JMP LDF97
B549          LB549:
B549 20 A5 B5   JSR LB5A5
B54C 8D 0C 8C   STA RTC+$0C
B54F 60         RTS
B550          LB550:
B550 0F 07 0F   .BYTE $F,$7,$F
B553 07 0F 03   .BYTE $7,$F,$3
B556 0F 03 0F   .BYTE $F,$3,$F
B559 01 0F 0F   .BYTE $1,$F,$F
B55C 07         .BYTE $7
B55D          LB55D:
B55D 08         PHP
B55E 78         SEI
B55F 20 A5 B5   JSR LB5A5
B562 AD 0C 8C   LDA RTC+$0C
B565 29 07      AND #$7
B567 8D 00 2B   STA L2B00
B56A A2 0B      LDX #$B
B56C A0 01      LDY #$1
B56E          LB56E:
B56E BD 00 8C   LDA RTC+$00,X
B571 3D 50 B5   AND LB550,X
B574 0A         ASL A
B575 0A         ASL A
B576 0A         ASL A
B577 0A         ASL A
B578 85 50      STA L50
B57A CA         DEX
B57B BD 00 8C   LDA RTC+$00,X
B57E 3D 50 B5   AND LB550,X
B581 18         CLC
B582 F8         SED
B583 65 50      ADC L50
B585 D8         CLD
B586 99 00 2B   STA L2B00,Y
B589 C8         INY
B58A CA         DEX
B58B 10 E1      BPL LB56E
B58D          LB58D:
B58D AD 05 8C   LDA RTC+$05
B590 29 04      AND #$4
B592 99 00 2B   STA L2B00,Y
B595 A9 00      LDA #$0
B597 8D 0D 8C   STA RTC+$0D
B59A 28         PLP
B59B 60         RTS
B59C          LB59C:
B59C 8D 0D 8C   STA RTC+$0D
B59F A2 4C      LDX #$4C
B5A1          LB5A1:
B5A1 CA         DEX
B5A2 D0 FD      BNE LB5A1
B5A4          LB5A4:
B5A5          LB5A5 = * + 1
              ; Instruction parameter jumped to.
B5A4 24 48      BIT L48
B5A6 A9 01      LDA #$1
B5A8 8D 0D 8C   STA RTC+$0D
B5AB AD 0D 8C   LDA RTC+$0D
B5AE 29 02      AND #$2
B5B0 D0 EA      BNE LB59C
B5B2          LB5B2:
B5B2 68         PLA
B5B3 60         RTS
B5B4          LB5B4:
B5B4 8A         TXA
B5B5 48         PHA
B5B6 20 5D B5   JSR LB55D
B5B9 A0 01      LDY #$1
B5BB 68         PLA
B5BC 48         PHA
B5BD AA         TAX
B5BE          LB5BE:
B5BE B9 00 2B   LDA L2B00,Y
B5C1 20 64 B4   JSR LB464
B5C4 9D 17 22   STA L2217,X
B5C7 E8         INX
B5C8 C8         INY
B5C9 C0 06      CPY #$6
B5CB 90 F1      BCC LB5BE
B5CD          LB5CD:
B5CD 68         PLA
B5CE AA         TAX
B5CF BD 1A 22   LDA L221A,X
B5D2 E9 0C      SBC #$C
B5D4 D0 03      BNE LB5D9
B5D6          LB5D6:
B5D6 9D 1A 22   STA L221A,X
B5D9          LB5D9:
B5D9 AD 07 2B   LDA L2B07
B5DC F0 09      BEQ LB5E7
B5DE          LB5DE:
B5DE A9 0C      LDA #$C
B5E0 18         CLC
B5E1 7D 1A 22   ADC L221A,X
B5E4 9D 1A 22   STA L221A,X
B5E7          LB5E7:
B5E7 60         RTS
B5E8          LB5E8:
B5E8 56         .BYTE $56
B5E9          LB5E9:
B5E9 49 2F      EOR #$2F
B5EB 4D 42 55   EOR L5542
B5EE 50 26      BVC LB616
B5F0 43 52 53   .BYTE $43,$52,$53
B5F3          LB5F3:
B5F3 4E 54 47   LSR L4754
B5F8          LB5F8 = * + 2
B5F6 4C 57 FF   JMP LFF57
B5F9 FF FF 9E   .BYTE $FF,$FF,$9E
B5FC FF FF FF   .BYTE $FF,$FF,$FF
B5FF FF 51 DD   .BYTE $FF,$51,$DD
B602 1C 9E 18   .BYTE $1C,$9E,$18
B605          LB605:
B605 21 09 24   .BYTE $21,$9,$24
B608 0C 00 1E   .BYTE $C,$0,$1E
B60B 12 27 03   .BYTE $12,$27,$3
B60E 15 18 0F   .BYTE $15,$18,$F
B611 1B 06 57   .BYTE $1B,$6,$57
B614 5A         .BYTE $5A
B615          LB615:
B616          LB616 = * + 1
              ; Instruction parameter jumped to.
B615 AD D6 2B   LDA L2BD6
B618 20 23 B0   JSR LB023
B61B A9 00      LDA #$0
B61D 8D B4 2B   STA L2BB4
B620 8D B5 2B   STA L2BB5
B623 20 A8 DF   JSR LDFA8
B626 A5 83      LDA L83
B628 29 8F      AND #$8F
B62A 10 07      BPL LB633
B62C          LB62C:
B62C 49 8F      EOR #$8F
B62E F0 03      BEQ LB633
B630          LB630:
B630 4C 94 C6   JMP LC694
B633          LB633:
B633 20 AC B7   JSR LB7AC
B636 B1 DC      LDA (LDC),Y
B638 A2 0F      LDX #$F
B63A          LB63A:
B63A DD E8 B5   CMP LB5E8,X
B63D F0 06      BEQ LB645
B63F          LB63F:
B63F CA         DEX
B640 10 F8      BPL LB63A
B642          LB642:
B642 4C 97 DF   JMP LDF97
B645          LB645:
B645 8E E2 2B   STX L2BE2
B648 BD 05 B6   LDA LB605,X
B64B 85 50      STA L50
B64D A9 FF      LDA #$FF
B64F 85 51      STA L51
B651 6C 50 00   JMP (L50)
B654          LB654:
B654 AD DE 2B   LDA L2BDE
B657 F0 03      BEQ LB65C
B659          LB659:
B659 4C 6F B6   JMP LB66F
B65C          LB65C:
B65C A9 00      LDA #$0
B65E A8         TAY
B65F 84 5A      STY L5A
B661          LB661:
B661 84 5B      STY L5B
B663          LB663:
B663 20 B5 DF   JSR LDFB5
B666 20 A9 F5   JSR LF5A9
B669 20 42 EE   JSR LEE42
B66C          LB66C:
B66C 4C 6B DB   JMP LDB6B
B66F          LB66F:
B66F A0 00      LDY #$0
B671 84 5A      STY L5A
B673 84 5B      STY L5B
B675 4C 33 FF   JMP LFF33
B678          LB678:
B678 A0 00      LDY #$0
B67A 20 B8 B6   JSR LB6B8
B67D          LB67D:
B67D 88         DEY
B67E 20 CF B6   JSR LB6CF
B681 D0 0A      BNE LB68D
B683          LB683:
B683 88         DEY
B684 20 CF B6   JSR LB6CF
B687 F0 FA      BEQ LB683
B689          LB689:
B689 C8         INY
B68A 20 90 B6   JSR LB690
B68D          LB68D:
B68D 4C 3C EE   JMP LEE3C
B690          LB690:
B690 20 E9 BA   JSR LBAE9
B693          LB693:
B693 20 9D B6   JSR LB69D
B696 90 1C      BCC LB6B4
B698          LB698:
B698 A9 74      LDA #$74
B69A 4C 6F B6   JMP LB66F
B69D          LB69D:
B69D C9 00      CMP #$0
B69F D0 03      BNE LB6A4
B6A1          LB6A1:
B6A1 AD E8 90   LDA L90E8
B6A4          LB6A4:
B6A4 48         PHA
B6A5 AA         TAX
B6A6 BD 00 82   LDA Partition_Typ+$00,X
B6A9 F0 0A      BEQ LB6B5
B6AB          LB6AB:
B6AB C9 06      CMP #$6
B6AD B0 06      BCS LB6B5
B6AF          LB6AF:
B6AF 68         PLA
B6B0 20 23 B0   JSR LB023
B6B3 18         CLC
B6B4          LB6B4:
B6B4 60         RTS
B6B5          LB6B5:
B6B5 68         PLA
B6B6 38         SEC
B6B7 60         RTS
B6B8          LB6B8:
B6B8 B9 00 02   LDA L200,Y
B6BB C9 3A      CMP #$3A
B6BD F0 0F      BEQ LB6CE
B6BF          LB6BF:
B6BF C9 2C      CMP #$2C
B6C1 F0 09      BEQ LB6CC
B6C3          LB6C3:
B6C3 C9 3D      CMP #$3D
B6C5 F0 05      BEQ LB6CC
B6C7          LB6C7:
B6C7 C8         INY
B6C8 C4 56      CPY L56
B6CA 90 EC      BCC LB6B8
B6CC          LB6CC:
B6CC 09 00      ORA #$0
B6CE          LB6CE:
B6CE 60         RTS
B6CF          LB6CF:
B6CF B9 00 02   LDA L200,Y
B6D2 C9 30      CMP #$30
B6D4 90 07      BCC LB6DD
B6D6          LB6D6:
B6D6 C9 3A      CMP #$3A
B6D8 B0 F2      BCS LB6CC
B6DA          LB6DA:
B6DA D9 00 02   CMP L200,Y
B6DD          LB6DD:
B6DD 60         RTS
B6DE          LB6DE:
B6DE A0 00      LDY #$0
B6E0 A2 00      LDX #$0
B6E2 A9 3A      LDA #$3A
B6E4 4C 61 B7   JMP LB761
B6E7          LB6E7:
B6E7 20 DE B6   JSR LB6DE
B6EA D0 05      BNE LB6F1
B6EC          LB6EC:
B6EC A9 34      LDA #$34
B6EE 4C 6F B6   JMP LB66F
B6F1          LB6F1:
B6F1 88         DEY
B6F2 88         DEY
B6F3 8C 00 2C   STY L2C00
B6F6 8A         TXA
B6F7 D0 F3      BNE LB6EC
B6F9          LB6F9:
B6F9 A9 3D      LDA #$3D
B6FB 20 61 B7   JSR LB761
B6FE 8A         TXA
B6FF F0 02      BEQ LB703
B701          LB701:
B701 A9 40      LDA #$40
B703          LB703:
B703 09 21      ORA #$21
B705 8D E3 2B   STA L2BE3
B708 E8         INX
B709 8E EA 2B   STX L2BEA
B70C 8E EB 2B   STX L2BEB
B70F AD E4 2B   LDA L2BE4
B712 F0 0D      BEQ LB721
B714          LB714:
B714 A9 80      LDA #$80
B716 0D E3 2B   ORA L2BE3
B719 8D E3 2B   STA L2BE3
B71C A9 00      LDA #$0
B71E 8D E4 2B   STA L2BE4
B721          LB721:
B721 98         TYA
B722 F0 29      BEQ LB74D
B724          LB724:
B724 9D 00 2C   STA L2C00,X
B727 AD EA 2B   LDA L2BEA
B72A 8D EC 2B   STA L2BEC
B72D A9 8D      LDA #$8D
B72F 20 61 B7   JSR LB761
B732 E8         INX
B733 8E EB 2B   STX L2BEB
B736 CA         DEX
B737 AD E4 2B   LDA L2BE4
B73A F0 02      BEQ LB73E
B73C          LB73C:
B73C A9 08      LDA #$8
B73E          LB73E:
B73E EC EA 2B   CPX L2BEA
B741 F0 02      BEQ LB745
B743          LB743:
B743 09 04      ORA #$4
B745          LB745:
B745 09 03      ORA #$3
B747 4D E3 2B   EOR L2BE3
B74A 8D E3 2B   STA L2BE3
B74D          LB74D:
B74D AD E3 2B   LDA L2BE3
B750 AE E2 2B   LDX L2BE2
B753 3D F8 B5   AND LB5F8,X
B756 D0 01      BNE LB759
B758          LB758:
B758 60         RTS
B759          LB759:
B759 8D DE 2B   STA L2BDE
B75C A9 30      LDA #$30
B75E 4C 6F B6   JMP LB66F
B761          LB761:
B761 8D E5 2B   STA L2BE5
B764          LB764:
B764 C4 56      CPY L56
B766 B0 2F      BCS LB797
B768          LB768:
B768 B1 DC      LDA (LDC),Y
B76A C8         INY
B76B CD E5 2B   CMP L2BE5
B76E F0 29      BEQ LB799
B770          LB770:
B770 C9 2A      CMP #$2A
B772 F0 04      BEQ LB778
B774          LB774:
B774 C9 3F      CMP #$3F
B776 D0 03      BNE LB77B
B778          LB778:
B778 EE E4 2B   INC L2BE4
B77B          LB77B:
B77B C9 2C      CMP #$2C
B77D D0 E5      BNE LB764
B77F          LB77F:
B77F 98         TYA
B780 9D 01 2C   STA L2C01,X
B783 AD E4 2B   LDA L2BE4
B786 29 7F      AND #$7F
B788 F0 08      BEQ LB792
B78A          LB78A:
B78A A9 80      LDA #$80
B78C 9D 18 2C   STA L2C18,X
B78F 8D E4 2B   STA L2BE4
B792          LB792:
B792 E8         INX
B793 E0 05      CPX #$5
B795 90 CD      BCC LB764
B797          LB797:
B797 A0 00      LDY #$0
B799          LB799:
B799 A5 56      LDA L56
B79B 9D 01 2C   STA L2C01,X
B79E AD E4 2B   LDA L2BE4
B7A1 29 7F      AND #$7F
B7A3 F0 05      BEQ LB7AA
B7A5          LB7A5:
B7A5 A9 80      LDA #$80
B7A7 9D 18 2C   STA L2C18,X
B7AA          LB7AA:
B7AA 98         TYA
B7AB 60         RTS
B7AC          LB7AC:
B7AC A4 DC      LDY LDC
B7AE F0 36      BEQ LB7E6
B7B0          LB7B0:
B7B0 88         DEY
B7B1 F0 32      BEQ LB7E5
B7B3          LB7B3:
B7B3 AD 00 02   LDA L200
B7B6 C9 55      CMP #$55
B7B8 D0 07      BNE LB7C1
B7BA          LB7BA:
B7BA AD 01 02   LDA L201
B7BD C9 30      CMP #$30
B7BF F0 04      BEQ LB7C5
B7C1          LB7C1:
B7C1 B9 00 02   LDA L200,Y
B7C5          LB7C5 = * + 1
              ; Instruction parameter jumped to.
B7C4 2C A9 00   BIT LA9
B7C7 C9 0D      CMP #$D
B7C9 F0 1B      BEQ LB7E6
B7CB          LB7CB:
B7CB 88         DEY
B7CC AD 00 02   LDA L200
B7CF C9 55      CMP #$55
B7D1 D0 07      BNE LB7DA
B7D3          LB7D3:
B7D3 AD 01 02   LDA L201
B7D6 C9 30      CMP #$30
B7D8 F0 04      BEQ LB7DE
B7DA          LB7DA:
B7DA B9 00 02   LDA L200,Y
B7DE          LB7DE = * + 1
              ; Instruction parameter jumped to.
B7DD 2C A9 00   BIT LA9
B7E0 C9 0D      CMP #$D
B7E2 F0 02      BEQ LB7E6
B7E4          LB7E4:
B7E4 C8         INY
B7E5          LB7E5:
B7E5 C8         INY
B7E6          LB7E6:
B7E6 84 56      STY L56
B7E8 C0 FF      CPY #$FF
B7EA A0 FF      LDY #$FF
B7EC 90 08      BCC LB7F6
B7EE          LB7EE:
B7EE 8C E2 2B   STY L2BE2
B7F1 A9 32      LDA #$32
B7F3 4C 6F B6   JMP LB66F
B7F6          LB7F6:
B7F6 A0 00      LDY #$0
B7F8 98         TYA
B7F9 85 DC      STA LDC
B7FB 8D F3 2B   STA L2BF3
B7FE 8D ED 2B   STA L2BED
B801 8D EE 2B   STA L2BEE
B804 85 97      STA L97
B806 8D EC 2B   STA L2BEC
B809 8D EA 2B   STA L2BEA
B80C 8D EB 2B   STA L2BEB
B80F 8D E4 2B   STA L2BE4
B812 8D DE 2B   STA L2BDE
B815 A2 05      LDX #$5
B817          LB817:
B817 9D FF 2B   STA L2BFF,X
B81A 9D 2F 2C   STA L2C2F,X
B81D 9D 37 2C   STA L2C37,X
B820 9D 3F 2C   STA L2C3F,X
B823 9D 0F 2C   STA L2C0F,X
B826 9D 17 2C   STA L2C17,X
B829 9D 1F 2C   STA L2C1F,X
B82C 9D 27 2C   STA L2C27,X
B82F CA         DEX
B830 D0 E5      BNE LB817
B832          LB832:
B832 60         RTS
B833          LB833:
B833 20 43 B8   JSR LB843
B836 90 0A      BCC LB842
B838          LB838:
B838 A9 74      LDA #$74
B83A 4C 6F B6   JMP LB66F
B83D          LB83D:
B83D 20 51 B8   JSR LB851
B840 B0 F6      BCS LB838
B842          LB842:
B842 60         RTS
B843          LB843:
B843 AD EB 2B   LDA L2BEB
B846 8D EA 2B   STA L2BEA
B849 A9 01      LDA #$1
B84B 8D EB 2B   STA L2BEB
B84E 8D EC 2B   STA L2BEC
B851          LB851:
B851 A2 00      LDX #$0
B853          LB853:
B853 86 97      STX L97
B855 20 66 B8   JSR LB866
B858 A6 97      LDX L97
B85A E8         INX
B85B EC EB 2B   CPX L2BEB
B85E 90 F3      BCC LB853
B860          LB860:
B860 AD 10 2C   LDA L2C10
B863 4C 9D B6   JMP LB69D
B866          LB866:
B866 AD E8 90   LDA L90E8
B869 E0 00      CPX #$0
B86B F0 03      BEQ LB870
B86D          LB86D:
B86D AD 10 2C   LDA L2C10
B870          LB870:
B870 9D 10 2C   STA L2C10,X
B873 BD 00 2C   LDA L2C00,X
B876 9D 08 2C   STA L2C08,X
B879 E8         INX
B87A BC 00 2C   LDY L2C00,X
B87D 84 50      STY L50
B87F AA         TAX
B880 A8         TAY
B881          LB881:
B881 BD 00 02   LDA L200,X
B884 C9 3A      CMP #$3A
B886 F0 0E      BEQ LB896
B888          LB888:
B888 C9 3D      CMP #$3D
B88A F0 09      BEQ LB895
B88C          LB88C:
B88C C9 2C      CMP #$2C
B88E F0 05      BEQ LB895
B890          LB890:
B890 E8         INX
B891 E4 50      CPX L50
B893 90 EC      BCC LB881
B895          LB895:
B895 60         RTS
B896          LB896:
B896 B9 00 02   LDA L200,Y
B899 C9 3E      CMP #$3E
B89B F0 F8      BEQ LB895
B89D          LB89D:
B89D C9 3C      CMP #$3C
B89F F0 F4      BEQ LB895
B8A1          LB8A1:
B8A1 E8         INX
B8A2 8A         TXA
B8A3 48         PHA
B8A4 A6 97      LDX L97
B8A6 9D 08 2C   STA L2C08,X
B8A9 A8         TAY
B8AA 88         DEY
B8AB F0 3E      BEQ LB8EB
B8AD          LB8AD:
B8AD 88         DEY
B8AE B9 00 02   LDA L200,Y
B8B1 C9 2F      CMP #$2F
B8B3 D0 20      BNE LB8D5
B8B5          LB8B5:
B8B5 B9 00 02   LDA L200,Y
B8B8 C9 2F      CMP #$2F
B8BA D0 06      BNE LB8C2
B8BC          LB8BC:
B8BC 98         TYA
B8BD 9D 08 2C   STA L2C08,X
B8C0 A9 2F      LDA #$2F
B8C2          LB8C2:
B8C2 C9 3D      CMP #$3D
B8C4 F0 09      BEQ LB8CF
B8C6          LB8C6:
B8C6 C9 2C      CMP #$2C
B8C8 F0 05      BEQ LB8CF
B8CA          LB8CA:
B8CA 88         DEY
B8CB C0 FF      CPY #$FF
B8CD D0 E6      BNE LB8B5
B8CF          LB8CF:
B8CF BC 08 2C   LDY L2C08,X
B8D2 F0 17      BEQ LB8EB
B8D4          LB8D4:
B8D4 88         DEY
B8D5          LB8D5:
B8D5 20 CF B6   JSR LB6CF
B8D8 D0 11      BNE LB8EB
B8DA          LB8DA:
B8DA 88         DEY
B8DB C0 FF      CPY #$FF
B8DD F0 05      BEQ LB8E4
B8DF          LB8DF:
B8DF 20 CF B6   JSR LB6CF
B8E2 F0 F6      BEQ LB8DA
B8E4          LB8E4:
B8E4 C8         INY
B8E5 20 E9 BA   JSR LBAE9
B8E8 A8         TAY
B8E9 D0 03      BNE LB8EE
B8EB          LB8EB:
B8EB AD E8 90   LDA L90E8
B8EE          LB8EE:
B8EE A6 97      LDX L97
B8F0 9D 10 2C   STA L2C10,X
B8F3 68         PLA
B8F4 9D 00 2C   STA L2C00,X
B8F7 60         RTS
B8F8          LB8F8:
B8F8 A0 00      LDY #$0
B8FA AD EA 2B   LDA L2BEA
B8FD CD EB 2B   CMP L2BEB
B900 F0 20      BEQ LB922
B902          LB902:
B902 CE EB 2B   DEC L2BEB
B905 AC EB 2B   LDY L2BEB
B908          LB908:
B908 B9 00 2C   LDA L2C00,Y
B90B A8         TAY
B90C B1 DC      LDA (LDC),Y
B90E AC E8 90   LDY L90E8
B911 F0 14      BEQ LB927
B913          LB913:
B913 A0 06      LDY #$6
B915 C9 42      CMP #$42
B917 F0 09      BEQ LB922
B919          LB919:
B919 88         DEY
B91A          LB91A:
B91A D9 92 C2   CMP LC292,Y
B91D F0 03      BEQ LB922
B91F          LB91F:
B91F 88         DEY
B920 D0 F8      BNE LB91A
B922          LB922:
B922 98         TYA
B923 8D EE 2B   STA L2BEE
B926 60         RTS
B927          LB927:
B927 A0 07      LDY #$7
B929          LB929:
B929 D9 99 C2   CMP LC299,Y
B92C F0 F4      BEQ LB922
B92E          LB92E:
B92E 88         DEY
B92F D0 F8      BNE LB929
B931          LB931:
B931 F0 EF      BEQ LB922
B933          LB933:
B933 AD 01 02   LDA L201
B936 C9 50      CMP #$50
B938 F0 11      BEQ LB94B
B93A          LB93A:
B93A C9 D0      CMP #$D0
B93C F0 07      BEQ LB945
B93E          LB93E:
B93E C9 44      CMP #$44
B940 F0 39      BEQ LB97B
B942          LB942:
B942 4C 21 AC   JMP LAC21
B945          LB945:
B945 AD 02 02   LDA L202
B948 4C 5E B9   JMP LB95E
B94B          LB94B:
B94B A5 56      LDA L56
B94D C9 02      CMP #$2
B94F D0 08      BNE LB959
B951          LB951:
B951 AD E3 90   LDA L90E3
B954 85 5A      STA L5A
B956 4C 74 B9   JMP LB974
B959          LB959:
B959 A0 02      LDY #$2
B95B 20 E9 BA   JSR LBAE9
B95E          LB95E:
B95E AA         TAX
B95F 48         PHA
B960 85 5A      STA L5A
B962 BD 00 82   LDA Partition_Typ+$00,X
B965 F0 04      BEQ LB96B
B967          LB967:
B967 C9 FF      CMP #$FF
B969 D0 05      BNE LB970
B96B          LB96B:
B96B A9 77      LDA #$77
B96D 4C 33 FF   JMP LFF33
B970          LB970:
B970 68         PLA
B971 20 51 F7   JSR LF751
B974          LB974:
B974 A0 00      LDY #$0
B976 A9 02      LDA #$2
B978 4C 61 B6   JMP LB661
B97B          LB97B:
B97B 20 DE B6   JSR LB6DE
B97E F0 3A      BEQ LB9BA
B980          LB980:
B980 88         DEY
B981 88         DEY
B982 8C 00 2C   STY L2C00
B985 20 33 B8   JSR LB833
B988 20 85 B0   JSR LB085
B98B D0 4E      BNE LB9DB
B98D          LB98D:
B98D AC 08 2C   LDY L2C08
B990 CC 00 2C   CPY L2C00
B993 D0 60      BNE LB9F5
B995          LB995:
B995 C8         INY
B996 C4 56      CPY L56
B998 D0 5B      BNE LB9F5
B99A          LB99A:
B99A 88         DEY
B99B B9 00 02   LDA L200,Y
B99E C9 5F      CMP #$5F
B9A0 F0 0A      BEQ LB9AC
B9A2          LB9A2:
B9A2 C9 2F      CMP #$2F
B9A4 D0 4F      BNE LB9F5
B9A6          LB9A6:
B9A6 20 10 B0   JSR LB010
B9A9          LB9A9:
B9A9 4C 5C B6   JMP LB65C
B9AC          LB9AC:
B9AC 20 7E A1   JSR LA17E
B9AF AD 22 22   LDA L2222
B9B2 F0 F5      BEQ LB9A9
B9B4          LB9B4:
B9B4 AC 23 22   LDY L2223
B9B7 4C 0A BA   JMP LBA0A
B9BA          LB9BA:
B9BA A5 56      LDA L56
B9BC C9 03      CMP #$3
B9BE D0 10      BNE LB9D0
B9C0          LB9C0:
B9C0 20 85 B0   JSR LB085
B9C3 D0 16      BNE LB9DB
B9C5          LB9C5:
B9C5 AD 02 02   LDA L202
B9C8 C9 5F      CMP #$5F
B9CA F0 E0      BEQ LB9AC
B9CC          LB9CC:
B9CC C9 2F      CMP #$2F
B9CE F0 D6      BEQ LB9A6
B9D0          LB9D0:
B9D0 A2 00      LDX #$0
B9D2 A0 02      LDY #$2
B9D4 A9 2F      LDA #$2F
B9D6 20 61 B7   JSR LB761
B9D9 D0 03      BNE LB9DE
B9DB          LB9DB:
B9DB 4C 94 DF   JMP LDF94
B9DE          LB9DE:
B9DE 88         DEY
B9DF 8C 08 2C   STY L2C08
B9E2 20 7D B6   JSR LB67D
B9E5 AD E8 90   LDA L90E8
B9E8 8D 10 2C   STA L2C10
B9EB 20 85 B0   JSR LB085
B9EE D0 EB      BNE LB9DB
B9F0          LB9F0:
B9F0 A9 00      LDA #$0
B9F2 8D 00 2C   STA L2C00
B9F5          LB9F5:
B9F5 A9 01      LDA #$1
B9F7 8D EB 2B   STA L2BEB
B9FA A9 00      LDA #$0
B9FC 20 20 BA   JSR LBA20
B9FF AD 00 2C   LDA L2C00
BA02 D0 0C      BNE LBA10
BA04          LBA04:
BA04 AD A7 2B   LDA L2BA7
BA07 AC A8 2B   LDY L2BA8
BA0A          LBA0A:
BA0A 20 13 B0   JSR LB013
BA0D 4C 5C B6   JMP LB65C
BA10          LBA10:
BA10 20 D9 BE   JSR LBED9
BA13 AC 28 2C   LDY L2C28
BA16 AD 20 2C   LDA L2C20
BA19 D0 EF      BNE LBA0A
BA1B          LBA1B:
BA1B A9 39      LDA #$39
BA1D 4C 6F B6   JMP LB66F
BA20          LBA20:
BA20 8D CD 2B   STA L2BCD
BA23 20 26 B0   JSR LB026
BA26 20 85 B0   JSR LB085
BA29 D0 0B      BNE LBA36
BA2B          LBA2B:
BA2B AE CD 2B   LDX L2BCD
BA2E BD 08 2C   LDA L2C08,X
BA31 DD 00 2C   CMP L2C00,X
BA34 D0 01      BNE LBA37
BA36          LBA36:
BA36 60         RTS
BA37          LBA37:
BA37 8D CC 2B   STA L2BCC
BA3A AD B4 2B   LDA L2BB4
BA3D 48         PHA
BA3E AD B5 2B   LDA L2BB5
BA41 48         PHA
BA42 BD 18 2C   LDA L2C18,X
BA45 48         PHA
BA46 BD 00 2C   LDA L2C00,X
BA49 48         PHA
BA4A AD EE 2B   LDA L2BEE
BA4D 48         PHA
BA4E BD 20 2C   LDA L2C20,X
BA51 48         PHA
BA52 A5 82      LDA L82
BA54 48         PHA
BA55 A9 06      LDA #$6
BA57 8D EE 2B   STA L2BEE
BA5A 8D B4 2B   STA L2BB4
BA5D 8D B5 2B   STA L2BB5
BA60          LBA60:
BA60 EE CC 2B   INC L2BCC
BA63 AE CC 2B   LDX L2BCC
BA66 E4 56      CPX L56
BA68 B0 60      BCS LBACA
BA6A          LBA6A:
BA6A BD 00 02   LDA L200,X
BA6D C9 3A      CMP #$3A
BA6F F0 59      BEQ LBACA
BA71          LBA71:
BA71 C9 2F      CMP #$2F
BA73 D0 0F      BNE LBA84
BA75          LBA75:
BA75 A9 01      LDA #$1
BA77 8D A7 2B   STA L2BA7
BA7A 8D A8 2B   STA L2BA8
BA7D A9 22      LDA #$22
BA7F 8D A9 2B   STA L2BA9
BA82 D0 DC      BNE LBA60
BA84          LBA84:
BA84 8A         TXA
BA85 AC CD 2B   LDY L2BCD
BA88 99 00 2C   STA L2C00,Y
BA8B          LBA8B:
BA8B E8         INX
BA8C E4 56      CPX L56
BA8E B0 07      BCS LBA97
BA90          LBA90:
BA90 BD 00 02   LDA L200,X
BA93 C9 2F      CMP #$2F
BA95 D0 F4      BNE LBA8B
BA97          LBA97:
BA97 A5 56      LDA L56
BA99 48         PHA
BA9A 8E CC 2B   STX L2BCC
BA9D 86 56      STX L56
BA9F A9 00      LDA #$0
BAA1 99 20 2C   STA L2C20,Y
BAA4 20 84 BE   JSR LBE84
BAA7 20 15 BF   JSR LBF15
BAAA F0 03      BEQ LBAAF
BAAC          LBAAC:
BAAC 4C 1B BA   JMP LBA1B
BAAF          LBAAF:
BAAF 68         PLA
BAB0 85 56      STA L56
BAB2 AC CD 2B   LDY L2BCD
BAB5 B9 20 2C   LDA L2C20,Y
BAB8 8D A7 2B   STA L2BA7
BABB B9 28 2C   LDA L2C28,Y
BABE 8D A8 2B   STA L2BA8
BAC1 18         CLC
BAC2 69 01      ADC #$1
BAC4 8D A9 2B   STA L2BA9
BAC7 4C 60 BA   JMP LBA60
BACA          LBACA:
BACA AE CD 2B   LDX L2BCD
BACD 68         PLA
BACE 85 82      STA L82
BAD0 68         PLA
BAD1 9D 20 2C   STA L2C20,X
BAD4 68         PLA
BAD5 8D EE 2B   STA L2BEE
BAD8 68         PLA
BAD9 9D 00 2C   STA L2C00,X
BADC 68         PLA
BADD 9D 18 2C   STA L2C18,X
BAE0 68         PLA
BAE1 8D B5 2B   STA L2BB5
BAE4 68         PLA
BAE5 8D B4 2B   STA L2BB4
BAE8 60         RTS
BAE9          LBAE9:
BAE9 08         PHP
BAEA 78         SEI
BAEB 98         TYA
BAEC 48         PHA
BAED A2 00      LDX #$0
BAEF          LBAEF:
BAEF B9 00 02   LDA L200,Y
BAF2 C9 30      CMP #$30
BAF4 90 0C      BCC LBB02
BAF6          LBAF6:
BAF6 C9 3A      CMP #$3A
BAF8 B0 08      BCS LBB02
BAFA          LBAFA:
BAFA C4 56      CPY L56
BAFC B0 04      BCS LBB02
BAFE          LBAFE:
BAFE C8         INY
BAFF E8         INX
BB00 D0 ED      BNE LBAEF
BB02          LBB02:
BB02 CA         DEX
BB03 E0 03      CPX #$3
BB05 90 03      BCC LBB0A
BB07          LBB07:
BB07 4C 94 DF   JMP LDF94
BB0A          LBB0A:
BB0A 68         PLA
BB0B A8         TAY
BB0C A9 00      LDA #$0
BB0E 8D 65 2A   STA L2A65
BB11          LBB11:
BB11 B9 00 02   LDA L200,Y
BB14 29 0F      AND #$F
BB16 8D 64 2A   STA L2A64
BB19 F0 11      BEQ LBB2C
BB1B          LBB1B:
BB1B 18         CLC
BB1C AD 65 2A   LDA L2A65
BB1F          LBB1F:
BB1F 7D 35 BB   ADC LBB35,X
BB22 B0 E3      BCS LBB07
BB24          LBB24:
BB24 CE 64 2A   DEC L2A64
BB27 D0 F6      BNE LBB1F
BB29          LBB29:
BB29 8D 65 2A   STA L2A65
BB2C          LBB2C:
BB2C C8         INY
BB2D CA         DEX
BB2E 10 E1      BPL LBB11
BB30          LBB30:
BB30 AD 65 2A   LDA L2A65
BB33 28         PLP
BB34 60         RTS
BB35          LBB35:
BB35 01 0A 64   .BYTE $1,$A,$64
BB38          LBB38:
BB38 A9 01      LDA #$1
BB3A 8D 00 2C   STA L2C00
BB3D A5 56      LDA L56
BB3F 8D 01 2C   STA L2C01
BB42 20 33 B8   JSR LB833
BB45 20 7E B0   JSR LB07E
BB48 C9 04      CMP #$4
BB4A F0 07      BEQ LBB53
BB4C          LBB4C:
BB4C C9 05      CMP #$5
BB4E F0 03      BEQ LBB53
BB50          LBB50:
BB50 4C 97 DF   JMP LDF97
BB53          LBB53:
BB53 20 D0 AE   JSR LAED0
BB56 AD 00 2C   LDA L2C00
BB59 C5 56      CMP L56
BB5B F0 61      BEQ LBBBE
BB5D          LBB5D:
BB5D 20 CF BE   JSR LBECF
BB60 AD 20 2C   LDA L2C20
BB63 F0 13      BEQ LBB78
BB65          LBB65:
BB65 20 F5 BB   JSR LBBF5
BB68 90 20      BCC LBB8A
BB6A          LBB6A:
BB6A A9 63      LDA #$63
BB6D          LBB6D = * + 1
              ; Instruction parameter jumped to.
BB6C 2C A9 62   BIT L62A9
BB70          LBB70 = * + 1
              ; Instruction parameter jumped to.
BB6F 2C A9 30   BIT L30A9
BB73          LBB73 = * + 1
              ; Instruction parameter jumped to.
BB72 2C A9 77   BIT L77A9
BB75 20 6F B6   JSR LB66F
BB78          LBB78:
BB78 20 F5 BB   JSR LBBF5
BB7B 90 F0      BCC LBB6D
BB7D          LBB7D:
BB7D AE EF 2B   LDX L2BEF
BB80 BD 06 02   LDA L206,X
BB83 C9 43      CMP #$43
BB85 D0 E9      BNE LBB70
BB87          LBB87:
BB87 4C 31 BC   JMP LBC31
BB8A          LBB8A:
BB8A AD 18 2C   LDA L2C18
BB8D 29 07      AND #$7
BB8F C9 05      CMP #$5
BB91 D0 DA      BNE LBB6D
BB93          LBB93:
BB93 20 AB BC   JSR LBCAB
BB96          LBB96:
BB96 20 1C D9   JSR LD91C
BB99 20 76 BC   JSR LBC76
BB9C D0 F8      BNE LBB96
BB9E          LBB9E:
BB9E 90 D3      BCC LBB73
BBA0          LBBA0:
BBA0 A0 02      LDY #$2
BBA2 B1 94      LDA (L94),Y
BBA4 D0 CD      BNE LBB73
BBA6          LBBA6:
BBA6 88         DEY
BBA7 A5 5A      LDA L5A
BBA9 AA         TAX
BBAA F1 94      SBC (L94),Y
BBAC C9 02      CMP #$2
BBAE F0 C3      BEQ LBB73
BBB0          LBBB0:
BBB0 90 C1      BCC LBB73
BBB2          LBBB2:
BBB2 B1 94      LDA (L94),Y
BBB4 48         PHA
BBB5 8A         TXA
BBB6 A8         TAY
BBB7 68         PLA
BBB8 20 13 B0   JSR LB013
BBBB 4C C1 BB   JMP LBBC1
BBBE          LBBBE:
BBBE 20 F4 AF   JSR LAFF4
BBC1          LBBC1:
BBC1 20 26 DB   JSR LDB26
BBC4 20 03 AF   JSR LAF03
BBC7 AD C7 2B   LDA L2BC7
BBCA 85 5A      STA L5A
BBCC AC C8 2B   LDY L2BC8
BBCF 88         DEY
BBD0 84 5B      STY L5B
BBD2 A9 02      LDA #$2
BBD4 A0 00      LDY #$0
BBD6 4C 63 B6   JMP LB663
BBD9          LBBD9:
BBD9 20 03 BC   JSR LBC03
BBDC          LBBDC:
BBDC 20 1C D9   JSR LD91C
BBDF A5 5A      LDA L5A
BBE1 C9 28      CMP #$28
BBE3 F0 0B      BEQ LBBF0
BBE5          LBBE5:
BBE5 20 39 A5   JSR LA539
BBE8 F0 06      BEQ LBBF0
BBEA          LBBEA:
BBEA 20 76 BC   JSR LBC76
BBED D0 ED      BNE LBBDC
BBEF          LBBEF:
BBEF 60         RTS
BBF0          LBBF0:
BBF0 A9 67      LDA #$67
BBF2 4C 33 FF   JMP LFF33
BBF5          LBBF5:
BBF5 A2 01      LDX #$1
BBF7 20 56 C1   JSR LC156
BBFA A5 56      LDA L56
BBFC 38         SEC
BBFD ED EF 2B   SBC L2BEF
BC00 C9 04      CMP #$4
BC02 60         RTS
BC03          LBC03:
BC03 AC EF 2B   LDY L2BEF
BC06 C8         INY
BC07 B9 00 02   LDA L200,Y
BC0A 85 5A      STA L5A
BC0C C8         INY
BC0D B9 00 02   LDA L200,Y
BC10 85 5B      STA L5B
BC12 C8         INY
BC13 B9 00 02   LDA L200,Y
BC16 8D A6 2B   STA L2BA6
BC19 C8         INY
BC1A B9 00 02   LDA L200,Y
BC1D 8D A5 2B   STA L2BA5
BC20 18         CLC
BC21 AD A6 2B   LDA L2BA6
BC24 6D A5 2B   ADC L2BA5
BC27 F0 03      BEQ LBC2C
BC29          LBC29:
BC29 4C 1C D9   JMP LD91C
BC2C          LBC2C:
BC2C A9 77      LDA #$77
BC2E 20 6F B6   JSR LB66F
BC31          LBC31:
BC31 20 D9 BB   JSR LBBD9
BC34 A9 05      LDA #$5
BC36 8D ED 2B   STA L2BED
BC39 A9 12      LDA #$12
BC3B 85 82      STA L82
BC3D 20 03 BC   JSR LBC03
BC40 20 C0 CB   JSR LCBC0
BC43 20 BD C3   JSR LC3BD
BC46 20 03 BC   JSR LBC03
BC49          LBC49:
BC49 20 1C D9   JSR LD91C
BC4C A5 5A      LDA L5A
BC4E 20 5C A3   JSR LA35C
BC51 20 76 BC   JSR LBC76
BC54 D0 F3      BNE LBC49
BC56          LBC56:
BC56 20 03 BC   JSR LBC03
BC59 A6 80      LDX L80
BC5B AD A6 2B   LDA L2BA6
BC5E 9D 48 2D   STA L2D48,X
BC61 AD A5 2B   LDA L2BA5
BC64 9D 68 2D   STA L2D68,X
BC67 A9 00      LDA #$0
BC69 20 EA CE   JSR LCEEA
BC6C A9 12      LDA #$12
BC6E 85 82      STA L82
BC70 20 1C CD   JSR LCD1C
BC73 4C 54 B6   JMP LB654
BC76          LBC76:
BC76 AD A6 2B   LDA L2BA6
BC79 D0 08      BNE LBC83
BC7B          LBC7B:
BC7B AD A5 2B   LDA L2BA5
BC7E F0 1E      BEQ LBC9E
BC80          LBC80:
BC80 CE A5 2B   DEC L2BA5
BC83          LBC83:
BC83 CE A6 2B   DEC L2BA6
BC86 E6 5B      INC L5B
BC88 AD C9 2B   LDA L2BC9
BC8B C5 5B      CMP L5B
BC8D D0 0F      BNE LBC9E
BC8F          LBC8F:
BC8F A9 00      LDA #$0
BC91 85 5B      STA L5B
BC93 A5 5A      LDA L5A
BC95 CD A7 2B   CMP L2BA7
BC98 F0 0C      BEQ LBCA6
BC9A          LBC9A:
BC9A E6 5A      INC L5A
BC9C 38         SEC
BC9E          LBC9E = * + 1
              ; Instruction parameter jumped to.
BC9D 24 18      BIT L18
BC9F AD A5 2B   LDA L2BA5
BCA2 0D A6 2B   ORA L2BA6
BCA5 60         RTS
BCA6          LBCA6:
BCA6 A9 67      LDA #$67
BCA8 4C 33 FF   JMP LFF33
BCAB          LBCAB:
BCAB A0 01      LDY #$1
BCAD B1 94      LDA (L94),Y
BCAF 85 5A      STA L5A
BCB1 C8         INY
BCB2 B1 94      LDA (L94),Y
BCB4 85 5B      STA L5B
BCB6 A0 1C      LDY #$1C
BCB8 B1 94      LDA (L94),Y
BCBA 8D A6 2B   STA L2BA6
BCBD C8         INY
BCBE B1 94      LDA (L94),Y
BCC0 8D A5 2B   STA L2BA5
BCC3 60         RTS
BCC4          LBCC4:
BCC4 20 1C D9   JSR LD91C
BCC7 20 5C A3   JSR LA35C
BCCA 20 76 BC   JSR LBC76
BCCD D0 F5      BNE LBCC4
BCCF          LBCCF:
BCCF 60         RTS
BCD0          LBCD0:
BCD0 AD 01 02   LDA L201
BCD3 C9 44      CMP #$44
BCD5 F0 03      BEQ LBCDA
BCD7          LBCD7:
BCD7 4C 9C B0   JMP LB09C
BCDA          LBCDA:
BCDA 20 F5 BD   JSR LBDF5
BCDD D0 F8      BNE LBCD7
BCDF          LBCDF:
BCDF 20 84 BE   JSR LBE84
BCE2 20 81 A4   JSR LA481
BCE5 A5 5A      LDA L5A
BCE7 8D 20 2C   STA L2C20
BCEA A5 5B      LDA L5B
BCEC 8D 28 2C   STA L2C28
BCEF          LBCEF:
BCEF A5 5A      LDA L5A
BCF1 8D CA 2B   STA L2BCA
BCF4 A5 5B      LDA L5B
BCF6 8D CB 2B   STA L2BCB
BCF9 20 FF A4   JSR LA4FF
BCFC A5 5B      LDA L5B
BCFE 48         PHA
BCFF A5 5A      LDA L5A
BD01 48         PHA
BD02 CD CA 2B   CMP L2BCA
BD05 D0 08      BNE LBD0F
BD07          LBD07:
BD07 AE CB 2B   LDX L2BCB
BD0A E8         INX
BD0B E4 5B      CPX L5B
BD0D F0 26      BEQ LBD35
BD0F          LBD0F:
BD0F AD CA 2B   LDA L2BCA
BD12 85 5A      STA L5A
BD14 AD CB 2B   LDA L2BCB
BD17 85 5B      STA L5B
BD19 20 91 A3   JSR LA391
BD1C 68         PLA
BD1D AA         TAX
BD1E 85 5A      STA L5A
BD20 68         PLA
BD21 85 5B      STA L5B
BD23 EC 20 2C   CPX L2C20
BD26 D0 C7      BNE LBCEF
BD28          LBD28:
BD28 CD 28 2C   CMP L2C28
BD2B D0 C2      BNE LBCEF
BD2D          LBD2D:
BD2D 20 91 A3   JSR LA391
BD30 A9 65      LDA #$65
BD32 4C 6F B6   JMP LB66F
BD35          LBD35:
BD35 68         PLA
BD36 68         PLA
BD37 A9 00      LDA #$0
BD39 8D 20 2C   STA L2C20
BD3C 20 20 BA   JSR LBA20
BD3F AD A8 2B   LDA L2BA8
BD42 48         PHA
BD43 AD A7 2B   LDA L2BA7
BD46 48         PHA
BD47 20 D9 BE   JSR LBED9
BD4A AD 20 2C   LDA L2C20
BD4D F0 05      BEQ LBD54
BD4F          LBD4F:
BD4F A9 63      LDA #$63
BD51 4C 6F B6   JMP LB66F
BD54          LBD54:
BD54 A9 06      LDA #$6
BD56 8D ED 2B   STA L2BED
BD59 AD CA 2B   LDA L2BCA
BD5C 85 5A      STA L5A
BD5E AD CB 2B   LDA L2BCB
BD61 85 5B      STA L5B
BD63 20 BD C3   JSR LC3BD
BD66 A6 80      LDX L80
BD68 A9 02      LDA #$2
BD6A 9D 48 2D   STA L2D48,X
BD6D A9 00      LDA #$0
BD6F 9D 68 2D   STA L2D68,X
BD72 20 F1 CD   JSR LCDF1
BD75 20 48 A3   JSR LA348
BD78 AE CB 2B   LDX L2BCB
BD7B 8E A8 2B   STX L2BA8
BD7E E8         INX
BD7F 8E A9 2B   STX L2BA9
BD82 AD CA 2B   LDA L2BCA
BD85 8D A7 2B   STA L2BA7
BD88 20 4B A7   JSR LA74B
BD8B 68         PLA
BD8C 8D 22 22   STA L2222
BD8F 68         PLA
BD90 8D 23 22   STA L2223
BD93 AD 30 2C   LDA L2C30
BD96 8D 24 22   STA L2224
BD99 AD 38 2C   LDA L2C38
BD9C 8D 25 22   STA L2225
BD9F AD 40 2C   LDA L2C40
BDA2 8D 26 22   STA L2226
BDA5 20 81 A1   JSR LA181
BDA8 20 D8 A7   JSR LA7D8
BDAB 4C 99 A1   JMP LA199
BDAE          LBDAE:
BDAE AD 01 02   LDA L201
BDB1 C9 44      CMP #$44
BDB3 F0 03      BEQ LBDB8
BDB5          LBDB5:
BDB5 4C 2D B1   JMP LB12D
BDB8          LBDB8:
BDB8 20 F5 BD   JSR LBDF5
BDBB D0 F8      BNE LBDB5
BDBD          LBDBD:
BDBD AD 08 2C   LDA L2C08
BDC0 48         PHA
BDC1 AE 00 2C   LDX L2C00
BDC4 CA         DEX
BDC5 8E 08 2C   STX L2C08
BDC8 A9 2F      LDA #$2F
BDCA 9D 00 02   STA L200,X
BDCD A9 00      LDA #$0
BDCF 20 20 BA   JSR LBA20
BDD2 68         PLA
BDD3 8D 08 2C   STA L2C08
BDD6 A9 00      LDA #$0
BDD8 8D BC 2B   STA L2BBC
BDDB 20 7C C0   JSR LC07C
BDDE F0 09      BEQ LBDE9
BDE0          LBDE0:
BDE0 A0 00      LDY #$0
BDE2 84 5A      STY L5A
BDE4 A9 01      LDA #$1
BDE6 4C 61 B6   JMP LB661
BDE9          LBDE9:
BDE9 AE 00 2C   LDX L2C00
BDEC CA         DEX
BDED A9 3A      LDA #$3A
BDEF 9D 00 02   STA L200,X
BDF2 4C 69 B2   JMP LB269
BDF5          LBDF5:
BDF5 A9 03      LDA #$3
BDF7 8D E2 2B   STA L2BE2
BDFA 20 E7 B6   JSR LB6E7
BDFD 20 33 B8   JSR LB833
BE00 4C 85 B0   JMP LB085
BE03          LBE03:
BE03 A2 01      LDX #$1
BE05          LBE05:
BE05 BD 00 02   LDA L200,X
BE08 DD 19 BE   CMP LBE19,X
BE0B D0 10      BNE LBE1D
BE0D          LBE0D:
BE0D E8         INX
BE0E E0 04      CPX #$4
BE10 90 F3      BCC LBE05
BE12          LBE12:
BE12 A2 01      LDX #$1
BE14 20 6C F7   JSR LF76C
BE19          LBE19 = * + 2
BE17 4C 5C B6   JMP LB65C
BE1A 45 4F 53   .BYTE $45,$4F,$53
BE1D          LBE1D:
BE1D AD 01 02   LDA L201
BE20 C9 2D      CMP #$2D
BE22 D0 07      BNE LBE2B
BE24          LBE24:
BE24 AD 02 02   LDA L202
BE27 C9 50      CMP #$50
BE29 F0 03      BEQ LBE2E
BE2B          LBE2B:
BE2B 4C 97 DF   JMP LDF97
BE2E          LBE2E:
BE2E A5 56      LDA L56
BE30 C9 04      CMP #$4
BE32 90 07      BCC LBE3B
BE34          LBE34:
BE34 AD 03 02   LDA L203
BE37 C9 FF      CMP #$FF
BE39 D0 03      BNE LBE3E
BE3B          LBE3B:
BE3B AD E8 90   LDA L90E8
BE3E          LBE3E:
BE3E 48         PHA
BE3F 4A         LSR A
BE40 4A         LSR A
BE41 4A         LSR A
BE42 20 0F F6   JSR LF60F
BE45 90 05      BCC LBE4C
BE47          LBE47:
BE47 A9 78      LDA #$78
BE49 4C 36 FF   JMP LFF36
BE4C          LBE4C:
BE4C 68         PLA
BE4D 48         PHA
BE4E 29 07      AND #$7
BE50 0A         ASL A
BE51 0A         ASL A
BE52 0A         ASL A
BE53 0A         ASL A
BE54 0A         ASL A
BE55 18         CLC
BE56 69 02      ADC #$2
BE58 85 68      STA L68
BE5A A0 00      LDY #$0
BE5C B1 68      LDA (L68),Y
BE5E 8D E7 2D   STA L2DE7
BE61          LBE61:
BE61 B1 68      LDA (L68),Y
BE63 99 00 23   STA L2300,Y
BE66 C8         INY
BE67 C0 1E      CPY #$1E
BE69 90 F6      BCC LBE61
BE6B          LBE6B:
BE6B 68         PLA
BE6C A0 02      LDY #$2
BE6E 99 00 23   STA L2300,Y
BE71 A9 1D      LDA #$1D
BE73 18         CLC
BE74 69 00      ADC #$0
BE76 8D 07 2E   STA L2E07
BE79 20 B2 F5   JSR LF5B2
BE7C E6 DE      INC LDE
BE7E A9 88      LDA #$88
BE80 8D C7 2D   STA L2DC7
BE83 60         RTS
BE84          LBE84:
BE84 A9 00      LDA #$0
BE86 85 50      STA L50
BE88 20 D0 AE   JSR LAED0
BE8B F0 05      BEQ LBE92
BE8D          LBE8D:
BE8D A9 74      LDA #$74
BE8F 4C 6F B6   JMP LB66F
BE92          LBE92:
BE92 4C 3C EE   JMP LEE3C
BE95          LBE95:
BE95 AE EB 2B   LDX L2BEB
BE98 CA         DEX
BE99          LBE99:
BE99 8E BD 2B   STX L2BBD
BE9C BD 10 2C   LDA L2C10,X
BE9F F0 0F      BEQ LBEB0
BEA1          LBEA1:
BEA1 20 B4 BE   JSR LBEB4
BEA4 20 23 B0   JSR LB023
BEA7 AD BD 2B   LDA L2BBD
BEAA 20 D1 BE   JSR LBED1
BEAD 20 B4 BE   JSR LBEB4
BEB0          LBEB0:
BEB0 CA         DEX
BEB1 10 E6      BPL LBE99
BEB3          LBEB3:
BEB3 60         RTS
BEB4          LBEB4:
BEB4 AE BD 2B   LDX L2BBD
BEB7 BD 10 2C   LDA L2C10,X
BEBA 48         PHA
BEBB AC EB 2B   LDY L2BEB
BEBE 88         DEY
BEBF          LBEBF:
BEBF 68         PLA
BEC0 48         PHA
BEC1 59 10 2C   EOR L2C10,Y
BEC4 99 10 2C   STA L2C10,Y
BEC7 88         DEY
BEC8 10 F5      BPL LBEBF
BECA          LBECA:
BECA 68         PLA
BECB 9D 10 2C   STA L2C10,X
BECE 60         RTS
BECF          LBECF:
BECF A9 00      LDA #$0
BED1          LBED1:
BED1 48         PHA
BED2 20 84 BE   JSR LBE84
BED5 68         PLA
BED6 20 20 BA   JSR LBA20
BED9          LBED9:
BED9 20 84 BE   JSR LBE84
BEDC A9 00      LDA #$0
BEDE 8D BC 2B   STA L2BBC
BEE1 20 7C C0   JSR LC07C
BEE4 D0 06      BNE LBEEC
BEE6          LBEE6:
BEE6 60         RTS
BEE7          LBEE7:
BEE7 20 F3 C0   JSR LC0F3
BEEA F0 10      BEQ LBEFC
BEEC          LBEEC:
BEEC 20 7C BF   JSR LBF7C
BEEF AD BE 2B   LDA L2BBE
BEF2 F0 01      BEQ LBEF5
BEF4          LBEF4:
BEF4 60         RTS
BEF5          LBEF5:
BEF5 AD BF 2B   LDA L2BBF
BEF8 30 ED      BMI LBEE7
BEFA          LBEFA:
BEFA 10 F0      BPL LBEEC
BEFC          LBEFC:
BEFC AD BE 2B   LDA L2BBE
BEFF F0 E5      BEQ LBEE6
BF01          LBF01:
BF01 60         RTS
BF02          LBF02:
BF02 20 E0 C0   JSR LC0E0
BF05 F0 1B      BEQ LBF22
BF07          LBF07:
BF07 D0 21      BNE LBF2A
BF09          LBF09:
BF09 A9 00      LDA #$0
BF0B          LBF0B:
BF0B 48         PHA
BF0C A9 00      LDA #$0
BF0E 8D BC 2B   STA L2BBC
BF11 68         PLA
BF12 20 20 BA   JSR LBA20
BF15          LBF15:
BF15 A9 00      LDA #$0
BF17 8D BC 2B   STA L2BBC
BF1A 20 7C C0   JSR LC07C
BF1D D0 0B      BNE LBF2A
BF1F          LBF1F:
BF1F 8D BE 2B   STA L2BBE
BF22          LBF22:
BF22 A9 FF      LDA #$FF
BF24 60         RTS
BF25          LBF25:
BF25 20 F3 C0   JSR LC0F3
BF28 F0 F8      BEQ LBF22
BF2A          LBF2A:
BF2A 20 7C BF   JSR LBF7C
BF2D AE BF 2B   LDX L2BBF
BF30 10 07      BPL LBF39
BF32          LBF32:
BF32 AD BE 2B   LDA L2BBE
BF35 F0 EE      BEQ LBF25
BF37          LBF37:
BF37 D0 42      BNE LBF7B
BF39          LBF39:
BF39 2C B4 2B   BIT L2BB4
BF3C 10 13      BPL LBF51
BF3E          LBF3E:
BF3E A2 00      LDX #$0
BF40 A0 17      LDY #$17
BF42          LBF42:
BF42 B1 94      LDA (L94),Y
BF44 DD 08 2B   CMP L2B08,X
BF47 90 08      BCC LBF51
BF49          LBF49:
BF49 D0 DA      BNE LBF25
BF4B          LBF4B:
BF4B E8         INX
BF4C C8         INY
BF4D C0 1C      CPY #$1C
BF4F 90 F1      BCC LBF42
BF51          LBF51:
BF51 2C B5 2B   BIT L2BB5
BF54 10 13      BPL LBF69
BF56          LBF56:
BF56 A2 00      LDX #$0
BF58 A0 17      LDY #$17
BF5A          LBF5A:
BF5A B1 94      LDA (L94),Y
BF5C DD 0D 2B   CMP L2B0D,X
BF5F 90 C4      BCC LBF25
BF61          LBF61:
BF61 D0 06      BNE LBF69
BF63          LBF63:
BF63 E8         INX
BF64 C8         INY
BF65 C0 1C      CPY #$1C
BF67 90 F1      BCC LBF5A
BF69          LBF69:
BF69 AE BF 2B   LDX L2BBF
BF6C AD EE 2B   LDA L2BEE
BF6F F0 0A      BEQ LBF7B
BF71          LBF71:
BF71 BD 18 2C   LDA L2C18,X
BF74 29 07      AND #$7
BF76 CD EE 2B   CMP L2BEE
BF79 D0 AA      BNE LBF25
BF7B          LBF7B:
BF7B 60         RTS
BF7C          LBF7C:
BF7C A2 FF      LDX #$FF
BF7E 8E BF 2B   STX L2BBF
BF81 E8         INX
BF82 8E E4 2B   STX L2BE4
BF85 20 2E C0   JSR LC02E
BF88 F0 06      BEQ LBF90
BF8A          LBF8A:
BF8A 60         RTS
BF8B          LBF8B:
BF8B 20 39 C0   JSR LC039
BF8E D0 FA      BNE LBF8A
BF90          LBF90:
BF90 BD 10 2C   LDA L2C10,X
BF93 CD E8 90   CMP L90E8
BF96 D0 F3      BNE LBF8B
BF98          LBF98:
BF98 BD 00 2C   LDA L2C00,X
BF9B AA         TAX
BF9C 20 56 C1   JSR LC156
BF9F A0 03      LDY #$3
BFA1 D0 13      BNE LBFB6
BFA3          LBFA3:
BFA3 BD 00 02   LDA L200,X
BFA6 D1 94      CMP (L94),Y
BFA9          LBFA9 = * + 1
              ; Instruction parameter accessed.
BFA8 F0 0A      BEQ LBFB4
BFAA          LBFAA:
BFAA C9 3F      CMP #$3F
BFAC D0 DD      BNE LBF8B
BFAE          LBFAE:
BFAE B1 94      LDA (L94),Y
BFB0 C9 A0      CMP #$A0
BFB2 F0 D7      BEQ LBF8B
BFB4          LBFB4:
BFB4 E8         INX
BFB5 C8         INY
BFB6          LBFB6:
BFB6 EC EF 2B   CPX L2BEF
BFB9 B0 0A      BCS LBFC5
BFBB          LBFBB:
BFBB BD 00 02   LDA L200,X
BFBE C9 2A      CMP #$2A
BFC0 D0 E1      BNE LBFA3
BFC2          LBFC2:
BFC2 4C 52 C0   JMP LC052
BFC5          LBFC5:
BFC5 C0 13      CPY #$13
BFC7 B0 06      BCS LBFCF
BFC9          LBFC9:
BFC9 B1 94      LDA (L94),Y
BFCB C9 A0      CMP #$A0
BFCD D0 BC      BNE LBF8B
BFCF          LBFCF:
BFCF AE EC 2B   LDX L2BEC
BFD2 8E BF 2B   STX L2BBF
BFD5 BD 18 2C   LDA L2C18,X
BFD8 29 80      AND #$80
BFDA 8D E4 2B   STA L2BE4
BFDD AD B8 2B   LDA L2BB8
BFE0 9D 40 2C   STA L2C40,X
BFE3 A5 5A      LDA L5A
BFE5 9D 30 2C   STA L2C30,X
BFE8 A5 5B      LDA L5B
BFEA 9D 38 2C   STA L2C38,X
BFED A0 00      LDY #$0
BFEF B1 94      LDA (L94),Y
BFF1 C8         INY
BFF2 48         PHA
BFF3 29 40      AND #$40
BFF5 85 50      STA L50
BFF7 68         PLA
BFF8 29 DF      AND #$DF
BFFA 30 02      BMI LBFFE
BFFC          LBFFC:
BFFC 09 20      ORA #$20
BFFE          LBFFE:
BFFE 29 27      AND #$27
C000 05 50      ORA L50
C002 85 50      STA L50
C004 A9 80      LDA #$80
C006 3D 18 2C   AND L2C18,X
C009 05 50      ORA L50
C00B 9D 18 2C   STA L2C18,X
C00E B1 94      LDA (L94),Y
C010 D0 07      BNE LC019
C012          LC012:
C012 CD E8 90   CMP L90E8
C015 D0 02      BNE LC019
C017          LC017:
C017 A9 01      LDA #$1
C019          LC019:
C019 9D 20 2C   STA L2C20,X
C01C C8         INY
C01D B1 94      LDA (L94),Y
C01F 9D 28 2C   STA L2C28,X
C022 AD F3 2B   LDA L2BF3
C025 D0 07      BNE LC02E
C027          LC027:
C027 A0 15      LDY #$15
C029 B1 94      LDA (L94),Y
C02B 8D F3 2B   STA L2BF3
C02E          LC02E:
C02E A9 FF      LDA #$FF
C030 8D BE 2B   STA L2BBE
C033 AD EB 2B   LDA L2BEB
C036 8D EC 2B   STA L2BEC
C039          LC039:
C039 CE EC 2B   DEC L2BEC
C03C 10 01      BPL LC03F
C03E          LC03E:
C03E 60         RTS
C03F          LC03F:
C03F AE EC 2B   LDX L2BEC
C042 BD 18 2C   LDA L2C18,X
C045 30 05      BMI LC04C
C047          LC047:
C047 BD 20 2C   LDA L2C20,X
C04A D0 ED      BNE LC039
C04C          LC04C:
C04C A9 00      LDA #$0
C04E 8D BE 2B   STA L2BBE
C051 60         RTS
C052          LC052:
C052 86 5C      STX L5C
C054 AE EF 2B   LDX L2BEF
C057 CA         DEX
C058 E4 5C      CPX L5C
C05A F0 1A      BEQ LC076
C05C          LC05C:
C05C A0 13      LDY #$13
C05E          LC05E:
C05E 88         DEY
C05F B1 94      LDA (L94),Y
C061 C9 A0      CMP #$A0
C063 F0 F9      BEQ LC05E
C065          LC065:
C065 BD 00 02   LDA L200,X
C068 D1 94      CMP (L94),Y
C06A F0 04      BEQ LC070
C06C          LC06C:
C06C C9 3F      CMP #$3F
C06E D0 09      BNE LC079
C070          LC070:
C070 88         DEY
C071 CA         DEX
C072 E4 5C      CPX L5C
C074 D0 EF      BNE LC065
C076          LC076:
C076 4C CF BF   JMP LBFCF
C079          LC079:
C079 4C 8B BF   JMP LBF8B
C07C          LC07C:
C07C A0 00      LDY #$0
C07E 8C BA 2B   STY L2BBA
C081 88         DEY
C082 8C BF 2B   STY L2BBF
C085 8C C0 2B   STY L2BC0
C088 AD A7 2B   LDA L2BA7
C08B 85 5A      STA L5A
C08D AD A9 2B   LDA L2BA9
C090 85 5B      STA L5B
C092 20 78 C3   JSR LC378
C095          LC095:
C095 AD C0 2B   LDA L2BC0
C098 D0 01      BNE LC09B
C09A          LC09A:
C09A 60         RTS
C09B          LC09B:
C09B A9 07      LDA #$7
C09D 8D C1 2B   STA L2BC1
C0A0 A9 00      LDA #$0
C0A2 20 E2 DC   JSR LDCE2
C0A5 8D C0 2B   STA L2BC0
C0A8          LC0A8:
C0A8 20 D4 DC   JSR LDCD4
C0AB CE C1 2B   DEC L2BC1
C0AE A0 00      LDY #$0
C0B0 B1 94      LDA (L94),Y
C0B2 D0 23      BNE LC0D7
C0B4          LC0B4:
C0B4 AD BA 2B   LDA L2BBA
C0B7 D0 3A      BNE LC0F3
C0B9          LC0B9:
C0B9 20 86 D9   JSR LD986
C0BC AD E8 90   LDA L90E8
C0BF 8D B9 2B   STA L2BB9
C0C2 A5 5A      LDA L5A
C0C4 8D BA 2B   STA L2BBA
C0C7 A5 5B      LDA L5B
C0C9 8D BB 2B   STA L2BBB
C0CC A5 94      LDA L94
C0CE AE BC 2B   LDX L2BBC
C0D1 8D BC 2B   STA L2BBC
C0D4 F0 1D      BEQ LC0F3
C0D6          LC0D6:
C0D6 60         RTS
C0D7          LC0D7:
C0D7 A2 01      LDX #$1
C0D9 EC BC 2B   CPX L2BBC
C0DC D0 2D      BNE LC10B
C0DE          LC0DE:
C0DE F0 13      BEQ LC0F3
C0E0          LC0E0:
C0E0 AD B6 2B   LDA L2BB6
C0E3 85 5A      STA L5A
C0E5 AD B7 2B   LDA L2BB7
C0E8 85 5B      STA L5B
C0EA 20 78 C3   JSR LC378
C0ED AD B8 2B   LDA L2BB8
C0F0 20 C6 DC   JSR LDCC6
C0F3          LC0F3:
C0F3 A9 FF      LDA #$FF
C0F5 8D BF 2B   STA L2BBF
C0F8 AD C1 2B   LDA L2BC1
C0FB 30 08      BMI LC105
C0FD          LC0FD:
C0FD A9 20      LDA #$20
C0FF 20 5B DC   JSR LDC5B
C102 4C A8 C0   JMP LC0A8
C105          LC105:
C105 20 5E 9F   JSR L9F5E
C108 4C 95 C0   JMP LC095
C10B          LC10B:
C10B A5 94      LDA L94
C10D 8D B8 2B   STA L2BB8
C110 20 86 D9   JSR LD986
C113 A5 5B      LDA L5B
C115 8D B7 2B   STA L2BB7
C118 A5 5A      LDA L5A
C11A 8D B6 2B   STA L2BB6
C11D 60         RTS
C11E          LC11E:
C11E 48         PHA
C11F 20 56 C1   JSR LC156
C122 20 38 C1   JSR LC138
C125 68         PLA
C126 38         SEC
C127 ED C2 2B   SBC L2BC2
C12A AA         TAX
C12B F0 0A      BEQ LC137
C12D          LC12D:
C12D 90 08      BCC LC137
C12F          LC12F:
C12F A9 A0      LDA #$A0
C131          LC131:
C131 91 94      STA (L94),Y
C133 C8         INY
C134 CA         DEX
C135 D0 FA      BNE LC131
C137          LC137:
C137 60         RTS
C138          LC138:
C138 98         TYA
C139 0A         ASL A
C13A A8         TAY
C13B B9 A0 00   LDA LA0,Y
C13E 85 94      STA L94
C140 B9 A1 00   LDA LA1,Y
C143 85 95      STA L95
C145 A0 00      LDY #$0
C147          LC147:
C147 BD 00 02   LDA L200,X
C14A 91 94      STA (L94),Y
C14C C8         INY
C14D F0 06      BEQ LC155
C14F          LC14F:
C14F E8         INX
C150 EC EF 2B   CPX L2BEF
C153 90 F2      BCC LC147
C155          LC155:
C155 60         RTS
C156          LC156:
C156 A9 00      LDA #$0
C158 8D C2 2B   STA L2BC2
C15B 8A         TXA
C15C 48         PHA
C15D          LC15D:
C15D BD 00 02   LDA L200,X
C160 C9 2C      CMP #$2C
C162 F0 13      BEQ LC177
C164          LC164:
C164 C9 3D      CMP #$3D
C166 F0 0F      BEQ LC177
C168          LC168:
C168 EE C2 2B   INC L2BC2
C16B E8         INX
C16C A9 0F      LDA #$F
C16E CD C2 2B   CMP L2BC2
C171 90 04      BCC LC177
C173          LC173:
C173 E4 56      CPX L56
C175 90 E6      BCC LC15D
C177          LC177:
C177 8E EF 2B   STX L2BEF
C17A 68         PLA
C17B AA         TAX
C17C 60         RTS
C17D          LC17D:
C17D A5 82      LDA L82
C17F 48         PHA
C180 A5 80      LDA L80
C182 48         PHA
C183 20 8D C1   JSR LC18D
C186 68         PLA
C187 85 80      STA L80
C189 68         PLA
C18A 85 82      STA L82
C18C 60         RTS
C18D          LC18D:
C18D A9 11      LDA #$11
C18F 85 82      STA L82
C191 20 60 DA   JSR LDA60
C194 20 D4 DC   JSR LDCD4
C197 AD BF 2B   LDA L2BBF
C19A 10 05      BPL LC1A1
C19C          LC19C:
C19C 20 50 C3   JSR LC350
C19F 18         CLC
C1A0 60         RTS
C1A1          LC1A1:
C1A1 A2 18      LDX #$18
C1A3 A0 1D      LDY #$1D
C1A5 2C B3 2B   BIT L2BB3
C1A8 10 04      BPL LC1AE
C1AA          LC1AA:
C1AA A9 00      LDA #$0
C1AC F0 02      BEQ LC1B0
C1AE          LC1AE:
C1AE B1 94      LDA (L94),Y
C1B0          LC1B0:
C1B0 8D C4 2B   STA L2BC4
C1B3 F0 02      BEQ LC1B7
C1B5          LC1B5:
C1B5 A2 16      LDX #$16
C1B7          LC1B7:
C1B7 88         DEY
C1B8 2C B3 2B   BIT L2BB3
C1BB 10 14      BPL LC1D1
C1BD          LC1BD:
C1BD A5 94      LDA L94
C1BF 4A         LSR A
C1C0 4A         LSR A
C1C1 4A         LSR A
C1C2 4A         LSR A
C1C3 4A         LSR A
C1C4 8D C3 2B   STA L2BC3
C1C7 A5 5B      LDA L5B
C1C9 0A         ASL A
C1CA 0A         ASL A
C1CB 0A         ASL A
C1CC 18         CLC
C1CD 6D C3 2B   ADC L2BC3
C1D1          LC1D1 = * + 1
              ; Instruction parameter jumped to.
C1D0 2C B1 94   BIT L94B1
C1D3 8D C3 2B   STA L2BC3
C1D6 E0 16      CPX #$16
C1D8 F0 0A      BEQ LC1E4
C1DA          LC1DA:
C1DA C9 0A      CMP #$A
C1DC 90 06      BCC LC1E4
C1DE          LC1DE:
C1DE CA         DEX
C1DF C9 64      CMP #$64
C1E1 90 01      BCC LC1E4
C1E3          LC1E3:
C1E3 CA         DEX
C1E4          LC1E4:
C1E4 20 BF C2   JSR LC2BF
C1E7 B1 94      LDA (L94),Y
C1E9 2C B3 2B   BIT L2BB3
C1EC 30 0D      BMI LC1FB
C1EE          LC1EE:
C1EE 48         PHA
C1EF 0A         ASL A
C1F0 10 05      BPL LC1F7
C1F2          LC1F2:
C1F2 A9 3C      LDA #$3C
C1F4 9D E1 2F   STA L2FE1,X
C1F7          LC1F7:
C1F7 68         PLA
C1F8 4C 06 C2   JMP LC206
C1FB          LC1FB:
C1FB C9 FF      CMP #$FF
C1FD D0 02      BNE LC201
C1FF          LC1FF:
C1FF A9 00      LDA #$0
C201          LC201:
C201 18         CLC
C202 69 07      ADC #$7
C204 38         SEC
C206          LC206 = * + 1
              ; Instruction parameter jumped to.
C205 2C 29 0F   BIT LF29
C208 A8         TAY
C209 B9 B0 C2   LDA LC2B0,Y
C20C 9D E0 2F   STA L2FE0,X
C20F CA         DEX
C210 B9 A1 C2   LDA LC2A1,Y
C213 9D E0 2F   STA L2FE0,X
C216 CA         DEX
C217 B9 92 C2   LDA LC292,Y
C21A 9D E0 2F   STA L2FE0,X
C21D CA         DEX
C21E CA         DEX
C21F B0 05      BCS LC226
C221          LC221:
C221 A9 2A      LDA #$2A
C223 9D E1 2F   STA L2FE1,X
C226          LC226:
C226 A9 A0      LDA #$A0
C228 9D E0 2F   STA L2FE0,X
C22B CA         DEX
C22C A0 12      LDY #$12
C22E          LC22E:
C22E B1 94      LDA (L94),Y
C230 9D E0 2F   STA L2FE0,X
C233 CA         DEX
C234 88         DEY
C235 C0 03      CPY #$3
C237 B0 F5      BCS LC22E
C239          LC239:
C239 A9 22      LDA #$22
C23B 9D E0 2F   STA L2FE0,X
C23E          LC23E:
C23E E8         INX
C23F E0 20      CPX #$20
C241 B0 0B      BCS LC24E
C243          LC243:
C243 BD E0 2F   LDA L2FE0,X
C246 C9 22      CMP #$22
C248 F0 04      BEQ LC24E
C24A          LC24A:
C24A C9 A0      CMP #$A0
C24C D0 F0      BNE LC23E
C24E          LC24E:
C24E A9 22      LDA #$22
C250 9D E0 2F   STA L2FE0,X
C253          LC253:
C253 E8         INX
C254 E0 20      CPX #$20
C256 B0 0A      BCS LC262
C258          LC258:
C258 A9 7F      LDA #$7F
C25A 3D E0 2F   AND L2FE0,X
C25D 9D E0 2F   STA L2FE0,X
C260 10 F1      BPL LC253
C262          LC262:
C262 A2 04      LDX #$4
C264 A0 1B      LDY #$1B
C266          LC266:
C266 B1 94      LDA (L94),Y
C268 9D AA 2B   STA L2BAA,X
C26B 88         DEY
C26C CA         DEX
C26D 10 F7      BPL LC266
C26F          LC26F:
C26F AD AD 2B   LDA L2BAD
C272 C9 0C      CMP #$C
C274 90 08      BCC LC27E
C276          LC276:
C276 E9 0C      SBC #$C
C278 8D AD 2B   STA L2BAD
C27B A9 80      LDA #$80
C27E          LC27E = * + 1
              ; Instruction parameter jumped to.
C27D 2C A9 00   BIT LA9
C280 8D AF 2B   STA L2BAF
C283 AD AD 2B   LDA L2BAD
C286 D0 05      BNE LC28D
C288          LC288:
C288 A9 0C      LDA #$C
C28A 8D AD 2B   STA L2BAD
C28D          LC28D:
C28D 20 25 BF   JSR LBF25
C290 38         SEC
C291 60         RTS
C292          LC292:
C292 44 53 50   .BYTE $44,$53,$50
C295 55 52 43   .BYTE $55,$52,$43
C299          LC299 = * + 1
C298 44 53 4E   .BYTE $44,$53,$4E
C29B 34 37 38   .BYTE $34,$37,$38
C29E 43 50 46   .BYTE $43,$50,$46
C2A1          LC2A1:
C2A1 45 45 52   .BYTE $45,$45,$52
C2A4 53 45 42   .BYTE $53,$45,$42
C2A7 49 59 41   .BYTE $49,$59,$41
C2AA 31 31 31   .BYTE $31,$31,$31
C2AD 38 52 4F   .BYTE $38,$52,$4F
C2B0          LC2B0:
C2B0 4C 51 47   JMP L4751
C2B3 52         .BYTE $52
C2B4          LC2B4:
C2B4 4C 4D 52   JMP L524D
C2B7 53 54 20   .BYTE $53,$54,$20
C2BA 20 20 31   .BYTE $20,$20,$31
C2BD 4E 52      .BYTE $4E,$52
C2BF          LC2BF:
C2BF A0 1B      LDY #$1B
C2C1 A9 20      LDA #$20
C2C3          LC2C3:
C2C3 99 DF 2F   STA L2FDF,Y
C2C6 88         DEY
C2C7 D0 FA      BNE LC2C3
C2C9          LC2C9:
C2C9 60         RTS
C2CA          LC2CA:
C2CA 43 4D 44   .BYTE $43,$4D,$44
C2CD 20 48 44   .BYTE $20,$48,$44
C2D0 20 20 20   .BYTE $20,$20,$20
C2D3 20 20 20   .BYTE $20,$20,$20
C2D6 20 20 20   .BYTE $20,$20,$20
C2D9 20 A0 A0   .BYTE $20,$A0,$A0
C2DC 48 44      .BYTE $48,$44
C2DE          LC2DE:
C2DE A0 31      LDY #$31
C2E0 48         PHA
C2E1          LC2E1:
C2E1 2C B3 2B   BIT L2BB3
C2E4 10 0D      BPL LC2F3
C2E6          LC2E6:
C2E6 A2 17      LDX #$17
C2E8          LC2E8:
C2E8 BD CA C2   LDA LC2CA,X
C2EB          LC2EB:
C2EB 9D 04 22   STA L2204,X
C2EE CA         DEX
C2EF 10 F7      BPL LC2E8
C2F1          LC2F1:
C2F1 30 06      BMI LC2F9
C2F3          LC2F3:
C2F3 20 D0 AE   JSR LAED0
C2F6 20 7E A1   JSR LA17E
C2F9          LC2F9:
C2F9 20 BF C2   JSR LC2BF
C2FC A9 FF      LDA #$FF
C2FE 85 50      STA L50
C300 A9 00      LDA #$0
C302 8D C3 2B   STA L2BC3
C305 8D C4 2B   STA L2BC4
C308 A9 22      LDA #$22
C30A 85 95      STA L95
C30C AC E8 90   LDY L90E8
C30F C0 FF      CPY #$FF
C311 F0 0B      BEQ LC31E
C313          LC313:
C313 B9 00 82   LDA Partition_Typ+$00,Y
C316 C9 01      CMP #$1
C318 F0 04      BEQ LC31E
C31A          LC31A:
C31A C9 04      CMP #$4
C31C 90 03      BCC LC321
C31E          LC31E:
C31E A9 04      LDA #$4
C321          LC321 = * + 1
              ; Instruction parameter jumped to.
C320 2C A9 90   BIT L90A9
C323 85 94      STA L94
C325 A0 00      LDY #$0
C327          LC327:
C327 B1 94      LDA (L94),Y
C329 C9 A0      CMP #$A0
C32B D0 02      BNE LC32F
C32D          LC32D:
C32D A9 20      LDA #$20
C32F          LC32F:
C32F 99 E2 2F   STA L2FE2,Y
C332 C8         INY
C333 C0 17      CPY #$17
C335 90 F0      BCC LC327
C337          LC337:
C337 A0 FF      LDY #$FF
C339 A9 04      LDA #$4
C33B 85 94      STA L94
C33D A9 12      LDA #$12
C33F 8D E0 2F   STA L2FE0
C342 A9 22      LDA #$22
C344 8D E1 2F   STA L2FE1
C347 8D F2 2F   STA L2FF2
C34A A9 20      LDA #$20
C34C 8D F3 2F   STA L2FF3
C34F 60         RTS
C350          LC350:
C350 20 BF C2   JSR LC2BF
C353 A0 0B      LDY #$B
C355          LC355:
C355 B9 61 C3   LDA LC361,Y
C358 99 E0 2F   STA L2FE0,Y
C35B 88         DEY
C35C 10 F7      BPL LC355
C35E          LC35E:
C35E 4C 7C C6   JMP LC67C
C361          LC361:
C361 42         .BYTE $42
C362          LC362:
C362 4C 4F 43   JMP L434F
C365 4B 53      .BYTE $4B,$53
C367          LC367:
C367 20 46 52   JSR L5246
C36A 45 45      EOR L45
C36D          LC36D = * + 1
              ; Instruction parameter jumped to.
C36C 2E A0 00   ROL LA0
C36F 98         TYA
C370 91 94      STA (L94),Y
C372 20 A7 D9   JSR LD9A7
C375 4C 65 D9   JMP LD965
C378          LC378:
C378 A9 01      LDA #$1
C37A          LC37A:
C37A 8D ED 2B   STA L2BED
C37D A9 11      LDA #$11
C37F 85 82      STA L82
C381 20 F7 CA   JSR LCAF7
C384 A9 02      LDA #$2
C386 4C C6 DC   JMP LDCC6
C389          LC389:
C389 A9 12      LDA #$12
C38B 85 82      STA L82
C38D 4C BD CB   JMP LCBBD
C390          LC390:
C390 20 86 D9   JSR LD986
C393 20 64 A4   JSR LA464
C396 A9 00      LDA #$0
C398 20 C6 DC   JSR LDCC6
C39B A5 5A      LDA L5A
C39D 20 EA CE   JSR LCEEA
C3A0 A5 5B      LDA L5B
C3A2 20 EA CE   JSR LCEEA
C3A5 20 85 D8   JSR LD885
C3A8 20 65 D9   JSR LD965
C3AB A9 00      LDA #$0
C3AD 20 C6 DC   JSR LDCC6
C3B0          LC3B0:
C3B0 20 EA CE   JSR LCEEA
C3B3 D0 FB      BNE LC3B0
C3B5          LC3B5:
C3B5 20 EA CE   JSR LCEEA
C3B8 A9 FF      LDA #$FF
C3BA 4C EA CE   JMP LCEEA
C3BD          LC3BD:
C3BD A5 82      LDA L82
C3BF 48         PHA
C3C0 A5 80      LDA L80
C3C2 48         PHA
C3C3 A5 5B      LDA L5B
C3C5 48         PHA
C3C6 A5 5A      LDA L5A
C3C8 48         PHA
C3C9 A9 00      LDA #$0
C3CB 8D 30 2C   STA L2C30
C3CE A9 11      LDA #$11
C3D0 85 82      STA L82
C3D2 20 86 D9   JSR LD986
C3D5 AD ED 2B   LDA L2BED
C3D8 48         PHA
C3D9 AD 10 2C   LDA L2C10
C3DC CD B9 2B   CMP L2BB9
C3DF F0 0C      BEQ LC3ED
C3E1          LC3E1:
C3E1 A2 01      LDX #$1
C3E3 8E BC 2B   STX L2BBC
C3E6 20 7C C0   JSR LC07C
C3E9 F0 2C      BEQ LC417
C3EB          LC3EB:
C3EB D0 40      BNE LC42D
C3ED          LC3ED:
C3ED AD BA 2B   LDA L2BBA
C3F0 F0 1B      BEQ LC40D
C3F2          LC3F2:
C3F2 C5 5A      CMP L5A
C3F4 D0 07      BNE LC3FD
C3F6          LC3F6:
C3F6 A5 5B      LDA L5B
C3F8 CD BB 2B   CMP L2BBB
C3FB F0 30      BEQ LC42D
C3FD          LC3FD:
C3FD AD BA 2B   LDA L2BBA
C400 85 5A      STA L5A
C402 AD BB 2B   LDA L2BBB
C405 85 5B      STA L5B
C407 20 AA D8   JSR LD8AA
C40A 4C 2D C4   JMP LC42D
C40D          LC40D:
C40D A9 01      LDA #$1
C40F 8D BC 2B   STA L2BBC
C412 20 F3 C0   JSR LC0F3
C415 D0 16      BNE LC42D
C417          LC417:
C417 20 90 C3   JSR LC390
C41A 38         SEC
C41B 6E 30 2C   ROR L2C30
C41E A5 5B      LDA L5B
C420 8D BB 2B   STA L2BBB
C423 A5 5A      LDA L5A
C425 8D BA 2B   STA L2BBA
C428 A9 02      LDA #$2
C42A 8D BC 2B   STA L2BBC
C42D          LC42D:
C42D AD BC 2B   LDA L2BBC
C430 20 C6 DC   JSR LDCC6
C433 68         PLA
C434 8D ED 2B   STA L2BED
C437 C9 04      CMP #$4
C439 D0 02      BNE LC43D
C43B          LC43B:
C43B 09 80      ORA #$80
C43D          LC43D:
C43D 20 EA CE   JSR LCEEA
C440 68         PLA
C441 8D 20 2C   STA L2C20
C444 20 EA CE   JSR LCEEA
C447 68         PLA
C448 8D 28 2C   STA L2C28
C44B 20 EA CE   JSR LCEEA
C44E 20 F2 DC   JSR LDCF2
C451 A8         TAY
C452 AD 00 2C   LDA L2C00
C455 AA         TAX
C456 A9 10      LDA #$10
C458 20 1E C1   JSR LC11E
C45B A0 10      LDY #$10
C45D A9 00      LDA #$0
C45F          LC45F:
C45F 91 94      STA (L94),Y
C461 C8         INY
C462 C0 1B      CPY #$1B
C464 90 F9      BCC LC45F
C466          LC466:
C466 AD ED 2B   LDA L2BED
C469 C9 04      CMP #$4
C46B D0 13      BNE LC480
C46D          LC46D:
C46D A0 10      LDY #$10
C46F AD F4 2B   LDA L2BF4
C472 91 94      STA (L94),Y
C474 C8         INY
C475 AD F5 2B   LDA L2BF5
C478 91 94      STA (L94),Y
C47A C8         INY
C47B AD F3 2B   LDA L2BF3
C47E 91 94      STA (L94),Y
C480          LC480:
C480 20 AD D8   JSR LD8AD
C483 2C 30 2C   BIT L2C30
C486 10 36      BPL LC4BE
C488          LC488:
C488 20 85 B0   JSR LB085
C48B D0 31      BNE LC4BE
C48D          LC48D:
C48D AD A7 2B   LDA L2BA7
C490 C9 01      CMP #$1
C492 D0 05      BNE LC499
C494          LC494:
C494 CD A8 2B   CMP L2BA8
C497 F0 25      BEQ LC4BE
C499          LC499:
C499 20 B2 A1   JSR LA1B2
C49C BD 00 22   LDA L2200,X
C49F C9 86      CMP #$86
C4A1 D0 1B      BNE LC4BE
C4A3          LC4A3:
C4A3 BD 01 22   LDA L2201,X
C4A6 CD A7 2B   CMP L2BA7
C4A9 D0 13      BNE LC4BE
C4AB          LC4AB:
C4AB BD 02 22   LDA L2202,X
C4AE CD A8 2B   CMP L2BA8
C4B1 D0 0B      BNE LC4BE
C4B3          LC4B3:
C4B3 FE 1C 22   INC L221C,X
C4B6 D0 03      BNE LC4BB
C4B8          LC4B8:
C4B8 FE 1D 22   INC L221D,X
C4BB          LC4BB:
C4BB 20 CF A1   JSR LA1CF
C4BE          LC4BE:
C4BE 68         PLA
C4BF 85 80      STA L80
C4C1 AA         TAX
C4C2 68         PLA
C4C3 85 82      STA L82
C4C5 AD BA 2B   LDA L2BBA
C4C8 8D 30 2C   STA L2C30
C4CB 9D E8 2C   STA L2CE8,X
C4CE AD BB 2B   LDA L2BBB
C4D1 8D 38 2C   STA L2C38
C4D4 9D 08 2D   STA L2D08,X
C4D7 AD BC 2B   LDA L2BBC
C4DA 8D 40 2C   STA L2C40
C4DD 9D 28 2D   STA L2D28,X
C4E0 AD ED 2B   LDA L2BED
C4E3 8D 18 2C   STA L2C18
C4E6 60         RTS
C4E7          LC4E7:
C4E7 A9 00      LDA #$0
C4E9 85 82      STA L82
C4EB A9 01      LDA #$1
C4ED 20 C2 DA   JSR LDAC2
C4F0 A9 00      LDA #$0
C4F2 20 C6 DC   JSR LDCC6
C4F5 A6 80      LDX L80
C4F7 A9 00      LDA #$0
C4F9 9D E8 2D   STA L2DE8,X
C4FC 20 F2 DC   JSR LDCF2
C4FF AA         TAX
C500 A9 00      LDA #$0
C502 9D 60 29   STA L2960,X
C505 A9 01      LDA #$1
C507 20 EA CE   JSR LCEEA
C50A A9 04      LDA #$4
C50C 20 EA CE   JSR LCEEA
C50F A9 01      LDA #$1
C511 20 EA CE   JSR LCEEA
C514 20 EA CE   JSR LCEEA
C517 AD E8 90   LDA L90E8
C51A D0 02      BNE LC51E
C51C          LC51C:
C51C A9 FF      LDA #$FF
C51E          LC51E:
C51E 20 EA CE   JSR LCEEA
C521 A9 00      LDA #$0
C523 20 EA CE   JSR LCEEA
C526 20 AD C5   JSR LC5AD
C529 D6 A0      DEC LA0,X
C52B D6 A0      DEC LA0,X
C52D A9 01      LDA #$1
C52F 8D B1 2B   STA L2BB1
C532 A9 00      LDA #$0
C534 20 EA CE   JSR LCEEA
C537          LC537:
C537 A9 01      LDA #$1
C539 20 EA CE   JSR LCEEA
C53C 20 EA CE   JSR LCEEA
C53F 20 7D C1   JSR LC17D
C542 90 2F      BCC LC573
C544          LC544:
C544 AD C3 2B   LDA L2BC3
C547 20 EA CE   JSR LCEEA
C54A AD C4 2B   LDA L2BC4
C54D 20 EA CE   JSR LCEEA
C550 20 AD C5   JSR LC5AD
C553 2C B3 2B   BIT L2BB3
C556 50 03      BVC LC55B
C558          LC558:
C558 20 BB C5   JSR LC5BB
C55B          LC55B:
C55B A9 00      LDA #$0
C55D 20 EA CE   JSR LCEEA
C560 D0 D5      BNE LC537
C562          LC562:
C562 A9 00      LDA #$0
C564 95 A0      STA LA0,X
C566 A9 88      LDA #$88
C568 A4 80      LDY L80
C56A 8D C5 2B   STA L2BC5
C56D 99 A8 2D   STA L2DA8,Y
C570 A5 84      LDA L84
C572 60         RTS
C573          LC573:
C573 2C B3 2B   BIT L2BB3
C576 10 0A      BPL LC582
C578          LC578:
C578 20 EA CE   JSR LCEEA
C57B D6 A0      DEC LA0,X
C57D D6 A0      DEC LA0,X
C57F 4C 91 C5   JMP LC591
C582          LC582:
C582 AD C3 2B   LDA L2BC3
C585 20 EA CE   JSR LCEEA
C588 AD C4 2B   LDA L2BC4
C58B 20 EA CE   JSR LCEEA
C58E 20 AD C5   JSR LC5AD
C591          LC591:
C591 D6 A0      DEC LA0,X
C593 D6 A0      DEC LA0,X
C595 A9 00      LDA #$0
C597 20 EA CE   JSR LCEEA
C59A 20 EA CE   JSR LCEEA
C59D 20 EA CE   JSR LCEEA
C5A0 B5 A0      LDA LA0,X
C5A2 38         SEC
C5A3 E9 01      SBC #$1
C5A5 A4 80      LDY L80
C5A7 99 E8 2D   STA L2DE8,Y
C5AA 4C 62 C5   JMP LC562
C5AD          LC5AD:
C5AD A0 00      LDY #$0
C5AF          LC5AF:
C5AF B9 E0 2F   LDA L2FE0,Y
C5B2 20 EA CE   JSR LCEEA
C5B5 C8         INY
C5B6 C0 1B      CPY #$1B
C5B8 D0 F5      BNE LC5AF
C5BA          LC5BA:
C5BA 60         RTS
C5BB          LC5BB:
C5BB A9 1F      LDA #$1F
C5BD 8D B2 2B   STA L2BB2
C5C0          LC5C0:
C5C0 D6 A0      DEC LA0,X
C5C2 CE B2 2B   DEC L2BB2
C5C5          LC5C5:
C5C5 A1 A0      LDA (LA0,X)
C5C7 C9 20      CMP #$20
C5C9 F0 F5      BEQ LC5C0
C5CB          LC5CB:
C5CB 2C B0 2B   BIT L2BB0
C5CE 30 0B      BMI LC5DB
C5D0          LC5D0:
C5D0 D6 A0      DEC LA0,X
C5D2 CE B2 2B   DEC L2BB2
C5D5 C9 3C      CMP #$3C
C5D7 F0 EC      BEQ LC5C5
C5D9          LC5D9:
C5D9 D0 0D      BNE LC5E8
C5DB          LC5DB:
C5DB 20 70 C6   JSR LC670
C5DE C9 3C      CMP #$3C
C5E0 F0 03      BEQ LC5E5
C5E2          LC5E2:
C5E2 20 6E C6   JSR LC66E
C5E5          LC5E5:
C5E5 20 6E C6   JSR LC66E
C5E8          LC5E8:
C5E8 20 1C C6   JSR LC61C
C5EB          LC5EB:
C5EB A9 29      LDA #$29
C5ED 2C B0 2B   BIT L2BB0
C5F0 10 02      BPL LC5F4
C5F2          LC5F2:
C5F2 A9 3F      LDA #$3F
C5F4          LC5F4:
C5F4 CD B2 2B   CMP L2BB2
C5F7 F0 08      BEQ LC601
C5F9          LC5F9:
C5F9 A9 01      LDA #$1
C5FB 20 70 C6   JSR LC670
C5FE 4C EB C5   JMP LC5EB
C601          LC601:
C601 EE B1 2B   INC L2BB1
C604 A9 06      LDA #$6
C606 2C B0 2B   BIT L2BB0
C609 10 02      BPL LC60D
C60B          LC60B:
C60B A9 04      LDA #$4
C60D          LC60D:
C60D CD B1 2B   CMP L2BB1
C610 D0 09      BNE LC61B
C612          LC612:
C612 A9 01      LDA #$1
C614 20 EA CE   JSR LCEEA
C617 D0 F9      BNE LC612
C619          LC619:
C619 D6 A0      DEC LA0,X
C61B          LC61B:
C61B 60         RTS
C61C          LC61C:
C61C A0 01      LDY #$1
C61E          LC61E:
C61E 20 58 C6   JSR LC658
C621 C8         INY
C622 C0 03      CPY #$3
C624 D0 12      BNE LC638
C626          LC626:
C626 2C B0 2B   BIT L2BB0
C629 10 0D      BPL LC638
C62B          LC62B:
C62B A0 00      LDY #$0
C62D 20 58 C6   JSR LC658
C630 20 6E C6   JSR LC66E
C633 20 6E C6   JSR LC66E
C636 A0 03      LDY #$3
C638          LC638:
C638 C0 05      CPY #$5
C63A 90 E2      BCC LC61E
C63C          LC63C:
C63C A9 20      LDA #$20
C63E 20 70 C6   JSR LC670
C641 A9 41      LDA #$41
C643 2C AF 2B   BIT L2BAF
C646 10 02      BPL LC64A
C648          LC648:
C648 A9 50      LDA #$50
C64A          LC64A:
C64A 20 70 C6   JSR LC670
C64D 2C B0 2B   BIT L2BB0
C650 10 05      BPL LC657
C652          LC652:
C652 A9 4D      LDA #$4D
C654 20 70 C6   JSR LC670
C657          LC657:
C657 60         RTS
C658          LC658:
C658 B9 77 C6   LDA LC677,Y
C65B 20 70 C6   JSR LC670
C65E B9 AA 2B   LDA L2BAA,Y
C661 20 7A B4   JSR LB47A
C664 48         PHA
C665 A5 50      LDA L50
C667 20 6B C6   JSR LC66B
C66A 68         PLA
C66B          LC66B:
C66B 09 30      ORA #$30
C66E          LC66E = * + 1
              ; Instruction parameter jumped to.
C66D 2C A9 20   BIT L20A9
C670          LC670:
C670 20 EA CE   JSR LCEEA
C673 EE B2 2B   INC L2BB2
C676 60         RTS
C677          LC677:
C677 2F         .BYTE $2F
C678          LC678:
C678 20 2F 20   JSR L202F
C67C          LC67C = * + 1
              ; Instruction parameter jumped to.
C67D          LC67D = * + 2
              ; Instruction parameter jumped to.
C67B 2E 8A 48   ROL L488A
C67E 98         TYA
C67F 48         PHA
C680 20 0B A6   JSR LA60B
C683 BD 50 2B   LDA L2B50,X
C686 8D C3 2B   STA L2BC3
C689 BD 60 2B   LDA L2B60,X
C68C 8D C4 2B   STA L2BC4
C68F 68         PLA
C690 A8         TAY
C691 68         PLA
C692 AA         TAX
C693 60         RTS
C694          LC694:
C694 A5 82      LDA L82
C696 85 4A      STA L4A
C698 20 AC B7   JSR LB7AC
C69B 8E E2 2B   STX L2BE2
C69E AE 00 02   LDX L200
C6A1 A5 4A      LDA L4A
C6A3 D0 2E      BNE LC6D3
C6A5          LC6A5:
C6A5 E0 2A      CPX #$2A
C6A7 D0 2A      BNE LC6D3
C6A9          LC6A9:
C6A9 20 C7 A2   JSR LA2C7
C6AC BD C0 2F   LDA L2FC0,X
C6AF F0 5E      BEQ LC70F
C6B1          LC6B1:
C6B1 85 5A      STA L5A
C6B3 BD D0 2F   LDA L2FD0,X
C6B6 85 5B      STA L5B
C6B8 AD E8 90   LDA L90E8
C6BB 8D 10 2C   STA L2C10
C6BE A9 02      LDA #$2
C6C0 8D 18 2C   STA L2C18
C6C3 20 3C EE   JSR LEE3C
C6C6 20 F7 CA   JSR LCAF7
C6C9 A9 04      LDA #$4
C6CB          LC6CB:
C6CB A6 80      LDX L80
C6CD 99 88 2D   STA L2D88,Y
C6D0 4C 54 B6   JMP LB654
C6D3          LC6D3:
C6D3 E0 24      CPX #$24
C6D5 D0 31      BNE LC708
C6D7          LC6D7:
C6D7 A5 4A      LDA L4A
C6D9 D0 03      BNE LC6DE
C6DB          LC6DB:
C6DB 4C 67 C9   JMP LC967
C6DE          LC6DE:
C6DE 20 DE B6   JSR LB6DE
C6E1 D0 06      BNE LC6E9
C6E3          LC6E3:
C6E3 20 78 B6   JSR LB678
C6E6 4C F6 C6   JMP LC6F6
C6E9          LC6E9:
C6E9 88         DEY
C6EA 88         DEY
C6EB 8C 00 2C   STY L2C00
C6EE 20 33 B8   JSR LB833
C6F1 A9 00      LDA #$0
C6F3 20 20 BA   JSR LBA20
C6F6          LC6F6:
C6F6 AD A7 2B   LDA L2BA7
C6F9 85 5A      STA L5A
C6FB AD A8 2B   LDA L2BA8
C6FE 85 5B      STA L5B
C700 20 F7 CA   JSR LCAF7
C703 A9 02      LDA #$2
C705 4C CB C6   JMP LC6CB
C708          LC708:
C708 E0 23      CPX #$23
C70A D0 0B      BNE LC717
C70C          LC70C:
C70C 4C 6C AE   JMP LAE6C
C70F          LC70F:
C70F A9 02      LDA #$2
C711 8D EE 2B   STA L2BEE
C714 20 03 AF   JSR LAF03
C717          LC717:
C717 20 DE B6   JSR LB6DE
C71A D0 04      BNE LC720
C71C          LC71C:
C71C A2 00      LDX #$0
C71E F0 0C      BEQ LC72C
C720          LC720:
C720 8A         TXA
C721 F0 05      BEQ LC728
C723          LC723:
C723 A9 30      LDA #$30
C725 4C 6F B6   JMP LB66F
C728          LC728:
C728 88         DEY
C729 F0 01      BEQ LC72C
C72B          LC72B:
C72B 88         DEY
C72C          LC72C:
C72C 8C 00 2C   STY L2C00
C72F A9 8D      LDA #$8D
C731 20 61 B7   JSR LB761
C734 E8         INX
C735 8E EB 2B   STX L2BEB
C738 20 33 B8   JSR LB833
C73B 20 84 BE   JSR LBE84
C73E 20 09 BF   JSR LBF09
C741 A2 00      LDX #$0
C743 8E F3 2B   STX L2BF3
C746 8E F0 2B   STX L2BF0
C749 8E ED 2B   STX L2BED
C74C E8         INX
C74D EC EA 2B   CPX L2BEA
C750 B0 10      BCS LC762
C752          LC752:
C752 20 FE C8   JSR LC8FE
C755 E8         INX
C756 EC EA 2B   CPX L2BEA
C759 B0 07      BCS LC762
C75B          LC75B:
C75B C0 04      CPY #$4
C75D F0 39      BEQ LC798
C75F          LC75F:
C75F 20 FE C8   JSR LC8FE
C762          LC762:
C762 A6 4A      LDX L4A
C764 86 82      STX L82
C766 E0 02      CPX #$2
C768 B0 0D      BCS LC777
C76A          LC76A:
C76A 8E F0 2B   STX L2BF0
C76D AD ED 2B   LDA L2BED
C770 D0 1C      BNE LC78E
C772          LC772:
C772 A9 02      LDA #$2
C774 8D ED 2B   STA L2BED
C777          LC777:
C777 AD ED 2B   LDA L2BED
C77A D0 12      BNE LC78E
C77C          LC77C:
C77C AD 18 2C   LDA L2C18
C77F 29 07      AND #$7
C781 8D ED 2B   STA L2BED
C784 AD 20 2C   LDA L2C20
C787 D0 05      BNE LC78E
C789          LC789:
C789 A9 01      LDA #$1
C78B 8D ED 2B   STA L2BED
C78E          LC78E:
C78E AD F0 2B   LDA L2BF0
C791 C9 01      CMP #$1
C793 F0 18      BEQ LC7AD
C795          LC795:
C795 4C 32 C8   JMP LC832
C798          LC798:
C798 BC 00 2C   LDY L2C00,X
C79B B9 00 02   LDA L200,Y
C79E 8D F3 2B   STA L2BF3
C7A1 AD 20 2C   LDA L2C20
C7A4 D0 BC      BNE LC762
C7A6          LC7A6:
C7A6 A9 01      LDA #$1
C7A8 8D F0 2B   STA L2BF0
C7AB D0 B5      BNE LC762
C7AD          LC7AD:
C7AD AD 18 2C   LDA L2C18
C7B0 29 80      AND #$80
C7B2 AA         TAX
C7B3 D0 15      BNE LC7CA
C7B5          LC7B5:
C7B5 A9 20      LDA #$20
C7B7 2C 18 2C   BIT L2C18
C7BA F0 06      BEQ LC7C2
C7BC          LC7BC:
C7BC 20 6D C3   JSR LC36D
C7BF 4C DF C8   JMP LC8DF
C7C2          LC7C2:
C7C2 AD 20 2C   LDA L2C20
C7C5 D0 03      BNE LC7CA
C7C7          LC7C7:
C7C7 4C DF C8   JMP LC8DF
C7CA          LC7CA:
C7CA AD 00 02   LDA L200
C7CD C9 40      CMP #$40
C7CF F0 0D      BEQ LC7DE
C7D1          LC7D1:
C7D1 8A         TXA
C7D2 D0 05      BNE LC7D9
C7D4          LC7D4:
C7D4 A9 63      LDA #$63
C7D6 4C 6F B6   JMP LB66F
C7D9          LC7D9:
C7D9 A9 33      LDA #$33
C7DB 4C 6F B6   JMP LB66F
C7DE          LC7DE:
C7DE AD 18 2C   LDA L2C18
C7E1 29 07      AND #$7
C7E3 CD ED 2B   CMP L2BED
C7E6 D0 71      BNE LC859
C7E8          LC7E8:
C7E8 C9 04      CMP #$4
C7EA F0 6D      BEQ LC859
C7EC          LC7EC:
C7EC 20 BD CB   JSR LCBBD
C7EF A5 80      LDA L80
C7F1 8D E0 2B   STA L2BE0
C7F4 A9 11      LDA #$11
C7F6 85 82      STA L82
C7F8 20 60 DA   JSR LDA60
C7FB AD B8 2B   LDA L2BB8
C7FE 20 C6 DC   JSR LDCC6
C801 A0 00      LDY #$0
C803 B1 94      LDA (L94),Y
C805 09 20      ORA #$20
C807 91 94      STA (L94),Y
C809 A0 1A      LDY #$1A
C80B A5 5A      LDA L5A
C80D 91 94      STA (L94),Y
C80F C8         INY
C810 A5 5B      LDA L5B
C812 91 94      STA (L94),Y
C814 AE E0 2B   LDX L2BE0
C817 AD 30 2C   LDA L2C30
C81A 9D E8 2C   STA L2CE8,X
C81D AD 38 2C   LDA L2C38
C820 9D 08 2D   STA L2D08,X
C823 AD 40 2C   LDA L2C40
C826 9D 28 2D   STA L2D28,X
C829 20 86 D9   JSR LD986
C82C 20 AD D8   JSR LD8AD
C82F 4C E5 C8   JMP LC8E5
C832          LC832:
C832 AD 20 2C   LDA L2C20
C835 D0 05      BNE LC83C
C837          LC837:
C837 A9 62      LDA #$62
C839 4C 6F B6   JMP LB66F
C83C          LC83C:
C83C AD F0 2B   LDA L2BF0
C83F C9 03      CMP #$3
C841 F0 0C      BEQ LC84F
C843          LC843:
C843 A9 20      LDA #$20
C845 2C 18 2C   BIT L2C18
C848 F0 05      BEQ LC84F
C84A          LC84A:
C84A A9 60      LDA #$60
C84C 4C 6F B6   JMP LB66F
C84F          LC84F:
C84F AD 18 2C   LDA L2C18
C852 29 07      AND #$7
C854 CD ED 2B   CMP L2BED
C857 F0 05      BEQ LC85E
C859          LC859:
C859 A9 64      LDA #$64
C85B 4C 6F B6   JMP LB66F
C85E          LC85E:
C85E A0 00      LDY #$0
C860 8C EC 2B   STY L2BEC
C863 AE F0 2B   LDX L2BF0
C866 E0 02      CPX #$2
C868 D0 1A      BNE LC884
C86A          LC86A:
C86A C9 04      CMP #$4
C86C F0 EB      BEQ LC859
C86E          LC86E:
C86E B1 94      LDA (L94),Y
C870 29 4F      AND #$4F
C872 91 94      STA (L94),Y
C874 A5 82      LDA L82
C876 48         PHA
C877 A9 11      LDA #$11
C879 85 82      STA L82
C87B 20 86 D9   JSR LD986
C87E 20 AD D8   JSR LD8AD
C881 68         PLA
C882 85 82      STA L82
C884          LC884:
C884 20 94 C8   JSR LC894
C887 AD F0 2B   LDA L2BF0
C88A C9 02      CMP #$2
C88C D0 57      BNE LC8E5
C88E          LC88E:
C88E 20 29 C9   JSR LC929
C891 4C 54 B6   JMP LB654
C894          LC894:
C894 A0 13      LDY #$13
C896 B1 94      LDA (L94),Y
C898 8D F4 2B   STA L2BF4
C89B C8         INY
C89C B1 94      LDA (L94),Y
C89E 8D F5 2B   STA L2BF5
C8A1 C8         INY
C8A2 B1 94      LDA (L94),Y
C8A4 AE F3 2B   LDX L2BF3
C8A7 8D F3 2B   STA L2BF3
C8AA 8A         TXA
C8AB F0 0A      BEQ LC8B7
C8AD          LC8AD:
C8AD CD F3 2B   CMP L2BF3
C8B0 F0 05      BEQ LC8B7
C8B2          LC8B2:
C8B2 A9 50      LDA #$50
C8B4 20 6F B6   JSR LB66F
C8B7          LC8B7:
C8B7 AE EC 2B   LDX L2BEC
C8BA BD 20 2C   LDA L2C20,X
C8BD 85 5A      STA L5A
C8BF BD 28 2C   LDA L2C28,X
C8C2 85 5B      STA L5B
C8C4 20 F7 CA   JSR LCAF7
C8C7 A4 80      LDY L80
C8C9 AE EC 2B   LDX L2BEC
C8CC BD 30 2C   LDA L2C30,X
C8CF 99 E8 2C   STA L2CE8,Y
C8D2 BD 38 2C   LDA L2C38,X
C8D5 99 08 2D   STA L2D08,Y
C8D8 BD 40 2C   LDA L2C40,X
C8DB 99 28 2D   STA L2D28,Y
C8DE 60         RTS
C8DF          LC8DF:
C8DF 20 BD CB   JSR LCBBD
C8E2 20 BD C3   JSR LC3BD
C8E5          LC8E5:
C8E5 A5 82      LDA L82
C8E7 C9 02      CMP #$2
C8E9 B0 10      BCS LC8FB
C8EB          LC8EB:
C8EB 20 89 D9   JSR LD989
C8EE 20 C7 A2   JSR LA2C7
C8F1 A5 5A      LDA L5A
C8F3 9D C0 2F   STA L2FC0,X
C8F6 A5 5B      LDA L5B
C8F8 9D D0 2F   STA L2FD0,X
C8FB          LC8FB:
C8FB 4C 54 B6   JMP LB654
C8FE          LC8FE:
C8FE BC 00 2C   LDY L2C00,X
C901 B9 00 02   LDA L200,Y
C904 A0 04      LDY #$4
C906          LC906:
C906 88         DEY
C907 30 08      BMI LC911
C909          LC909:
C909 D9 1F C9   CMP LC91F,Y
C90C D0 F8      BNE LC906
C90E          LC90E:
C90E 8C F0 2B   STY L2BF0
C911          LC911:
C911 A0 06      LDY #$6
C913          LC913:
C913 88         DEY
C914 30 08      BMI LC91E
C916          LC916:
C916 D9 23 C9   CMP LC923,Y
C919 D0 F8      BNE LC913
C91B          LC91B:
C91B 8C ED 2B   STY L2BED
C91E          LC91E:
C91E 60         RTS
C91F          LC91F:
C91F 52 57 41   .BYTE $52,$57,$41
C922          LC922:
C923          LC923 = * + 1
C922 4D 44 53   EOR L5344
C925 50 55      BVC LC97C
C927          LC927:
C929          LC929 = * + 2
              ; Instruction parameter jumped to.
C927 4C 43 20   JMP L2043
C92A DB D9      .BYTE $DB,$D9
C92C A5 5A      LDA L5A
C92E F0 06      BEQ LC936
C930          LC930:
C930 20 5E 9F   JSR L9F5E
C933 4C 29 C9   JMP LC929
C936          LC936:
C936 A6 80      LDX L80
C938 BD 48 2D   LDA L2D48,X
C93B D0 03      BNE LC940
C93D          LC93D:
C93D DE 68 2D   DEC L2D68,X
C940          LC940:
C940 DE 48 2D   DEC L2D48,X
C943 A6 5B      LDX L5B
C945 E8         INX
C946 8A         TXA
C947 D0 0A      BNE LC953
C949          LC949:
C949 A9 00      LDA #$0
C94B 20 C6 DC   JSR LDCC6
C94E 20 DD A0   JSR LA0DD
C951 A9 02      LDA #$2
C953          LC953:
C953 20 C6 DC   JSR LDCC6
C956 A6 80      LDX L80
C958 A9 01      LDA #$1
C95A 9D A8 2D   STA L2DA8,X
C95D A9 80      LDA #$80
C95F 05 80      ORA L80
C961 A6 82      LDX L82
C963 9D 48 2C   STA L2C48,X
C966 60         RTS
C967          LC967:
C967 A9 0C      LDA #$C
C969 8D E2 2B   STA L2BE2
C96C A0 01      LDY #$1
C96E 8C B3 2B   STY L2BB3
C971 A6 56      LDX L56
C973 CA         DEX
C974 F0 33      BEQ LC9A9
C976          LC976:
C976 20 B8 B6   JSR LB6B8
C979 F0 55      BEQ LC9D0
C97B          LC97B:
C97C          LC97C = * + 1
              ; Instruction parameter jumped to.
C97B A0 01      LDY #$1
C97D          LC97D:
C97E          LC97E = * + 1
              ; Instruction parameter jumped to.
C97D AD 01 02   LDA L201
C980 C9 3D      CMP #$3D
C982 D0 14      BNE LC998
C984          LC984:
C984 AD 02 02   LDA L202
C987 C9 54      CMP #$54
C989 F0 04      BEQ LC98F
C98B          LC98B:
C98B C9 50      CMP #$50
C98D D0 09      BNE LC998
C98F          LC98F:
C98F A0 03      LDY #$3
C991 8C B3 2B   STY L2BB3
C994 C4 56      CPY L56
C996 F0 11      BEQ LC9A9
C998          LC998:
C998 88         DEY
C999          LC999:
C999 C8         INY
C99A 20 CF B6   JSR LB6CF
C99D F0 FA      BEQ LC999
C99F          LC99F:
C99F C4 56      CPY L56
C9A1 D0 2D      BNE LC9D0
C9A3          LC9A3:
C9A3 AC B3 2B   LDY L2BB3
C9A6 20 90 B6   JSR LB690
C9A9          LC9A9:
C9A9 AD E8 90   LDA L90E8
C9AC 8D 10 2C   STA L2C10
C9AF EE EA 2B   INC L2BEA
C9B2 EE EB 2B   INC L2BEB
C9B5 AC B3 2B   LDY L2BB3
C9B8 A9 2A      LDA #$2A
C9BA 99 00 02   STA L200,Y
C9BD 8C 00 2C   STY L2C00
C9C0 8C 08 2C   STY L2C08
C9C3 C8         INY
C9C4 84 56      STY L56
C9C6 8C 01 2C   STY L2C01
C9C9 A9 80      LDA #$80
C9CB 8D 18 2C   STA L2C18
C9CE 30 18      BMI LC9E8
C9D0          LC9D0:
C9D0 20 DE B6   JSR LB6DE
C9D3 D0 08      BNE LC9DD
C9D5          LC9D5:
C9D5 20 F6 B7   JSR LB7F6
C9D8 AC B3 2B   LDY L2BB3
C9DB C8         INY
C9DC C8         INY
C9DD          LC9DD:
C9DD 88         DEY
C9DE 88         DEY
C9DF 8C 00 2C   STY L2C00
C9E2 20 F9 B6   JSR LB6F9
C9E5 20 3D B8   JSR LB83D
C9E8          LC9E8:
C9E8 AD 01 02   LDA L201
C9EB C9 3D      CMP #$3D
C9ED D0 4F      BNE LCA3E
C9EF          LC9EF:
C9EF AD 02 02   LDA L202
C9F2 C9 50      CMP #$50
C9F4 F0 45      BEQ LCA3B
C9F6          LC9F6:
C9F6 C9 54      CMP #$54
C9F8 D0 44      BNE LCA3E
C9FA          LC9FA:
C9FA A9 40      LDA #$40
C9FC 8D B3 2B   STA L2BB3
C9FF 4E B0 2B   LSR L2BB0
CA02 AC EA 2B   LDY L2BEA
CA05          LCA05:
CA05 CC EB 2B   CPY L2BEB
CA08 B0 39      BCS LCA43
CA0A          LCA0A:
CA0A BE 00 2C   LDX L2C00,Y
CA0D BD 00 02   LDA L200,X
CA10 C9 3C      CMP #$3C
CA12 D0 07      BNE LCA1B
CA14          LCA14:
CA14 6E B4 2B   ROR L2BB4
CA17 18         CLC
CA18 20 8A CA   JSR LCA8A
CA1B          LCA1B:
CA1B C9 3E      CMP #$3E
CA1D D0 07      BNE LCA26
CA1F          LCA1F:
CA1F 6E B5 2B   ROR L2BB5
CA22 38         SEC
CA23 20 8A CA   JSR LCA8A
CA26          LCA26:
CA26 C9 4C      CMP #$4C
CA28 D0 03      BNE LCA2D
CA2A          LCA2A:
CA2A 6E B0 2B   ROR L2BB0
CA2D          LCA2D:
CA2D C9 4E      CMP #$4E
CA2F D0 05      BNE LCA36
CA31          LCA31:
CA31 A9 00      LDA #$0
CA33 8D B3 2B   STA L2BB3
CA36          LCA36:
CA36 C8         INY
CA37 D0 CC      BNE LCA05
CA39          LCA39:
CA39 F0 08      BEQ LCA43
CA3B          LCA3B:
CA3B A9 80      LDA #$80
CA3E          LCA3E = * + 1
              ; Instruction parameter jumped to.
CA3D 2C A9 00   BIT LA9
CA40 8D B3 2B   STA L2BB3
CA43          LCA43:
CA43 2C B3 2B   BIT L2BB3
CA46 10 0F      BPL LCA57
CA48          LCA48:
CA48 A9 00      LDA #$0
CA4A A8         TAY
CA4B          LCA4B:
CA4B 99 10 2C   STA L2C10,Y
CA4E C8         INY
CA4F CC EA 2B   CPY L2BEA
CA52 90 F7      BCC LCA4B
CA54          LCA54:
CA54 20 23 B0   JSR LB023
CA57          LCA57:
CA57 A9 00      LDA #$0
CA59 8D EE 2B   STA L2BEE
CA5C AC EA 2B   LDY L2BEA
CA5F CC EB 2B   CPY L2BEB
CA62 F0 03      BEQ LCA67
CA64          LCA64:
CA64 20 08 B9   JSR LB908
CA67          LCA67:
CA67 20 84 BE   JSR LBE84
CA6A A9 00      LDA #$0
CA6C 20 20 BA   JSR LBA20
CA6F 20 E1 C2   JSR LC2E1
CA72 20 15 BF   JSR LBF15
CA75 20 E7 C4   JSR LC4E7
CA78 20 FE CE   JSR LCEFE
CA7B A6 80      LDX L80
CA7D 9D C8 2D   STA L2DC8,X
CA80 A9 04      LDA #$4
CA82 9D 88 2D   STA L2D88,X
CA85 A9 00      LDA #$0
CA87 85 DC      STA LDC
CA89 60         RTS
CA8A          LCA8A:
CA8A 48         PHA
CA8B 98         TYA
CA8C 48         PHA
CA8D A9 04      LDA #$4
CA8F 90 02      BCC LCA93
CA91          LCA91:
CA91 A9 09      LDA #$9
CA93          LCA93:
CA93 48         PHA
CA94 A0 00      LDY #$0
CA96 86 51      STX L51
CA98          LCA98:
CA98 A6 51      LDX L51
CA9A 8A         TXA
CA9B 18         CLC
CA9C 79 F2 CA   ADC LCAF2,Y
CA9F AA         TAX
CAA0 20 DB CA   JSR LCADB
CAA3 99 AA 2B   STA L2BAA,Y
CAA6 C8         INY
CAA7 C0 05      CPY #$5
CAA9 90 ED      BCC LCA98
CAAB          LCAAB:
CAAB AD AD 2B   LDA L2BAD
CAAE E9 0C      SBC #$C
CAB0 D0 03      BNE LCAB5
CAB2          LCAB2:
CAB2 8D AD 2B   STA L2BAD
CAB5          LCAB5:
CAB5 E8         INX
CAB6 E8         INX
CAB7 BD 00 02   LDA L200,X
CABA 29 7F      AND #$7F
CABC C9 41      CMP #$41
CABE F0 09      BEQ LCAC9
CAC0          LCAC0:
CAC0 AD AD 2B   LDA L2BAD
CAC3 18         CLC
CAC4 69 0C      ADC #$C
CAC6 8D AD 2B   STA L2BAD
CAC9          LCAC9:
CAC9 68         PLA
CACA A8         TAY
CACB A2 04      LDX #$4
CACD          LCACD:
CACD BD AA 2B   LDA L2BAA,X
CAD0 99 08 2B   STA L2B08,Y
CAD3 88         DEY
CAD4 CA         DEX
CAD5 10 F6      BPL LCACD
CAD7          LCAD7:
CAD7 68         PLA
CAD8 A8         TAY
CAD9 68         PLA
CADA 60         RTS
CADB          LCADB:
CADB BD 00 02   LDA L200,X
CADE 29 0F      AND #$F
CAE0 0A         ASL A
CAE1 85 50      STA L50
CAE3 0A         ASL A
CAE4 0A         ASL A
CAE5 65 50      ADC L50
CAE7 85 50      STA L50
CAE9 E8         INX
CAEA BD 00 02   LDA L200,X
CAED 29 0F      AND #$F
CAEF 65 50      ADC L50
CAF1 60         RTS
CAF2          LCAF2:
CAF2 07         .BYTE $7
CAF3          LCAF3:
CAF3 01 04      ORA (L4,X)
CAF5 0A         ASL A
CAF7          LCAF7 = * + 1
              ; Instruction parameter jumped to.
CAF6 0D A9 01   ORA L1A9
CAF9 20 C2 DA   JSR LDAC2
CAFC 20 92 CB   JSR LCB92
CAFF AD ED 2B   LDA L2BED
CB02 48         PHA
CB03 0A         ASL A
CB04 9D 88 2D   STA L2D88,X
CB07 20 5A D8   JSR LD85A
CB0A A6 80      LDX L80
CB0C A5 5A      LDA L5A
CB0E D0 05      BNE LCB15
CB10          LCB10:
CB10 A5 5B      LDA L5B
CB12 9D E8 2D   STA L2DE8,X
CB15          LCB15:
CB15 68         PLA
CB16 C9 04      CMP #$4
CB18 D0 6A      BNE LCB84
CB1A          LCB1A:
CB1A A4 82      LDY L82
CB1C B9 48 2C   LDA L2C48,Y
CB1F 09 40      ORA #$40
CB21 99 48 2C   STA L2C48,Y
CB24 AD F3 2B   LDA L2BF3
CB27 9D 08 2E   STA L2E08,X
CB2A 20 76 DC   JSR LDC76
CB2D 10 03      BPL LCB32
CB2F          LCB2F:
CB2F 4C EC DA   JMP LDAEC
CB32          LCB32:
CB32 A6 80      LDX L80
CB34 9D A8 2C   STA L2CA8,X
CB37 AC F4 2B   LDY L2BF4
CB3A 84 5A      STY L5A
CB3C AC F5 2B   LDY L2BF5
CB3F 84 5B      STY L5B
CB41 20 76 D9   JSR LD976
CB44 20 B9 D9   JSR LD9B9
CB47 20 65 D9   JSR LD965
CB4A A9 02      LDA #$2
CB4C 20 98 D0   JSR LD098
CB4F A6 80      LDX L80
CB51 A0 00      LDY #$0
CB53 B1 94      LDA (L94),Y
CB55 38         SEC
CB56 E9 FE      SBC #$FE
CB58 F0 02      BEQ LCB5C
CB5A          LCB5A:
CB5A A9 20      LDA #$20
CB5C          LCB5C:
CB5C 9D A8 2E   STA L2EA8,X
CB5F D0 11      BNE LCB72
CB61          LCB61:
CB61 AD F4 2B   LDA L2BF4
CB64 9D 88 2E   STA L2E88,X
CB67 AD F5 2B   LDA L2BF5
CB6A 9D 68 2E   STA L2E68,X
CB6D A9 FF      LDA #$FF
CB6F 9D 48 2E   STA L2E48,X
CB72          LCB72:
CB72 A6 80      LDX L80
CB74 A9 02      LDA #$2
CB76 9D 28 2E   STA L2E28,X
CB79 A9 00      LDA #$0
CB7B 20 C6 DC   JSR LDCC6
CB7E 20 2B D3   JSR LD32B
CB81 4C 89 D9   JMP LD989
CB84          LCB84:
CB84 20 08 A0   JSR LA008
CB87 A6 80      LDX L80
CB89 9D C8 2D   STA L2DC8,X
CB8C A9 88      LDA #$88
CB8E 9D A8 2D   STA L2DA8,X
CB91 60         RTS
CB92          LCB92:
CB92 A6 80      LDX L80
CB94 BD 68 2C   LDA L2C68,X
CB97 0A         ASL A
CB98 30 06      BMI LCBA0
CB9A          LCB9A:
CB9A A8         TAY
CB9B A9 02      LDA #$2
CB9D 99 A0 00   STA LA0,Y
CBA0          LCBA0:
CBA0 BD 88 2C   LDA L2C88,X
CBA3 09 80      ORA #$80
CBA5 9D 88 2C   STA L2C88,X
CBA8 0A         ASL A
CBA9 30 06      BMI LCBB1
CBAB          LCBAB:
CBAB A8         TAY
CBAC A9 02      LDA #$2
CBAE 99 A0 00   STA LA0,Y
CBB1          LCBB1:
CBB1 A9 00      LDA #$0
CBB3 9D E8 2D   STA L2DE8,X
CBB6 9D 48 2D   STA L2D48,X
CBB9 9D 68 2D   STA L2D68,X
CBBC 60         RTS
CBBD          LCBBD:
CBBD 20 81 A4   JSR LA481
CBC0          LCBC0:
CBC0 A9 01      LDA #$1
CBC2 20 BF DA   JSR LDABF
CBC5 20 73 D9   JSR LD973
CBC8 20 92 CB   JSR LCB92
CBCB A6 80      LDX L80
CBCD AD ED 2B   LDA L2BED
CBD0 48         PHA
CBD1 0A         ASL A
CBD2 9D 88 2D   STA L2D88,X
CBD5 68         PLA
CBD6 C9 04      CMP #$4
CBD8 F0 06      BEQ LCBE0
CBDA          LCBDA:
CBDA A9 01      LDA #$1
CBDC 9D A8 2D   STA L2DA8,X
CBDF 60         RTS
CBE0          LCBE0:
CBE0 A4 82      LDY L82
CBE2 B9 48 2C   LDA L2C48,Y
CBE5 29 3F      AND #$3F
CBE7 09 40      ORA #$40
CBE9 99 48 2C   STA L2C48,Y
CBEC AD F3 2B   LDA L2BF3
CBEF 9D 08 2E   STA L2E08,X
CBF2 20 76 DC   JSR LDC76
CBF5 10 03      BPL LCBFA
CBF7          LCBF7:
CBF7 4C EC DA   JMP LDAEC
CBFA          LCBFA:
CBFA 48         PHA
CBFB 20 7E B0   JSR LB07E
CBFE C9 01      CMP #$1
CC00 F0 04      BEQ LCC06
CC02          LCC02:
CC02 C9 04      CMP #$4
CC04 90 03      BCC LCC09
CC06          LCC06:
CC06 A9 00      LDA #$0
CC09          LCC09 = * + 1
              ; Instruction parameter jumped to.
CC08 2C A9 20   BIT L20A9
CC0B A6 80      LDX L80
CC0D 9D A8 2E   STA L2EA8,X
CC10 68         PLA
CC11 9D A8 2C   STA L2CA8,X
CC14 20 7D D0   JSR LD07D
CC17 20 F3 A3   JSR LA3F3
CC1A A5 5A      LDA L5A
CC1C 8D F4 2B   STA L2BF4
CC1F A5 5B      LDA L5B
CC21 8D F5 2B   STA L2BF5
CC24 A6 80      LDX L80
CC26 BD A8 2C   LDA L2CA8,X
CC29 20 76 D9   JSR LD976
CC2C A9 00      LDA #$0
CC2E 20 A6 D0   JSR LD0A6
CC31 A9 00      LDA #$0
CC33 20 DA CC   JSR LCCDA
CC36 A9 11      LDA #$11
CC38 20 DA CC   JSR LCCDA
CC3B A9 00      LDA #$0
CC3D 20 DA CC   JSR LCCDA
CC40 AD F3 2B   LDA L2BF3
CC43 20 DA CC   JSR LCCDA
CC46 A5 5A      LDA L5A
CC48 20 DA CC   JSR LCCDA
CC4B A5 5B      LDA L5B
CC4D 20 DA CC   JSR LCCDA
CC50 A9 10      LDA #$10
CC52 20 A6 D0   JSR LD0A6
CC55 20 89 D9   JSR LD989
CC58 A5 5A      LDA L5A
CC5A 20 DA CC   JSR LCCDA
CC5D A5 5B      LDA L5B
CC5F 20 DA CC   JSR LCCDA
CC62 20 B3 D9   JSR LD9B3
CC65 20 65 D9   JSR LD965
CC68 20 BE D7   JSR LD7BE
CC6B D0 03      BNE LCC70
CC6D          LCC6D:
CC6D 20 92 CC   JSR LCC92
CC70          LCC70:
CC70 A9 02      LDA #$2
CC72 20 C6 DC   JSR LDCC6
CC75 A6 80      LDX L80
CC77 38         SEC
CC78 A9 00      LDA #$0
CC7A FD 08 2E   SBC L2E08,X
CC7D 9D 28 2E   STA L2E28,X
CC80 20 E2 D4   JSR LD4E2
CC83 20 3C D0   JSR LD03C
CC86 20 A7 D9   JSR LD9A7
CC89 20 65 D9   JSR LD965
CC8C 20 48 A3   JSR LA348
CC8F 4C 72 CB   JMP LCB72
CC92          LCC92:
CC92 A6 80      LDX L80
CC94 BD A8 2C   LDA L2CA8,X
CC97 20 7D D0   JSR LD07D
CC9A 20 A6 D0   JSR LD0A6
CC9D AD F4 2B   LDA L2BF4
CCA0 20 DA CC   JSR LCCDA
CCA3 AD F5 2B   LDA L2BF5
CCA6 20 DA CC   JSR LCCDA
CCA9 A9 FE      LDA #$FE
CCAB 20 DA CC   JSR LCCDA
CCAE AD F4 2B   LDA L2BF4
CCB1 20 DA CC   JSR LCCDA
CCB4 AD F5 2B   LDA L2BF5
CCB7 20 DA CC   JSR LCCDA
CCBA 20 F3 A3   JSR LA3F3
CCBD A6 80      LDX L80
CCBF A5 5A      LDA L5A
CCC1 9D 88 2E   STA L2E88,X
CCC4 8D F4 2B   STA L2BF4
CCC7 A5 5B      LDA L5B
CCC9 9D 68 2E   STA L2E68,X
CCCC 8D F5 2B   STA L2BF5
CCCF A9 FF      LDA #$FF
CCD1 9D 48 2E   STA L2E48,X
CCD4 20 D9 D7   JSR LD7D9
CCD7 4C 89 D9   JMP LD989
CCDA          LCCDA:
CCDA 48         PHA
CCDB A6 80      LDX L80
CCDD BD A8 2C   LDA L2CA8,X
CCE0 4C F6 CE   JMP LCEF6
CCE3          LCCE3:
CCE3 A5 82      LDA L82
CCE5 D0 0B      BNE LCCF2
CCE7          LCCE7:
CCE7 A9 00      LDA #$0
CCE9 8D C5 2B   STA L2BC5
CCEC 20 04 DB   JSR LDB04
CCEF          LCCEF:
CCEF 4C 6B DB   JMP LDB6B
CCF2          LCCF2:
CCF2 C9 0F      CMP #$F
CCF4 F0 14      BEQ LCD0A
CCF6          LCCF6:
CCF6 20 1C CD   JSR LCD1C
CCF9 A5 82      LDA L82
CCFB C9 02      CMP #$2
CCFD 90 F0      BCC LCCEF
CCFF          LCCFF:
CCFF AD DE 2B   LDA L2BDE
CD02 D0 03      BNE LCD07
CD04          LCD04:
CD04 4C 5C B6   JMP LB65C
CD07          LCD07:
CD07 4C 6C B6   JMP LB66C
CD0A          LCD0A:
CD0A A9 0E      LDA #$E
CD0C 85 82      STA L82
CD0E          LCD0E:
CD0E 20 1C CD   JSR LCD1C
CD11 C6 82      DEC L82
CD13 10 F9      BPL LCD0E
CD15          LCD15:
CD15 AD DE 2B   LDA L2BDE
CD18 F0 EA      BEQ LCD04
CD1A          LCD1A:
CD1A D0 EB      BNE LCD07
CD1C          LCD1C:
CD1C A6 82      LDX L82
CD1E BD 48 2C   LDA L2C48,X
CD21 C9 FF      CMP #$FF
CD23 D0 01      BNE LCD26
CD25          LCD25:
CD25 60         RTS
CD26          LCD26:
CD26 29 3F      AND #$3F
CD28 85 80      STA L80
CD2A AA         TAX
CD2B BD C8 2C   LDA L2CC8,X
CD2E 20 23 B0   JSR LB023
CD31 20 AC DA   JSR LDAAC
CD34 C9 07      CMP #$7
CD36 F0 0F      BEQ LCD47
CD38          LCD38:
CD38 C9 04      CMP #$4
CD3A F0 11      BEQ LCD4D
CD3C          LCD3C:
CD3C 20 92 DA   JSR LDA92
CD3F B0 09      BCS LCD4A
CD41          LCD41:
CD41 20 AF CD   JSR LCDAF
CD44 20 F1 CD   JSR LCDF1
CD47          LCD47:
CD47 20 53 A3   JSR LA353
CD4A          LCD4A:
CD4A 4C 04 DB   JMP LDB04
CD4D          LCD4D:
CD4D 20 54 DA   JSR LDA54
CD50 20 79 DB   JSR LDB79
CD53 20 A6 D3   JSR LD3A6
CD56 A6 99      LDX L99
CD58 86 54      STX L54
CD5A 20 BE D7   JSR LD7BE
CD5D F0 2B      BEQ LCD8A
CD5F          LCD5F:
CD5F E6 54      INC L54
CD61 A9 00      LDA #$0
CD63 85 51      STA L51
CD65 85 52      STA L52
CD67 A5 9A      LDA L9A
CD69 38         SEC
CD6A E9 0E      SBC #$E
CD6C 85 53      STA L53
CD6E 20 05 D1   JSR LD105
CD71 A6 80      LDX L80
CD73 A5 51      LDA L51
CD75 9D 48 2D   STA L2D48,X
CD78 A5 52      LDA L52
CD7A 9D 68 2D   STA L2D68,X
CD7D          LCD7D:
CD7D A9 40      LDA #$40
CD7F 20 FD D9   JSR LD9FD
CD82 F0 03      BEQ LCD87
CD84          LCD84:
CD84 20 F1 CD   JSR LCDF1
CD87          LCD87:
CD87 4C 04 DB   JMP LDB04
CD8A          LCD8A:
CD8A A5 9A      LDA L9A
CD8C 38         SEC
CD8D E9 0E      SBC #$E
CD8F 85 53      STA L53
CD91 AD F6 2B   LDA L2BF6
CD94 85 88      STA L88
CD96 20 1A D1   JSR LD11A
CD99 A2 00      LDX #$0
CD9B A9 02      LDA #$2
CD9D 20 4F D1   JSR LD14F
CDA0 A6 80      LDX L80
CDA2 A5 8B      LDA L8B
CDA4 9D 48 2D   STA L2D48,X
CDA7 A5 8C      LDA L8C
CDA9 9D 68 2D   STA L2D68,X
CDAC 4C 7D CD   JMP LCD7D
CDAF          LCDAF:
CDAF A6 80      LDX L80
CDB1 BD 48 2D   LDA L2D48,X
CDB4 1D 68 2D   ORA L2D68,X
CDB7 D0 0C      BNE LCDC5
CDB9          LCDB9:
CDB9 20 D4 DC   JSR LDCD4
CDBC C9 02      CMP #$2
CDBE D0 05      BNE LCDC5
CDC0          LCDC0:
CDC0 A9 0D      LDA #$D
CDC2 20 EA CE   JSR LCEEA
CDC5          LCDC5:
CDC5 20 D4 DC   JSR LDCD4
CDC8 C9 02      CMP #$2
CDCA D0 0F      BNE LCDDB
CDCC          LCDCC:
CDCC A6 80      LDX L80
CDCE BD 48 2D   LDA L2D48,X
CDD1 D0 03      BNE LCDD6
CDD3          LCDD3:
CDD3 DE 68 2D   DEC L2D68,X
CDD6          LCDD6:
CDD6 DE 48 2D   DEC L2D48,X
CDD9 A9 00      LDA #$0
CDDB          LCDDB:
CDDB 38         SEC
CDDC E9 01      SBC #$1
CDDE 48         PHA
CDDF A9 00      LDA #$0
CDE1 20 C6 DC   JSR LDCC6
CDE4 20 EA CE   JSR LCEEA
CDE7 68         PLA
CDE8 20 EA CE   JSR LCEEA
CDEB 20 85 D8   JSR LD885
CDEE 4C 65 D9   JMP LD965
CDF1          LCDF1:
CDF1 A5 82      LDA L82
CDF3 48         PHA
CDF4 A6 80      LDX L80
CDF6 BD E8 2C   LDA L2CE8,X
CDF9 85 5A      STA L5A
CDFB BD 08 2D   LDA L2D08,X
CDFE 85 5B      STA L5B
CE00 20 A2 A1   JSR LA1A2
CE03 A4 80      LDY L80
CE05 BE 28 2D   LDX L2D28,Y
CE08 BD 00 22   LDA L2200,X
CE0B 29 20      AND #$20
CE0D D0 0C      BNE LCE1B
CE0F          LCE0F:
CE0F A9 80      LDA #$80
CE11 1D 00 22   ORA L2200,X
CE14 29 8F      AND #$8F
CE16 9D 00 22   STA L2200,X
CE19 D0 40      BNE LCE5B
CE1B          LCE1B:
CE1B B9 88 2D   LDA L2D88,Y
CE1E 29 0F      AND #$F
CE20 C9 08      CMP #$8
CE22 F0 37      BEQ LCE5B
CE24          LCE24:
CE24 BD 00 22   LDA L2200,X
CE27 29 8F      AND #$8F
CE29 9D 00 22   STA L2200,X
CE2C BD 01 22   LDA L2201,X
CE2F 85 5A      STA L5A
CE31 BD 02 22   LDA L2202,X
CE34 85 5B      STA L5B
CE36 BD 1A 22   LDA L221A,X
CE39 D0 0C      BNE LCE47
CE3B          LCE3B:
CE3B 85 5A      STA L5A
CE3D BD 1B 22   LDA L221B,X
CE40 85 5B      STA L5B
CE42 A9 67      LDA #$67
CE44 4C 33 FF   JMP LFF33
CE47          LCE47:
CE47 9D 01 22   STA L2201,X
CE4A BD 1B 22   LDA L221B,X
CE4D 9D 02 22   STA L2202,X
CE50 A9 00      LDA #$0
CE52 9D 1A 22   STA L221A,X
CE55 9D 1B 22   STA L221B,X
CE58 20 2B B3   JSR LB32B
CE5B          LCE5B:
CE5B 68         PLA
CE5C 85 82      STA L82
CE5E 20 92 DA   JSR LDA92
CE61 A4 80      LDY L80
CE63 BE 28 2D   LDX L2D28,Y
CE66 B9 48 2D   LDA L2D48,Y
CE69 9D 1C 22   STA L221C,X
CE6C B9 68 2D   LDA L2D68,Y
CE6F 9D 1D 22   STA L221D,X
CE72 20 B4 B5   JSR LB5B4
CE75 A4 80      LDY L80
CE77 B9 E8 2C   LDA L2CE8,Y
CE7A 85 5A      STA L5A
CE7C B9 08 2D   LDA L2D08,Y
CE7F 85 5B      STA L5B
CE81 4C A5 A1   JMP LA1A5
CE84          LCE84:
CE84 A9 11      LDA #$11
CE86 85 82      STA L82
CE88 20 A3 CE   JSR LCEA3
CE8B 85 84      STA L84
CE8D A6 80      LDX L80
CE8F BD A8 2D   LDA L2DA8,X
CE92 29 08      AND #$8
CE94 85 81      STA L81
CE96 D0 0A      BNE LCEA2
CE98          LCE98:
CE98 20 AC DA   JSR LDAAC
CE9B F0 05      BEQ LCEA2
CE9D          LCE9D:
CE9D A9 80      LDA #$80
CE9F 20 EB D9   JSR LD9EB
CEA2          LCEA2:
CEA2 60         RTS
CEA3          LCEA3:
CEA3 20 60 DA   JSR LDA60
CEA6 20 3C EE   JSR LEE3C
CEA9 20 AC DA   JSR LDAAC
CEAC D0 06      BNE LCEB4
CEAE          LCEAE:
CEAE 20 A5 9F   JSR L9FA5
CEB1 4C B7 CE   JMP LCEB7
CEB4          LCEB4:
CEB4 20 2B 9F   JSR L9F2B
CEB7          LCEB7:
CEB7 A6 80      LDX L80
CEB9 BD C8 2D   LDA L2DC8,X
CEBC 60         RTS
CEBD          LCEBD:
CEBD A2 12      LDX #$12
CEBF 86 82      STX L82
CEC1 20 92 DA   JSR LDA92
CEC4 20 3C EE   JSR LEE3C
CEC7 20 AC DA   JSR LDAAC
CECA 90 05      BCC LCED1
CECC          LCECC:
CECC A9 20      LDA #$20
CECE 20 F2 D9   JSR LD9F2
CED1          LCED1:
CED1 A5 82      LDA L82
CED3 C9 0F      CMP #$F
CED5 D0 03      BNE LCEDA
CED7          LCED7:
CED7 4C AD A0   JMP LA0AD
CEDA          LCEDA:
CEDA 20 AC DA   JSR LDAAC
CEDD B0 03      BCS LCEE2
CEDF          LCEDF:
CEDF 4C C1 A0   JMP LA0C1
CEE2          LCEE2:
CEE2 D0 03      BNE LCEE7
CEE4          LCEE4:
CEE4 4C 63 A1   JMP LA163
CEE7          LCEE7:
CEE7 4C 68 A1   JMP LA168
CEEA          LCEEA:
CEEA 48         PHA
CEEB 20 F2 DC   JSR LDCF2
CEEE 10 06      BPL LCEF6
CEF0          LCEF0:
CEF0 68         PLA
CEF1 A9 61      LDA #$61
CEF3 4C 6F B6   JMP LB66F
CEF6          LCEF6:
CEF6 0A         ASL A
CEF7 AA         TAX
CEF8 68         PLA
CEF9 81 A0      STA (LA0,X)
CEFB F6 A0      INC LA0,X
CEFD 60         RTS
CEFE          LCEFE:
CEFE A6 80      LDX L80
CF00 BD 68 2C   LDA L2C68,X
CF03 10 03      BPL LCF08
CF05          LCF05:
CF05 BD 88 2C   LDA L2C88,X
CF08          LCF08:
CF08 29 BF      AND #$BF
CF0A 0A         ASL A
CF0B AA         TAX
CF0C A4 80      LDY L80
CF0E B9 E8 2D   LDA L2DE8,Y
CF11 F0 12      BEQ LCF25
CF13          LCF13:
CF13 A1 A0      LDA (LA0,X)
CF15 48         PHA
CF16 B5 A0      LDA LA0,X
CF18 D9 E8 2D   CMP L2DE8,Y
CF1B D0 04      BNE LCF21
CF1D          LCF1D:
CF1D A9 FF      LDA #$FF
CF1F 95 A0      STA LA0,X
CF21          LCF21:
CF21 68         PLA
CF22 F6 A0      INC LA0,X
CF24 60         RTS
CF25          LCF25:
CF25 A1 A0      LDA (LA0,X)
CF27 F6 A0      INC LA0,X
CF29 60         RTS
CF2A          LCF2A:
CF2A 20 EA CE   JSR LCEEA
CF2D F0 01      BEQ LCF30
CF2F          LCF2F:
CF2F 60         RTS
CF30          LCF30:
CF30 20 F3 A3   JSR LA3F3
CF33 A9 00      LDA #$0
CF35 20 C6 DC   JSR LDCC6
CF38 A5 5A      LDA L5A
CF3A 20 EA CE   JSR LCEEA
CF3D A5 5B      LDA L5B
CF3F 20 EA CE   JSR LCEEA
CF42 20 85 D8   JSR LD885
CF45 20 79 DB   JSR LDB79
CF48 20 73 D9   JSR LD973
CF4B A9 02      LDA #$2
CF4D 4C C6 DC   JMP LDCC6
CF50          LCF50:
CF50 20 88 CF   JSR LCF88
CF53 20 CD CF   JSR LCFCD
CF56 A5 90      LDA L90
CF58 85 9B      STA L9B
CF5A 20 D0 CF   JSR LCFD0
CF5D E6 9B      INC L9B
CF5F E6 9B      INC L9B
CF61 20 BE D7   JSR LD7BE
CF64 F0 0D      BEQ LCF73
CF66          LCF66:
CF66 A5 8B      LDA L8B
CF68 85 99      STA L99
CF6A A5 90      LDA L90
CF6C 0A         ASL A
CF6D 18         CLC
CF6E 69 10      ADC #$10
CF70 85 9A      STA L9A
CF72 60         RTS
CF73          LCF73:
CF73 A5 90      LDA L90
CF75 0A         ASL A
CF76 18         CLC
CF77 69 10      ADC #$10
CF79 85 9A      STA L9A
CF7B 20 D3 CF   JSR LCFD3
CF7E A5 90      LDA L90
CF80 85 99      STA L99
CF82 A5 8B      LDA L8B
CF84 8D F6 2B   STA L2BF6
CF87 60         RTS
CF88          LCF88:
CF88 20 FF CF   JSR LCFFF
CF8B 85 92      STA L92
CF8D A6 80      LDX L80
CF8F BD 48 2D   LDA L2D48,X
CF92 85 90      STA L90
CF94 BD 68 2D   LDA L2D68,X
CF97 85 91      STA L91
CF99 D0 04      BNE LCF9F
CF9B          LCF9B:
CF9B A5 90      LDA L90
CF9D F0 0B      BEQ LCFAA
CF9F          LCF9F:
CF9F A5 90      LDA L90
CFA1 38         SEC
CFA2 E9 01      SBC #$1
CFA4 85 90      STA L90
CFA6 B0 02      BCS LCFAA
CFA8          LCFA8:
CFA8 C6 91      DEC L91
CFAA          LCFAA:
CFAA BD 08 2E   LDA L2E08,X
CFAD 85 50      STA L50
CFAF          LCFAF:
CFAF 46 50      LSR L50
CFB1 90 03      BCC LCFB6
CFB3          LCFB3:
CFB3 20 13 D0   JSR LD013
CFB6          LCFB6:
CFB6 20 0B D0   JSR LD00B
CFB9 A5 50      LDA L50
CFBB D0 F2      BNE LCFAF
CFBD          LCFBD:
CFBD A5 98      LDA L98
CFBF 18         CLC
CFC0 65 8B      ADC L8B
CFC2 85 8B      STA L8B
CFC4 90 06      BCC LCFCC
CFC6          LCFC6:
CFC6 E6 8C      INC L8C
CFC8 D0 02      BNE LCFCC
CFCA          LCFCA:
CFCA E6 8D      INC L8D
CFCC          LCFCC:
CFCC 60         RTS
CFCD          LCFCD:
CFCD A9 FE      LDA #$FE
CFD0          LCFD0 = * + 1
              ; Instruction parameter jumped to.
CFCF 2C A9 78   BIT L78A9
CFD3          LCFD3 = * + 1
              ; Instruction parameter jumped to.
CFD2 2C A9 06   BIT L6A9
CFD5 85 50      STA L50
CFD7 A9 00      LDA #$0
CFD9 85 90      STA L90
CFDB 85 91      STA L91
CFDD A2 18      LDX #$18
CFDF          LCFDF:
CFDF 06 8B      ASL L8B
CFE1 26 8C      ROL L8C
CFE3 26 8D      ROL L8D
CFE5 26 90      ROL L90
CFE7 26 91      ROL L91
CFE9 A5 90      LDA L90
CFEB 38         SEC
CFEC E5 50      SBC L50
CFEE A8         TAY
CFEF A5 91      LDA L91
CFF1 E9 00      SBC #$0
CFF3 90 06      BCC LCFFB
CFF5          LCFF5:
CFF5 E6 8B      INC L8B
CFF7 85 91      STA L91
CFF9 84 90      STY L90
CFFB          LCFFB:
CFFB CA         DEX
CFFC D0 E1      BNE LCFDF
CFFE          LCFFE:
CFFE 60         RTS
CFFF          LCFFF:
CFFF A9 00      LDA #$0
D001 85 8B      STA L8B
D003 85 8C      STA L8C
D005 85 8D      STA L8D
D007 60         RTS
D008          LD008:
D008 20 0B D0   JSR LD00B
D00B          LD00B:
D00B 18         CLC
D00C 26 90      ROL L90
D00E 26 91      ROL L91
D010 26 92      ROL L92
D012 60         RTS
D013          LD013:
D013 18         CLC
D014 A2 FD      LDX #$FD
D016          LD016:
D016 B5 8E      LDA L8E,X
D018 75 93      ADC L93,X
D01A 95 8E      STA L8E,X
D01C E8         INX
D01D D0 F7      BNE LD016
D01F          LD01F:
D01F 60         RTS
D020          LD020:
D020 20 4F D0   JSR LD04F
D023 A5 5A      LDA L5A
D025 91 94      STA (L94),Y
D027 C8         INY
D028 A5 5B      LDA L5B
D02A 91 94      STA (L94),Y
D02C 4C D5 D2   JMP LD2D5
D02F          LD02F:
D02F 20 4F D0   JSR LD04F
D032 B1 94      LDA (L94),Y
D034 85 5A      STA L5A
D036 C8         INY
D037 B1 94      LDA (L94),Y
D039 85 5B      STA L5B
D03B 60         RTS
D03C          LD03C:
D03C 20 4F D0   JSR LD04F
D03F A9 00      LDA #$0
D041 91 94      STA (L94),Y
D043 C8         INY
D044 A6 80      LDX L80
D046 BD 28 2E   LDA L2E28,X
D049 AA         TAX
D04A CA         DEX
D04B 8A         TXA
D04C 91 94      STA (L94),Y
D04E 60         RTS
D04F          LD04F:
D04F 20 F2 DC   JSR LDCF2
D052 0A         ASL A
D053 AA         TAX
D054 B5 A1      LDA LA1,X
D056 85 95      STA L95
D058 A9 00      LDA #$0
D05A 85 94      STA L94
D05C A0 00      LDY #$0
D05E 60         RTS
D05F          LD05F:
D05F 48         PHA
D060 A9 00      LDA #$0
D062 85 50      STA L50
D064 85 52      STA L52
D066 98         TYA
D067 18         CLC
D068 69 03      ADC #$3
D06A 85 51      STA L51
D06C 8A         TXA
D06D 18         CLC
D06E 69 03      ADC #$3
D070 85 53      STA L53
D072 68         PLA
D073 A8         TAY
D074 88         DEY
D075          LD075:
D075 B1 50      LDA (L50),Y
D077 91 52      STA (L52),Y
D079 88         DEY
D07A 10 F9      BPL LD075
D07C          LD07C:
D07C 60         RTS
D07D          LD07D:
D07D A8         TAY
D07E 18         CLC
D07F 69 03      ADC #$3
D081 85 51      STA L51
D083 A9 00      LDA #$0
D085 85 50      STA L50
D087 A8         TAY
D088          LD088:
D088 91 50      STA (L50),Y
D08A C8         INY
D08B D0 FB      BNE LD088
D08D          LD08D:
D08D 60         RTS
D08E          LD08E:
D08E A9 00      LDA #$0
D090 20 98 D0   JSR LD098
D093 A0 02      LDY #$2
D095 B1 94      LDA (L94),Y
D097 60         RTS
D098          LD098:
D098 85 94      STA L94
D09A A6 80      LDX L80
D09C BD A8 2C   LDA L2CA8,X
D09F AA         TAX
D0A0 18         CLC
D0A1 69 03      ADC #$3
D0A3 85 95      STA L95
D0A5 60         RTS
D0A6          LD0A6:
D0A6 48         PHA
D0A7 20 98 D0   JSR LD098
D0AA 48         PHA
D0AB 8A         TXA
D0AC 0A         ASL A
D0AD AA         TAX
D0AE 68         PLA
D0AF 95 A1      STA LA1,X
D0B1 68         PLA
D0B2 95 A0      STA LA0,X
D0B4 60         RTS
D0B5          LD0B5:
D0B5 20 56 D1   JSR LD156
D0B8 30 0F      BMI LD0C9
D0BA          LD0BA:
D0BA 50 14      BVC LD0D0
D0BC          LD0BC:
D0BC A6 80      LDX L80
D0BE BD A8 2C   LDA L2CA8,X
D0C1 20 D9 D0   JSR LD0D9
D0C4 20 56 D1   JSR LD156
D0C7 10 07      BPL LD0D0
D0C9          LD0C9:
D0C9 20 A6 D3   JSR LD3A6
D0CC 2C 20 D5   BIT LD520
D0CF 60         RTS
D0D0          LD0D0:
D0D0 A5 9A      LDA L9A
D0D2 20 A6 D0   JSR LD0A6
D0D5 2C 21 D5   BIT LD521
D0D8 60         RTS
D0D9          LD0D9:
D0D9 85 9C      STA L9C
D0DB A9 80      LDA #$80
D0DD D0 04      BNE LD0E3
D0DF          LD0DF:
D0DF 85 9C      STA L9C
D0E1 A9 90      LDA #$90
D0E3          LD0E3:
D0E3 85 55      STA L55
D0E5 B1 94      LDA (L94),Y
D0E7 85 5A      STA L5A
D0E9 C8         INY
D0EA B1 94      LDA (L94),Y
D0EC 85 5B      STA L5B
D0EE A5 9C      LDA L9C
D0F0 20 76 D9   JSR LD976
D0F3 A6 9C      LDX L9C
D0F5 4C 60 D9   JMP LD960
D0F8          LD0F8:
D0F8 A6 80      LDX L80
D0FA BD A8 2C   LDA L2CA8,X
D0FD 4C D7 DC   JMP LDCD7
D100          LD100:
D100 A9 78      LDA #$78
D102 20 10 D1   JSR LD110
D105          LD105:
D105 CA         DEX
D106 10 F8      BPL LD100
D108          LD108:
D108 A5 53      LDA L53
D10A 4A         LSR A
D10B 20 10 D1   JSR LD110
D10E A5 54      LDA L54
D110          LD110:
D110 18         CLC
D111 65 51      ADC L51
D113 85 51      STA L51
D115 90 02      BCC LD119
D117          LD117:
D117 E6 52      INC L52
D119          LD119:
D119 60         RTS
D11A          LD11A:
D11A 20 FF CF   JSR LCFFF
D11D 20 46 D1   JSR LD146
D120 A4 88      LDY L88
D122          LD122:
D122 88         DEY
D123 30 0A      BMI LD12F
D125          LD125:
D125 A2 02      LDX #$2
D127 A9 D6      LDA #$D6
D129 20 4F D1   JSR LD14F
D12C 4C 22 D1   JMP LD122
D12F          LD12F:
D12F A4 54      LDY L54
D131          LD131:
D131 88         DEY
D132 30 0A      BMI LD13E
D134          LD134:
D134 A2 00      LDX #$0
D136 A9 79      LDA #$79
D138 20 4F D1   JSR LD14F
D13B 4C 31 D1   JMP LD131
D13E          LD13E:
D13E A5 53      LDA L53
D140 4A         LSR A
D141 A2 00      LDX #$0
D143 4C 4F D1   JMP LD14F
D146          LD146:
D146 A2 00      LDX #$0
D148 86 90      STX L90
D14A 86 91      STX L91
D14C 86 92      STX L92
D14E 60         RTS
D14F          LD14F:
D14F 86 91      STX L91
D151 85 90      STA L90
D153 4C 13 D0   JMP LD013
D156          LD156:
D156 20 BE D7   JSR LD7BE
D159 D0 0C      BNE LD167
D15B          LD15B:
D15B AD F6 2B   LDA L2BF6
D15E 20 18 D8   JSR LD818
D161 F0 04      BEQ LD167
D163          LD163:
D163 2C 22 D5   BIT LD522
D166 60         RTS
D167          LD167:
D167 20 8E D0   JSR LD08E
D16A C5 99      CMP L99
D16C D0 0E      BNE LD17C
D16E          LD16E:
D16E A4 9A      LDY L9A
D170 B1 94      LDA (L94),Y
D172 F0 04      BEQ LD178
D174          LD174:
D174 2C 21 D5   BIT LD521
D177 60         RTS
D178          LD178:
D178 2C 23 D5   BIT LD523
D17B 60         RTS
D17C          LD17C:
D17C A5 99      LDA L99
D17E C9 06      CMP #$6
D180 B0 0A      BCS LD18C
D182          LD182:
D182 0A         ASL A
D183 A8         TAY
D184 A9 04      LDA #$4
D186 85 94      STA L94
D188 B1 94      LDA (L94),Y
D18A D0 04      BNE LD190
D18C          LD18C:
D18C 2C 22 D5   BIT LD522
D18F 60         RTS
D190          LD190:
D190 2C 20 D5   BIT LD520
D193 60         RTS
D194          LD194:
D194 A9 20      LDA #$20
D196 20 F2 D9   JSR LD9F2
D199 A9 80      LDA #$80
D19B 20 FD D9   JSR LD9FD
D19E D0 46      BNE LD1E6
D1A0          LD1A0:
D1A0 A6 80      LDX L80
D1A2 FE 48 2D   INC L2D48,X
D1A5 D0 03      BNE LD1AA
D1A7          LD1A7:
D1A7 FE 68 2D   INC L2D68,X
D1AA          LD1AA:
D1AA A6 80      LDX L80
D1AC BD 28 2E   LDA L2E28,X
D1AF F0 30      BEQ LD1E1
D1B1          LD1B1:
D1B1 20 D4 DC   JSR LDCD4
D1B4 A6 80      LDX L80
D1B6 DD 28 2E   CMP L2E28,X
D1B9 90 03      BCC LD1BE
D1BB          LD1BB:
D1BB 20 07 D2   JSR LD207
D1BE          LD1BE:
D1BE A6 80      LDX L80
D1C0 BD 28 2E   LDA L2E28,X
D1C3 20 C6 DC   JSR LDCC6
D1C6 A1 A0      LDA (LA0,X)
D1C8 85 84      STA L84
D1CA A9 20      LDA #$20
D1CC 20 F2 D9   JSR LD9F2
D1CF 20 06 D5   JSR LD506
D1D2          LD1D2:
D1D2 48         PHA
D1D3 90 29      BCC LD1FE
D1D5          LD1D5:
D1D5 A9 00      LDA #$0
D1D7 20 E2 DC   JSR LDCE2
D1DA D0 22      BNE LD1FE
D1DC          LD1DC:
D1DC 68         PLA
D1DD C9 02      CMP #$2
D1DF F0 12      BEQ LD1F3
D1E1          LD1E1:
D1E1 A9 80      LDA #$80
D1E3 20 EB D9   JSR LD9EB
D1E6          LD1E6:
D1E6 20 B7 DA   JSR LDAB7
D1E9 B5 A0      LDA LA0,X
D1EB 99 E8 2D   STA L2DE8,Y
D1EE A9 0D      LDA #$D
D1F0 85 84      STA L84
D1F2 60         RTS
D1F3          LD1F3:
D1F3 20 FF D1   JSR LD1FF
D1F6 A6 80      LDX L80
D1F8 A9 00      LDA #$0
D1FA 9D 28 2E   STA L2E28,X
D1FD 60         RTS
D1FE          LD1FE:
D1FE 68         PLA
D1FF          LD1FF:
D1FF A6 80      LDX L80
D201 9D 28 2E   STA L2E28,X
D204 4C 47 D3   JMP LD347
D207          LD207:
D207 20 DB D9   JSR LD9DB
D20A 20 FF DC   JSR LDCFF
D20D 50 16      BVC LD225
D20F          LD20F:
D20F 20 A7 D9   JSR LD9A7
D212 20 79 DB   JSR LDB79
D215 A9 02      LDA #$2
D217 20 C6 DC   JSR LDCC6
D21A 20 03 DA   JSR LDA03
D21D D0 14      BNE LD233
D21F          LD21F:
D21F 20 A1 D9   JSR LD9A1
D222 4C 65 D9   JMP LD965
D225          LD225:
D225 20 79 DB   JSR LDB79
D228 20 03 DA   JSR LDA03
D22B D0 06      BNE LD233
D22D          LD22D:
D22D 20 A1 D9   JSR LD9A1
D230 20 65 D9   JSR LD965
D233          LD233:
D233 20 DB D9   JSR LD9DB
D236 A5 5A      LDA L5A
D238 F0 09      BEQ LD243
D23A          LD23A:
D23A 20 79 DB   JSR LDB79
D23D 20 A1 D9   JSR LD9A1
D240 4C 79 DB   JMP LDB79
D243          LD243:
D243 60         RTS
D244          LD244:
D244 20 D5 D2   JSR LD2D5
D247 20 F2 DC   JSR LDCF2
D24A 0A         ASL A
D24B AA         TAX
D24C A5 84      LDA L84
D24E 81 A0      STA (LA0,X)
D250 B4 A0      LDY LA0,X
D252 C8         INY
D253 D0 09      BNE LD25E
D255          LD255:
D255 A4 80      LDY L80
D257 B9 28 2E   LDA L2E28,Y
D25A F0 0A      BEQ LD266
D25C          LD25C:
D25C A0 02      LDY #$2
D25E          LD25E:
D25E 98         TYA
D25F A4 80      LDY L80
D261 D9 28 2E   CMP L2E28,Y
D264 D0 05      BNE LD26B
D266          LD266:
D266 A9 20      LDA #$20
D268 4C EB D9   JMP LD9EB
D26B          LD26B:
D26B F6 A0      INC LA0,X
D26D D0 0B      BNE LD27A
D26F          LD26F:
D26F AD F7 2B   LDA L2BF7
D272 09 10      ORA #$10
D274 8D F7 2B   STA L2BF7
D277 4C 07 D2   JMP LD207
D27A          LD27A:
D27A 60         RTS
D27B          LD27B:
D27B A9 A0      LDA #$A0
D27D 20 FD D9   JSR LD9FD
D280 D0 27      BNE LD2A9
D282          LD282:
D282 A5 84      LDA L84
D284 20 44 D2   JSR LD244
D287 A5 81      LDA L81
D289 F0 0D      BEQ LD298
D28B          LD28B:
D28B 60         RTS
D28C          LD28C:
D28C A9 20      LDA #$20
D28E 20 FD D9   JSR LD9FD
D291 F0 05      BEQ LD298
D293          LD293:
D293 A9 51      LDA #$51
D295 8D DE 2B   STA L2BDE
D298          LD298:
D298 20 C3 D2   JSR LD2C3
D29B 20 2B D3   JSR LD32B
D29E AD DE 2B   LDA L2BDE
D2A1 F0 03      BEQ LD2A6
D2A3          LD2A3:
D2A3 4C 6F B6   JMP LB66F
D2A6          LD2A6:
D2A6 4C A8 DF   JMP LDFA8
D2A9          LD2A9:
D2A9 29 80      AND #$80
D2AB D0 05      BNE LD2B2
D2AD          LD2AD:
D2AD A5 81      LDA L81
D2AF F0 DB      BEQ LD28C
D2B1          LD2B1:
D2B1 60         RTS
D2B2          LD2B2:
D2B2 A5 84      LDA L84
D2B4 48         PHA
D2B5 20 25 D5   JSR LD525
D2B8 68         PLA
D2B9 85 84      STA L84
D2BB A9 80      LDA #$80
D2BD 20 F2 D9   JSR LD9F2
D2C0 4C 82 D2   JMP LD282
D2C3          LD2C3:
D2C3 A9 20      LDA #$20
D2C5 20 FD D9   JSR LD9FD
D2C8 D0 0A      BNE LD2D4
D2CA          LD2CA:
D2CA A9 00      LDA #$0
D2CC 85 84      STA L84
D2CE 20 44 D2   JSR LD244
D2D1 4C C3 D2   JMP LD2C3
D2D4          LD2D4:
D2D4 60         RTS
D2D5          LD2D5:
D2D5 A9 40      LDA #$40
D2D7 20 EB D9   JSR LD9EB
D2DA 20 FF DC   JSR LDCFF
D2DD 09 40      ORA #$40
D2DF A6 44      LDX L44
D2E1 9D 68 2C   STA L2C68,X
D2E4 60         RTS
D2E5          LD2E5:
D2E5 20 FF DC   JSR LDCFF
D2E8 29 BF      AND #$BF
D2EA A6 44      LDX L44
D2EC 9D 68 2C   STA L2C68,X
D2EF 60         RTS
D2F0          LD2F0:
D2F0 A9 80      LDA #$80
D2F2 20 FD D9   JSR LD9FD
D2F5 D0 3F      BNE LD336
D2F7          LD2F7:
D2F7 20 B7 DA   JSR LDAB7
D2FA B5 A0      LDA LA0,X
D2FC D9 E8 2D   CMP L2DE8,Y
D2FF F0 2A      BEQ LD32B
D301          LD301:
D301 F6 A0      INC LA0,X
D303 D0 0E      BNE LD313
D305          LD305:
D305 AD F7 2B   LDA L2BF7
D308 09 10      ORA #$10
D30A 8D F7 2B   STA L2BF7
D30D 20 07 D2   JSR LD207
D310          LD310:
D310 20 B7 DA   JSR LDAB7
D313          LD313:
D313 A1 A0      LDA (LA0,X)
D315          LD315:
D315 99 C8 2D   STA L2DC8,Y
D318 A9 89      LDA #$89
D31A 99 A8 2D   STA L2DA8,Y
D31D B5 A0      LDA LA0,X
D31F D9 E8 2D   CMP L2DE8,Y
D322 F0 01      BEQ LD325
D324          LD324:
D324 60         RTS
D325          LD325:
D325 A9 81      LDA #$81
D327 99 A8 2D   STA L2DA8,Y
D32A 60         RTS
D32B          LD32B:
D32B 20 94 D1   JSR LD194
D32E 20 B7 DA   JSR LDAB7
D331 A5 84      LDA L84
D333 4C 15 D3   JMP LD315
D336          LD336:
D336 A6 80      LDX L80
D338 A9 0D      LDA #$D
D33A 9D C8 2D   STA L2DC8,X
D33D A9 81      LDA #$81
D33F 9D A8 2D   STA L2DA8,X
D342 A9 50      LDA #$50
D344 20 6F B6   JSR LB66F
D347          LD347:
D347 A6 80      LDX L80
D349 BD 28 2E   LDA L2E28,X
D34C 85 86      STA L86
D34E C6 86      DEC L86
D350 C9 02      CMP #$2
D352 D0 04      BNE LD358
D354          LD354:
D354 A9 FF      LDA #$FF
D356 85 86      STA L86
D358          LD358:
D358 BD 08 2E   LDA L2E08,X
D35B 85 87      STA L87
D35D 20 D4 DC   JSR LDCD4
D360 A6 80      LDX L80
D362 C5 86      CMP L86
D364 90 19      BCC LD37F
D366          LD366:
D366 F0 17      BEQ LD37F
D368          LD368:
D368 20 79 DB   JSR LDB79
D36B 20 8D D3   JSR LD38D
D36E 90 08      BCC LD378
D370          LD370:
D370 A6 80      LDX L80
D372 9D E8 2D   STA L2DE8,X
D375 4C 79 DB   JMP LDB79
D378          LD378:
D378 20 79 DB   JSR LDB79
D37B A9 FF      LDA #$FF
D37D 85 86      STA L86
D37F          LD37F:
D37F 20 8D D3   JSR LD38D
D382 B0 03      BCS LD387
D384          LD384:
D384 20 D4 DC   JSR LDCD4
D387          LD387:
D387 A6 80      LDX L80
D389 9D E8 2D   STA L2DE8,X
D38C 60         RTS
D38D          LD38D:
D38D 20 4F D0   JSR LD04F
D390 A4 86      LDY L86
D392          LD392:
D392 B1 94      LDA (L94),Y
D394 D0 0D      BNE LD3A3
D396          LD396:
D396 88         DEY
D397 C0 02      CPY #$2
D399 90 04      BCC LD39F
D39B          LD39B:
D39B C6 87      DEC L87
D39D D0 F3      BNE LD392
D39F          LD39F:
D39F C6 87      DEC L87
D3A1 18         CLC
D3A2 60         RTS
D3A3          LD3A3:
D3A3 98         TYA
D3A4 38         SEC
D3A5 60         RTS
D3A6          LD3A6:
D3A6 20 BE D7   JSR LD7BE
D3A9 D0 03      BNE LD3AE
D3AB          LD3AB:
D3AB 20 01 D8   JSR LD801
D3AE          LD3AE:
D3AE 20 8E D0   JSR LD08E
D3B1 85 99      STA L99
D3B3 A9 04      LDA #$4
D3B5 85 94      STA L94
D3B7 A0 0A      LDY #$A
D3B9 D0 04      BNE LD3BF
D3BB          LD3BB:
D3BB 88         DEY
D3BC 88         DEY
D3BD 30 27      BMI LD3E6
D3BF          LD3BF:
D3BF B1 94      LDA (L94),Y
D3C1 F0 F8      BEQ LD3BB
D3C3          LD3C3:
D3C3 98         TYA
D3C4 4A         LSR A
D3C5 C5 99      CMP L99
D3C7 F0 0A      BEQ LD3D3
D3C9          LD3C9:
D3C9 85 99      STA L99
D3CB A6 80      LDX L80
D3CD BD A8 2C   LDA L2CA8,X
D3D0 20 D9 D0   JSR LD0D9
D3D3          LD3D3:
D3D3 A0 00      LDY #$0
D3D5 84 94      STY L94
D3D7 B1 94      LDA (L94),Y
D3D9 D0 0B      BNE LD3E6
D3DB          LD3DB:
D3DB C8         INY
D3DC B1 94      LDA (L94),Y
D3DE A8         TAY
D3DF 88         DEY
D3E0 84 9A      STY L9A
D3E2 98         TYA
D3E3 4C A6 D0   JMP LD0A6
D3E6          LD3E6:
D3E6 A9 67      LDA #$67
D3E8 20 33 FF   JSR LFF33
D3EB          LD3EB:
D3EB 20 AC B7   JSR LB7AC
D3EE AD 01 02   LDA L201
D3F1 85 82      STA L82
D3F3 20 60 DA   JSR LDA60
D3F6 90 05      BCC LD3FD
D3F8          LD3F8:
D3F8 A9 70      LDA #$70
D3FA 20 6F B6   JSR LB66F
D3FD          LD3FD:
D3FD A9 A0      LDA #$A0
D3FF 20 F2 D9   JSR LD9F2
D402 20 AC DA   JSR LDAAC
D405 F0 05      BEQ LD40C
D407          LD407:
D407 A9 64      LDA #$64
D409 20 6F B6   JSR LB66F
D40C          LD40C:
D40C AD 02 02   LDA L202
D40F 9D 48 2D   STA L2D48,X
D412 AD 03 02   LDA L203
D415 9D 68 2D   STA L2D68,X
D418 A6 80      LDX L80
D41A A9 89      LDA #$89
D41C 9D A8 2D   STA L2DA8,X
D41F AD 04 02   LDA L204
D422 F0 11      BEQ LD435
D424          LD424:
D424 38         SEC
D425 E9 01      SBC #$1
D427 F0 0C      BEQ LD435
D429          LD429:
D429 DD 08 2E   CMP L2E08,X
D42C 90 07      BCC LD435
D42E          LD42E:
D42E A9 51      LDA #$51
D430 8D DE 2B   STA L2BDE
D433 A9 00      LDA #$0
D435          LD435:
D435 85 98      STA L98
D437 20 50 CF   JSR LCF50
D43A 20 B5 D0   JSR LD0B5
D43D 50 08      BVC LD447
D43F          LD43F:
D43F A9 80      LDA #$80
D441 20 EB D9   JSR LD9EB
D444 4C 36 D3   JMP LD336
D447          LD447:
D447 20 57 D4   JSR LD457
D44A A9 80      LDA #$80
D44C 20 FD D9   JSR LD9FD
D44F F0 03      BEQ LD454
D451          LD451:
D451 4C 36 D3   JMP LD336
D454          LD454:
D454 4C 54 B6   JMP LB654
D457          LD457:
D457 20 7F D4   JSR LD47F
D45A A5 9B      LDA L9B
D45C 20 C6 DC   JSR LDCC6
D45F A6 80      LDX L80
D461 BD 08 2E   LDA L2E08,X
D464 38         SEC
D465 E5 98      SBC L98
D467 B0 03      BCS LD46C
D469          LD469:
D469 4C E6 D3   JMP LD3E6
D46C          LD46C:
D46C 18         CLC
D46D 65 9B      ADC L9B
D46F 90 03      BCC LD474
D471          LD471:
D471 69 01      ADC #$1
D473 38         SEC
D474          LD474:
D474 20 D2 D1   JSR LD1D2
D477 4C 10 D3   JMP LD310
D47A          LD47A:
D47A A9 51      LDA #$51
D47C 20 6F B6   JSR LB66F
D47F          LD47F:
D47F A5 94      LDA L94
D481 85 88      STA L88
D483 A5 95      LDA L95
D485 85 89      STA L89
D487 20 BD D4   JSR LD4BD
D48A F0 22      BEQ LD4AE
D48C          LD48C:
D48C 20 54 DA   JSR LDA54
D48F 20 2F D0   JSR LD02F
D492 A5 5A      LDA L5A
D494 F0 19      BEQ LD4AF
D496          LD496:
D496 20 79 DB   JSR LDB79
D499 20 BD D4   JSR LD4BD
D49C D0 11      BNE LD4AF
D49E          LD49E:
D49E 20 2F D0   JSR LD02F
D4A1 A5 5A      LDA L5A
D4A3 F0 09      BEQ LD4AE
D4A5          LD4A5:
D4A5 20 79 DB   JSR LDB79
D4A8 20 A1 D9   JSR LD9A1
D4AB 4C 79 DB   JMP LDB79
D4AE          LD4AE:
D4AE 60         RTS
D4AF          LD4AF:
D4AF A0 00      LDY #$0
D4B1 B1 88      LDA (L88),Y
D4B3 85 5A      STA L5A
D4B5 C8         INY
D4B6 B1 88      LDA (L88),Y
D4B8 85 5B      STA L5B
D4BA 4C 6E D8   JMP LD86E
D4BD          LD4BD:
D4BD 20 89 D9   JSR LD989
D4C0 A0 00      LDY #$0
D4C2 B1 88      LDA (L88),Y
D4C4 C5 5A      CMP L5A
D4C6 F0 01      BEQ LD4C9
D4C8          LD4C8:
D4C8 60         RTS
D4C9          LD4C9:
D4C9 C8         INY
D4CA B1 88      LDA (L88),Y
D4CC C5 5B      CMP L5B
D4CE D0 11      BNE LD4E1
D4D0          LD4D0:
D4D0 AD F7 2B   LDA L2BF7
D4D3 29 10      AND #$10
D4D5 F0 0A      BEQ LD4E1
D4D7          LD4D7:
D4D7 AD F7 2B   LDA L2BF7
D4DA 29 EF      AND #$EF
D4DC 8D F7 2B   STA L2BF7
D4DF 49 10      EOR #$10
D4E1          LD4E1:
D4E1 60         RTS
D4E2          LD4E2:
D4E2 20 4F D0   JSR LD04F
D4E5 A0 02      LDY #$2
D4E7 A9 00      LDA #$0
D4E9          LD4E9:
D4E9 91 94      STA (L94),Y
D4EB C8         INY
D4EC D0 FB      BNE LD4E9
D4EE          LD4EE:
D4EE 20 06 D5   JSR LD506
D4F1          LD4F1:
D4F1 9D 28 2E   STA L2E28,X
D4F4 A8         TAY
D4F5 A9 FF      LDA #$FF
D4F7 91 94      STA (L94),Y
D4F9 20 06 D5   JSR LD506
D4FC 90 F3      BCC LD4F1
D4FE          LD4FE:
D4FE D0 05      BNE LD505
D500          LD500:
D500 A9 00      LDA #$0
D502 9D 28 2E   STA L2E28,X
D505          LD505:
D505 60         RTS
D506          LD506:
D506 A6 80      LDX L80
D508 BD 28 2E   LDA L2E28,X
D50B 38         SEC
D50C F0 0E      BEQ LD51C
D50E          LD50E:
D50E 18         CLC
D50F 7D 08 2E   ADC L2E08,X
D512 90 0B      BCC LD51F
D514          LD514:
D514 D0 06      BNE LD51C
D516          LD516:
D516 A9 02      LDA #$2
D518 2C 24 D5   BIT LD524
D51B 60         RTS
D51C          LD51C:
D51C 69 01      ADC #$1
D51E 38         SEC
D51F          LD51F:
D51F 60         RTS
D520          LD520:
D521          LD521 = * + 1
D522          LD522 = * + 2
D520 7F 3F FF   .BYTE $7F,$3F,$FF
D523          LD523:
D524          LD524 = * + 1
D523 BF 00      .BYTE $BF,$0
D525          LD525:
D525 20 87 D6   JSR LD687
D528 20 50 CF   JSR LCF50
D52B          LD52B:
D52B 20 7C C6   JSR LC67C
D52E A4 80      LDY L80
D530 BE 08 2E   LDX L2E08,Y
D533 CA         DEX
D534 8A         TXA
D535 18         CLC
D536 65 9B      ADC L9B
D538 90 0C      BCC LD546
D53A          LD53A:
D53A E6 9A      INC L9A
D53C E6 9A      INC L9A
D53E D0 06      BNE LD546
D540          LD540:
D540 E6 99      INC L99
D542 A9 10      LDA #$10
D544 85 9A      STA L9A
D546          LD546:
D546 A5 86      LDA L86
D548 18         CLC
D549 69 02      ADC #$2
D54B 20 A6 D0   JSR LD0A6
D54E A5 99      LDA L99
D550 C9 06      CMP #$6
D552 90 11      BCC LD565
D554          LD554:
D554 20 BE D7   JSR LD7BE
D557 D0 07      BNE LD560
D559          LD559:
D559 85 99      STA L99
D55B EE F6 2B   INC L2BF6
D55E D0 05      BNE LD565
D560          LD560:
D560 A9 52      LDA #$52
D562 20 6F B6   JSR LB66F
D565          LD565:
D565 A5 9A      LDA L9A
D567 38         SEC
D568 E5 86      SBC L86
D56A B0 03      BCS LD56F
D56C          LD56C:
D56C E9 0F      SBC #$F
D56E 18         CLC
D56F          LD56F:
D56F 48         PHA
D570 20 BE D7   JSR LD7BE
D573 F0 1E      BEQ LD593
D575          LD575:
D575 68         PLA
D576 85 53      STA L53
D578 A5 99      LDA L99
D57A E5 85      SBC L85
D57C 85 54      STA L54
D57E A2 00      LDX #$0
D580 86 51      STX L51
D582 86 52      STX L52
D584 AA         TAX
D586          LD586 = * + 1
              ; Instruction parameter jumped to.
D585 20 05 D1   JSR LD105
D588 A5 52      LDA L52
D58A D0 2F      BNE LD5BB
D58C          LD58C:
D58C A6 51      LDX L51
D58E CA         DEX
D58F D0 2A      BNE LD5BB
D591          LD591:
D591 F0 26      BEQ LD5B9
D593          LD593:
D593 68         PLA
D594 85 53      STA L53
D596 A5 99      LDA L99
D598 E5 85      SBC L85
D59A B0 04      BCS LD5A0
D59C          LD59C:
D59C E6 88      INC L88
D59E 69 06      ADC #$6
D5A0          LD5A0:
D5A0 85 54      STA L54
D5A2 AD F6 2B   LDA L2BF6
D5A5 38         SEC
D5A6 E5 88      SBC L88
D5A8 85 88      STA L88
D5AA 20 1A D1   JSR LD11A
D5AD A5 8C      LDA L8C
D5AF D0 0A      BNE LD5BB
D5B1          LD5B1:
D5B1 A6 8B      LDX L8B
D5B3 D0 01      BNE LD5B6
D5B5          LD5B5:
D5B5 60         RTS
D5B6          LD5B6:
D5B6 CA         DEX
D5B7 D0 02      BNE LD5BB
D5B9          LD5B9:
D5B9 E6 87      INC L87
D5BB          LD5BB:
D5BB CD C4 2B   CMP L2BC4
D5BE 90 09      BCC LD5C9
D5C0          LD5C0:
D5C0 D0 9E      BNE LD560
D5C2          LD5C2:
D5C2 AD C3 2B   LDA L2BC3
D5C5 C5 51      CMP L51
D5C7 90 97      BCC LD560
D5C9          LD5C9:
D5C9 A9 01      LDA #$1
D5CB 20 E2 DC   JSR LDCE2
D5CE 18         CLC
D5CF 69 01      ADC #$1
D5D1 A6 80      LDX L80
D5D3 9D 28 2E   STA L2E28,X
D5D6 20 F3 A3   JSR LA3F3
D5D9 20 20 D0   JSR LD020
D5DC A5 87      LDA L87
D5DE D0 15      BNE LD5F5
D5E0          LD5E0:
D5E0 20 A7 D9   JSR LD9A7
D5E3          LD5E3:
D5E3 20 79 DB   JSR LDB79
D5E6 20 73 D9   JSR LD973
D5E9 20 F3 A3   JSR LA3F3
D5EC 20 20 D0   JSR LD020
D5EF 20 E2 D4   JSR LD4E2
D5F2 4C 01 D6   JMP LD601
D5F5          LD5F5:
D5F5 20 79 DB   JSR LDB79
D5F8 20 73 D9   JSR LD973
D5FB 20 E2 D4   JSR LD4E2
D5FE 20 3C D0   JSR LD03C
D601          LD601:
D601 20 A7 D9   JSR LD9A7
D604 20 2F D0   JSR LD02F
D607 A5 5A      LDA L5A
D609 48         PHA
D60A A5 5B      LDA L5B
D60C 48         PHA
D60D 20 89 D9   JSR LD989
D610 A5 5B      LDA L5B
D612 48         PHA
D613 A5 5A      LDA L5A
D615 48         PHA
D616 20 F8 D0   JSR LD0F8
D619 AA         TAX
D61A D0 0A      BNE LD626
D61C          LD61C:
D61C 20 A8 D6   JSR LD6A8
D61F A9 10      LDA #$10
D621 20 A6 D0   JSR LD0A6
D624 E6 85      INC L85
D626          LD626:
D626 68         PLA
D627 20 DA CC   JSR LCCDA
D62A 68         PLA
D62B 20 DA CC   JSR LCCDA
D62E 68         PLA
D62F 85 5B      STA L5B
D631 68         PLA
D632 85 5A      STA L5A
D634 F0 1B      BEQ LD651
D636          LD636:
D636 20 BE D7   JSR LD7BE
D639 D0 07      BNE LD642
D63B          LD63B:
D63B A5 8A      LDA L8A
D63D CD F6 2B   CMP L2BF6
D640 90 A1      BCC LD5E3
D642          LD642:
D642 A5 85      LDA L85
D644 C5 99      CMP L99
D646 D0 9B      BNE LD5E3
D648          LD648:
D648 20 F8 D0   JSR LD0F8
D64B C5 9A      CMP L9A
D64D 90 94      BCC LD5E3
D64F          LD64F:
D64F F0 A4      BEQ LD5F5
D651          LD651:
D651 20 F8 D0   JSR LD0F8
D654 48         PHA
D655 A9 00      LDA #$0
D657 20 98 D0   JSR LD098
D65A A9 00      LDA #$0
D65C A8         TAY
D65D 91 94      STA (L94),Y
D65F C8         INY
D660 68         PLA
D661 38         SEC
D662 E9 01      SBC #$1
D664 91 94      STA (L94),Y
D666 20 B3 D9   JSR LD9B3
D669 20 65 D9   JSR LD965
D66C 20 48 A3   JSR LA348
D66F 20 50 CF   JSR LCF50
D672 20 79 DB   JSR LDB79
D675 20 B5 D0   JSR LD0B5
D678 70 03      BVS LD67D
D67A          LD67A:
D67A 4C 57 D4   JMP LD457
D67D          LD67D:
D67D A9 80      LDA #$80
D67F 20 EB D9   JSR LD9EB
D682 A9 50      LDA #$50
D684 20 6F B6   JSR LB66F
D687          LD687:
D687 20 A6 D3   JSR LD3A6
D68A 20 7F D4   JSR LD47F
D68D 20 BE D7   JSR LD7BE
D690 D0 07      BNE LD699
D692          LD692:
D692 AD F6 2B   LDA L2BF6
D695 85 8A      STA L8A
D697 85 88      STA L88
D699          LD699:
D699 A5 9A      LDA L9A
D69B 85 86      STA L86
D69D A5 99      LDA L99
D69F 85 85      STA L85
D6A1 A9 00      LDA #$0
D6A3 85 87      STA L87
D6A5 85 98      STA L98
D6A7 60         RTS
D6A8          LD6A8:
D6A8 20 F3 A3   JSR LA3F3
D6AB 20 79 DB   JSR LDB79
D6AE 20 54 DA   JSR LDA54
D6B1 20 F2 DC   JSR LDCF2
D6B4 48         PHA
D6B5 20 7D D0   JSR LD07D
D6B8 A6 80      LDX L80
D6BA BD A8 2C   LDA L2CA8,X
D6BD A8         TAY
D6BE 68         PLA
D6BF AA         TAX
D6C0 20 BE D7   JSR LD7BE
D6C3 D0 03      BNE LD6C8
D6C5          LD6C5:
D6C5 4C 97 D7   JMP LD797
D6C8          LD6C8:
D6C8 A9 10      LDA #$10
D6CA 20 5F D0   JSR LD05F
D6CD A9 00      LDA #$0
D6CF 20 98 D0   JSR LD098
D6D2 A0 02      LDY #$2
D6D4 B1 94      LDA (L94),Y
D6D6 48         PHA
D6D7 A9 00      LDA #$0
D6D9 20 C6 DC   JSR LDCC6
D6DC 68         PLA
D6DD 18         CLC
D6DE 69 01      ADC #$1
D6E0 91 94      STA (L94),Y
D6E2 0A         ASL A
D6E3 69 04      ADC #$4
D6E5 85 88      STA L88
D6E7 A8         TAY
D6E8 38         SEC
D6E9 E9 02      SBC #$2
D6EB 85 89      STA L89
D6ED          LD6ED:
D6ED A5 5A      LDA L5A
D6EF 85 86      STA L86
D6F1 91 94      STA (L94),Y
D6F3 C8         INY
D6F4 A5 5B      LDA L5B
D6F6 85 87      STA L87
D6F8 91 94      STA (L94),Y
D6FA A0 00      LDY #$0
D6FC 98         TYA
D6FD 91 94      STA (L94),Y
D6FF C8         INY
D700 A9 11      LDA #$11
D702 91 94      STA (L94),Y
D704 A9 10      LDA #$10
D706 20 C6 DC   JSR LDCC6
D709 20 9B D9   JSR LD99B
D70C 20 65 D9   JSR LD965
D70F A6 80      LDX L80
D711 BD A8 2C   LDA L2CA8,X
D714 48         PHA
D715 20 FF DC   JSR LDCFF
D718 A6 80      LDX L80
D71A 9D A8 2C   STA L2CA8,X
D71D 68         PLA
D71E A6 44      LDX L44
D720 9D 68 2C   STA L2C68,X
D723 A9 00      LDA #$0
D725 20 C6 DC   JSR LDCC6
D728 A0 00      LDY #$0
D72A A5 5A      LDA L5A
D72C 91 94      STA (L94),Y
D72E C8         INY
D72F A5 5B      LDA L5B
D731 91 94      STA (L94),Y
D733 20 BE D7   JSR LD7BE
D736 D0 41      BNE LD779
D738          LD738:
D738 A5 85      LDA L85
D73A C9 FF      CMP #$FF
D73C D0 3B      BNE LD779
D73E          LD73E:
D73E A5 5B      LDA L5B
D740 48         PHA
D741 A5 5A      LDA L5A
D743 48         PHA
D744 20 A7 D9   JSR LD9A7
D747 20 65 D9   JSR LD965
D74A 20 79 DB   JSR LDB79
D74D 20 D6 D7   JSR LD7D6
D750 E6 8A      INC L8A
D752 A5 8A      LDA L8A
D754 0A         ASL A
D755 18         CLC
D756 69 03      ADC #$3
D758 20 A6 D0   JSR LD0A6
D75B 68         PLA
D75C 20 DA CC   JSR LCCDA
D75F 68         PLA
D760 20 DA CC   JSR LCCDA
D763 20 D9 D7   JSR LD7D9
D766 A5 8A      LDA L8A
D768 48         PHA
D769 4C 24 D8   JMP LD824
D76C          LD76C:
D76C 20 F2 DC   JSR LDCF2
D76F A6 80      LDX L80
D771 20 D9 D0   JSR LD0D9
D774 A9 00      LDA #$0
D776 20 C6 DC   JSR LDCC6
D779          LD779:
D779 C6 89      DEC L89
D77B C6 89      DEC L89
D77D A4 88      LDY L88
D77F A5 86      LDA L86
D781 91 94      STA (L94),Y
D783 C8         INY
D784 A5 87      LDA L87
D786 91 94      STA (L94),Y
D788 20 A7 D9   JSR LD9A7
D78B 20 65 D9   JSR LD965
D78E A4 89      LDY L89
D790 C0 03      CPY #$3
D792 B0 D8      BCS LD76C
D794          LD794:
D794 4C 79 DB   JMP LDB79
D797          LD797:
D797 A5 85      LDA L85
D799 C9 05      CMP #$5
D79B B0 03      BCS LD7A0
D79D          LD79D:
D79D 4C C8 D6   JMP LD6C8
D7A0          LD7A0:
D7A0 A9 FF      LDA #$FF
D7A2 85 85      STA L85
D7A4 A9 00      LDA #$0
D7A6 20 C6 DC   JSR LDCC6
D7A9 A0 02      LDY #$2
D7AB 91 94      STA (L94),Y
D7AD A6 80      LDX L80
D7AF BD 08 2E   LDA L2E08,X
D7B2 C8         INY
D7B3 91 94      STA (L94),Y
D7B5 C8         INY
D7B6 F0 03      BEQ LD7BB
D7B8          LD7B8:
D7B8 4C ED D6   JMP LD6ED
D7BB          LD7BB:
D7BB 4C C8 D6   JMP LD6C8
D7BE          LD7BE:
D7BE 8E F8 2B   STX L2BF8
D7C1 A6 80      LDX L80
D7C3 BD A8 2E   LDA L2EA8,X
D7C6 AE F8 2B   LDX L2BF8
D7C9 29 20      AND #$20
D7CB 60         RTS
D7CC          LD7CC:
D7CC A6 80      LDX L80
D7CE A9 FE      LDA #$FE
D7D0 DD 48 2E   CMP L2E48,X
D7D3 D0 01      BNE LD7D6
D7D5          LD7D5:
D7D5 60         RTS
D7D6          LD7D6:
D7D6 A9 80      LDA #$80
D7D9          LD7D9 = * + 1
              ; Instruction parameter jumped to.
D7D8 2C A9 90   BIT L90A9
D7DB 48         PHA
D7DC A6 80      LDX L80
D7DE BD 88 2E   LDA L2E88,X
D7E1 85 5A      STA L5A
D7E3 BD 68 2E   LDA L2E68,X
D7E6 85 5B      STA L5B
D7E8 A9 FF      LDA #$FF
D7EA 9D 48 2E   STA L2E48,X
D7ED BD A8 2C   LDA L2CA8,X
D7F0 85 9C      STA L9C
D7F2 20 76 D9   JSR LD976
D7F5 68         PLA
D7F6 20 5C D9   JSR LD95C
D7F9 A6 80      LDX L80
D7FB A9 FE      LDA #$FE
D7FD 9D 48 2E   STA L2E48,X
D800 60         RTS
D801          LD801:
D801 A9 5A      LDA #$5A
D803 8D F6 2B   STA L2BF6
D806 20 18 D8   JSR LD818
D809 D0 01      BNE LD80C
D80B          LD80B:
D80B 60         RTS
D80C          LD80C:
D80C CE F6 2B   DEC L2BF6
D80F AD F6 2B   LDA L2BF6
D812 20 2A D8   JSR LD82A
D815 D0 F5      BNE LD80C
D817          LD817:
D817 60         RTS
D818          LD818:
D818 A6 80      LDX L80
D81A DD 48 2E   CMP L2E48,X
D81D D0 01      BNE LD820
D81F          LD81F:
D81F 60         RTS
D820          LD820:
D820 48         PHA
D821 20 CC D7   JSR LD7CC
D824          LD824:
D824 A9 03      LDA #$3
D826 20 98 D0   JSR LD098
D829 68         PLA
D82A          LD82A:
D82A AA         TAX
D82B 0A         ASL A
D82C A8         TAY
D82D B1 94      LDA (L94),Y
D82F D0 03      BNE LD834
D831          LD831:
D831 09 FF      ORA #$FF
D833 60         RTS
D834          LD834:
D834 85 5A      STA L5A
D836 C8         INY
D837 B1 94      LDA (L94),Y
D839 85 5B      STA L5B
D83B 8A         TXA
D83C 48         PHA
D83D A9 FF      LDA #$FF
D83F A6 80      LDX L80
D841 9D 48 2E   STA L2E48,X
D844 BD A8 2C   LDA L2CA8,X
D847 85 9C      STA L9C
D849 20 76 D9   JSR LD976
D84C A9 80      LDA #$80
D84E 20 5C D9   JSR LD95C
D851 A6 80      LDX L80
D853 68         PLA
D854 9D 48 2E   STA L2E48,X
D857 A9 00      LDA #$0
D859 60         RTS
D85A          LD85A:
D85A 20 73 D9   JSR LD973
D85D 20 82 D8   JSR LD882
D860 20 65 D9   JSR LD965
D863 20 FE CE   JSR LCEFE
D866 85 5A      STA L5A
D868 20 FE CE   JSR LCEFE
D86B 85 5B      STA L5B
D86D 60         RTS
D86E          LD86E:
D86E 20 5A D8   JSR LD85A
D871 A5 5A      LDA L5A
D873 D0 01      BNE LD876
D875          LD875:
D875 60         RTS
D876          LD876:
D876 20 79 DB   JSR LDB79
D879 20 73 D9   JSR LD973
D87C 20 82 D8   JSR LD882
D87F 4C 79 DB   JMP LDB79
D882          LD882:
D882 A9 80      LDA #$80
D885          LD885 = * + 1
              ; Instruction parameter jumped to.
D884 2C A9 90   BIT L90A9
D887 85 55      STA L55
D889 20 F2 DC   JSR LDCF2
D88C AA         TAX
D88D 20 BB D8   JSR LD8BB
D890 8A         TXA
D891 48         PHA
D892 0A         ASL A
D893 AA         TAX
D894 A9 00      LDA #$0
D896 95 A0      STA LA0,X
D898 20 AC DA   JSR LDAAC
D89B C9 04      CMP #$4
D89D B0 08      BCS LD8A7
D89F          LD89F:
D89F FE 48 2D   INC L2D48,X
D8A2 D0 03      BNE LD8A7
D8A4          LD8A4:
D8A4 FE 68 2D   INC L2D68,X
D8A7          LD8A7:
D8A7 68         PLA
D8A8 AA         TAX
D8A9 60         RTS
D8AA          LD8AA:
D8AA A9 80      LDA #$80
D8AD          LD8AD = * + 1
              ; Instruction parameter jumped to.
D8AC 2C A9 90   BIT L90A9
D8AF 85 55      STA L55
D8B1 A5 9C      LDA L9C
D8B3 20 76 D9   JSR LD976
D8B6 A6 9C      LDX L9C
D8B8 4C 60 D9   JMP LD960
D8BB          LD8BB:
D8BB A5 55      LDA L55
D8BD          LD8BD:
D8BD 48         PHA
D8BE 86 9C      STX L9C
D8C0 2C DF 2B   BIT L2BDF
D8C3 50 03      BVC LD8C8
D8C5          LD8C5:
D8C5 4C 4F D9   JMP LD94F
D8C8          LD8C8:
D8C8 8A         TXA
D8C9 0A         ASL A
D8CA AA         TAX
D8CB BD 01 28   LDA L2801,X
D8CE 85 55      STA L55
D8D0 BD 00 28   LDA L2800,X
D8D3 F0 30      BEQ LD905
D8D5          LD8D5:
D8D5 AA         TAX
D8D6 20 7F AF   JSR LAF7F
D8D9 A5 9C      LDA L9C
D8DB 0A         ASL A
D8DC AA         TAX
D8DD AD C8 2B   LDA L2BC8
D8E0 F0 07      BEQ LD8E9
D8E2          LD8E2:
D8E2 DD 00 28   CMP L2800,X
D8E5 F0 1E      BEQ LD905
D8E7          LD8E7:
D8E7 90 1C      BCC LD905
D8E9          LD8E9:
D8E9 68         PLA
D8EA 48         PHA
D8EB C9 90      CMP #$90
D8ED D0 60      BNE LD94F
D8EF          LD8EF:
D8EF 20 87 A2   JSR LA287
D8F2 BD 70 2B   LDA L2B70,X
D8F5 20 6B AF   JSR LAF6B
D8F8 D0 4D      BNE LD947
D8FA          LD8FA:
D8FA AD C9 2B   LDA L2BC9
D8FD F0 50      BEQ LD94F
D8FF          LD8FF:
D8FF C5 55      CMP L55
D901 F0 02      BEQ LD905
D903          LD903:
D903 B0 4A      BCS LD94F
D905          LD905:
D905 20 0D D9   JSR LD90D
D908          LD908:
D908 A9 66      LDA #$66
D90A 4C 33 FF   JMP LFF33
D90D          LD90D:
D90D A5 9C      LDA L9C
D90F 0A         ASL A
D910 AA         TAX
D911 BD 00 28   LDA L2800,X
D914 85 5A      STA L5A
D916 BD 01 28   LDA L2801,X
D919 85 5B      STA L5B
D91B 60         RTS
D91C          LD91C:
D91C 8A         TXA
D91D 48         PHA
D91E A6 5A      LDX L5A
D920 20 7F AF   JSR LAF7F
D923 A5 5A      LDA L5A
D925 F0 E1      BEQ LD908
D927          LD927:
D927 AD C8 2B   LDA L2BC8
D92A F0 06      BEQ LD932
D92C          LD92C:
D92C C5 5A      CMP L5A
D92E F0 D8      BEQ LD908
D930          LD930:
D930 90 D6      BCC LD908
D932          LD932:
D932 A5 5A      LDA L5A
D934 CD C7 2B   CMP L2BC7
D937 90 CF      BCC LD908
D939          LD939:
D939 AD C9 2B   LDA L2BC9
D93C F0 06      BEQ LD944
D93E          LD93E:
D93E C5 5B      CMP L5B
D940 F0 C6      BEQ LD908
D942          LD942:
D942 90 C4      BCC LD908
D944          LD944:
D944 68         PLA
D945 AA         TAX
D946 60         RTS
D947          LD947:
D947 20 0D D9   JSR LD90D
D94A A9 73      LDA #$73
D94C 4C 33 FF   JMP LFF33
D94F          LD94F:
D94F A6 9C      LDX L9C
D951 68         PLA
D952 85 55      STA L55
D954 4C 4B FF   JMP LFF4B
D957          LD957:
D957 A9 80      LDA #$80
D959 2C A9 90   BIT L90A9
D95C          LD95C:
D95C A6 9C      LDX L9C
D95E 85 55      STA L55
D960          LD960:
D960 A5 55      LDA L55
D962 20 BD D8   JSR LD8BD
D965          LD965:
D965 B5 20      LDA L20,X
D967 20 4B FF   JSR LFF4B
D96A 18         CLC
D96B 48         PHA
D96C A9 00      LDA #$0
D96E 8D DF 2B   STA L2BDF
D971 68         PLA
D972 60         RTS
D973          LD973:
D973 20 F2 DC   JSR LDCF2
D976          LD976:
D976 0A         ASL A
D977 A8         TAY
D978 A5 5A      LDA L5A
D97A 99 00 28   STA L2800,Y
D97D A5 5B      LDA L5B
D97F 99 01 28   STA L2801,Y
D982 A9 00      LDA #$0
D984 AA         TAX
D985 60         RTS
D986          LD986:
D986 20 60 DA   JSR LDA60
D989          LD989:
D989 20 F2 DC   JSR LDCF2
D98C 85 9C      STA L9C
D98E 0A         ASL A
D98F A8         TAY
D990 B9 00 28   LDA L2800,Y
D993 85 5A      STA L5A
D995 B9 01 28   LDA L2801,Y
D998 85 5B      STA L5B
D99A 60         RTS
D99B          LD99B:
D99B A9 90      LDA #$90
D99D 85 55      STA L55
D99F D0 24      BNE LD9C5
D9A1          LD9A1:
D9A1 A9 80      LDA #$80
D9A3 85 55      STA L55
D9A5 D0 1E      BNE LD9C5
D9A7          LD9A7:
D9A7 A9 90      LDA #$90
D9A9 85 55      STA L55
D9AB D0 24      BNE LD9D1
D9AD          LD9AD:
D9AD A9 80      LDA #$80
D9AF 85 55      STA L55
D9B1 D0 1E      BNE LD9D1
D9B3          LD9B3:
D9B3 A9 90      LDA #$90
D9B5 85 55      STA L55
D9B7 D0 02      BNE LD9BB
D9B9          LD9B9:
D9B9 A9 80      LDA #$80
D9BB          LD9BB:
D9BB 85 55      STA L55
D9BD A6 80      LDX L80
D9BF BD A8 2C   LDA L2CA8,X
D9C2 AA         TAX
D9C3 10 13      BPL LD9D8
D9C5          LD9C5:
D9C5 20 73 D9   JSR LD973
D9C8 20 F2 DC   JSR LDCF2
D9CB AA         TAX
D9CC A9 00      LDA #$0
D9CE 9D 60 29   STA L2960,X
D9D1          LD9D1:
D9D1 20 E5 D2   JSR LD2E5
D9D4 20 F2 DC   JSR LDCF2
D9D7 AA         TAX
D9D8          LD9D8:
D9D8 4C BB D8   JMP LD8BB
D9DB          LD9DB:
D9DB A9 00      LDA #$0
D9DD 20 C6 DC   JSR LDCC6
D9E0 20 FE CE   JSR LCEFE
D9E3 85 5A      STA L5A
D9E5 20 FE CE   JSR LCEFE
D9E8 85 5B      STA L5B
D9EA 60         RTS
D9EB          LD9EB:
D9EB A6 80      LDX L80
D9ED 1D 88 2D   ORA L2D88,X
D9F0 D0 07      BNE LD9F9
D9F2          LD9F2:
D9F2 A6 80      LDX L80
D9F4 49 FF      EOR #$FF
D9F6 3D 88 2D   AND L2D88,X
D9F9          LD9F9:
D9F9 9D 88 2D   STA L2D88,X
D9FC 60         RTS
D9FD          LD9FD:
D9FD A6 80      LDX L80
D9FF 3D 88 2D   AND L2D88,X
DA02 60         RTS
DA03          LDA03:
DA03 20 F2 DC   JSR LDCF2
DA06 AA         TAX
DA07 BD 60 29   LDA L2960,X
DA0A 29 FE      AND #$FE
DA0C C9 90      CMP #$90
DA0E 60         RTS
DA0F          LDA0F:
DA0F A2 00      LDX #$0
DA11          LDA11:
DA11 86 52      STX L52
DA13 BD 48 2C   LDA L2C48,X
DA16 C9 FF      CMP #$FF
DA18 D0 08      BNE LDA22
DA1A          LDA1A:
DA1A A6 52      LDX L52
DA1C E8         INX
DA1D E0 10      CPX #$10
DA1F 90 F0      BCC LDA11
DA21          LDA21:
DA21 60         RTS
DA22          LDA22:
DA22 86 52      STX L52
DA24 29 3F      AND #$3F
DA26 A8         TAY
DA27 AE BF 2B   LDX L2BBF
DA2A B9 88 2D   LDA L2D88,Y
DA2D DD 18 2C   CMP L2C18,X
DA30 D0 E8      BNE LDA1A
DA32          LDA32:
DA32 B9 C8 2C   LDA L2CC8,Y
DA35 DD 10 2C   CMP L2C10,X
DA38 D0 E0      BNE LDA1A
DA3A          LDA3A:
DA3A B9 E8 2C   LDA L2CE8,Y
DA3D DD 30 2C   CMP L2C30,X
DA40 D0 D8      BNE LDA1A
DA42          LDA42:
DA42 B9 08 2D   LDA L2D08,Y
DA45 DD 38 2C   CMP L2C38,X
DA48 D0 D0      BNE LDA1A
DA4A          LDA4A:
DA4A B9 28 2D   LDA L2D28,Y
DA4D DD 40 2C   CMP L2C40,X
DA50 D0 C8      BNE LDA1A
DA52          LDA52:
DA52 18         CLC
DA53 60         RTS
DA54          LDA54:
DA54 20 FF DC   JSR LDCFF
DA57 50 06      BVC LDA5F
DA59          LDA59:
DA59 20 A7 D9   JSR LD9A7
DA5C 20 65 D9   JSR LD965
DA5F          LDA5F:
DA5F 60         RTS
DA60          LDA60:
DA60 A5 82      LDA L82
DA62 C9 13      CMP #$13
DA64 90 02      BCC LDA68
DA66          LDA66:
DA66 29 0F      AND #$F
DA68          LDA68:
DA68 C9 0F      CMP #$F
DA6A D0 02      BNE LDA6E
DA6C          LDA6C:
DA6C A9 10      LDA #$10
DA6E          LDA6E:
DA6E AA         TAX
DA6F 38         SEC
DA70 BD 48 2C   LDA L2C48,X
DA73 30 1C      BMI LDA91
DA75          LDA75:
DA75 29 3F      AND #$3F
DA77 85 80      STA L80
DA79 AA         TAX
DA7A C9 1F      CMP #$1F
DA7C F0 04      BEQ LDA82
DA7E          LDA7E:
DA7E C9 1E      CMP #$1E
DA80 D0 06      BNE LDA88
DA82          LDA82:
DA82 AD D6 2B   LDA L2BD6
DA85 4C 8B DA   JMP LDA8B
DA88          LDA88:
DA88 BD C8 2C   LDA L2CC8,X
DA8B          LDA8B:
DA8B 20 23 B0   JSR LB023
DA8E A5 80      LDA L80
DA90 18         CLC
DA91          LDA91:
DA91 60         RTS
DA92          LDA92:
DA92 A5 82      LDA L82
DA94 C9 13      CMP #$13
DA96 90 02      BCC LDA9A
DA98          LDA98:
DA98 29 0F      AND #$F
DA9A          LDA9A:
DA9A AA         TAX
DA9B BD 48 2C   LDA L2C48,X
DA9E A8         TAY
DA9F 0A         ASL A
DAA0 90 06      BCC LDAA8
DAA2          LDAA2:
DAA2 30 06      BMI LDAAA
DAA4          LDAA4:
DAA4 98         TYA
DAA5 4C 75 DA   JMP LDA75
DAA8          LDAA8:
DAA8 30 FA      BMI LDAA4
DAAA          LDAAA:
DAAA 38         SEC
DAAB 60         RTS
DAAC          LDAAC:
DAAC A6 80      LDX L80
DAAE BD 88 2D   LDA L2D88,X
DAB1 4A         LSR A
DAB2 29 07      AND #$7
DAB4 C9 04      CMP #$4
DAB6 60         RTS
DAB7          LDAB7:
DAB7 20 F2 DC   JSR LDCF2
DABA 0A         ASL A
DABB AA         TAX
DABC A4 80      LDY L80
DABE 60         RTS
DABF          LDABF:
DABF 38         SEC
DAC0 B0 01      BCS LDAC3
DAC2          LDAC2:
DAC2 18         CLC
DAC3          LDAC3:
DAC3 08         PHP
DAC4 85 50      STA L50
DAC6 20 04 DB   JSR LDB04
DAC9 20 48 DB   JSR LDB48
DACC AD E8 90   LDA L90E8
DACF 9D C8 2C   STA L2CC8,X
DAD2 8A         TXA
DAD3 A6 82      LDX L82
DAD5 28         PLP
DAD6 90 02      BCC LDADA
DAD8          LDAD8:
DAD8 09 80      ORA #$80
DADA          LDADA:
DADA 9D 48 2C   STA L2C48,X
DADD 29 3F      AND #$3F
DADF A8         TAY
DAE0 20 68 DC   JSR LDC68
DAE3 C6 50      DEC L50
DAE5 30 1C      BMI LDB03
DAE7          LDAE7:
DAE7 20 76 DC   JSR LDC76
DAEA 10 08      BPL LDAF4
DAEC          LDAEC:
DAEC 20 68 DC   JSR LDC68
DAEF A9 70      LDA #$70
DAF1 4C 6F B6   JMP LB66F
DAF4          LDAF4:
DAF4 99 68 2C   STA L2C68,Y
DAF7 C6 50      DEC L50
DAF9 30 08      BMI LDB03
DAFB          LDAFB:
DAFB 20 76 DC   JSR LDC76
DAFE 30 EC      BMI LDAEC
DB00          LDB00:
DB00 99 88 2C   STA L2C88,Y
DB03          LDB03:
DB03 60         RTS
DB04          LDB04:
DB04 A5 82      LDA L82
DB06 C9 0F      CMP #$F
DB08 D0 01      BNE LDB0B
DB0A          LDB0A:
DB0A 60         RTS
DB0B          LDB0B:
DB0B AA         TAX
DB0C BD 48 2C   LDA L2C48,X
DB0F C9 FF      CMP #$FF
DB11 F0 F7      BEQ LDB0A
DB13          LDB13:
DB13 29 3F      AND #$3F
DB15 85 80      STA L80
DB17 A9 FF      LDA #$FF
DB19 9D 48 2C   STA L2C48,X
DB1C A6 80      LDX L80
DB1E A9 00      LDA #$0
DB20 9D A8 2D   STA L2DA8,X
DB23 4C 68 DC   JMP LDC68
DB26          LDB26:
DB26 A9 0E      LDA #$E
DB28 85 82      STA L82
DB2A          LDB2A:
DB2A A6 82      LDX L82
DB2C BD 48 2C   LDA L2C48,X
DB2F C9 FF      CMP #$FF
DB31 F0 10      BEQ LDB43
DB33          LDB33:
DB33 29 3F      AND #$3F
DB35 85 80      STA L80
DB37 AA         TAX
DB38 BD C8 2C   LDA L2CC8,X
DB3B CD E8 90   CMP L90E8
DB3E D0 03      BNE LDB43
DB40          LDB40:
DB40 20 04 DB   JSR LDB04
DB43          LDB43:
DB43 C6 82      DEC L82
DB45 10 E3      BPL LDB2A
DB47          LDB47:
DB47 60         RTS
DB48          LDB48:
DB48 A9 00      LDA #$0
DB4A 85 80      STA L80
DB4C          LDB4C:
DB4C A2 12      LDX #$12
DB4E          LDB4E:
DB4E BD 48 2C   LDA L2C48,X
DB51 29 3F      AND #$3F
DB53 C5 80      CMP L80
DB55 F0 07      BEQ LDB5E
DB57          LDB57:
DB57 CA         DEX
DB58 10 F4      BPL LDB4E
DB5A          LDB5A:
DB5A A5 80      LDA L80
DB5C AA         TAX
DB5D 60         RTS
DB5E          LDB5E:
DB5E E6 80      INC L80
DB60 A5 80      LDA L80
DB62 C9 20      CMP #$20
DB64 90 E6      BCC LDB4C
DB66          LDB66:
DB66 A9 70      LDA #$70
DB68 4C 6F B6   JMP LB66F
DB6B          LDB6B:
DB6B A9 11      LDA #$11
DB6D 85 82      STA L82
DB6F 20 04 DB   JSR LDB04
DB72 A9 12      LDA #$12
DB74 85 82      STA L82
DB76 4C 04 DB   JMP LDB04
DB79          LDB79:
DB79 A6 80      LDX L80
DB7B BD 68 2C   LDA L2C68,X
DB7E 30 03      BMI LDB83
DB80          LDB80:
DB80 BD 88 2C   LDA L2C88,X
DB83          LDB83:
DB83 C9 FF      CMP #$FF
DB85 F0 1C      BEQ LDBA3
DB87          LDB87:
DB87 BD 68 2C   LDA L2C68,X
DB8A 49 80      EOR #$80
DB8C 9D 68 2C   STA L2C68,X
DB8F 48         PHA
DB90 BD 88 2C   LDA L2C88,X
DB93 49 80      EOR #$80
DB95 9D 88 2C   STA L2C88,X
DB98 A8         TAY
DB99 68         PLA
DB9A 10 01      BPL LDB9D
DB9C          LDB9C:
DB9C 98         TYA
DB9D          LDB9D:
DB9D 29 BF      AND #$BF
DB9F AA         TAX
DBA0 4C 65 D9   JMP LD965
DBA3          LDBA3:
DBA3 BD 68 2C   LDA L2C68,X
DBA6 10 03      BPL LDBAB
DBA8          LDBA8:
DBA8 BD 88 2C   LDA L2C88,X
DBAB          LDBAB:
DBAB 29 BF      AND #$BF
DBAD A8         TAY
DBAE 20 76 DC   JSR LDC76
DBB1 10 05      BPL LDBB8
DBB3          LDBB3:
DBB3 A9 70      LDA #$70
DBB5 4C 6F B6   JMP LB66F
DBB8          LDBB8:
DBB8 A6 80      LDX L80
DBBA 09 80      ORA #$80
DBBC BC 68 2C   LDY L2C68,X
DBBF 10 05      BPL LDBC6
DBC1          LDBC1:
DBC1 9D 68 2C   STA L2C68,X
DBC4 30 03      BMI LDBC9
DBC6          LDBC6:
DBC6 9D 88 2C   STA L2C88,X
DBC9          LDBC9:
DBC9 A5 5A      LDA L5A
DBCB 48         PHA
DBCC A5 5B      LDA L5B
DBCE 48         PHA
DBCF A9 01      LDA #$1
DBD1 85 52      STA L52
DBD3 BD 68 2C   LDA L2C68,X
DBD6 10 03      BPL LDBDB
DBD8          LDBD8:
DBD8 BD 88 2C   LDA L2C88,X
DBDB          LDBDB:
DBDB 29 BF      AND #$BF
DBDD A8         TAY
DBDE 18         CLC
DBDF 69 03      ADC #$3
DBE1 85 53      STA L53
DBE3 A0 00      LDY #$0
DBE5 B1 52      LDA (L52),Y
DBE7 85 5B      STA L5B
DBE9 A9 00      LDA #$0
DBEB 85 52      STA L52
DBED BD 68 2C   LDA L2C68,X
DBF0 10 03      BPL LDBF5
DBF2          LDBF2:
DBF2 BD 88 2C   LDA L2C88,X
DBF5          LDBF5:
DBF5 29 BF      AND #$BF
DBF7 A8         TAY
DBF8 18         CLC
DBF9 69 03      ADC #$3
DBFB 85 53      STA L53
DBFD A0 00      LDY #$0
DBFF B1 52      LDA (L52),Y
DC01 85 5A      STA L5A
DC03 F0 2E      BEQ LDC33
DC05          LDC05:
DC05 20 AC DA   JSR LDAAC
DC08 F0 0B      BEQ LDC15
DC0A          LDC0A:
DC0A 20 03 DA   JSR LDA03
DC0D D0 06      BNE LDC15
DC0F          LDC0F:
DC0F 20 48 DC   JSR LDC48
DC12 4C 2A DC   JMP LDC2A
DC15          LDC15:
DC15 A6 80      LDX L80
DC17 BD 68 2C   LDA L2C68,X
DC1A 49 80      EOR #$80
DC1C 9D 68 2C   STA L2C68,X
DC1F BD 88 2C   LDA L2C88,X
DC22 49 80      EOR #$80
DC24 9D 88 2C   STA L2C88,X
DC27 20 A1 D9   JSR LD9A1
DC2A          LDC2A:
DC2A 68         PLA
DC2B 85 5B      STA L5B
DC2D 68         PLA
DC2E 85 5A      STA L5A
DC30 4C 3C DC   JMP LDC3C
DC33          LDC33:
DC33 68         PLA
DC34 85 5B      STA L5B
DC36 68         PLA
DC37 85 5A      STA L5A
DC39 20 48 DC   JSR LDC48
DC3C          LDC3C:
DC3C 20 F2 DC   JSR LDCF2
DC3F AA         TAX
DC40 4C 65 D9   JMP LD965
DC43          LDC43:
DC43 A9 70      LDA #$70
DC45 4C 6F B6   JMP LB66F
DC48          LDC48:
DC48 A6 80      LDX L80
DC4A BD 68 2C   LDA L2C68,X
DC4D 49 80      EOR #$80
DC4F 9D 68 2C   STA L2C68,X
DC52 BD 88 2C   LDA L2C88,X
DC55 49 80      EOR #$80
DC57 9D 88 2C   STA L2C88,X
DC5A 60         RTS
DC5B          LDC5B:
DC5B 85 50      STA L50
DC5D 20 D4 DC   JSR LDCD4
DC60 18         CLC
DC61 65 50      ADC L50
DC63 95 A0      STA LA0,X
DC65 85 94      STA L94
DC67 60         RTS
DC68          LDC68:
DC68 A6 80      LDX L80
DC6A A9 FF      LDA #$FF
DC6C 9D 68 2C   STA L2C68,X
DC6F 9D 88 2C   STA L2C88,X
DC72 9D A8 2C   STA L2CA8,X
DC75 60         RTS
DC76          LDC76:
DC76 98         TYA
DC77 48         PHA
DC78 20 94 DC   JSR LDC94
DC7B 30 13      BMI LDC90
DC7D          LDC7D:
DC7D B5 20      LDA L20,X
DC7F 30 FC      BMI LDC7D
DC81          LDC81:
DC81 A9 00      LDA #$0
DC83 95 20      STA L20,X
DC85 9D 60 29   STA L2960,X
DC88 8A         TXA
DC89 0A         ASL A
DC8A A8         TAY
DC8B A9 02      LDA #$2
DC8D 99 A0 00   STA LA0,Y
DC90          LDC90:
DC90 68         PLA
DC91 A8         TAY
DC92 8A         TXA
DC93 60         RTS
DC94          LDC94:
DC94 A9 1E      LDA #$1E
DC96 85 41      STA L41
DC98          LDC98:
DC98 C6 41      DEC L41
DC9A 30 05      BMI LDCA1
DC9C          LDC9C:
DC9C 20 A5 DC   JSR LDCA5
DC9F F0 F7      BEQ LDC98
DCA1          LDCA1:
DCA1 A5 41      LDA L41
DCA3 AA         TAX
DCA4 60         RTS
DCA5          LDCA5:
DCA5 A2 1F      LDX #$1F
DCA7          LDCA7:
DCA7 BD 68 2C   LDA L2C68,X
DCAA 29 1F      AND #$1F
DCAC C5 41      CMP L41
DCAE F0 15      BEQ LDCC5
DCB0          LDCB0:
DCB0 BD 88 2C   LDA L2C88,X
DCB3 29 1F      AND #$1F
DCB5 C5 41      CMP L41
DCB7 F0 0C      BEQ LDCC5
DCB9          LDCB9:
DCB9 BD A8 2C   LDA L2CA8,X
DCBC 29 1F      AND #$1F
DCBE C5 41      CMP L41
DCC0 F0 03      BEQ LDCC5
DCC2          LDCC2:
DCC2 CA         DEX
DCC3 10 E2      BPL LDCA7
DCC5          LDCC5:
DCC5 60         RTS
DCC6          LDCC6:
DCC6 85 50      STA L50
DCC8 20 F2 DC   JSR LDCF2
DCCB 0A         ASL A
DCCC AA         TAX
DCCD A5 50      LDA L50
DCCF 95 A0      STA LA0,X
DCD1 4C D9 DC   JMP LDCD9
DCD4          LDCD4:
DCD4 20 F2 DC   JSR LDCF2
DCD7          LDCD7:
DCD7 0A         ASL A
DCD8 AA         TAX
DCD9          LDCD9:
DCD9 B5 A1      LDA LA1,X
DCDB 85 95      STA L95
DCDD B5 A0      LDA LA0,X
DCDF 85 94      STA L94
DCE1 60         RTS
DCE2          LDCE2:
DCE2 85 52      STA L52
DCE4 20 F2 DC   JSR LDCF2
DCE7 AA         TAX
DCE8 18         CLC
DCE9 69 03      ADC #$3
DCEB 85 53      STA L53
DCED A0 00      LDY #$0
DCEF B1 52      LDA (L52),Y
DCF1 60         RTS
DCF2          LDCF2:
DCF2 A6 80      LDX L80
DCF4 BD 68 2C   LDA L2C68,X
DCF7 10 03      BPL LDCFC
DCF9          LDCF9:
DCF9 BD 88 2C   LDA L2C88,X
DCFC          LDCFC:
DCFC 29 BF      AND #$BF
DCFE 60         RTS
DCFF          LDCFF:
DCFF A6 80      LDX L80
DD01 86 44      STX L44
DD03 BD 68 2C   LDA L2C68,X
DD06 10 09      BPL LDD11
DD08          LDD08:
DD08 8A         TXA
DD09 18         CLC
DD0A 69 20      ADC #$20
DD0C 85 44      STA L44
DD0E BD 88 2C   LDA L2C88,X
DD11          LDD11:
DD11 85 51      STA L51
DD13 29 1F      AND #$1F
DD15 24 51      BIT L51
DD17 60         RTS
DD18          LDD18:
DD18 A6 80      LDX L80
DD1A BD 68 2C   LDA L2C68,X
DD1D 30 03      BMI LDD22
DD1F          LDD1F:
DD1F BD 88 2C   LDA L2C88,X
DD22          LDD22:
DD22 C9 FF      CMP #$FF
DD24 60         RTS
DD25          LDD25:
DD25 A6 80      LDX L80
DD27 09 80      ORA #$80
DD29 BC 68 2C   LDY L2C68,X
DD2C 10 04      BPL LDD32
DD2E          LDD2E:
DD2E 9D 68 2C   STA L2C68,X
DD31 60         RTS
DD32          LDD32:
DD32 9D 88 2C   STA L2C88,X
DD35 60         RTS
DD36          LDD36:
DD36 AD 01 02   LDA L201
DD39 C9 30      CMP #$30
DD3B F0 11      BEQ LDD4E
DD3D          LDD3D:
DD3D 29 0F      AND #$F
DD3F 0A         ASL A
DD40 A8         TAY
DD41 88         DEY
DD42 B1 62      LDA (L62),Y
DD44 85 65      STA L65
DD46 88         DEY
DD47 B1 62      LDA (L62),Y
DD49 85 64      STA L64
DD4B 4C 9D DD   JMP LDD9D
DD4E          LDD4E:
DD4E A5 56      LDA L56
DD50 C9 03      CMP #$3
DD52 B0 09      BCS LDD5D
DD54          LDD54:
DD54 A9 A6      LDA #$A6
DD56 85 62      STA L62
DD58 A9 DD      LDA #$DD
DD5A 85 63      STA L63
DD5C 60         RTS
DD5D          LDD5D:
DD5D 78         SEI
DD5E 20 7E B0   JSR LB07E
DD61 C9 01      CMP #$1
DD63 F0 13      BEQ LDD78
DD65          LDD65:
DD65 C9 04      CMP #$4
DD67 F0 12      BEQ LDD7B
DD69          LDD69:
DD69 C9 05      CMP #$5
DD6B F0 0E      BEQ LDD7B
DD6D          LDD6D:
DD6D C9 03      CMP #$3
DD6F F0 0D      BEQ LDD7E
DD71          LDD71:
DD71 C9 02      CMP #$2
DD73 F0 09      BEQ LDD7E
DD75          LDD75:
DD75 4C 97 DF   JMP LDF97
DD78          LDD78:
DD78 A9 00      LDA #$0
DD7B          LDD7B = * + 1
              ; Instruction parameter jumped to.
DD7A 2C A9 80   BIT L80A9
DD7E          LDD7E = * + 1
              ; Instruction parameter jumped to.
DD7D 2C A9 40   BIT L40A9
DD80 8D E8 2B   STA L2BE8
DD83 20 3C EE   JSR LEE3C
DD86 A9 00      LDA #$0
DD88 85 6E      STA L6E
DD8A AD 02 02   LDA L202
DD8D 85 4C      STA L4C
DD8F 29 1F      AND #$1F
DD91 0A         ASL A
DD92 AA         TAX
DD93 BD BA DD   LDA LDDBA,X
DD96 85 64      STA L64
DD98 BD BB DD   LDA LDDBB,X
DD9B 85 65      STA L65
DD9D          LDD9D:
DD9D 20 A3 DD   JSR LDDA3
DDA0 4C 54 B6   JMP LB654
DDA3          LDDA3:
DDA3 6C 64 00   JMP (L64)
DDA6 ED AA      .WORD LAAED
DDA8 2B AB      .WORD LAB2B
DDAA 00 05 03   .BYTE $0,$5,$3
DDAD 05 06 05   .BYTE $5,$6,$5
DDB0 09 05 0C   .BYTE $9,$5,$C
DDB3 05 0F 05   .BYTE $5,$F,$5
DDB6 7C 9A      .WORD L9A7C
DDB8 5C F4      .WORD LF45C
DDBA          LDDBA:
DDBB          LDDBB = * + 1
DDBA C9 E4      .WORD LE4C9
DDBC E7 E3      .WORD LE3E7
DDBE 1B E5      .WORD LE51B
DDC0 1E E5      .BYTE $1E,$E5
DDC2 9A E5      .WORD LE59A
DDC4 E7 E3      .WORD LE3E7
DDC6 1E E6      .WORD LE61E
DDC8 1E E6      .WORD LE61E
DDCA 8E E7      .WORD LE78E
DDCC 8E E7      .WORD LE78E
DDCE C8 E5      .WORD LE5C8
DDD0 E7 E3      .WORD LE3E7
DDD2 AD E5      .WORD LE5AD
DDD4 E7 E3      .WORD LE3E7
DDD6 7B E6      .WORD LE67B
DDD8 7B E6      .WORD LE67B
DDDA C9 E4      .WORD LE4C9
DDDC E7 E3      .WORD LE3E7
DDDE 1B E5      .WORD LE51B
DDE0 1E E5      .BYTE $1E,$E5
DDE2 9A E5      .WORD LE59A
DDE4 E7 E3      .WORD LE3E7
DDE6 1E E6      .WORD LE61E
DDE8 1E E6      .WORD LE61E
DDEA 5C DD 5C   .BYTE $5C,$DD,$5C
DDED DD         .BYTE $DD
DDEE C8 E5      .WORD LE5C8
DDF0 E7 E3      .WORD LE3E7
DDF2 06 E7      .WORD LE706
DDF4 06 E7      .WORD LE706
DDF6 11 E7      .WORD LE711
DDF8 DD E2      .WORD LE2DD
DDFA          LDDFA:
DDFA 26 43 4F   .BYTE $26,$43,$4F
DDFD 50 59 52   .BYTE $50,$59,$52
DE00 49 47 48   .BYTE $49,$47,$48
DE03 54 20 43   .BYTE $54,$20,$43
DE06          LDE06:
DE06 4D 44 20   EOR L2044
DE09 38         SEC
DE0A 39 A6 5E   AND L5EA6,Y
DE0D 9A         TXS
DE0E 20 FD DE   JSR LDEFD
DE11 20 6B DB   JSR LDB6B
DE14 4C 1C F5   JMP LF51C
DE17          LDE17:
DE17 20 CB DE   JSR LDECB
DE1A A2 00      LDX #$0
DE1C          LDE1C:
DE1C BD FA DD   LDA LDDFA,X
DE1F 9D 00 02   STA L200,X
DE22 E8         INX
DE23 E0 11      CPX #$11
DE25 90 F5      BCC LDE1C
DE27          LDE27:
DE27 86 56      STX L56
DE29          LDE29:
DE29 A0 01      LDY #$1
DE2B 8C 00 2C   STY L2C00
DE2E 20 33 B8   JSR LB833
DE31 20 CF BE   JSR LBECF
DE34 AD 20 2C   LDA L2C20
DE37 D0 05      BNE LDE3E
DE39          LDE39:
DE39 A9 39      LDA #$39
DE3B 4C 6F B6   JMP LB66F
DE3E          LDE3E:
DE3E A9 FF      LDA #$FF
DE40 85 85      STA L85
DE42 AD 28 2C   LDA L2C28
DE45 85 5B      STA L5B
DE47 AD 20 2C   LDA L2C20
DE4A 85 5A      STA L5A
DE4C A9 03      LDA #$3
DE4E 20 7A C3   JSR LC37A
DE51          LDE51:
DE51 A9 00      LDA #$0
DE53 8D D2 2B   STA L2BD2
DE58          LDE58 = * + 2
              ; Instruction parameter jumped to.
DE56 20 B7 DE   JSR LDEB7
DE59          LDE59:
DE59 85 87      STA L87
DE5B 20 C1 DE   JSR LDEC1
DE5E 20 B7 DE   JSR LDEB7
DE61 85 88      STA L88
DE63 20 C1 DE   JSR LDEC1
DE66 20 B7 DE   JSR LDEB7
DE69 8D D3 2B   STA L2BD3
DE6C 20 C1 DE   JSR LDEC1
DE6F A5 85      LDA L85
DE71 F0 06      BEQ LDE79
DE73          LDE73:
DE73 A5 88      LDA L88
DE75 48         PHA
DE76 A5 87      LDA L87
DE78 48         PHA
DE79          LDE79:
DE79 20 B7 DE   JSR LDEB7
DE7C A0 00      LDY #$0
DE7E 84 85      STY L85
DE80 91 87      STA (L87),Y
DE82 20 C1 DE   JSR LDEC1
DE85 E6 87      INC L87
DE87 D0 02      BNE LDE8B
DE89          LDE89:
DE89 E6 88      INC L88
DE8B          LDE8B:
DE8B CE D3 2B   DEC L2BD3
DE8E D0 E9      BNE LDE79
DE90          LDE90:
DE90 20 84 CE   JSR LCE84
DE93 AD D2 2B   LDA L2BD2
DE96 C5 84      CMP L84
DE98 D0 10      BNE LDEAA
DE9A          LDE9A:
DE9A A5 81      LDA L81
DE9C D0 B3      BNE LDE51
DE9E          LDE9E:
DE9E 20 6B DB   JSR LDB6B
DEA1 68         PLA
DEA2 85 87      STA L87
DEA4 68         PLA
DEA5 85 88      STA L88
DEA7 6C 87 00   JMP (L87)
DEAA          LDEAA:
DEAA A9 50      LDA #$50
DEAD          LDEAD = * + 1
              ; Instruction parameter jumped to.
DEAC 2C A9 51   BIT L51A9
DEAF 48         PHA
DEB0 20 89 D9   JSR LD989
DEB3 68         PLA
DEB4 4C 33 FF   JMP LFF33
DEB7          LDEB7:
DEB7 20 84 CE   JSR LCE84
DEBA A5 81      LDA L81
DEBC F0 EF      BEQ LDEAD
DEBE          LDEBE:
DEBE A5 84      LDA L84
DEC0 60         RTS
DEC1          LDEC1:
DEC1 18         CLC
DEC2 6D D2 2B   ADC L2BD2
DEC5 69 00      ADC #$0
DEC7 8D D2 2B   STA L2BD2
DECA 60         RTS
DECB          LDECB:
DECB AD 37 FF   LDA LFF37
DECE 8D CE 2B   STA L2BCE
DED1 AD 38 FF   LDA LFF38
DED4 8D CF 2B   STA L2BCF
DED7 AD 34 FF   LDA LFF34
DEDA 8D D0 2B   STA L2BD0
DEDD AD 35 FF   LDA LFF35
DEE0 8D D1 2B   STA L2BD1
DEE3 A2 36      LDX #$36
DEE5 20 EA DE   JSR LDEEA
DEE8 A2 33      LDX #$33
DEEA          LDEEA:
DEEA A9 0B      LDA #$B
DEEC A0 DE      LDY #$DE
DEEE          LDEEE:
DEEE 48         PHA
DEEF 20 00 F7   JSR LF700
DEF2 68         PLA
DEF3 9D 01 FF   STA LFF01,X
DEF6 98         TYA
DEF7 9D 02 FF   STA LFF02,X
DEFA 4C F5 F6   JMP LF6F5
DEFD          LDEFD:
DEFD A2 36      LDX #$36
DEFF AD CE 2B   LDA L2BCE
DF02 AC CF 2B   LDY L2BCF
DF05 20 EE DE   JSR LDEEE
DF08 A2 33      LDX #$33
DF0A AD D0 2B   LDA L2BD0
DF0D AC D1 2B   LDY L2BD1
DF10 4C EE DE   JMP LDEEE
DF13          LDF13:
DF13 C9 10      CMP #$10
DF15 B0 04      BCS LDF1B
DF17          LDF17:
DF17 A8         TAY
DF18 B9 84 DF   LDA LDF84,Y
DF1B          LDF1B:
DF1B 48         PHA
DF1C 8A         TXA
DF1D 85 9C      STA L9C
DF1F 0A         ASL A
DF20 A8         TAY
DF21 B9 00 28   LDA L2800,Y
DF24 85 5A      STA L5A
DF26 B9 01 28   LDA L2801,Y
DF29 85 5B      STA L5B
DF2B AD E2 2B   LDA L2BE2
DF2E C9 00      CMP #$0
DF30 D0 08      BNE LDF3A
DF32          LDF32:
DF32 A9 FF      LDA #$FF
DF34 8D E2 2B   STA L2BE2
DF37 20 03 AF   JSR LAF03
DF3A          LDF3A:
DF3A 68         PLA
DF3B          LDF3B:
DF3B 20 B5 DF   JSR LDFB5
DF3E          LDF3E:
DF3E A6 5E      LDX L5E
DF40 9A         TXS
DF41 20 A9 F5   JSR LF5A9
DF44 20 6B DB   JSR LDB6B
DF47 20 2C EE   JSR LEE2C
DF4A A5 83      LDA L83
DF4C 29 0F      AND #$F
DF4E 85 82      STA L82
DF50 C9 0F      CMP #$F
DF52 F0 2D      BEQ LDF81
DF54          LDF54:
DF54 24 46      BIT L46
DF56 70 08      BVS LDF60
DF58          LDF58:
DF58 10 0C      BPL LDF66
DF5A          LDF5A:
DF5A 20 60 DA   JSR LDA60
DF5D 4C 71 DF   JMP LDF71
DF60          LDF60:
DF60 20 92 DA   JSR LDA92
DF63 4C 71 DF   JMP LDF71
DF66          LDF66:
DF66 AA         TAX
DF67 BD 48 2C   LDA L2C48,X
DF6A C9 FF      CMP #$FF
DF6C F0 13      BEQ LDF81
DF6E          LDF6E:
DF6E 20 75 DA   JSR LDA75
DF71          LDF71:
DF71 20 C7 A2   JSR LA2C7
DF74 A9 00      LDA #$0
DF76 9D 40 2B   STA L2B40,X
DF79 20 AC DA   JSR LDAAC
DF7C B0 03      BCS LDF81
DF7E          LDF7E:
DF7E 20 04 DB   JSR LDB04
DF81          LDF81:
DF81 4C 30 FF   JMP LFF30
DF84          LDF84:
DF84 00 00 40   .BYTE $0,$0,$40
DF87 41 66 44   .BYTE $41,$66,$44
DF8A 45 46 26   .BYTE $45,$46,$26
DF8D 47 76 42   .BYTE $47,$76,$42
DF90 43 76 48   .BYTE $43,$76,$48
DF93 74         .BYTE $74
DF94          LDF94:
DF94 A9 30      LDA #$30
DF97          LDF97 = * + 1
              ; Instruction parameter jumped to.
DF96 2C A9 31   BIT L31A9
DF99 2C A9 32   BIT L32A9
DF9C 2C A9 33   BIT L33A9
DF9F 2C A9 34   BIT L34A9
DFA2 20 AD DF   JSR LDFAD
DFA5 4C 3E DF   JMP LDF3E
DFA8          LDFA8:
DFA8 20 42 EE   JSR LEE42
DFAB A9 00      LDA #$0
DFAD          LDFAD:
DFAD 48         PHA
DFAE A9 00      LDA #$0
DFB0 85 5A      STA L5A
DFB2 85 5B      STA L5B
DFB4 68         PLA
DFB5          LDFB5:
DFB5 85 50      STA L50
DFB7 8A         TXA
DFB8 48         PHA
DFB9 98         TYA
DFBA 48         PHA
DFBB A5 50      LDA L50
DFBD A2 00      LDX #$0
DFBF          LDFBF:
DFBF DD AD E0   CMP LE0AD,X
DFC2 F0 03      BEQ LDFC7
DFC4          LDFC4:
DFC4 E8         INX
DFC5 D0 F8      BNE LDFBF
DFC7          LDFC7:
DFC7 48         PHA
DFC8 8A         TXA
DFC9 0A         ASL A
DFCA AA         TAX
DFCB BD D6 E0   LDA LE0D6,X
DFCE 85 DF      STA LDF
DFD0 BD D5 E0   LDA LE0D5,X
DFD3 85 DE      STA LDE
DFD5 68         PLA
DFD6 48         PHA
DFD7 A2 00      LDX #$0
DFD9 20 53 E0   JSR LE053
DFDC AD 00 23   LDA L2300
DFDF 8D E7 2D   STA L2DE7
DFE2 20 96 E0   JSR LE096
DFE5 A0 00      LDY #$0
DFE7          LDFE7:
DFE7 B1 DE      LDA (LDE),Y
DFE9 F0 06      BEQ LDFF1
DFEB          LDFEB:
DFEB 20 98 E0   JSR LE098
DFEE C8         INY
DFEF D0 F6      BNE LDFE7
DFF1          LDFF1:
DFF1 68         PLA
DFF2 A8         TAY
DFF3 29 F0      AND #$F0
DFF5 C9 40      CMP #$40
DFF7 D0 27      BNE LE020
DFF9          LDFF9:
DFF9 98         TYA
DFFA 48         PHA
DFFB A4 9C      LDY L9C
DFFD B9 C0 28   LDA L28C0,Y
E000          LE000:
              ; Instruction opcode accessed.
              ; Instruction opcode accessed.
E000 20 4A E0   JSR LE04A
E003 B9 E0 28   LDA L28E0,Y
E006 20 4A E0   JSR LE04A
E009 68         PLA
E00A C9 40      CMP #$40
E00C D0 12      BNE LE020
E00E          LE00E:
E00E B9 00 29   LDA L2900,Y
E011 20 41 E0   JSR LE041
E014 B9 20 29   LDA L2920,Y
E017 20 41 E0   JSR LE041
E01A B9 40 29   LDA L2940,Y
E01D 20 41 E0   JSR LE041
E020          LE020:
E020 A5 5A      LDA L5A
E022 20 65 E0   JSR LE065
E025 A5 5B      LDA L5B
E027 20 65 E0   JSR LE065
E02A CA         DEX
E02B 8A         TXA
E02C 18         CLC
E02D 69 00      ADC #$0
E02F 8D 07 2E   STA L2E07
E032 20 B2 F5   JSR LF5B2
E035 E6 DE      INC LDE
E037 A9 88      LDA #$88
E039 8D C7 2D   STA L2DC7
E03C 68         PLA
E03D A8         TAY
E03E 68         PLA
E03F AA         TAX
E040 60         RTS
E041          LE041:
E041 20 8D E0   JSR LE08D
E044 20 53 E0   JSR LE053
E047 A4 9C      LDY L9C
E049 60         RTS
E04A          LE04A:
E04A 20 8D E0   JSR LE08D
E04D 20 5C E0   JSR LE05C
E050 A4 9C      LDY L9C
E052 60         RTS
E053          LE053:
E053 48         PHA
E054 4A         LSR A
E055 4A         LSR A
E056 4A         LSR A
E057 4A         LSR A
E058 20 5E E0   JSR LE05E
E05B 68         PLA
E05C          LE05C:
E05C 29 0F      AND #$F
E05E          LE05E:
E05E A8         TAY
E05F          LE05F:
E05F B9 9D E0   LDA LE09D,Y
E062 4C 98 E0   JMP LE098
E065          LE065:
E065 48         PHA
E066 20 96 E0   JSR LE096
E069 68         PLA
E06A C9 64      CMP #$64
E06C 90 05      BCC LE073
E06E          LE06E:
E06E A0 64      LDY #$64
E070 20 7A E0   JSR LE07A
E073          LE073:
E073 A0 0A      LDY #$A
E075 20 7A E0   JSR LE07A
E078 A0 01      LDY #$1
E07A          LE07A:
E07A 84 50      STY L50
E07C A0 00      LDY #$0
E07E          LE07E:
E07E C5 50      CMP L50
E080 90 05      BCC LE087
E082          LE082:
E082 E5 50      SBC L50
E084 C8         INY
E085 D0 F7      BNE LE07E
E087          LE087:
E087 48         PHA
E088 20 5F E0   JSR LE05F
E08B 68         PLA
E08C 60         RTS
E08D          LE08D:
E08D 48         PHA
E08E A9 20      LDA #$20
E090 9D 00 23   STA L2300,X
E093 E8         INX
E094 68         PLA
E095 60         RTS
E096          LE096:
E096 A9 2C      LDA #$2C
E098          LE098:
E098 9D 00 23   STA L2300,X
E09B E8         INX
E09C 60         RTS
E09D          LE09D:
E09D 30 31 32   .BYTE $30,$31,$32
E0A0 33 34 35   .BYTE $33,$34,$35
E0A3 36 37 38   .BYTE $36,$37,$38
E0A6 39 41 42   .BYTE $39,$41,$42
E0A9 43 44 45   .BYTE $43,$44,$45
E0AD          LE0AD = * + 1
E0AC 46 00 52   .BYTE $46,$0,$52
E0AF 50 51 26   .BYTE $50,$51,$26
E0B2 30 31 32   .BYTE $30,$31,$32
E0B5 33 34 60   .BYTE $33,$34,$60
E0B8 63 64 65   .BYTE $63,$64,$65
E0BB 66 67 61   .BYTE $66,$67,$61
E0BE 39 62 01   .BYTE $39,$62,$1
E0C1 70 71 72   .BYTE $70,$71,$72
E0C4 73 74 75   .BYTE $73,$74,$75
E0C7 76 77 78   .BYTE $76,$77,$78
E0CA 02         .BYTE $2
E0CB          LE0CB:
E0CB 38         SEC
E0CC 40         RTI
E0CD 41 42 43   .BYTE $41,$42,$43
E0D0 44 45 46   .BYTE $44,$45,$46
E0D5          LE0D5 = * + 2
E0D3 47 48 25   .BYTE $47,$48,$25
E0D6          LE0D6:
E0D6 E1 29 E1   .BYTE $E1,$29,$E1
E0D9 37 E1 4A   .BYTE $37,$E1,$4A
E0DC E1 5D E1   .BYTE $E1,$5D,$E1
E0DF 6E E1 6E   .BYTE $6E,$E1,$6E
E0E2 E1 6E E1   .BYTE $E1,$6E,$E1
E0E5 6E E1 6E   .BYTE $6E,$E1,$6E
E0E8 E1 7B E1   .BYTE $E1,$7B,$E1
E0EB 8B E1      .WORD LE18B
E0ED 97 E1      .WORD LE197
E0EF AA E1      .BYTE $AA,$E1
E0F1 B3 E1      .WORD LE1B3
E0F3 B3 E1      .WORD LE1B3
E0F5 C1 E1      .WORD LE1C1
E0F7 CF E1      .WORD LE1CF
E0F9 CF E1      .WORD LE1CF
E0FB DE E1 EF   .BYTE $DE,$E1,$EF
E0FE E1 FA E1   .BYTE $E1,$FA,$E1
E101 0A E2 19   .BYTE $A,$E2,$19
E104 E2 2A E2   .BYTE $E2,$2A,$E2
E107 3A E2 47   .BYTE $3A,$E2,$47
E10A E2 56 E2   .BYTE $E2,$56,$E2
E10D 71 E2 7E   .BYTE $71,$E2,$7E
E110 E2 C6 E2   .BYTE $E2,$C6,$E2
E113 91 E2 9C   .BYTE $91,$E2,$9C
E116 E2 9C E2   .BYTE $E2,$9C,$E2
E119 9C E2 A9   .BYTE $9C,$E2,$A9
E11C E2 A9 E2   .BYTE $E2,$A9,$E2
E11F A9 E2 A9   .BYTE $A9,$E2,$A9
E122 E2 BA E2   .BYTE $E2,$BA,$E2
E125 20 4F 4B   .BYTE $20,$4F,$4B
E128 00         .BYTE $0
E129          LE129:
E129 46 49      LSR L49
E12B 4C 45 20   JMP L2045
E12E 54 4F 4F   .BYTE $54,$4F,$4F
E131 20         .BYTE $20
E132          LE132:
E132 4C 4F 4E   JMP L4E4F
E135 47 00 52   .BYTE $47,$0,$52
E138 45 43 4F   .BYTE $45,$43,$4F
E13B 52 44 20   .BYTE $52,$44,$20
E13E 4E 4F 54   .BYTE $4E,$4F,$54
E141 20 50 52   .BYTE $20,$50,$52
E144 45 53 45   .BYTE $45,$53,$45
E147 4E 54 00   .BYTE $4E,$54,$0
E14A 4F 56 45   .BYTE $4F,$56,$45
E14D 52 46      .BYTE $52,$46
E14F          LE14F:
E14F 4C 4F 57   JMP L574F
E152 20 49 4E   .BYTE $20,$49,$4E
E155 20 52 45   .BYTE $20,$52,$45
E158 43 4F 52   .BYTE $43,$4F,$52
E15B 44 00 57   .BYTE $44,$0,$57
E15E 52 49 54   .BYTE $52,$49,$54
E161 45 20 50   .BYTE $45,$20,$50
E164 52 4F 54   .BYTE $52,$4F,$54
E167 45 43 54   .BYTE $45,$43,$54
E16A 20 4F 4E   .BYTE $20,$4F,$4E
E16D 00 53 59   .BYTE $0,$53,$59
E170 4E 54 41   .BYTE $4E,$54,$41
E173 58 20 45   .BYTE $58,$20,$45
E176 52 52 4F   .BYTE $52,$52,$4F
E179 52 00 57   .BYTE $52,$0,$57
E17C 52         .BYTE $52
E17D          LE17D:
E17D 49 54      EOR #$54
E17F 45 20      EOR L20
E181 46 49      LSR L49
E183 4C 45 20   JMP L2045
E186 4F 50 45   .BYTE $4F,$50,$45
E189 4E 00      .BYTE $4E,$0
E18B          LE18B:
E18B 46 49      LSR L49
E18D 4C 45 20   JMP L2045
E190 45 58 49   .BYTE $45,$58,$49
E193 53 54 53   .BYTE $53,$54,$53
E196 00         .BYTE $0
E197          LE197:
E197 46 49      LSR L49
E199 4C 45 20   JMP L2045
E19C 54 59 50   .BYTE $54,$59,$50
E19F 45 20 4D   .BYTE $45,$20,$4D
E1A2 49 53 4D   .BYTE $49,$53,$4D
E1A5 41 54 43   .BYTE $41,$54,$43
E1A8 48 00 4E   .BYTE $48,$0,$4E
E1AB 4F 20 42   .BYTE $4F,$20,$42
E1AE          LE1AE:
E1AE 4C 4F 43   JMP L434F
E1B1 4B 00      .BYTE $4B,$0
E1B3          LE1B3:
E1B3 49 4C      EOR #$4C
E1B5 4C 45 47   JMP L4745
E1B8 41         .BYTE $41
E1B9          LE1B9:
E1B9 4C 20 42   JMP L4220
E1BC          LE1BC:
E1BC 4C 4F 43   JMP L434F
E1BF 4B 00      .BYTE $4B,$0
E1C1          LE1C1:
E1C1 46 49      LSR L49
E1C3 4C 45 20   JMP L2045
E1C6 4E 4F 54   .BYTE $4E,$4F,$54
E1C9 20 4F 50   .BYTE $20,$4F,$50
E1CC 45 4E 00   .BYTE $45,$4E,$0
E1CF          LE1CF:
E1CF 46 49      LSR L49
E1D1 4C 45 20   JMP L2045
E1D4 4E 4F 54   .BYTE $4E,$4F,$54
E1D7 20 46 4F   .BYTE $20,$46,$4F
E1DA 55         .BYTE $55
E1DB          LE1DB:
E1DB 4E 44 00   LSR L44
E1DE 20 46 49   JSR L4946
E1E1 4C 45 53   JMP L5345
E1E4 20 53 43   .BYTE $20,$53,$43
E1E7 52 41 54   .BYTE $52,$41,$54
E1EA 43 48 45   .BYTE $43,$48,$45
E1ED 44 00 4E   .BYTE $44,$0,$4E
E1F0 4F 20 43   .BYTE $4F,$20,$43
E1F3 48 41      .BYTE $48,$41
E1F5          LE1F5:
E1F5 4E 4E 45   LSR L454E
E1F8 4C 00 44   JMP L4400
E1FB 49 52 45   .BYTE $49,$52,$45
E1FE 43 54 4F   .BYTE $43,$54,$4F
E201 52 59 20   .BYTE $52,$59,$20
E204 45 52 52   .BYTE $45,$52,$52
E207 4F 52 00   .BYTE $4F,$52,$0
E20A 50 41 52   .BYTE $50,$41,$52
E20D 54         .BYTE $54
E20E          LE20E:
E20E 49 54      EOR #$54
E210 49 4F      EOR #$4F
E212          LE212:
E212 4E 20 46   LSR L4620
E215 55 4C      EOR L4C,X
E217 4C 00 43   JMP L4300
E21A 4D 44 20   .BYTE $4D,$44,$20
E21D 48 44 20   .BYTE $48,$44,$20
E220 44 4F 53   .BYTE $44,$4F,$53
E223 20 56 31   .BYTE $20,$56,$31
E226 2E 39 30   .BYTE $2E,$39,$30
E229 00 44 52   .BYTE $0,$44,$52
E22C 49 56 45   .BYTE $49,$56,$45
E22F 20 4E 4F   .BYTE $20,$4E,$4F
E232 54 20 52   .BYTE $54,$20,$52
E235 45 41 44   .BYTE $45,$41,$44
E238 59 00 46   .BYTE $59,$0,$46
E23B 4F 52 4D   .BYTE $4F,$52,$4D
E23E 41 54 20   .BYTE $41,$54,$20
E241 45 52 52   .BYTE $45,$52,$52
E244 4F 52 00   .BYTE $4F,$52,$0
E247 48 41 52   .BYTE $48,$41,$52
E24A 44 57 41   .BYTE $44,$57,$41
E24D 52 45 20   .BYTE $52,$45,$20
E250 45 52 52   .BYTE $45,$52,$52
E253 4F 52 00   .BYTE $4F,$52,$0
E256 53 45 4C   .BYTE $53,$45,$4C
E259 45 43 54   .BYTE $45,$43,$54
E25C 45 44 20   .BYTE $45,$44,$20
E25F 50 41 52   .BYTE $50,$41,$52
E262 54         .BYTE $54
E263          LE263:
E263 49 54      EOR #$54
E265 49 4F      EOR #$4F
E267 4E 20 49   LSR L4920
E26A 4C 4C 45   JMP L454C
E26D 47 41      .BYTE $47,$41
E26F          LE26F:
E26F 4C 00 53   JMP L5300
E272 59 53 54   .BYTE $59,$53,$54
E275 45 4D 20   .BYTE $45,$4D,$20
E278 45 52 52   .BYTE $45,$52,$52
E27B 4F 52 00   .BYTE $4F,$52,$0
E27E 50 41 52   .BYTE $50,$41,$52
E281 54 49 54   .BYTE $54,$49,$54
E284 49 4F 4E   .BYTE $49,$4F,$4E
E287          LE287:
E287 20 53 45   JSR L4553
E28A 4C 45 43   JMP L4345
E28D 54 45 44   .BYTE $54,$45,$44
E290 00 53 43   .BYTE $0,$53,$43
E293 53 49 20   .BYTE $53,$49,$20
E296 45 52 52   .BYTE $45,$52,$52
E299 4F 52 00   .BYTE $4F,$52,$0
E29C 53 54 41   .BYTE $53,$54,$41
E29F 54 55 53   .BYTE $54,$55,$53
E2A2 20 45 52   .BYTE $20,$45,$52
E2A5 52 4F 52   .BYTE $52,$4F,$52
E2A8 00 43 4F   .BYTE $0,$43,$4F
E2AB 4E 54 52   .BYTE $4E,$54,$52
E2AE 4F         .BYTE $4F
E2AF          LE2AF:
E2AF 4C 4C 45   JMP L454C
E2B2 52 20 45   .BYTE $52,$20,$45
E2B5 52 52 4F   .BYTE $52,$52,$4F
E2B8 52 00      .BYTE $52,$0
E2BA          LE2BA:
E2BA 49 4C      EOR #$4C
E2BC 4C 45 47   JMP L4745
E2BF 41         .BYTE $41
E2C0          LE2C0:
E2C0 4C 20 4A   JMP L4A20
E2C3 4F 42 00   .BYTE $4F,$42,$0
E2C6 44 49 52   .BYTE $44,$49,$52
E2C9 45 43 54   .BYTE $45,$43,$54
E2CC 4F 52 59   .BYTE $4F,$52,$59
E2CF 20 4E 4F   .BYTE $20,$4E,$4F
E2D2 54 20 46   .BYTE $54,$20,$46
E2D5 4F 55      .BYTE $4F,$55
E2D7          LE2D7:
E2D7 4E 44 00   LSR L44
E2DA          LE2DA:
E2DA 4C 54 B6   JMP LB654
E2DD          LE2DD:
E2DD A5 46      LDA L46
E2DF 29 04      AND #$4
E2E1 F0 F7      BEQ LE2DA
E2E3          LE2E3:
E2E3 A0 03      LDY #$3
E2E5 20 B8 B6   JSR LB6B8
E2E8 F0 02      BEQ LE2EC
E2EA          LE2EA:
E2EA A0 04      LDY #$4
E2EC          LE2EC:
E2EC C0 04      CPY #$4
E2EE 90 01      BCC LE2F1
E2F0          LE2F0:
E2F0 88         DEY
E2F1          LE2F1:
E2F1 8C 00 2C   STY L2C00
E2F4 A5 56      LDA L56
E2F6 8D 01 2C   STA L2C01
E2F9 AD 03 02   LDA L203
E2FC C9 2A      CMP #$2A
E2FE D0 0E      BNE LE30E
E300          LE300:
E300 20 C7 A2   JSR LA2C7
E303 BD C0 2F   LDA L2FC0,X
E306 F0 06      BEQ LE30E
E308          LE308:
E308 BC D0 2F   LDY L2FD0,X
E30B 4C 5B E3   JMP LE35B
E30E          LE30E:
E30E 20 43 B8   JSR LB843
E311 B0 22      BCS LE335
E313          LE313:
E313 20 D0 AE   JSR LAED0
E316 D0 1D      BNE LE335
E318          LE318:
E318 A9 01      LDA #$1
E31A 8D EA 2B   STA L2BEA
E31D 8D EB 2B   STA L2BEB
E320 20 CF BE   JSR LBECF
E323 AD 20 2C   LDA L2C20
E326 F0 10      BEQ LE338
E328          LE328:
E328 AD 18 2C   LDA L2C18
E32B 29 03      AND #$3
E32D C9 02      CMP #$2
E32F F0 1A      BEQ LE34B
E331          LE331:
E331 24 4C      BIT L4C
E333 30 16      BMI LE34B
E335          LE335:
E335 A9 0F      LDA #$F
E338          LE338 = * + 1
              ; Instruction parameter jumped to.
E337 2C A9 02   BIT L2A9
E33A 48         PHA
E33B 20 10 E4   JSR LE410
E33E 68         PLA
E33F C9 0F      CMP #$F
E341 F0 03      BEQ LE346
E343          LE343:
E343 A9 62      LDA #$62
E346          LE346 = * + 1
              ; Instruction parameter jumped to.
E345 2C A9 74   BIT L74A9
E348 4C 6F B6   JMP LB66F
E34B          LE34B:
E34B 20 C7 A2   JSR LA2C7
E34E AD 28 2C   LDA L2C28
E351 A8         TAY
E352 9D D0 2F   STA L2FD0,X
E355 AD 20 2C   LDA L2C20
E358 9D C0 2F   STA L2FC0,X
E35B          LE35B:
E35B 85 5A      STA L5A
E35D 84 5B      STY L5B
E35F A9 02      LDA #$2
E362          LE362 = * + 1
              ; Instruction parameter jumped to.
E361 2C A9 00   BIT LA9
E364 85 96      STA L96
E366 A2 00      LDX #$0
E368 A9 AA      LDA #$AA
E36A 20 A8 E3   JSR LE3A8
E36D 20 B9 97   JSR L97B9
E370 A0 01      LDY #$1
E372 B1 68      LDA (L68),Y
E374 85 5B      STA L5B
E376 88         DEY
E377 B1 68      LDA (L68),Y
E379 85 5A      STA L5A
E37B D0 0F      BNE LE38C
E37D          LE37D:
E37D A9 1F      LDA #$1F
E37F 20 48 FF   JSR LFF48
E382 A6 5B      LDX L5B
E384 CA         DEX
E385 8A         TXA
E386 38         SEC
E387 E5 96      SBC L96
E389 4C 90 E3   JMP LE390
E38C          LE38C:
E38C A2 FE      LDX #$FE
E38E A9 00      LDA #$0
E390          LE390:
E390 20 48 FF   JSR LFF48
E393 A0 02      LDY #$2
E395          LE395:
E395 B1 68      LDA (L68),Y
E397 20 48 FF   JSR LFF48
E39A C8         INY
E39B CA         DEX
E39C D0 F7      BNE LE395
E39E          LE39E:
E39E 20 9B 97   JSR L979B
E3A1 A5 5A      LDA L5A
E3A3 D0 BD      BNE LE362
E3A5          LE3A5:
E3A5 4C 54 B6   JMP LB654
E3A8          LE3A8:
E3A8 48         PHA
E3A9 8A         TXA
E3AA 20 76 D9   JSR LD976
E3AD 68         PLA
E3AE 20 25 E8   JSR LE825
E3B1 C9 02      CMP #$2
E3B3 B0 01      BCS LE3B6
E3B5          LE3B5:
E3B5 60         RTS
E3B6          LE3B6:
E3B6 48         PHA
E3B7 A9 02      LDA #$2
E3B9 20 10 E4   JSR LE410
E3BC 68         PLA
E3BD 4C 13 DF   JMP LDF13
E3C0          LE3C0:
E3C0 8D E1 2B   STA L2BE1
E3C3 A5 6A      LDA L6A
E3C5 2C E8 2B   BIT L2BE8
E3C8 10 11      BPL LE3DB
E3CA          LE3CA:
E3CA 29 80      AND #$80
E3CC 09 20      ORA #$20
E3CE 0D E1 2B   ORA L2BE1
E3D1 25 70      AND L70
E3D3 05 71      ORA L71
E3D5          LE3D5:
E3D5 85 6A      STA L6A
E3D7 AD E1 2B   LDA L2BE1
E3DA 60         RTS
E3DB          LE3DB:
E3DB 29 F0      AND #$F0
E3DD 0D E1 2B   ORA L2BE1
E3E0 4C D5 E3   JMP LE3D5
E3E3          LE3E3:
E3E3 20 25 E8   JSR LE825
E3E7          LE3E7 = * + 1
              ; Instruction parameter jumped to.
E3E6 2C A9 4F   BIT L4FA9
E3E9          LE3E9:
E3E9 20 C0 E3   JSR LE3C0
E3EC C9 02      CMP #$2
E3EE 90 11      BCC LE401
E3F0          LE3F0:
E3F0 24 4C      BIT L4C
E3F2 70 0D      BVS LE401
E3F4          LE3F4:
E3F4 20 01 E4   JSR LE401
E3F7          LE3F7:
E3F7 AD E1 2B   LDA L2BE1
E3FA 29 0F      AND #$F
E3FC A2 00      LDX #$0
E3FE 4C 36 FF   JMP LFF36
E401          LE401:
E401 A5 6A      LDA L6A
E403 2C E8 2B   BIT L2BE8
E406 50 08      BVC LE410
E408          LE408:
E408 29 0F      AND #$F
E40A D0 02      BNE LE40E
E40C          LE40C:
E40C A9 01      LDA #$1
E40E          LE40E:
E40E 05 6A      ORA L6A
E410          LE410:
E410 48         PHA
E411 20 B9 97   JSR L97B9
E414 68         PLA
E415 20 48 FF   JSR LFF48
E418 4C 9B 97   JMP L979B
E41B          LE41B:
E41B 48         PHA
E41C          LE41C:
E41C 2C 01 88   BIT PIO+$01
E41F 30 19      BMI LE43A
E421          LE421:
E421 AD 00 80   LDA VIA1+$00
E424 30 14      BMI LE43A
E426          LE426:
E426 29 04      AND #$4
E428 C5 6E      CMP L6E
E42A F0 F0      BEQ LE41C
E42C          LE42C:
E42C 85 6E      STA L6E
E42E 68         PLA
E42F 8D 0A 80   STA VIA1+$0A
E432 A9 04      LDA #$4
E434          LE434:
E434 2C 0D 80   BIT VIA1+$0D
E437 F0 FB      BEQ LE434
E439          LE439:
E439 60         RTS
E43A          LE43A:
E43A 4C 3C FF   JMP LFF3C
E43D          LE43D:
E43D 2C 0A 80   BIT VIA1+$0A
E440 AD 00 80   LDA VIA1+$00
E443 49 08      EOR #$8
E445 8D 00 80   STA VIA1+$00
E448 A9 04      LDA #$4
E44A          LE44A:
E44A 2C 01 88   BIT PIO+$01
E44D 30 EB      BMI LE43A
E44F          LE44F:
E44F 2C 00 80   BIT VIA1+$00
E452 30 E6      BMI LE43A
E454          LE454:
E454 2C 0D 80   BIT VIA1+$0D
E457 F0 F1      BEQ LE44A
E459          LE459:
E459 AD 0A 80   LDA VIA1+$0A
E45C 60         RTS
E45D          LE45D:
E45D 2C 01 88   BIT PIO+$01
E460 30 D8      BMI LE43A
E462          LE462:
E462 AD 00 80   LDA VIA1+$00
E465 30 D3      BMI LE43A
E467          LE467:
E467 29 04      AND #$4
E469 C5 6E      CMP L6E
E46B F0 F0      BEQ LE45D
E46D          LE46D:
E46D 85 6E      STA L6E
E46F 60         RTS
E470          LE470:
E470 A2 01      LDX #$1
E473          LE473 = * + 1
              ; Instruction parameter jumped to.
E472 2C A2 02   BIT L2A2
E475          LE475:
E475 A0 00      LDY #$0
E477 20 B9 97   JSR L97B9
E47A          LE47A:
E47A B1 68      LDA (L68),Y
E47C 20 48 FF   JSR LFF48
E47F C8         INY
E480 D0 F8      BNE LE47A
E482          LE482:
E482 CA         DEX
E483 F0 05      BEQ LE48A
E485          LE485:
E485 E6 69      INC L69
E487 4C 7A E4   JMP LE47A
E48A          LE48A:
E48A 4C 9B 97   JMP L979B
E48D          LE48D:
E48D A2 01      LDX #$1
E490          LE490 = * + 1
              ; Instruction parameter jumped to.
E48F 2C A2 02   BIT L2A2
E492          LE492:
E492 A0 00      LDY #$0
E494 20 9B 97   JSR L979B
E497          LE497:
E497 20 45 FF   JSR LFF45
E49A 91 68      STA (L68),Y
E49C C8         INY
E49D D0 F8      BNE LE497
E49F          LE49F:
E49F CA         DEX
E4A0 F0 05      BEQ LE4A7
E4A2          LE4A2:
E4A2 E6 69      INC L69
E4A4 4C 97 E4   JMP LE497
E4A7          LE4A7:
E4A7 4C 6C 97   JMP L976C
E4AA          LE4AA:
E4AA 20 BF E4   JSR LE4BF
E4AD          LE4AD:
E4AD AD 03 02   LDA L203
E4B0 85 5A      STA L5A
E4B2 AD 04 02   LDA L204
E4B5 85 5B      STA L5B
E4B7          LE4B7:
E4B7 A9 00      LDA #$0
E4B9 20 76 D9   JSR LD976
E4BC A9 00      LDA #$0
E4BE 60         RTS
E4BF          LE4BF:
E4BF A5 4C      LDA L4C
E4C1 29 10      AND #$10
E4C3 A2 00      LDX #$0
E4C5 9D 40 28   STA L2840,X
E4C8 60         RTS
E4C9          LE4C9:
E4C9 2C E8 2B   BIT L2BE8
E4CC 30 1B      BMI LE4E9
E4CE          LE4CE:
E4CE A9 20      LDA #$20
E4D0 24 4C      BIT L4C
E4D2 D0 0C      BNE LE4E0
E4D4          LE4D4:
E4D4 20 AD E4   JSR LE4AD
E4D7 A9 80      LDA #$80
E4D9 20 E3 E3   JSR LE3E3
E4DC 24 4C      BIT L4C
E4DE 30 03      BMI LE4E3
E4E0          LE4E0:
E4E0 20 70 E4   JSR LE470
E4E3          LE4E3:
E4E3 20 E0 E7   JSR LE7E0
E4E6 4C CE E4   JMP LE4CE
E4E9          LE4E9:
E4E9 24 4C      BIT L4C
E4EB 30 11      BMI LE4FE
E4ED          LE4ED:
E4ED 20 AA E4   JSR LE4AA
E4F0 A9 B2      LDA #$B2
E4F2 20 E3 E3   JSR LE3E3
E4F5 20 73 E4   JSR LE473
E4F8 20 AD E7   JSR LE7AD
E4FB 4C ED E4   JMP LE4ED
E4FE          LE4FE:
E4FE 24 71      BIT L71
E500 30 11      BMI LE513
E502          LE502:
E502 20 AD E4   JSR LE4AD
E505 A9 80      LDA #$80
E507 20 E3 E3   JSR LE3E3
E50A 20 70 E4   JSR LE470
E50D 20 AD E7   JSR LE7AD
E510 4C 02 E5   JMP LE502
E513          LE513:
E513 A9 8D      LDA #$8D
E515 2C A9 0B   BIT LBA9
E518          LE518:
E518 4C E9 E3   JMP LE3E9
E51B          LE51B:
E51B A9 00      LDA #$0
E51D 2C A9 4F   BIT L4FA9
E520 8D E1 2B   STA L2BE1
E523 2C E8 2B   BIT L2BE8
E526 30 2D      BMI LE555
E528          LE528:
E528 24 4C      BIT L4C
E52A 30 0B      BMI LE537
E52C          LE52C:
E52C A9 00      LDA #$0
E52E 85 68      STA L68
E530 A9 03      LDA #$3
E532 85 69      STA L69
E534 20 8D E4   JSR LE48D
E537          LE537:
E537 A9 20      LDA #$20
E539 24 4C      BIT L4C
E53B D0 12      BNE LE54F
E53D          LE53D:
E53D AD E1 2B   LDA L2BE1
E540 C9 02      CMP #$2
E542 B0 D4      BCS LE518
E544          LE544:
E544 20 AD E4   JSR LE4AD
E547 A9 90      LDA #$90
E549 20 E3 E3   JSR LE3E3
E54C 20 5D E4   JSR LE45D
E54F          LE54F:
E54F 20 E0 E7   JSR LE7E0
E552 4C 2C E5   JMP LE52C
E555          LE555:
E555 24 4C      BIT L4C
E557 30 1E      BMI LE577
E559          LE559:
E559 20 5F EE   JSR LEE5F
E55C 20 90 E4   JSR LE490
E55F AD E1 2B   LDA L2BE1
E562 C9 02      CMP #$2
E564 B0 B2      BCS LE518
E566          LE566:
E566 20 AA E4   JSR LE4AA
E569 A9 B4      LDA #$B4
E56B 20 E3 E3   JSR LE3E3
E56E 20 5D E4   JSR LE45D
E571 20 AD E7   JSR LE7AD
E574 4C 59 E5   JMP LE559
E577          LE577:
E577 A9 00      LDA #$0
E579 85 68      STA L68
E57B A9 03      LDA #$3
E57D 85 69      STA L69
E57F 20 8D E4   JSR LE48D
E582 AD E1 2B   LDA L2BE1
E585 C9 02      CMP #$2
E587 B0 8F      BCS LE518
E589          LE589:
E589 20 AD E4   JSR LE4AD
E58C A9 90      LDA #$90
E58E 20 E3 E3   JSR LE3E3
E591 20 5D E4   JSR LE45D
E594 20 AD E7   JSR LE7AD
E597 4C 77 E5   JMP LE577
E59A          LE59A:
E59A A5 4C      LDA L4C
E59C 4A         LSR A
E59D 90 03      BCC LE5A2
E59F          LE59F:
E59F 4C E7 E3   JMP LE3E7
E5A2          LE5A2:
E5A2 A9 00      LDA #$0
E5A4 85 6A      STA L6A
E5A6 A2 00      LDX #$0
E5A8 A9 C0      LDA #$C0
E5AA 4C E3 E3   JMP LE3E3
E5AD          LE5AD:
E5AD A9 20      LDA #$20
E5AF 24 4C      BIT L4C
E5B1 10 03      BPL LE5B6
E5B3          LE5B3:
E5B3 4C 01 E4   JMP LE401
E5B6          LE5B6:
E5B6 F0 0A      BEQ LE5C2
E5B8          LE5B8:
E5B8 AD 04 02   LDA L204
E5BB 85 71      STA L71
E5BD AD 05 02   LDA L205
E5C0 85 70      STA L70
E5C2          LE5C2:
E5C2 AD 03 02   LDA L203
E5C5 85 6A      STA L6A
E5C7 60         RTS
E5C8          LE5C8:
E5C8 20 9A E5   JSR LE59A
E5CB 2C E8 2B   BIT L2BE8
E5CE 30 01      BMI LE5D1
E5D0          LE5D0:
E5D0 60         RTS
E5D1          LE5D1:
E5D1 24 4C      BIT L4C
E5D3 10 0E      BPL LE5E3
E5D5          LE5D5:
E5D5 20 AA E4   JSR LE4AA
E5D8 A9 01      LDA #$1
E5DA 8D 01 28   STA L2801
E5DD A9 A8      LDA #$A8
E5DF 20 25 E8   JSR LE825
E5E3          LE5E3 = * + 1
              ; Instruction parameter jumped to.
E5E2 2C A9 00   BIT LA9
E5E5 20 E9 E3   JSR LE3E9
E5E8 20 B9 97   JSR L97B9
E5EB A9 0A      LDA #$A
E5ED 20 48 FF   JSR LFF48
E5F0 24 4C      BIT L4C
E5F2 10 04      BPL LE5F8
E5F4          LE5F4:
E5F4 AD 03 02   LDA L203
E5F8          LE5F8 = * + 1
              ; Instruction parameter jumped to.
E5F7 2C A9 00   BIT LA9
E5FA 20 48 FF   JSR LFF48
E5FD A9 01      LDA #$1
E5FF 20 48 FF   JSR LFF48
E602 A9 0A      LDA #$A
E604 20 48 FF   JSR LFF48
E607 A9 01      LDA #$1
E609 20 48 FF   JSR LFF48
E60C A5 4C      LDA L4C
E60E 29 20      AND #$20
E610 F0 0B      BEQ LE61D
E612          LE612:
E612 A2 01      LDX #$1
E614          LE614:
E614 8A         TXA
E615 20 48 FF   JSR LFF48
E618 E8         INX
E619 E0 0B      CPX #$B
E61B 90 F7      BCC LE614
E61D          LE61D:
E61D 60         RTS
E61E          LE61E:
E61E A9 01      LDA #$1
E620 24 4C      BIT L4C
E622 F0 08      BEQ LE62C
E624          LE624:
E624 A9 4F      LDA #$4F
E626 20 C0 E3   JSR LE3C0
E629 4C F7 E3   JMP LE3F7
E62C          LE62C:
E62C 2C E8 2B   BIT L2BE8
E62F 30 0D      BMI LE63E
E631          LE631:
E631 2C 03 02   BIT L203
E634 30 05      BMI LE63B
E636          LE636:
E636 A9 01      LDA #$1
E638 4C C0 E3   JMP LE3C0
E63B          LE63B:
E63B 4C 7E E6   JMP LE67E
E63E          LE63E:
E63E 30 46      BMI LE686
E640          LE640:
E640 A2 00      LDX #$0
E642          LE642:
E642 BD 5D E6   LDA LE65D,X
E645 9D 00 02   STA L200,X
E648 E8         INX
E649 E0 0C      CPX #$C
E64B 90 F5      BCC LE642
E64D          LE64D:
E64D 86 56      STX L56
E64F A2 01      LDX #$1
E651 8E 00 2C   STX L2C00
E654 A9 0A      LDA #$A
E656 8D 01 2C   STA L2C01
E659 CA         DEX
E65A 4C 0F FF   JMP LFF0F
E65D          LE65D:
E65D 4E 30 3A   .BYTE $4E,$30,$3A
E660 43 4D 44   .BYTE $43,$4D,$44
E663 20 48 44   .BYTE $20,$48,$44
E666          LE666:
E666 2C 38 39   .BYTE $2C,$38,$39
E669 02 4F 0A   .BYTE $2,$4F,$A
E66C          LE66C:
E66C 00 E5 01   .BYTE $0,$E5,$1
E66F 02 00 0A   .BYTE $2,$0,$A
E672          LE672:
E672 00 00 01   .BYTE $0,$0,$1
E675 02 4F 0A   .BYTE $2,$4F,$A
E678 4F 00      .BYTE $4F,$0
E67A          LE67A:
E67B          LE67B = * + 1
              ; Instruction parameter jumped to.
E67A 01 A9      ORA (LA9,X)
E67C          LE67C:
E67D          LE67D = * + 1
              ; Instruction parameter jumped to.
E67E          LE67E = * + 2
              ; Instruction parameter jumped to.
E67C 0E 2C A9   ASL LA92C
E67F          LE67F:
E680          LE680 = * + 1
              ; Instruction parameter jumped to.
E67F 06 20      ASL L20
E681          LE681:
E681 C0 E3      CPY #$E3
E683 4C 97 DF   JMP LDF97
E686          LE686:
E686 A2 03      LDX #$3
E688          LE688:
E688 E4 56      CPX L56
E68A F0 12      BEQ LE69E
E68C          LE68C:
E68C BD 00 02   LDA L200,X
E68F DD 6C E6   CMP LE66C,X
E692 90 E7      BCC LE67B
E694          LE694:
E694 DD 72 E6   CMP LE672,X
E697 90 02      BCC LE69B
E699          LE699:
E69A          LE69A = * + 1
              ; Instruction parameter jumped to.
E699 D0 E0      BNE LE67B
E69B          LE69B:
E69B E8         INX
E69C D0 EA      BNE LE688
E69E          LE69E:
E69E E0 09      CPX #$9
E6A0 B0 09      BCS LE6AB
E6A2          LE6A2:
E6A2 BD 66 E6   LDA LE666,X
E6A5 9D 00 02   STA L200,X
E6A8 E8         INX
E6A9 D0 F3      BNE LE69E
E6AB          LE6AB:
E6AB A2 00      LDX #$0
E6AD AD 07 02   LDA L207
E6B0          LE6B0:
E6B0 9D 00 50   STA L5000,X
E6B3 9D 00 51   STA L5100,X
E6B6 E8         INX
E6B7 D0 F7      BNE LE6B0
E6B9          LE6B9:
E6B9 A5 4C      LDA L4C
E6BB 29 EF      AND #$EF
E6BD 85 4C      STA L4C
E6BF          LE6BF:
E6BF AD 06 02   LDA L206
E6C2 85 5A      STA L5A
E6C4 AD 08 02   LDA L208
E6C7 85 5B      STA L5B
E6C9 20 BF E4   JSR LE4BF
E6CC 20 B7 E4   JSR LE4B7
E6CF A9 B4      LDA #$B4
E6D1 20 25 E8   JSR LE825
E6D4 C9 02      CMP #$2
E6D6 90 03      BCC LE6DB
E6D8          LE6D8:
E6D8 4C 7E E6   JMP LE67E
E6DB          LE6DB:
E6DB EE 08 02   INC L208
E6DE AD 08 02   LDA L208
E6E1 C9 0B      CMP #$B
E6E3 90 DA      BCC LE6BF
E6E5          LE6E5:
E6E5 A9 01      LDA #$1
E6E7 8D 08 02   STA L208
E6EA A5 4C      LDA L4C
E6EC 49 10      EOR #$10
E6EE 85 4C      STA L4C
E6F0 29 10      AND #$10
E6F2 D0 CB      BNE LE6BF
E6F4          LE6F4:
E6F4 EE 06 02   INC L206
E6F7 AD 06 02   LDA L206
E6FA CD 04 02   CMP L204
E6FD 90 C0      BCC LE6BF
E6FF          LE6FF:
E6FF F0 BE      BEQ LE6BF
E701          LE701:
E701 A9 00      LDA #$0
E703 4C C0 E3   JMP LE3C0
E706          LE706:
E706 2C E8 2B   BIT L2BE8
E709 30 01      BMI LE70C
E70B          LE70B:
E70B 60         RTS
E70C          LE70C:
E70C A9 00      LDA #$0
E70E 4C E9 E3   JMP LE3E9
E711          LE711:
E711 78         SEI
E712 AE 04 02   LDX L204
E715 A5 56      LDA L56
E717 C9 04      CMP #$4
E719 B0 03      BCS LE71E
E71B          LE71B:
E71B 4C 97 DF   JMP LDF97
E71E          LE71E:
E71E AD 03 02   LDA L203
E721 C9 42      CMP #$42
E723 D0 1A      BNE LE73F
E725          LE725:
E725 8A         TXA
E726 C9 30      CMP #$30
E728 F0 04      BEQ LE72E
E72A          LE72A:
E72A C9 31      CMP #$31
E72C D0 ED      BNE LE71B
E72E          LE72E:
E72E 48         PHA
E72F A5 46      LDA L46
E731 29 FB      AND #$FB
E733 85 46      STA L46
E735 68         PLA
E736 29 01      AND #$1
E738 0A         ASL A
E739 0A         ASL A
E73A 05 46      ORA L46
E73C 85 46      STA L46
E73E 60         RTS
E73F          LE73F:
E73F C9 53      CMP #$53
E741 D0 03      BNE LE746
E743          LE743:
E743 86 57      STX L57
E745 60         RTS
E746          LE746:
E746 C9 52      CMP #$52
E748 D0 03      BNE LE74D
E74A          LE74A:
E74A 86 61      STX L61
E74C 60         RTS
E74D          LE74D:
E74D C9 54      CMP #$54
E74F F0 08      BEQ LE759
E751          LE751:
E751 C9 56      CMP #$56
E753 F0 04      BEQ LE759
E755          LE755:
E755 C9 4D      CMP #$4D
E757 D0 01      BNE LE75A
E759          LE759:
E759 60         RTS
E75A          LE75A:
E75A C9 4D      CMP #$4D
E75C F0 11      BEQ LE76F
E75E          LE75E:
E75E C9 04      CMP #$4
E760 90 B9      BCC LE71B
E762          LE762:
E762 C9 1F      CMP #$1F
E764 B0 B5      BCS LE71B
E766          LE766:
E766 09 40      ORA #$40
E768 85 78      STA L78
E76A 49 60      EOR #$60
E76C 85 77      STA L77
E76E 60         RTS
E76F          LE76F:
E76F A9 00      LDA #$0
E771 85 6E      STA L6E
E773 85 68      STA L68
E775 AD 05 02   LDA L205
E778 85 69      STA L69
E77A E0 57      CPX #$57
E77C F0 0A      BEQ LE788
E77E          LE77E:
E77E E0 52      CPX #$52
E780 D0 99      BNE LE71B
E782          LE782:
E782 AE 06 02   LDX L206
E785 4C 75 E4   JMP LE475
E788          LE788:
E788 AE 06 02   LDX L206
E78B 4C 92 E4   JMP LE492
E78E          LE78E:
E78E 2C E8 2B   BIT L2BE8
E791 70 03      BVS LE796
E793          LE793:
E793 4C 7B E6   JMP LE67B
E796          LE796:
E796 24 4C      BIT L4C
E798 30 0D      BMI LE7A7
E79A          LE79A:
E79A A5 56      LDA L56
E79C C9 04      CMP #$4
E79E 90 F3      BCC LE793
E7A0          LE7A0:
E7A0 AD 03 02   LDA L203
E7A3 8D E9 2B   STA L2BE9
E7A6 60         RTS
E7A7          LE7A7:
E7A7 AD E9 2B   LDA L2BE9
E7AA 4C 10 E4   JMP LE410
E7AD          LE7AD:
E7AD CE 05 02   DEC L205
E7B0 D0 03      BNE LE7B5
E7B2          LE7B2:
E7B2 68         PLA
E7B3 68         PLA
E7B4 60         RTS
E7B5          LE7B5:
E7B5 EE 04 02   INC L204
E7B8 AD 04 02   LDA L204
E7BB 24 4C      BIT L4C
E7BD 10 0D      BPL LE7CC
E7BF          LE7BF:
E7BF C9 28      CMP #$28
E7C1 90 08      BCC LE7CB
E7C3          LE7C3:
E7C3 A9 00      LDA #$0
E7C5 8D 04 02   STA L204
E7C8          LE7C8:
E7C8 EE 03 02   INC L203
E7CB          LE7CB:
E7CB 60         RTS
E7CC          LE7CC:
E7CC C9 0B      CMP #$B
E7CE 90 FB      BCC LE7CB
E7D0          LE7D0:
E7D0 A9 01      LDA #$1
E7D2 8D 04 02   STA L204
E7D5 A5 4C      LDA L4C
E7D7 49 10      EOR #$10
E7D9 85 4C      STA L4C
E7DB 29 10      AND #$10
E7DD F0 E9      BEQ LE7C8
E7DF          LE7DF:
E7DF 60         RTS
E7E0          LE7E0:
E7E0 CE 05 02   DEC L205
E7E3 D0 03      BNE LE7E8
E7E5          LE7E5:
E7E5 68         PLA
E7E6 68         PLA
E7E7 60         RTS
E7E8          LE7E8:
E7E8 2C E8 2B   BIT L2BE8
E7EB 50 21      BVC LE80E
E7ED          LE7ED:
E7ED A2 00      LDX #$0
E7EF AD 03 02   LDA L203
E7F2          LE7F2:
E7F2 DD C3 EA   CMP LEAC3,X
E7F5 90 03      BCC LE7FA
E7F7          LE7F7:
E7F7 E8         INX
E7F8 D0 F8      BNE LE7F2
E7FA          LE7FA:
E7FA CA         DEX
E7FB AD 04 02   LDA L204
E7FE 18         CLC
E7FF 6D E9 2B   ADC L2BE9
E802 DD DC EA   CMP LEADC,X
E805 90 03      BCC LE80A
E807          LE807:
E807 FD DC EA   SBC LEADC,X
E80A          LE80A:
E80A 8D 04 02   STA L204
E80D 60         RTS
E80E          LE80E:
E80E EE 04 02   INC L204
E811 D0 08      BNE LE81B
E813          LE813:
E813 EE 03 02   INC L203
E816 D0 03      BNE LE81B
E818          LE818:
E818 EE 03 02   INC L203
E81B          LE81B:
E81B 60         RTS
E81C          LE81C:
E81C 20 25 E8   JSR LE825
E81F B0 01      BCS LE822
E821          LE821:
E821 60         RTS
E822          LE822:
E822 4C 36 FF   JMP LFF36
E825          LE825:
E825 08         PHP
E826 78         SEI
E827 E0 20      CPX #$20
E829 90 06      BCC LE831
E82B          LE82B:
E82B A9 0E      LDA #$E
E82D 28         PLP
E82E C9 02      CMP #$2
E830 60         RTS
E831          LE831:
E831 95 20      STA L20,X
E833 9D 60 29   STA L2960,X
E836 AD 61 2A   LDA L2A61
E839 29 3F      AND #$3F
E83B 8D 62 2A   STA L2A62
E83E          LE83E:
E83E 98         TYA
E83F 48         PHA
E840 8A         TXA
E841 48         PHA
E842 20 60 E8   JSR LE860
E845 68         PLA
E846 AA         TAX
E847 68         PLA
E848 A8         TAY
E849 B5 20      LDA L20,X
E84B C9 02      CMP #$2
E84D B0 04      BCS LE853
E84F          LE84F:
E84F 28         PLP
E850 C9 02      CMP #$2
E852 60         RTS
E853          LE853:
E853 CE 62 2A   DEC L2A62
E856 30 F7      BMI LE84F
E858          LE858:
E858 BD 60 29   LDA L2960,X
E85B 95 20      STA L20,X
E85D 4C 3E E8   JMP LE83E
E860          LE860:
E860 08         PHP
E861 78         SEI
E862 20 8C E8   JSR LE88C
E865 A2 00      LDX #$0
E867          LE867:
E867 B5 20      LDA L20,X
E869 10 17      BPL LE882
E86B          LE86B:
E86B 8D 56 2A   STA L2A56
E86E 8E 57 2A   STX L2A57
E871 4A         LSR A
E872 A9 C2      LDA #$C2
E874 B0 03      BCS LE879
E876          LE876:
E876 20 24 E9   JSR LE924
E879          LE879:
E879 20 14 EC   JSR LEC14
E87C 20 DF E8   JSR LE8DF
E87F AE 57 2A   LDX L2A57
E882          LE882:
E882 E8         INX
E883 E0 20      CPX #$20
E885 90 E0      BCC LE867
E887          LE887:
E887 20 FB E8   JSR LE8FB
E88A 28         PLP
E88B 60         RTS
E88C          LE88C:
E88C 20 7E B0   JSR LB07E
E88F A2 00      LDX #$0
E891 C9 01      CMP #$1
E893 F0 3E      BEQ LE8D3
E895          LE895:
E895 C9 04      CMP #$4
E897 90 20      BCC LE8B9
E899          LE899:
E899 C9 06      CMP #$6
E89B B0 36      BCS LE8D3
E89D          LE89D:
E89D B5 02      LDA L2,X
E89F 10 11      BPL LE8B2
E8A1          LE8A1:
E8A1 95 20      STA L20,X
E8A3 8A         TXA
E8A4 0A         ASL A
E8A5 A8         TAY
E8A6 B9 0B 00   LDA LB,Y
E8A9 99 00 28   STA L2800,Y
E8AC B9 0C 00   LDA LC,Y
E8AF 99 01 28   STA L2801,Y
E8B2          LE8B2:
E8B2 E8         INX
E8B3 E0 0B      CPX #$B
E8B5 90 E6      BCC LE89D
E8B7          LE8B7:
E8B7 B0 1A      BCS LE8D3
E8B9          LE8B9:
E8B9 B5 00      LDA L0,X
E8BB 10 11      BPL LE8CE
E8BD          LE8BD:
E8BD 95 20      STA L20,X
E8BF 8A         TXA
E8C0 0A         ASL A
E8C1 A8         TAY
E8C2 B9 06 00   LDA L6,Y
E8C5 99 00 28   STA L2800,Y
E8C8 B9 07 00   LDA L7,Y
E8CB 99 01 28   STA L2801,Y
E8CE          LE8CE:
E8CE E8         INX
E8CF          LE8CF:
E8CF E0 05      CPX #$5
E8D1 90 E6      BCC LE8B9
E8D3          LE8D3:
E8D3 A2 0A      LDX #$A
E8D5          LE8D5:
E8D5 B5 00      LDA L0,X
E8D7 29 7F      AND #$7F
E8D9 95 00      STA L0,X
E8DB CA         DEX
E8DC 10 F7      BPL LE8D5
E8DE          LE8DE:
E8DE 60         RTS
E8DF          LE8DF:
E8DF 20 7E B0   JSR LB07E
E8E2 AE 57 2A   LDX L2A57
E8E5 C9 01      CMP #$1
E8E7          LE8E7:
E8E7 F0 11      BEQ LE8FA
E8E9          LE8E9:
E8E9 C9 04      CMP #$4
E8EB 90 09      BCC LE8F6
E8ED          LE8ED:
E8ED C9 06      CMP #$6
E8EF B0 09      BCS LE8FA
E8F1          LE8F1:
E8F1 B5 20      LDA L20,X
E8F3 95 02      STA L2,X
E8F5 60         RTS
E8F6          LE8F6:
E8F6 B5 20      LDA L20,X
E8F8 95 00      STA L0,X
E8FA          LE8FA:
E8FA 60         RTS
E8FB          LE8FB:
E8FB A9 02      LDA #$2
E8FD 25 49      AND L49
E8FF F0 14      BEQ LE915
E901          LE901:
E901 CE 60 2A   DEC L2A60
E904 D0 0D      BNE LE913
E906          LE906:
E906 A9 19      LDA #$19
E909          LE909 = * + 1
              ; Instruction parameter jumped to.
E908 8D 60 2A   STA L2A60
E90B AD 00 8F   LDA LED
E90E 49 02      EOR #$2
E910 8D 00 8F   STA LED
E913          LE913:
E913 A9 02      LDA #$2
E915          LE915:
E915 09 20      ORA #$20
E917 2D 00 8F   AND LED
E91A 45 49      EOR L49
E91C 49 DF      EOR #$DF
E91E 29 EF      AND #$EF
E920 8D 00 8F   STA LED
E923 60         RTS
E924          LE924:
E924 A2 2A      LDX #$2A
E926 AD 56 2A   LDA L2A56
E929          LE929:
E92B          LE92B = * + 2
              ; Instruction parameter jumped to.
E929 DD 44 E9   CMP LE944,X
E92C          LE92C:
E92D          LE92D = * + 1
              ; Instruction parameter jumped to.
E92C F0 06      BEQ LE934
E92E          LE92E:
E92E CA         DEX
E92F 10 F8      BPL LE929
E931          LE931:
E931 A9 C1      LDA #$C1
E933 60         RTS
E934          LE934:
E934 8A         TXA
E935 0A         ASL A
E936 AA         TAX
E937 BD 6F E9   LDA LE96F,X
E93A 85 E8      STA LE8
E93C BD 70 E9   LDA LE970,X
E93F 85 E9      STA LE9
E941 6C E8 00   JMP (LE8)
E944          LE944:
E944 80         .BYTE $80
E945          LE945:
E945 90 A0      BCC LE8E7
E947          LE947:
E947 B0 C0      BCS LE909
E949          LE949:
E949 D0 E0      BNE LE92B
E94B          LE94B:
E94B F0 82      BEQ LE8CF
E94D 84 86 88   .BYTE $84,$86,$88
E950 8A 8C 8E   .BYTE $8A,$8C,$8E
E953 92 94 96   .BYTE $92,$94,$96
E956 98 9A 9C   .BYTE $98,$9A,$9C
E959 9E A2 A4   .BYTE $9E,$A2,$A4
E95C A6 A8 AA   .BYTE $A6,$A8,$AA
E95F AC B2      .WORD LB2AC
E961 B4 B6      .WORD LB6B4
E963 B8 CC CE   .BYTE $B8,$CC,$CE
E966 EC EE F2   .BYTE $EC,$EE,$F2
E969 F4 F6 F8   .BYTE $F4,$F6,$F8
E96C FA FC FE   .BYTE $FA,$FC,$FE
E96F          LE96F:
E970          LE970 = * + 1
E96F 05 ED      .WORD LED05
E971 23 ED      .WORD LED23
E973 43 ED      .WORD LED43
E975 20 ED      .WORD LED20
E977 68 ED      .WORD LED68
E979 79 ED      .WORD LED79
E97B 79 ED      .WORD LED79
E97D 7F ED      .WORD LED7F
E97F 74 EC      .BYTE $74,$EC
E981 20 ED      .WORD LED20
E983 20 ED      .WORD LED20
E985 20 ED      .WORD LED20
E987 20 ED      .WORD LED20
E989 20 ED      .WORD LED20
E98B 20 ED      .WORD LED20
E98D 20 ED      .WORD LED20
E98F 3C EE      .WORD LEE3C
E991 4D EE      .WORD LEE4D
E993 2C EE      .WORD LEE2C
E995 42 EE      .WORD LEE42
E997 20 ED      .WORD LED20
E999 20 ED      .WORD LED20
E99B 20 ED      .WORD LED20
E99D 85 ED      .WORD LED85
E99F 9E ED      .WORD LED9E
E9A1 5C ED      .WORD LED5C
E9A3 C2 EC      .WORD LECC2
E9A5 D9 EC      .WORD LECD9
E9A7 F9 ED      .WORD LEDF9
E9A9 02 EE      .WORD LEE02
E9AB 56 EE      .WORD LEE56
E9AD 4B ED      .WORD LED4B
E9AF 9E EC      .WORD LEC9E
E9B1 A9 EC      .WORD LECA9
E9B3 A4 ED A1   .BYTE $A4,$ED,$A1
E9B6 ED FB F0   .BYTE $ED,$FB,$F0
E9B9 3D EF 3A   .BYTE $3D,$EF,$3A
E9BC EF 14      .BYTE $EF,$14
E9BE          LE9BE:
E9BE EE 17 EE   INC LEE17
E9C1 AC ED A9   LDY LA9ED
E9C5          LE9C5 = * + 1
              ; Instruction parameter jumped to.
E9C6          LE9C6 = * + 2
              ; Instruction parameter jumped to.
E9C4 ED 38 24   SBC L2438
E9C7          LE9C7:
E9C7 18         CLC
E9C8 6E 5C 2A   ROR L2A5C
E9CB 20 7B EA   JSR LEA7B
E9CE          LE9CE:
E9CE 20 70 EA   JSR LEA70
E9D1 20 93 EA   JSR LEA93
E9D4 90 04      BCC LE9DA
E9D6          LE9D6:
E9D6 A9 C0      LDA #$C0
E9D8 38         SEC
E9D9 60         RTS
E9DA          LE9DA:
E9DA AC 5E 2A   LDY L2A5E
E9DD AD 5A 2A   LDA L2A5A
E9E0 D9 00 83   CMP Partition_SizeHi+$00,Y
E9E3 90 0A      BCC LE9EF
E9E5          LE9E5:
E9E5 D0 EF      BNE LE9D6
E9E7          LE9E7:
E9E7 AD 5B 2A   LDA L2A5B
E9EA D9 00 86   CMP Partition_SizeLo+$00,Y
E9ED B0 E7      BCS LE9D6
E9EF          LE9EF:
E9EF 18         CLC
E9F0 AD 5B 2A   LDA L2A5B
E9F3 79 00 8B   ADC Partition_StartLo+$00,Y
E9F7          LE9F7 = * + 1
              ; Instruction parameter jumped to.
E9F6 8D 65 2A   STA L2A65
E9F9 AD 5A 2A   LDA L2A5A
E9FC 79 00 8A   ADC Partition_StartMi+$00,Y
E9FF 8D 64 2A   STA L2A64
EA02 A9 00      LDA #$0
EA04 79 00 87   ADC Partition_StartHi+$00,Y
EA07 8D 63 2A   STA L2A63
EA0A          LEA0A:
EA0A A0 FF      LDY #$FF
EA0C          LEA0C:
EA0C C8         INY
EA0D AD 63 2A   LDA L2A63
EA10 D9 38 90   CMP L9038,Y
EA13 90 14      BCC LEA29
EA15          LEA15:
EA15 D0 F5      BNE LEA0C
EA17          LEA17:
EA17 AD 64 2A   LDA L2A64
EA1A D9 70 90   CMP L9070,Y
EA1D 90 0A      BCC LEA29
EA1F          LEA1F:
EA1F D0 EB      BNE LEA0C
EA21          LEA21:
EA21 AD 65 2A   LDA L2A65
EA24 D9 A8 90   CMP L90A8,Y
EA27 B0 E3      BCS LEA0C
EA29          LEA29:
EA29 88         DEY
EA2A B9 00 90   LDA L9000,Y
EA2D 30 A7      BMI LE9D6
EA2F          LEA2F:
EA2F AE 57 2A   LDX L2A57
EA32 20 5F EA   JSR LEA5F
EA35 38         SEC
EA36 AD 65 2A   LDA L2A65
EA39 F9 A8 90   SBC L90A8,Y
EA3C 9D 40 29   STA L2940,X
EA3F AD 64 2A   LDA L2A64
EA42 F9 70 90   SBC L9070,Y
EA45 9D 20 29   STA L2920,X
EA48 AD 63 2A   LDA L2A63
EA4B F9 38 90   SBC L9038,Y
EA4E 9D 00 29   STA L2900,X
EA51          LEA51:
EA51 A9 00      LDA #$0
EA53 85 66      STA L66
EA55 AD 57 2A   LDA L2A57
EA58 18         CLC
EA59 69 03      ADC #$3
EA5B 85 67      STA L67
EA5D 18         CLC
EA5E          LEA5E:
EA5E 60         RTS
EA5F          LEA5F:
EA5F 48         PHA
EA60 29 07      AND #$7
EA62 9D E0 28   STA L28E0,X
EA65 68         PLA
EA66 4A         LSR A
EA67 4A         LSR A
EA68 4A         LSR A
EA69 4A         LSR A
EA6A 29 07      AND #$7
EA6C 9D C0 28   STA L28C0,X
EA6F 60         RTS
EA70          LEA70:
EA70 AE 57 2A   LDX L2A57
EA73 AD E8 90   LDA L90E8
EA76 8D 5E 2A   STA L2A5E
EA79 A8         TAY
EA7A 60         RTS
EA7B          LEA7B:
EA7B AD 57 2A   LDA L2A57
EA7E 0A         ASL A
EA7F AA         TAX
EA80 BD 00 28   LDA L2800,X
EA83 8D 58 2A   STA L2A58
EA86 BD 01 28   LDA L2801,X
EA89 8D 59 2A   STA L2A59
EA8C BD 40 28   LDA L2840,X
EA8F 8D 5F 2A   STA L2A5F
EA92 60         RTS
EA93          LEA93:
EA93 AC 5E 2A   LDY L2A5E
EA96 B9 00 82   LDA Partition_Typ+$00,Y
EA99 F0 C3      BEQ LEA5E
EA9B          LEA9B:
EA9B C9 FF      CMP #$FF
EA9D D0 02      BNE LEAA1
EA9F          LEA9F:
EA9F A9 00      LDA #$0
EAA1          LEAA1:
EAA1 0A         ASL A
EAA2 AA         TAX
EAA3 BD B3 EA   LDA LEAB3,X
EAA6 85 E8      STA LE8
EAA8 BD B4 EA   LDA LEAB4,X
EAAB 85 E9      STA LE9
EAAD 2C 5C 2A   BIT L2A5C
EAB0 6C E8 00   JMP (LE8)
EAB3          LEAB3:
EAB4          LEAB4 = * + 1
EAB3 E4 EA      .BYTE $E4,$EA
EAB5 FD EA      .WORD LEAFD
EAB7 09 EB      .WORD LEB09
EAB9 16 EB      .WORD LEB16
EABB 79 EB      .WORD LEB79
EABD 58 EB      .WORD LEB58
EABF E4 EA E4   .BYTE $E4,$EA,$E4
EAC3          LEAC3 = * + 1
EAC2 EA 01 12   .BYTE $EA,$1,$12
EAC5 19 1F 24   .BYTE $19,$1F,$24
EAC8 35 3C 42   .BYTE $35,$3C,$42
EACC          LEACC = * + 1
EACB 47 00 01   .BYTE $47,$0,$1
EACE 01 02 02   .BYTE $1,$2,$2
EAD1 04 04      .BYTE $4,$4
EAD3          LEAD3:
EAD4          LEAD4 = * + 1
EAD3 05 00      ORA L0
EAD5 65 EA      ADC LEA
EAD7 56 AB      LSR LAB,X
EAD9 10 95      BPL LEA70
EADC          LEADC = * + 1
EADB 01 15 13   .BYTE $1,$15,$13
EADE 12 11 15   .BYTE $12,$11,$15
EAE1 13 12      .BYTE $13,$12
EAE3          LEAE3:
EAE3 11 30      ORA (L30),Y
EAE5 09 AD      ORA #$AD
EAE7 58         CLI
EAE8 2A         ROL A
EAE9          LEAE9:
EAE9 20 F2 EA   JSR LEAF2
EAEC 4C 94 EB   JMP LEB94
EAEF          LEAEF:
EAEF AD 58 2A   LDA L2A58
EAF2          LEAF2:
EAF2 8D 5A 2A   STA L2A5A
EAF5 AD 59 2A   LDA L2A59
EAF8 8D 5B 2A   STA L2A5B
EAFB 18         CLC
EAFC 60         RTS
EAFD          LEAFD:
EAFD 30 F0      BMI LEAEF
EAFF          LEAFF:
EAFF AE 58 2A   LDX L2A58
EB02 F0 10      BEQ LEB14
EB04          LEB04:
EB04 CA         DEX
EB05 8A         TXA
EB06 4C E9 EA   JMP LEAE9
EB09          LEB09:
EB09 30 09      BMI LEB14
EB0B          LEB0B:
EB0B AD 58 2A   LDA L2A58
EB0E F0 04      BEQ LEB14
EB10          LEB10:
EB10 C9 24      CMP #$24
EB12 90 0D      BCC LEB21
EB14          LEB14:
EB14 38         SEC
EB15 60         RTS
EB16          LEB16:
EB16 30 FC      BMI LEB14
EB18          LEB18:
EB18 AD 58 2A   LDA L2A58
EB1B F0 F7      BEQ LEB14
EB1D          LEB1D:
EB1D C9 47      CMP #$47
EB1F B0 F3      BCS LEB14
EB21          LEB21:
EB21 A2 00      LDX #$0
EB23          LEB23:
EB23 DD C3 EA   CMP LEAC3,X
EB26 90 03      BCC LEB2B
EB28          LEB28:
EB28 E8         INX
EB29 D0 F8      BNE LEB23
EB2B          LEB2B:
EB2B CA         DEX
EB2C BD DC EA   LDA LEADC,X
EB2F CD 59 2A   CMP L2A59
EB32 F0 E0      BEQ LEB14
EB34          LEB34:
EB34 90 DE      BCC LEB14
EB36          LEB36:
EB36 8D 66 2A   STA L2A66
EB39 8A         TXA
EB3A 48         PHA
EB3B AD 58 2A   LDA L2A58
EB3E 38         SEC
EB3F FD C3 EA   SBC LEAC3,X
EB42 20 FD EB   JSR LEBFD
EB45 68         PLA
EB46 A8         TAY
EB47 BE CC EA   LDX LEACC,Y
EB4A B9 D4 EA   LDA LEAD4,Y
EB4D A0 00      LDY #$0
EB4F 20 E5 EB   JSR LEBE5
EB52 AD 59 2A   LDA L2A59
EB55 4C 91 EB   JMP LEB91
EB58          LEB58:
EB58 30 47      BMI LEBA1
EB5A          LEB5A:
EB5A AD 56 2A   LDA L2A56
EB5D C9 80      CMP #$80
EB5F D0 1A      BNE LEB7B
EB61          LEB61:
EB61 AD 58 2A   LDA L2A58
EB64 C9 01      CMP #$1
EB66 D0 13      BNE LEB7B
EB68          LEB68:
EB68 AD 59 2A   LDA L2A59
EB6B D0 0E      BNE LEB7B
EB6D          LEB6D:
EB6D A9 28      LDA #$28
EB6F 8D 58 2A   STA L2A58
EB72 A9 05      LDA #$5
EB74 8D 59 2A   STA L2A59
EB77 D0 02      BNE LEB7B
EB79          LEB79:
EB79 30 26      BMI LEBA1
EB7B          LEB7B:
EB7B A9 28      LDA #$28
EB7D 8D 66 2A   STA L2A66
EB80 AE 58 2A   LDX L2A58
EB83 F0 1A      BEQ LEB9F
EB85          LEB85:
EB85 CA         DEX
EB86 8A         TXA
EB87 20 FD EB   JSR LEBFD
EB8A AD 59 2A   LDA L2A59
EB8D C9 28      CMP #$28
EB8F B0 0E      BCS LEB9F
EB91          LEB91:
EB91 20 C4 EB   JSR LEBC4
EB94          LEB94:
EB94 4E 5A 2A   LSR L2A5A
EB97 6E 5B 2A   ROR L2A5B
EB9A 6E 5D 2A   ROR L2A5D
EB9D 18         CLC
EB9E 60         RTS
EB9F          LEB9F:
EB9F 38         SEC
EBA0 60         RTS
EBA1          LEBA1:
EBA1 AD 58 2A   LDA L2A58
EBA4 C9 50      CMP #$50
EBA6 B0 F7      BCS LEB9F
EBA8          LEBA8:
EBA8 A9 14      LDA #$14
EBAA 8D 66 2A   STA L2A66
EBAD AD 58 2A   LDA L2A58
EBB0 20 FD EB   JSR LEBFD
EBB3 AE 59 2A   LDX L2A59
EBB6 CA         DEX
EBB7 8A         TXA
EBB8 C9 0A      CMP #$A
EBBA B0 E3      BCS LEB9F
EBBC          LEBBC:
EBBC AE 5F 2A   LDX L2A5F
EBBF F0 03      BEQ LEBC4
EBC1          LEBC1:
EBC1 18         CLC
EBC2 69 0A      ADC #$A
EBC4          LEBC4:
EBC4 20 E1 EB   JSR LEBE1
EBC7 AD 65 2A   LDA L2A65
EBCA 8D 5B 2A   STA L2A5B
EBCD AD 64 2A   LDA L2A64
EBD0 8D 5A 2A   STA L2A5A
EBD3 18         CLC
EBD4 60         RTS
EBD5          LEBD5:
EBD5 A9 00      LDA #$0
EBD7 8D 65 2A   STA L2A65
EBDA 8D 64 2A   STA L2A64
EBDD 8D 63 2A   STA L2A63
EBE0 60         RTS
EBE1          LEBE1:
EBE1 A2 00      LDX #$0
EBE3 A0 00      LDY #$0
EBE5          LEBE5:
EBE5 18         CLC
EBE6 48         PHA
EBE7 6D 65 2A   ADC L2A65
EBEA 8D 65 2A   STA L2A65
EBED 8A         TXA
EBEE 6D 64 2A   ADC L2A64
EBF1 8D 64 2A   STA L2A64
EBF4 98         TYA
EBF5 6D 63 2A   ADC L2A63
EBF8 8D 63 2A   STA L2A63
EBFB          LEBFB:
EBFB 68         PLA
EBFC 60         RTS
EBFD          LEBFD:
EBFD A2 00      LDX #$0
EBFF A0 00      LDY #$0
EC01 48         PHA
EC02 20 D5 EB   JSR LEBD5
EC05 AD 66 2A   LDA L2A66
EC08 F0 F1      BEQ LEBFB
EC0A          LEC0A:
EC0A 68         PLA
EC0B          LEC0B:
EC0B 20 E5 EB   JSR LEBE5
EC0E CE 66 2A   DEC L2A66
EC11 D0 F8      BNE LEC0B
EC13          LEC13:
EC13 60         RTS
EC14          LEC14:
EC14 C9 02      CMP #$2
EC16 D0 15      BNE LEC2D
EC18          LEC18:
EC18 20 7C EF   JSR LEF7C
EC1B C9 00      CMP #$0
EC1D D0 0E      BNE LEC2D
EC1F          LEC1F:
EC1F AD 13 2A   LDA L2A13
EC22 29 0F      AND #$F
EC24 C9 01      CMP #$1
EC26 F0 03      BEQ LEC2B
EC28          LEC28:
EC28 A9 02      LDA #$2
EC2B          LEC2B = * + 1
              ; Instruction parameter jumped to.
EC2A 2C A9 00   BIT LA9
EC2D          LEC2D:
EC2D A2 00      LDX #$0
EC2F          LEC2F:
EC2F DD 5E EC   CMP LEC5E,X
EC32 F0 09      BEQ LEC3D
EC34          LEC34:
EC34 E8         INX
EC35 E0 0B      CPX #$B
EC37 90 F6      BCC LEC2F
EC39          LEC39:
EC39 A9 0D      LDA #$D
EC3B D0 03      BNE LEC40
EC3D          LEC3D:
EC3D BD 69 EC   LDA LEC69,X
EC40          LEC40:
EC40 AE 57 2A   LDX L2A57
EC43 C9 00      CMP #$0
EC45 F0 14      BEQ LEC5B
EC47          LEC47:
EC47 48         PHA
EC48 AD 11 2A   LDA L2A11
EC4B 9D 00 29   STA L2900,X
EC4E AD 13 2A   LDA L2A13
EC51 9D 20 29   STA L2920,X
EC54 AD 1D 2A   LDA L2A1D
EC57 9D 40 29   STA L2940,X
EC5A 68         PLA
EC5B          LEC5B:
EC5B 95 20      STA L20,X
EC5D 60         RTS
EC5E          LEC5E:
EC5E 00 02      .BYTE $0,$2
EC60          LEC60:
EC60 08         PHP
EC61 10 18      BPL LEC7B
EC63 85 86 87   .BYTE $85,$86,$87
EC66 C0 C1 C3   .BYTE $C0,$C1,$C3
EC69          LEC69:
EC69 00 02 03   .BYTE $0,$2,$3
EC6C 0B 0C 05   .BYTE $B,$C,$5
EC6F 06 07 04   .BYTE $6,$7,$4
EC72 0E         .BYTE $E
EC73          LEC73:
EC73 08         PHP
EC74 A9 20      LDA #$20
EC76 8D 06 80   STA VIA1+$06
EC79 A9 4E      LDA #$4E
EC7B          LEC7B:
EC7B 8D 07 80   STA VIA1+$07
EC7E 8D 05 80   STA VIA1+$05
EC81 AD 0B 80   LDA VIA1+$0B
EC84 09 40      ORA #$40
EC86 8D 0B 80   STA VIA1+$0B
EC89 A9 FF      LDA #$FF
EC8B 8D 50 2A   STA L2A50
EC8E A9 19      LDA #$19
EC90 8D 60 2A   STA L2A60
EC93 A9 01      LDA #$1
EC95 8D 61 2A   STA L2A61
EC98 20 80 F1   JSR LF180
EC9B A9 00      LDA #$0
EC9D 60         RTS
EC9E          LEC9E:
EC9E 20 C7 E9   JSR LE9C7
ECA1 B0 35      BCS LECD8
ECA3          LECA3:
ECA3 20 B4 EC   JSR LECB4
ECA6 4C 0A ED   JMP LED0A
ECA9          LECA9:
ECA9 20 C7 E9   JSR LE9C7
ECAC B0 2A      BCS LECD8
ECAE          LECAE:
ECAE 20 B4 EC   JSR LECB4
ECB1 4C 28 ED   JMP LED28
ECB4          LECB4:
ECB4 AE 57 2A   LDX L2A57
ECB7 BD 80 28   LDA L2880,X
ECBA 85 66      STA L66
ECBC BD 60 28   LDA L2860,X
ECBF 85 67      STA L67
ECC1 60         RTS
ECC2          LECC2:
ECC2 20 C7 E9   JSR LE9C7
ECC5 B0 11      BCS LECD8
ECC7          LECC7:
ECC7 20 78 EE   JSR LEE78
ECCA F0 07      BEQ LECD3
ECCC          LECCC:
ECCC A9 08      LDA #$8
ECCE          LECCE:
ECCE 20 A2 EE   JSR LEEA2
ECD1 D0 05      BNE LECD8
ECD3          LECD3:
ECD3 20 68 EE   JSR LEE68
ECD6 A9 00      LDA #$0
ECD8          LECD8:
ECD8 60         RTS
ECD9          LECD9:
ECD9 20 C7 E9   JSR LE9C7
ECDC B0 FA      BCS LECD8
ECDE          LECDE:
ECDE 20 68 EE   JSR LEE68
ECE1 20 78 EE   JSR LEE78
ECE4 F0 1B      BEQ LED01
ECE6          LECE6:
ECE6 A0 00      LDY #$0
ECE8          LECE8:
ECE8 B1 68      LDA (L68),Y
ECEA 99 00 52   STA L5200,Y
ECED C8         INY
ECEE D0 F8      BNE LECE8
ECF0          LECF0:
ECF0 20 CC EC   JSR LECCC
ECF3 C9 00      CMP #$0
ECF5 D0 E1      BNE LECD8
ECF7          LECF7:
ECF7 A0 00      LDY #$0
ECF9          LECF9:
ECF9 B9 00 52   LDA L5200,Y
ECFC 91 68      STA (L68),Y
ECFE C8         INY
ECFF D0 F8      BNE LECF9
ED01          LED01:
ED01 A9 0A      LDA #$A
ED03 D0 C9      BNE LECCE
ED05          LED05:
ED05 20 C7 E9   JSR LE9C7
ED08 B0 18      BCS LED22
ED0A          LED0A:
ED0A 20 78 EE   JSR LEE78
ED0D F0 07      BEQ LED16
ED0F          LED0F:
ED0F A9 08      LDA #$8
ED11 20 A2 EE   JSR LEEA2
ED14 D0 0C      BNE LED22
ED16          LED16:
ED16 20 68 EE   JSR LEE68
ED19          LED19:
ED19 B1 68      LDA (L68),Y
ED1B 91 66      STA (L66),Y
ED1D C8         INY
ED1E D0 F9      BNE LED19
ED20          LED20:
ED20 A9 00      LDA #$0
ED22          LED22:
ED22 60         RTS
ED23          LED23:
ED23 20 C7 E9   JSR LE9C7
ED26 B0 22      BCS LED4A
ED28          LED28:
ED28 20 78 EE   JSR LEE78
ED2B F0 07      BEQ LED34
ED2D          LED2D:
ED2D A9 08      LDA #$8
ED2F 20 A2 EE   JSR LEEA2
ED32 D0 16      BNE LED4A
ED34          LED34:
ED34 20 68 EE   JSR LEE68
ED37          LED37:
ED37 B1 66      LDA (L66),Y
ED39 91 68      STA (L68),Y
ED3B C8         INY
ED3C D0 F9      BNE LED37
ED3E          LED3E:
ED3E A9 0A      LDA #$A
ED40 4C A2 EE   JMP LEEA2
ED43          LED43:
ED43 20 C7 E9   JSR LE9C7
ED46 B0 02      BCS LED4A
ED48          LED48:
ED48 A9 00      LDA #$0
ED4A          LED4A:
ED4A 60         RTS
ED4B          LED4B:
ED4B 20 7B EA   JSR LEA7B
ED4E A9 00      LDA #$0
ED50 8D 59 2A   STA L2A59
ED53 4E 5C 2A   LSR L2A5C
ED56 20 CE E9   JSR LE9CE
ED59 90 06      BCC LED61
ED5B          LED5B:
ED5B 60         RTS
ED5C          LED5C:
ED5C 20 C5 E9   JSR LE9C5
ED5F B0 FA      BCS LED5B
ED61          LED61:
ED61 A9 0B      LDA #$B
ED63 A0 00      LDY #$0
ED65 4C 46 EF   JMP LEF46
ED68          LED68:
ED68 20 70 EA   JSR LEA70
ED6B A9 00      LDA #$0
ED6D 8D 5A 2A   STA L2A5A
ED70 8D 5B 2A   STA L2A5B
ED73 20 DA E9   JSR LE9DA
ED76 90 E9      BCC LED61
ED78          LED78:
ED78 60         RTS
ED79          LED79:
ED79 20 51 EA   JSR LEA51
ED7C 6C 66 00   JMP (L66)
ED7F          LED7F:
ED7F 20 51 EA   JSR LEA51
ED82 A9 00      LDA #$0
ED84 60         RTS
ED85          LED85:
ED85 20 8B ED   JSR LED8B
ED88 4C AC ED   JMP LEDAC
ED8B          LED8B:
ED8B AE 57 2A   LDX L2A57
ED8E A9 03      LDA #$3
ED90 9D 60 28   STA L2860,X
ED93 A9 00      LDA #$0
ED95 9D 80 28   STA L2880,X
ED98 A9 01      LDA #$1
ED9A 9D A0 28   STA L28A0,X
ED9D 60         RTS
ED9E          LED9E:
ED9E 20 8B ED   JSR LED8B
EDA1 A0 0A      LDY #$A
EDA3 2C A0 08   BIT L8A0
EDA6 38         SEC
EDA7 B0 06      BCS LEDAF
EDA9          LEDA9:
EDA9 A0 0A      LDY #$A
EDAC          LEDAC = * + 1
              ; Instruction parameter jumped to.
EDAB 2C A0 08   BIT L8A0
EDAE 18         CLC
EDAF          LEDAF:
EDAF AE 57 2A   LDX L2A57
EDB2 BD 60 28   LDA L2860,X
EDB5 48         PHA
EDB6 BD 80 28   LDA L2880,X
EDB9 48         PHA
EDBA 98         TYA
EDBB 48         PHA
EDBC BD A0 28   LDA L28A0,X
EDBF 48         PHA
EDC0 90 1B      BCC LEDDD
EDC2          LEDC2:
EDC2 BD 40 28   LDA L2840,X
EDC5 8D 65 2A   STA L2A65
EDC8 8A         TXA
EDC9 0A         ASL A
EDCA AA         TAX
EDCB BD 01 28   LDA L2801,X
EDCE 8D 64 2A   STA L2A64
EDD1 BD 00 28   LDA L2800,X
EDD4 8D 63 2A   STA L2A63
EDD7 20 0A EA   JSR LEA0A
EDDA 4C E0 ED   JMP LEDE0
EDDD          LEDDD:
EDDD 20 C5 E9   JSR LE9C5
EDE0          LEDE0:
EDE0 90 07      BCC LEDE9
EDE2          LEDE2:
EDE2 68         PLA
EDE3 68         PLA
EDE4 68         PLA
EDE5 68         PLA
EDE6 A9 C0      LDA #$C0
EDE8 60         RTS
EDE9          LEDE9:
EDE9 68         PLA
EDEA A8         TAY
EDEB 68         PLA
EDEC 38         SEC
EDED 20 D2 EE   JSR LEED2
EDF0 68         PLA
EDF1 85 68      STA L68
EDF3 68         PLA
EDF4 85 69      STA L69
EDF6 4C 4A EF   JMP LEF4A
EDF9          LEDF9:
EDF9 20 C5 E9   JSR LE9C5
EDFC B0 15      BCS LEE13
EDFE          LEDFE:
EDFE A9 08      LDA #$8
EE00 D0 07      BNE LEE09
EE02          LEE02:
EE02 20 C5 E9   JSR LE9C5
EE05 B0 0C      BCS LEE13
EE07          LEE07:
EE07 A9 0A      LDA #$A
EE09          LEE09:
EE09 20 A2 EE   JSR LEEA2
EE0C D0 05      BNE LEE13
EE0E          LEE0E:
EE0E 20 5F EE   JSR LEE5F
EE11 A9 00      LDA #$0
EE13          LEE13:
EE13 60         RTS
EE14          LEE14:
EE14 A0 01      LDY #$1
EE17          LEE17 = * + 1
              ; Instruction parameter accessed.
EE16 2C A0 00   BIT LA0
EE19 A9 00      LDA #$0
EE1B AE 57 2A   LDX L2A57
EE1E 9D 00 29   STA L2900,X
EE21 9D 20 29   STA L2920,X
EE24 9D 40 29   STA L2940,X
EE27 A9 1B      LDA #$1B
EE29 4C 46 EF   JMP LEF46
EE2C          LEE2C:
EE2C A9 50      LDA #$50
EE2E 8D DE 2B   STA L2BDE
EE31 A9 32      LDA #$32
EE33 8D 60 2A   STA L2A60
EE36 A9 02      LDA #$2
EE38 2C A9 40   BIT L40A9
EE3C          LEE3C = * + 1
              ; Instruction parameter jumped to.
EE3B 2C A9 01   BIT L1A9
EE3E 05 49      ORA L49
EE40 D0 0F      BNE LEE51
EE42          LEE42:
EE42 A9 00      LDA #$0
EE44 8D DE 2B   STA L2BDE
EE47 A9 FD      LDA #$FD
EE49 2C A9 BF   BIT LBFA9
EE4D          LEE4D = * + 1
              ; Instruction parameter jumped to.
EE4C 2C A9 FE   BIT LFEA9
EE4F 25 49      AND L49
EE51          LEE51:
EE51 85 49      STA L49
EE53          LEE53:
EE53 A9 00      LDA #$0
EE55 60         RTS
EE56          LEE56:
EE56 A9 80      LDA #$80
EE58 25 49      AND L49
EE5A F0 F7      BEQ LEE53
EE5C          LEE5C:
EE5C A9 C3      LDA #$C3
EE5E 60         RTS
EE5F          LEE5F:
EE5F A0 00      LDY #$0
EE61 84 68      STY L68
EE63 A9 50      LDA #$50
EE65 85 69      STA L69
EE67 60         RTS
EE68          LEE68:
EE68 A0 00      LDY #$0
EE6A 84 68      STY L68
EE6C A9 50      LDA #$50
EE6E 85 69      STA L69
EE70 2C 5D 2A   BIT L2A5D
EE73 10 02      BPL LEE77
EE75          LEE75:
EE75 E6 69      INC L69
EE77          LEE77:
EE77 60         RTS
EE78          LEE78:
EE78 AE 57 2A   LDX L2A57
EE7B BD C0 28   LDA L28C0,X
EE7E CD 50 2A   CMP L2A50
EE81 D0 1E      BNE LEEA1
EE83          LEE83:
EE83 BD E0 28   LDA L28E0,X
EE86 CD 51 2A   CMP L2A51
EE89 D0 16      BNE LEEA1
EE8B          LEE8B:
EE8B BD 00 29   LDA L2900,X
EE8E CD 52 2A   CMP L2A52
EE91 D0 0E      BNE LEEA1
EE93          LEE93:
EE93 BD 20 29   LDA L2920,X
EE96 CD 53 2A   CMP L2A53
EE99 D0 06      BNE LEEA1
EE9B          LEE9B:
EE9B BD 40 29   LDA L2940,X
EE9E CD 54 2A   CMP L2A54
EEA1          LEEA1:
EEA1 60         RTS
EEA2          LEEA2:
EEA2 A2 FF      LDX #$FF
EEA4 8E 50 2A   STX L2A50
EEA7 20 44 EF   JSR LEF44
EEAA D0 23      BNE LEECF
EEAC          LEEAC:
EEAC AE 57 2A   LDX L2A57
EEAF BD C0 28   LDA L28C0,X
EEB2 8D 50 2A   STA L2A50
EEB5 BD E0 28   LDA L28E0,X
EEB8 8D 51 2A   STA L2A51
EEBB BD 00 29   LDA L2900,X
EEBE 8D 52 2A   STA L2A52
EEC1 BD 20 29   LDA L2920,X
EEC4 8D 53 2A   STA L2A53
EEC7 BD 40 29   LDA L2940,X
EECA 8D 54 2A   STA L2A54
EECD A9 00      LDA #$0
EECF          LEECF:
EECF 4C 76 EF   JMP LEF76
EED2          LEED2:
EED2 08         PHP
EED3 48         PHA
EED4 20 07 EF   JSR LEF07
EED7 68         PLA
EED8 8D 00 2A   STA L2A00
EEDB A9 00      LDA #$0
EEDD AE 57 2A   LDX L2A57
EEE0 8C 04 2A   STY L2A04
EEE3 28         PLP
EEE4 90 0F      BCC LEEF5
EEE6          LEEE6:
EEE6 BD 40 29   LDA L2940,X
EEE9 8D 03 2A   STA L2A03
EEEC BD 20 29   LDA L2920,X
EEEF 8D 02 2A   STA L2A02
EEF2 BD 00 29   LDA L2900,X
EEF5          LEEF5:
EEF5 8D 01 2A   STA L2A01
EEF8 BD E0 28   LDA L28E0,X
EEFB 0A         ASL A
EEFC 0A         ASL A
EEFD 0A         ASL A
EEFE 0A         ASL A
EEFF 0A         ASL A
EF00 0D 01 2A   ORA L2A01
EF03 8D 01 2A   STA L2A01
EF06 60         RTS
EF07          LEF07:
EF07 A9 00      LDA #$0
EF09 A2 4F      LDX #$4F
EF0B          LEF0B:
EF0B 9D 00 2A   STA L2A00,X
EF0E CA         DEX
EF0F 10 FA      BPL LEF0B
EF11          LEF11:
EF11 A2 FF      LDX #$FF
EF13 8E 10 2A   STX L2A10
EF16 8E 30 2A   STX L2A30
EF19 A9 00      LDA #$0
EF1B 85 E0      STA LE0
EF1D A9 2A      LDA #$2A
EF1F 85 E1      STA LE1
EF21 A9 10      LDA #$10
EF23 85 E2      STA LE2
EF25 A9 2A      LDA #$2A
EF27 85 E3      STA LE3
EF29 A9 30      LDA #$30
EF2B 85 E4      STA LE4
EF2D A9 2A      LDA #$2A
EF2F 85 E5      STA LE5
EF31 A9 00      LDA #$0
EF33 85 68      STA L68
EF35 A9 50      LDA #$50
EF37 85 69      STA L69
EF39 60         RTS
EF3A          LEF3A:
EF3A A9 01      LDA #$1
EF3C 2C A9 00   BIT LA9
EF3F A0 00      LDY #$0
EF41 18         CLC
EF42 90 03      BCC LEF47
EF44          LEF44:
EF44 A0 01      LDY #$1
EF46          LEF46:
EF46 38         SEC
EF47          LEF47:
EF47 20 D2 EE   JSR LEED2
EF4A          LEF4A:
EF4A AD 00 2A   LDA L2A00
EF4D C9 0A      CMP #$A
EF4F D0 0B      BNE LEF5C
EF51          LEF51:
EF51 A9 80      LDA #$80
EF53 25 49      AND L49
EF55 F0 05      BEQ LEF5C
EF57          LEF57:
EF57 A9 C3      LDA #$C3
EF59 4C 76 EF   JMP LEF76
EF5C          LEF5C:
EF5C AE 57 2A   LDX L2A57
EF5F BD C0 28   LDA L28C0,X
EF62 20 13 F1   JSR LF113
EF65 D0 05      BNE LEF6C
EF67          LEF67:
EF67 A9 85      LDA #$85
EF69 4C 76 EF   JMP LEF76
EF6C          LEF6C:
EF6C 20 97 EF   JSR LEF97
EF6F C9 00      CMP #$0
EF71 D0 03      BNE LEF76
EF73          LEF73:
EF73 AD 10 2A   LDA L2A10
EF76          LEF76:
EF76 8D 10 2A   STA L2A10
EF79 C9 00      CMP #$0
EF7B 60         RTS
EF7C          LEF7C:
EF7C A9 03      LDA #$3
EF7E A0 1B      LDY #$1B
EF80 18         CLC
EF81 20 D2 EE   JSR LEED2
EF84 A9 11      LDA #$11
EF86 85 68      STA L68
EF88 A9 2A      LDA #$2A
EF8A 85 69      STA L69
EF8C 4C 4A EF   JMP LEF4A
EF8F          LEF8F:
EF8F AD 00 8F   LDA LED
EF92 29 EF      AND #$EF
EF94 8D 00 8F   STA LED
EF97          LEF97:
EF97 A9 20      LDA #$20
EF99          LEF99:
EF99 2C 00 84   BIT VIA2+$00
EF9C 70 FB      BVS LEF99
EF9E          LEF9E:
EF9E 30 08      BMI LEFA8
EFA0          LEFA0:
EFA0 D0 F7      BNE LEF99
EFA2          LEFA2:
EFA2 20 DB F0   JSR LF0DB
EFA5 A9 00      LDA #$0
EFA7 60         RTS
EFA8          LEFA8:
EFA8 F0 2B      BEQ LEFD5
EFAA          LEFAA:
EFAA AD 00 84   LDA VIA2+$00
EFAD 29 07      AND #$7
EFAF C9 00      CMP #$0
EFB1 D0 03      BNE LEFB6
EFB3          LEFB3:
EFB3 4C DD EF   JMP LEFDD
EFB6          LEFB6:
EFB6 C9 04      CMP #$4
EFB8 D0 03      BNE LEFBD
EFBA          LEFBA:
EFBA 4C 14 F0   JMP LF014
EFBD          LEFBD:
EFBD C9 01      CMP #$1
EFBF D0 03      BNE LEFC4
EFC1          LEFC1:
EFC1 4C 38 F0   JMP LF038
EFC4          LEFC4:
EFC4 C9 05      CMP #$5
EFC6 D0 03      BNE LEFCB
EFC8          LEFC8:
EFC8 4C 79 F0   JMP LF079
EFCB          LEFCB:
EFCB C9 07      CMP #$7
EFCD D0 03      BNE LEFD2
EFCF          LEFCF:
EFCF 4C AA F0   JMP LF0AA
EFD2          LEFD2:
EFD2 A9 87      LDA #$87
EFD5          LEFD5 = * + 1
              ; Instruction parameter jumped to.
EFD4 2C A9 86   BIT L86A9
EFD7 48         PHA
EFD8 20 FB F0   JSR LF0FB
EFDB 68         PLA
EFDC 60         RTS
EFDD          LEFDD:
EFDD A4 68      LDY L68
EFDF A9 00      LDA #$0
EFE1 85 68      STA L68
EFE3 A9 FF      LDA #$FF
EFE5 8D 03 84   STA VIA2+$03
EFE8 A9 A0      LDA #$A0
EFEA 8D 00 84   STA VIA2+$00
EFED          LEFED:
EFED AD 00 84   LDA VIA2+$00
EFF0 C9 A0      CMP #$A0
EFF2 D0 1B      BNE LF00F
EFF4          LEFF4:
EFF4 B1 68      LDA (L68),Y
EFF6 49 FF      EOR #$FF
EFF8 AA         TAX
EFF9 AD 00 8F   LDA LED
EFFC 29 EF      AND #$EF
EFFE 1D 00 93   ORA L9300,X
F001 8D 00 8F   STA LED
F004 8E 01 84   STX VIA2+$01
F007 C8         INY
F008 D0 E3      BNE LEFED
F00A          LF00A:
F00A E6 69      INC L69
F00C 4C ED EF   JMP LEFED
F00F          LF00F:
F00F 84 68      STY L68
F011 4C 8F EF   JMP LEF8F
F014          LF014:
F014 A4 68      LDY L68
F016 A9 00      LDA #$0
F018 85 68      STA L68
F01A 8D 03 84   STA VIA2+$03
F01D A9 AC      LDA #$AC
F01F 8D 00 84   STA VIA2+$00
F022          LF022:
F022 AD 00 84   LDA VIA2+$00
F025 C9 AC      CMP #$AC
F027 D0 E6      BNE LF00F
F029          LF029:
F029 AD 01 84   LDA VIA2+$01
F02C 49 FF      EOR #$FF
F02E 91 68      STA (L68),Y
F030 C8         INY
F031 D0 EF      BNE LF022
F033          LF033:
F033 E6 69      INC L69
F035 4C 22 F0   JMP LF022
F038          LF038:
F038 09 20      ORA #$20
F03A A0 FF      LDY #$FF
F03C 8C 03 84   STY VIA2+$03
F03F C8         INY
F040 8D 00 84   STA VIA2+$00
F043 8D 55 2A   STA L2A55
F046          LF046:
F046 2C 00 84   BIT VIA2+$00
F049 70 FB      BVS LF046
F04B          LF04B:
F04B AD 55 2A   LDA L2A55
F04E          LF04E:
F04E CD 00 84   CMP VIA2+$00
F051 F0 FB      BEQ LF04E
F053          LF053:
F053 09 80      ORA #$80
F055 CD 00 84   CMP VIA2+$00
F058 D0 1C      BNE LF076
F05A          LF05A:
F05A B1 E0      LDA (LE0),Y
F05C 49 FF      EOR #$FF
F05E AA         TAX
F05F AD 00 8F   LDA LED
F062 29 EF      AND #$EF
F064 1D 00 93   ORA L9300,X
F067 8D 00 8F   STA LED
F06A 8E 01 84   STX VIA2+$01
F06D E6 E0      INC LE0
F06F D0 D5      BNE LF046
F071          LF071:
F071 E6 E1      INC LE1
F073 4C 46 F0   JMP LF046
F076          LF076:
F076 4C 8F EF   JMP LEF8F
F079          LF079:
F079 09 28      ORA #$28
F07B A0 00      LDY #$0
F07D 8C 03 84   STY VIA2+$03
F080 8D 00 84   STA VIA2+$00
F083 8D 55 2A   STA L2A55
F086          LF086:
F086 2C 00 84   BIT VIA2+$00
F089 70 FB      BVS LF086
F08B          LF08B:
F08B AD 55 2A   LDA L2A55
F08E          LF08E:
F08E CD 00 84   CMP VIA2+$00
F091 F0 FB      BEQ LF08E
F093          LF093:
F093 09 80      ORA #$80
F095 CD 00 84   CMP VIA2+$00
F098 D0 DC      BNE LF076
F09A          LF09A:
F09A AD 01 84   LDA VIA2+$01
F09D 49 FF      EOR #$FF
F09F 91 E2      STA (LE2),Y
F0A1 E6 E2      INC LE2
F0A3 D0 E1      BNE LF086
F0A5          LF0A5:
F0A5 E6 E3      INC LE3
F0A7 4C 86 F0   JMP LF086
F0AA          LF0AA:
F0AA 09 28      ORA #$28
F0AC A0 00      LDY #$0
F0AE 8C 03 84   STY VIA2+$03
F0B1 8D 00 84   STA VIA2+$00
F0B4 8D 55 2A   STA L2A55
F0B7          LF0B7:
F0B7 2C 00 84   BIT VIA2+$00
F0BA 70 FB      BVS LF0B7
F0BC          LF0BC:
F0BC AD 55 2A   LDA L2A55
F0BF          LF0BF:
F0BF CD 00 84   CMP VIA2+$00
F0C2 F0 FB      BEQ LF0BF
F0C4          LF0C4:
F0C4 09 80      ORA #$80
F0C6 CD 00 84   CMP VIA2+$00
F0C9 D0 AB      BNE LF076
F0CB          LF0CB:
F0CB AD 01 84   LDA VIA2+$01
F0CE 49 FF      EOR #$FF
F0D0 91 E4      STA (LE4),Y
F0D2 E6 E4      INC LE4
F0D4 D0 E1      BNE LF0B7
F0D6          LF0D6:
F0D6 E6 E5      INC LE5
F0D8 4C B7 F0   JMP LF0B7
F0DB          LF0DB:
F0DB A9 DB      LDA #$DB
F0DD 8D 0C 84   STA VIA2+$0C
F0E0 A9 00      LDA #$0
F0E2 8D 03 84   STA VIA2+$03
F0E5 A9 08      LDA #$8
F0E7 8D 00 84   STA VIA2+$00
F0EA AD 02 88   LDA PIO+$02
F0ED 29 E3      AND #$E3
F0EF 8D 02 88   STA PIO+$02
F0F2 AD 00 8F   LDA LED
F0F5 29 EF      AND #$EF
F0F7 8D 00 8F   STA LED
F0FA 60         RTS
F0FB          LF0FB:
F0FB 20 DB F0   JSR LF0DB
F0FE AD 02 88   LDA PIO+$02
F101 09 08      ORA #$8
F103 8D 02 88   STA PIO+$02
F106 A2 28      LDX #$28
F108          LF108:
F108 CA         DEX
F109 D0 FD      BNE LF108
F10B          LF10B:
F10B 29 F7      AND #$F7
F10D 8D 02 88   STA PIO+$02
F110 A9 00      LDA #$0
F112 60         RTS
F113          LF113:
F113 08         PHP
F114 78         SEI
F115 AA         TAX
F116          LF116:
F116 A9 20      LDA #$20
F118 2D 00 84   AND VIA2+$00
F11B F0 02      BEQ LF11F
F11D          LF11D:
F11D D0 F7      BNE LF116
F11F          LF11F:
F11F 38         SEC
F120          LF120:
F120 2A         ROL A
F121 CA         DEX
F122 10 FC      BPL LF120
F124          LF124:
F124 A2 FF      LDX #$FF
F126 8E 03 84   STX VIA2+$03
F129 0D E5 90   ORA L90E5
F12C 49 FF      EOR #$FF
F12E AA         TAX
F12F AD 00 8F   LDA LED
F132 29 EF      AND #$EF
F134 1D 00 93   ORA L9300,X
F137 8D 00 8F   STA LED
F13A 8E 01 84   STX VIA2+$01
F13D A9 00      LDA #$0
F13F 8D 00 84   STA VIA2+$00
F142 A9 FB      LDA #$FB
F144 A2 10      LDX #$10
F146 8D 0C 84   STA VIA2+$0C
F149 8E 00 84   STX VIA2+$00
F14C A2 00      LDX #$0
F14E A0 00      LDY #$0
F150          LF150:
F150 AD 00 84   LDA VIA2+$00
F153 29 20      AND #$20
F155 D0 15      BNE LF16C
F157          LF157:
F157 CA         DEX
F158 D0 F6      BNE LF150
F15A          LF15A:
F15A 88         DEY
F15B D0 F3      BNE LF150
F15D          LF15D:
F15D A9 DB      LDA #$DB
F15F 8D 0C 84   STA VIA2+$0C
F162 A2 54      LDX #$54
F164          LF164:
F164 CA         DEX
F165 D0 FD      BNE LF164
F167          LF167:
F167 AD 00 84   LDA VIA2+$00
F16A 29 20      AND #$20
F16C          LF16C:
F16C A2 08      LDX #$8
F16E 8E 00 84   STX VIA2+$00
F171 A2 DB      LDX #$DB
F173 8E 0C 84   STX VIA2+$0C
F176 28         PLP
F177 AA         TAX
F178 D0 05      BNE LF17F
F17A          LF17A:
F17A 20 DB F0   JSR LF0DB
F17D A2 00      LDX #$0
F17F          LF17F:
F17F 60         RTS
F180          LF180:
F180 08         PHP
F181 78         SEI
F182 20 14 F7   JSR LF714
F185 A2 00      LDX #$0
F187          LF187:
F187 8A         TXA
F188 8D 65 2A   STA L2A65
F18B 4A         LSR A
F18C 4A         LSR A
F18D 4A         LSR A
F18E 4A         LSR A
F18F 4D 65 2A   EOR L2A65
F192 29 0F      AND #$F
F194 A8         TAY
F195 B9 A3 F1   LDA LF1A3,Y
F198 9D 00 93   STA L9300,X
F19B E8         INX
F19C D0 E9      BNE LF187
F19E          LF19E:
F19E 20 0B F7   JSR LF70B
F1A1 28         PLP
F1A2 60         RTS
F1A3          LF1A3:
F1A3 10 00 00   .BYTE $10,$0,$0
F1A6          LF1A6:
F1A6 10 00      BPL LF1A8
F1A8          LF1A8:
F1A8 10 10      BPL LF1BA
F1AA 00 00 10   .BYTE $0,$0,$10
F1AD 10 00 10   .BYTE $10,$0,$10
F1B0 00 00 10   .BYTE $0,$0,$10
F1B3          LF1B3:
F1B4          LF1B4 = * + 1
              ; Instruction parameter jumped to.
F1B3 09 20      ORA #$20
F1B5          LF1B5:
F1B5 48         PHA
F1B6          LF1B6:
F1B6 78         SEI
F1B7 20 5A 97   JSR L975A
F1BA          LF1BA:
F1BA A9 00      LDA #$0
F1BC 8D 00 80   STA VIA1+$00
F1BF A9 7A      LDA #$7A
F1C1 8D 02 80   STA VIA1+$02
F1C4 68         PLA
F1C5          LF1C5:
F1C5 78         SEI
F1C6 48         PHA
F1C7 20 75 97   JSR L9775
F1CA 20 5A 97   JSR L975A
F1CD 20 8A F2   JSR LF28A
F1D0 A9 00      LDA #$0
F1D2 8D D5 2B   STA L2BD5
F1D5 68         PLA
F1D6          LF1D6:
F1D6 78         SEI
F1D7 8D D4 2B   STA L2BD4
F1DA 20 5A 97   JSR L975A
F1DD AD 00 80   LDA VIA1+$00
F1E0 29 01      AND #$1
F1E2 F0 49      BEQ LF22D
F1E4          LF1E4:
F1E4 20 6C 97   JSR L976C
F1E7 2C D5 2B   BIT L2BD5
F1EA 10 06      BPL LF1F2
F1EC          LF1EC:
F1EC 20 06 F4   JSR LF406
F1EF 20 FF F3   JSR LF3FF
F1F2          LF1F2:
F1F2 20 06 F4   JSR LF406
F1F5 8A         TXA
F1F6 48         PHA
F1F7 20 75 97   JSR L9775
F1FA A2 08      LDX #$8
F1FC          LF1FC:
F1FC A9 14      LDA #$14
F1FE          LF1FE:
F1FE E9 01      SBC #$1
F200 D0 FC      BNE LF1FE
F202          LF202:
F202 6E D4 2B   ROR L2BD4
F205 B0 06      BCS LF20D
F207          LF207:
F207 20 63 97   JSR L9763
F20A 4C 10 F2   JMP LF210
F20D          LF20D:
F20D 20 5A 97   JSR L975A
F210          LF210:
F210 20 6C 97   JSR L976C
F213 A9 14      LDA #$14
F215          LF215:
F215 E9 01      SBC #$1
F217 D0 FC      BNE LF215
F219          LF219:
F219 AD 00 80   LDA VIA1+$00
F21C 29 FD      AND #$FD
F21E 09 08      ORA #$8
F220 8D 00 80   STA VIA1+$00
F223 CA         DEX
F224 D0 D6      BNE LF1FC
F226          LF226:
F226 20 FF F3   JSR LF3FF
F229 68         PLA
F22A AA         TAX
F22B 18         CLC
F22C 60         RTS
F22D          LF22D:
F22D 20 37 F2   JSR LF237
F230 38         SEC
F231 60         RTS
F232          LF232:
F232 A9 3F      LDA #$3F
F234 20 B5 F1   JSR LF1B5
F237          LF237:
F237 20 4D F2   JSR LF24D
F23A A9 14      LDA #$14
F23C          LF23C:
F23C E9 01      SBC #$1
F23E D0 FC      BNE LF23C
F240          LF240:
F240 20 6C 97   JSR L976C
F243 20 5A 97   JSR L975A
F246 18         CLC
F247 60         RTS
F248          LF248:
F248 A9 6F      LDA #$6F
F24A 20 C5 F1   JSR LF1C5
F24D          LF24D:
F24D AD 00 80   LDA VIA1+$00
F250 09 50      ORA #$50
F252 8D 00 80   STA VIA1+$00
F255 A9 3A      LDA #$3A
F257 8D 02 80   STA VIA1+$02
F25A          LF25A:
F25A 60         RTS
F25B          LF25B:
F25B 20 B3 F1   JSR LF1B3
F25E B0 FA      BCS LF25A
F260          LF260:
F260 20 48 F2   JSR LF248
F263 B0 F5      BCS LF25A
F265          LF265:
F265 A2 00      LDX #$0
F267          LF267:
F267 BD 84 F2   LDA LF284,X
F26A 20 D6 F1   JSR LF1D6
F26D E8         INX
F26E E0 06      CPX #$6
F270 90 F5      BCC LF267
F272          LF272:
F272 A5 77      LDA L77
F274 20 D6 F1   JSR LF1D6
F277 A9 80      LDA #$80
F279 8D D5 2B   STA L2BD5
F27C A5 78      LDA L78
F27E 20 D6 F1   JSR LF1D6
F281 4C 32 F2   JMP LF232
F284          LF284:
F284 4D 2D 57   .BYTE $4D,$2D,$57
F287 77 00 02   .BYTE $77,$0,$2
F28A          LF28A:
F28A 8A         TXA
F28B A2 00      LDX #$0
F28D          LF28D:
F28D CA         DEX
F28E D0 FD      BNE LF28D
F290          LF290:
F290 A2 90      LDX #$90
F292          LF292:
F292 CA         DEX
F293 D0 FD      BNE LF292
F295          LF295:
F295 AA         TAX
F296 60         RTS
F297          LF297:
F297 AD E4 90   LDA L90E4
F29A 10 19      BPL LF2B5
F29C          LF29C:
F29C 29 7F      AND #$7F
F29E 38         SEC
F29F ED E6 2B   SBC L2BE6
F2A2 D0 03      BNE LF2A7
F2A4          LF2A4:
F2A4 8D E6 2B   STA L2BE6
F2A7          LF2A7:
F2A7 A5 49      LDA L49
F2A9 29 FB      AND #$FB
F2AB 29 F7      AND #$F7
F2AD 85 49      STA L49
F2AF AD E1 90   LDA L90E1
F2B2 20 CA F2   JSR LF2CA
F2B5          LF2B5:
F2B5 AE E6 2B   LDX L2BE6
F2B8 F0 22      BEQ LF2DC
F2BA          LF2BA:
F2BA E0 08      CPX #$8
F2BC D0 03      BNE LF2C1
F2BE          LF2BE:
F2BE A9 04      LDA #$4
F2C1          LF2C1 = * + 1
              ; Instruction parameter jumped to.
F2C0 2C A9 08   BIT L8A9
F2C3 05 49      ORA L49
F2C5 85 49      STA L49
F2C7 8A         TXA
F2C8 09 80      ORA #$80
F2CA          LF2CA:
F2CA 20 5A F7   JSR LF75A
F2CD 29 7F      AND #$7F
F2CF 48         PHA
F2D0 20 5B F2   JSR LF25B
F2D3 68         PLA
F2D4 09 20      ORA #$20
F2D6 85 77      STA L77
F2D8 49 60      EOR #$60
F2DA 85 78      STA L78
F2DC          LF2DC:
F2DC 60         RTS
F2DD          LF2DD:
F2DD 08         PHP
F2DE 78         SEI
F2DF A9 08      LDA #$8
F2E1 2D 01 88   AND PIO+$01
F2E4 D0 13      BNE LF2F9
F2E6          LF2E6:
F2E6 20 EC F3   JSR LF3EC
F2E9 B0 50      BCS LF33B
F2EB          LF2EB:
F2EB A9 80      LDA #$80
F2ED 45 49      EOR L49
F2EF 85 49      STA L49
F2F1 A9 00      LDA #$0
F2F3 8D F9 2B   STA L2BF9
F2F6 4C 2A F3   JMP LF32A
F2F9          LF2F9:
F2F9 2C E7 2B   BIT L2BE7
F2FC 30 24      BMI LF322
F2FE          LF2FE:
F2FE AD E6 2B   LDA L2BE6
F301 F0 09      BEQ LF30C
F303          LF303:
F303 09 80      ORA #$80
F305 CD E4 90   CMP L90E4
F308 F0 20      BEQ LF32A
F30A          LF30A:
F30A D0 16      BNE LF322
F30C          LF30C:
F30C A9 02      LDA #$2
F30E 2D 01 88   AND PIO+$01
F311 F0 0A      BEQ LF31D
F313          LF313:
F313 A9 04      LDA #$4
F315 2D 01 88   AND PIO+$01
F318 D0 17      BNE LF331
F31A          LF31A:
F31A A9 09      LDA #$9
F31D          LF31D = * + 1
              ; Instruction parameter jumped to.
F31C 2C A9 08   BIT L8A9
F31F 8D E6 2B   STA L2BE6
F322          LF322:
F322 20 0D F4   JSR LF40D
F325 D0 03      BNE LF32A
F327          LF327:
F327 20 97 F2   JSR LF297
F32A          LF32A:
F32A 58         CLI
F32B 20 2A F4   JSR LF42A
F32E 20 21 F4   JSR LF421
F331          LF331:
F331 A9 00      LDA #$0
F333 8D E7 2B   STA L2BE7
F336 8D E6 2B   STA L2BE6
F339 28         PLP
F33A 60         RTS
F33B          LF33B:
F33B A5 49      LDA L49
F33D 2C 4E F3   BIT LF34E
F340 D0 E8      BNE LF32A
F342          LF342:
F342 48         PHA
F343 A9 00      LDA #$0
F345 85 50      STA L50
F347 85 51      STA L51
F349 85 52      STA L52
F34B 85 53      STA L53
F34E          LF34E = * + 1
              ; Instruction parameter accessed.
F34D A9 01      LDA #$1
F34F 85 49      STA L49
F351 58         CLI
F352 48         PHA
F353          LF353:
F353 20 2A F4   JSR LF42A
F356          LF356:
F356 68         PLA
F357 85 49      STA L49
F359          LF359:
F359 A2 FA      LDX #$FA
F35B          LF35B:
F35B AD 01 88   LDA PIO+$01
F35E 29 0E      AND #$E
F360 49 0E      EOR #$E
F362 D0 0F      BNE LF373
F364          LF364:
F364 20 8A F2   JSR LF28A
F367 CA         DEX
F368 D0 F1      BNE LF35B
F36A          LF36A:
F36A A5 49      LDA L49
F36C 49 01      EOR #$1
F36E 85 49      STA L49
F370 4C 59 F3   JMP LF359
F373          LF373:
F373 A2 01      LDX #$1
F375 86 49      STX L49
F377 48         PHA
F378 20 EC F3   JSR LF3EC
F37B 68         PLA
F37C B0 31      BCS LF3AF
F37E          LF37E:
F37E 4A         LSR A
F37F C9 04      CMP #$4
F381 90 02      BCC LF385
F383          LF383:
F383 A9 03      LDA #$3
F385          LF385:
F385 AA         TAX
F386 E4 53      CPX L53
F388 86 53      STX L53
F38A D0 02      BNE LF38E
F38C          LF38C:
F38C F6 4F      INC L4F,X
F38E          LF38E:
F38E B5 4F      LDA L4F,X
F390 DD E8 F3   CMP LF3E8,X
F393 B0 05      BCS LF39A
F395          LF395:
F395 20 C1 F3   JSR LF3C1
F398 90 04      BCC LF39E
F39A          LF39A:
F39A A9 00      LDA #$0
F39C 95 4F      STA L4F,X
F39E          LF39E:
F39E B4 4F      LDY L4F,X
F3A0 B9 DF F3   LDA LF3DF,Y
F3A3 09 01      ORA #$1
F3A5 48         PHA
F3A6 E0 03      CPX #$3
F3A8 D0 A9      BNE LF353
F3AA          LF3AA:
F3AA 20 2D F4   JSR LF42D
F3AD F0 A7      BEQ LF356
F3AF          LF3AF:
F3AF 68         PLA
F3B0 85 49      STA L49
F3B2 20 2A F4   JSR LF42A
F3B5 28         PLP
F3B6 20 C1 F3   JSR LF3C1
F3B9 D0 03      BNE LF3BE
F3BB          LF3BB:
F3BB AD E3 90   LDA L90E3
F3BE          LF3BE:
F3BE 4C 5E B9   JMP LB95E
F3C1          LF3C1:
F3C1 A9 00      LDA #$0
F3C3 18         CLC
F3C4 A4 50      LDY L50
F3C6          LF3C6:
F3C6 88         DEY
F3C7 30 04      BMI LF3CD
F3C9          LF3C9:
F3C9 69 64      ADC #$64
F3CB D0 F9      BNE LF3C6
F3CD          LF3CD:
F3CD A4 51      LDY L51
F3CF          LF3CF:
F3CF 88         DEY
F3D0 30 06      BMI LF3D8
F3D2          LF3D2:
F3D2 69 0A      ADC #$A
F3D4 B0 08      BCS LF3DE
F3D6          LF3D6:
F3D6 90 F7      BCC LF3CF
F3D8          LF3D8:
F3D8 65 52      ADC L52
F3DA B0 02      BCS LF3DE
F3DC          LF3DC:
F3DC C9 FF      CMP #$FF
F3DE          LF3DE:
F3DE 60         RTS
F3DF          LF3DF:
F3DF 00 80 08   .BYTE $0,$80,$8
F3E2 88 04 84   .BYTE $88,$4,$84
F3E5 0C 8C 40   .BYTE $C,$8C,$40
F3E8          LF3E8:
F3E8 C0 03      CPY #$3
F3EA 0A         ASL A
F3EB 0A         ASL A
F3EC          LF3EC:
F3EC A0 1E      LDY #$1E
F3EE          LF3EE:
F3EE 20 21 F4   JSR LF421
F3F1 A9 08      LDA #$8
F3F3 2D 01 88   AND PIO+$01
F3F6 D0 05      BNE LF3FD
F3F8          LF3F8:
F3F8 88         DEY
F3F9 D0 F3      BNE LF3EE
F3FB          LF3FB:
F3FB 38         SEC
F3FD          LF3FD = * + 1
              ; Instruction parameter jumped to.
F3FC 24 18      BIT L18
F3FE 60         RTS
F3FF          LF3FF:
F3FF AD 00 80   LDA VIA1+$00
F402 6A         ROR A
F403 90 FA      BCC LF3FF
F405          LF405:
F405 60         RTS
F406          LF406:
F406 AD 00 80   LDA VIA1+$00
F409 6A         ROR A
F40A B0 FA      BCS LF406
F40C          LF40C:
F40C 60         RTS
F40D          LF40D:
F40D A9 01      LDA #$1
F40F 25 49      AND L49
F411 D0 0D      BNE LF420
F413          LF413:
F413 A9 F0      LDA #$F0
F415 2D 00 80   AND VIA1+$00
F418 8D 00 80   STA VIA1+$00
F41B AD 00 80   LDA VIA1+$00
F41E 29 05      AND #$5
F420          LF420:
F420 60         RTS
F421          LF421:
F421 A2 4B      LDX #$4B
F423          LF423:
F423 20 8A F2   JSR LF28A
F426 CA         DEX
F427 D0 FA      BNE LF423
F429          LF429:
F429 60         RTS
F42A          LF42A:
F42A 20 21 F4   JSR LF421
F42D          LF42D:
F42D AD 01 88   LDA PIO+$01
F430 29 0E      AND #$E
F432 49 0E      EOR #$E
F434 D0 F7      BNE LF42D
F436          LF436:
F436 60         RTS
F437          LF437:
F437 78         SEI
F438 D8         CLD
F439 A2 8F      LDX #$8F
F43B 9A         TXS
F43C 20 20 F7   JSR LF720
F43F AD E1 90   LDA L90E1
F442 20 5A F7   JSR LF75A
F445 AD E2 90   LDA L90E2
F448 20 51 F7   JSR LF751
F44B 20 00 F7   JSR LF700
F44E A9 00      LDA #$0
F450 85 49      STA L49
F452 AA         TAX
F453          LF453:
F453 9D 00 91   STA L9100,X
F456 9D 00 92   STA L9200,X
F459 E8         INX
F45A D0 F7      BNE LF453
F45C          LF45C:
F45C 78         SEI
F45D D8         CLD
F45E A9 DB      LDA #$DB
F460 8D 0C 84   STA VIA2+$0C
F463 A9 08      LDA #$8
F465 8D 00 84   STA VIA2+$00
F468 A9 18      LDA #$18
F46A 8D 02 84   STA VIA2+$02
F46D A9 00      LDA #$0
F46F 8D 03 84   STA VIA2+$03
F472 A9 00      LDA #$0
F474 8D 0A 84   STA VIA2+$0A
F477 A9 7F      LDA #$7F
F479 8D 0E 84   STA VIA2+$0E
F47C 8D 0D 84   STA VIA2+$0D
F47F A9 FF      LDA #$FF
F481 8D 0F 80   STA VIA1+$0F
F484 A9 3A      LDA #$3A
F486 8D 03 80   STA VIA1+$03
F489 A9 D5      LDA #$D5
F48B 8D 00 80   STA VIA1+$00
F48E A9 3A      LDA #$3A
F490 8D 02 80   STA VIA1+$02
F493 A9 00      LDA #$0
F495 8D 09 80   STA VIA1+$09
F498 A9 05      LDA #$5
F49A 8D 08 80   STA VIA1+$08
F49D A9 7F      LDA #$7F
F49F 8D 0E 80   STA VIA1+$0E
F4A2 8D 0D 80   STA VIA1+$0D
F4A5 A9 00      LDA #$0
F4A7 8D 0C 80   STA VIA1+$0C
F4AA A9 0C      LDA #$C
F4AC 8D 0B 80   STA VIA1+$0B
F4AF A9 C6      LDA #$C6
F4B1 8D 0E 80   STA VIA1+$0E
F4B4 A9 92      LDA #$92
F4B6 A2 E2      LDX #$E2
F4B8 20 F8 90   JSR L90F8
F4BB A9 02      LDA #$2
F4BD 85 01      STA L1
F4BF A0 00      LDY #$0
F4C1 84 00      STY L0
F4C3 98         TYA
F4C4          LF4C4:
F4C4 91 00      STA (L0),Y
F4C6 C8         INY
F4C7 D0 FB      BNE LF4C4
F4C9          LF4C9:
F4C9 E6 01      INC L1
F4CB A6 01      LDX L1
F4CD E0 80      CPX #$80
F4CF 90 F3      BCC LF4C4
F4D1          LF4D1:
F4D1 A9 80      LDA #$80
F4D3 8D DA 2B   STA L2BDA
F4D6          LF4D6:
F4D6 78         SEI
F4D7 A4 49      LDY L49
F4D9 A2 00      LDX #$0
F4DB 8A         TXA
F4DC          LF4DC:
F4DC 95 00      STA L0,X
F4DE 9D 00 01   STA L100,X
F4E1 E8         INX
F4E2 D0 F8      BNE LF4DC
F4E4          LF4E4:
F4E4 84 49      STY L49
F4E6 A2 8F      LDX #$8F
F4E8 9A         TXS
F4E9 86 5E      STX L5E
F4EB 20 CE F5   JSR LF5CE
F4EE AD E3 90   LDA L90E3
F4F1 8D D6 2B   STA L2BD6
F4F4 20 23 B0   JSR LB023
F4F7 20 27 F5   JSR LF527
F4FA A0 32      LDY #$32
F4FC          LF4FC:
F4FC 20 8A F2   JSR LF28A
F4FF 88         DEY
F500 D0 FA      BNE LF4FC
F502          LF502:
F502 A2 00      LDX #$0
F504 A9 82      LDA #$82
F506 20 1C E8   JSR LE81C
F509 A0 00      LDY #$0
F50B          LF50B:
F50B CA         DEX
F50C D0 FD      BNE LF50B
F50E          LF50E:
F50E 88         DEY
F50F D0 FA      BNE LF50B
F511          LF511:
F511 20 03 AF   JSR LAF03
F514 2C DA 2B   BIT L2BDA
F517 10 03      BPL LF51C
F519          LF519:
F519 4C 17 DE   JMP LDE17
F51C          LF51C:
F51C A9 73      LDA #$73
F51E 20 AD DF   JSR LDFAD
F521 20 44 97   JSR L9744
F524 4C 30 FF   JMP LFF30
F527          LF527:
F527 A9 FF      LDA #$FF
F529 A2 00      LDX #$0
F52B          LF52B:
F52B 9D 48 2C   STA L2C48,X
F52E E8         INX
F52F E0 13      CPX #$13
F531 90 F8      BCC LF52B
F533          LF533:
F533 A2 00      LDX #$0
F535          LF535:
F535 9D 68 2C   STA L2C68,X
F538 9D 88 2C   STA L2C88,X
F53B 9D A8 2C   STA L2CA8,X
F53E E8         INX
F53F E0 20      CPX #$20
F541 90 F2      BCC LF535
F543          LF543:
F543 A9 1E      LDA #$1E
F545 09 80      ORA #$80
F547 8D 57 2C   STA L2C57
F54A A9 1F      LDA #$1F
F54C 8D 58 2C   STA L2C58
F54F A9 01      LDA #$1
F551 8D C6 2D   STA L2DC6
F554 A9 1E      LDA #$1E
F556 8D 86 2C   STA L2C86
F559 A9 88      LDA #$88
F55B 8D C7 2D   STA L2DC7
F55E A9 1F      LDA #$1F
F560 8D 87 2C   STA L2C87
F563 A2 00      LDX #$0
F565 A0 03      LDY #$3
F567          LF567:
F567 A9 00      LDA #$0
F569 95 A0      STA LA0,X
F56B E8         INX
F56C 98         TYA
F56D 95 A0      STA LA0,X
F56F C8         INY
F570 E8         INX
F571 E0 40      CPX #$40
F573 90 F2      BCC LF567
F575          LF575:
F575 20 A9 F5   JSR LF5A9
F578 20 B2 F5   JSR LF5B2
F57B 20 54 DD   JSR LDD54
F57E 20 BB F5   JSR LF5BB
F581 A9 02      LDA #$2
F583 8D 61 2A   STA L2A61
F586 A9 04      LDA #$4
F588 85 46      STA L46
F58A A9 01      LDA #$1
F58C 85 57      STA L57
F58E A9 02      LDA #$2
F590 85 61      STA L61
F592 A9 05      LDA #$5
F594 8D E9 2B   STA L2BE9
F597 A9 00      LDA #$0
F599 8D E7 2B   STA L2BE7
F59C 8D E6 2B   STA L2BE6
F59F 85 71      STA L71
F5A1 A9 FF      LDA #$FF
F5A3 85 70      STA L70
F5A5 8D FA 2B   STA L2BFA
F5A8 60         RTS
F5A9          LF5A9:
F5A9 A9 00      LDA #$0
F5AB 85 DC      STA LDC
F5AD A9 02      LDA #$2
F5AF 85 DD      STA LDD
F5B1 60         RTS
F5B2          LF5B2:
F5B2 A9 00      LDA #$0
F5B4 85 DE      STA LDE
F5B6 A9 23      LDA #$23
F5B8 85 DF      STA LDF
F5BA 60         RTS
F5BB          LF5BB:
F5BB AD E4 90   LDA L90E4
F5BE 30 03      BMI LF5C3
F5C0          LF5C0:
F5C0 AD E1 90   LDA L90E1
F5C3          LF5C3:
F5C3 29 1F      AND #$1F
F5C5 09 20      ORA #$20
F5C7 85 77      STA L77
F5C9 49 60      EOR #$60
F5CB 85 78      STA L78
F5CD 60         RTS
F5CE          LF5CE:
F5CE 08         PHP
F5CF 78         SEI
F5D0 20 00 F7   JSR LF700
F5D3 A2 00      LDX #$0
F5D5 A0 00      LDY #$0
F5D7          LF5D7:
F5D7 BD 00 FE   LDA LFE00,X
F5DA 99 01 FF   STA LFF01,Y
F5DD BD 01 FE   LDA LFE01,X
F5E0 99 02 FF   STA LFF02,Y
F5E3 C8         INY
F5E4 C8         INY
F5E5 C8         INY
F5E6 E8         INX
F5E7 E8         INX
F5E8 E0 3E      CPX #$3E
F5EA 90 EB      BCC LF5D7
F5EC          LF5EC:
F5EC 20 F5 F6   JSR LF6F5
F5EF 28         PLP
F5F0 60         RTS
F5F1          LF5F1:
F5F1 A2 00      LDX #$0
F5F3 20 EB F6   JSR LF6EB
F5F6 A9 00      LDA #$0
F5F8 8D A0 28   STA L28A0
F5FB          LF5FB:
F5FB 20 0F F6   JSR LF60F
F5FE B0 0E      BCS LF60E
F600          LF600:
F600 20 24 F6   JSR LF624
F603 EE A0 28   INC L28A0
F606 AD A0 28   LDA L28A0
F609 C9 20      CMP #$20
F60B 90 EE      BCC LF5FB
F60D          LF60D:
F60D 18         CLC
F60E          LF60E:
F60E 60         RTS
F60F          LF60F:
F60F 18         CLC
F610 6D E7 90   ADC L90E7
F613 8D 01 28   STA L2801
F616 A9 00      LDA #$0
F618 AA         TAX
F619 6D E6 90   ADC L90E6
F61C 8D 00 28   STA L2800
F61F A9 AA      LDA #$AA
F621 4C C9 F6   JMP LF6C9
F624          LF624:
F624 20 00 F7   JSR LF700
F627 AD A0 28   LDA L28A0
F62A 0A         ASL A
F62B 0A         ASL A
F62C 0A         ASL A
F62D AA         TAX
F62E A9 02      LDA #$2
F630 85 68      STA L68
F632          LF632:
F632 A0 00      LDY #$0
F634 B1 68      LDA (L68),Y
F636 9D 00 82   STA Partition_Typ+$00,X
F639 A0 1C      LDY #$1C
F63B B1 68      LDA (L68),Y
F63D 9D 00 83   STA Partition_SizeHi+$00,X
F640 C8         INY
F641 B1 68      LDA (L68),Y
F643 9D 00 86   STA Partition_SizeLo+$00,X
F646 A0 13      LDY #$13
F648 B1 68      LDA (L68),Y
F64A 9D 00 87   STA Partition_StartHi+$00,X
F64D C8         INY
F64E B1 68      LDA (L68),Y
F650 9D 00 8A   STA Partition_StartMi+$00,X
F653 C8         INY
F654 B1 68      LDA (L68),Y
F656 9D 00 8B   STA Partition_StartLo+$00,X
F659 E8         INX
F65A A5 68      LDA L68
F65C 18         CLC
F65D 69 20      ADC #$20
F65F 85 68      STA L68
F661 90 CF      BCC LF632
F663          LF663:
F663 4C F5 F6   JMP LF6F5
F666          LF666:
F666 20 EB F6   JSR LF6EB
F669 A9 50      LDA #$50
F66B 9D 60 28   STA L2860,X
F66E 8A         TXA
F66F 0A         ASL A
F670 AA         TAX
F671 A9 00      LDA #$0
F673 9D 00 28   STA L2800,X
F676 A9 02      LDA #$2
F678 9D 01 28   STA L2801,X
F67B 8A         TXA
F67C 4A         LSR A
F67D AA         TAX
F67E A9 01      LDA #$1
F680 9D A0 28   STA L28A0,X
F683 A9 00      LDA #$0
F685 9D 80 28   STA L2880,X
F688 A9 FC      LDA #$FC
F68A 4C C9 F6   JMP LF6C9
F68D          LF68D:
F68D 20 66 F6   JSR LF666
F690 90 01      BCC LF693
F692          LF692:
F692 60         RTS
F693          LF693:
F693 8A         TXA
F694 48         PHA
F695 A2 0F      LDX #$F
F697          LF697:
F697 BD F0 51   LDA L51F0,X
F69A DD B9 F6   CMP LF6B9,X
F69D D0 16      BNE LF6B5
F69F          LF69F:
F69F CA         DEX
F6A0 10 F5      BPL LF697
F6A2          LF6A2:
F6A2 20 00 F7   JSR LF700
F6A5 A2 00      LDX #$0
F6A7          LF6A7:
F6A7 BD 00 51   LDA L5100,X
F6AA 9D 00 90   STA L9000,X
F6AD E8         INX
F6AE D0 F7      BNE LF6A7
F6B0          LF6B0:
F6B0 20 F5 F6   JSR LF6F5
F6B3 18         CLC
F6B5          LF6B5 = * + 1
              ; Instruction parameter jumped to.
F6B4 24 38      BIT L38
F6B6 68         PLA
F6B7 AA         TAX
F6B8 60         RTS
F6B9          LF6B9:
F6B9 43 4D 44   .BYTE $43,$4D,$44
F6BC 20 48 44   .BYTE $20,$48,$44
F6BF 20         .BYTE $20
F6C0          LF6C0:
F6C0 20 8D 03   JSR L38D
F6C3 88         DEY
F6C4 8E 02 88   STX PIO+$02
F6C7 EA         NOP
F6C8 60         RTS
F6C9          LF6C9:
F6C9 08         PHP
F6CA 78         SEI
F6CB 95 20      STA L20,X
F6CD AD E8 90   LDA L90E8
F6D0 48         PHA
F6D1 A9 00      LDA #$0
F6D3 20 63 F7   JSR LF763
F6D6 20 00 F7   JSR LF700
F6D9 B5 20      LDA L20,X
F6DB 20 25 E8   JSR LE825
F6DE 68         PLA
F6DF 20 63 F7   JSR LF763
F6E2 20 F5 F6   JSR LF6F5
F6E5 B5 20      LDA L20,X
F6E7 28         PLP
F6E8 C9 02      CMP #$2
F6EA 60         RTS
F6EB          LF6EB:
F6EB 48         PHA
F6EC 08         PHP
F6ED 58         CLI
F6EE          LF6EE:
F6EE B5 20      LDA L20,X
F6F0 30 FC      BMI LF6EE
F6F2          LF6F2:
F6F2 28         PLP
F6F3 68         PLA
F6F4 60         RTS
F6F5          LF6F5:
F6F5 48         PHA
F6F6 AD 00 8F   LDA LED
F6F9 29 DF      AND #$DF
F6FB 8D 00 8F   STA LED
F6FE 68         PLA
F6FF 60         RTS
F700          LF700:
F700 48         PHA
F701 AD 00 8F   LDA LED
F704 09 20      ORA #$20
F706 8D 00 8F   STA LED
F709 68         PLA
F70A 60         RTS
F70B          LF70B:
F70B 48         PHA
F70C AD DB 2B   LDA L2BDB
F70F 8D 00 8F   STA LED
F712 68         PLA
F713 60         RTS
F714          LF714:
F714 48         PHA
F715 AD 00 8F   LDA LED
F718 8D DB 2B   STA L2BDB
F71B 20 00 F7   JSR LF700
F71E 68         PLA
F71F 60         RTS
F720          LF720:
F720 48         PHA
F721 AD 02 88   LDA PIO+$02
F724 09 02      ORA #$2
F726 8D 02 88   STA PIO+$02
F729 68         PLA
F72A 60         RTS
F72B          LF72B:
F72B 48         PHA
F72C AD 02 88   LDA PIO+$02
F72F 29 FD      AND #$FD
F731 8D 02 88   STA PIO+$02
F734 68         PLA
F735 60         RTS
F736          LF736:
F736 20 14 F7   JSR LF714
F739 8D E0 90   STA L90E0
F73C 4C 0B F7   JMP LF70B
F73F          LF73F:
F73F 20 14 F7   JSR LF714
F742 8D E1 90   STA L90E1
F745 4C 0B F7   JMP LF70B
F748          LF748:
F748 20 14 F7   JSR LF714
F74B 8D E2 90   STA L90E2
F74E 4C 0B F7   JMP LF70B
F751          LF751:
F751 20 14 F7   JSR LF714
F754 8D E3 90   STA L90E3
F757 4C 0B F7   JMP LF70B
F75A          LF75A:
F75A 20 14 F7   JSR LF714
F75D 8D E4 90   STA L90E4
F760 4C 0B F7   JMP LF70B
F763          LF763:
F763 20 14 F7   JSR LF714
F766 8D E8 90   STA L90E8
F769 4C 0B F7   JMP LF70B
F76C          LF76C:
F76C 8A         TXA
F76D 0A         ASL A
F76E 0A         ASL A
F76F 0A         ASL A
F770 0A         ASL A
F771 0A         ASL A
F772 0A         ASL A
F773 48         PHA
F774 A2 00      LDX #$0
F776 20 66 F6   JSR LF666
F779 B0 41      BCS LF7BC
F77B          LF77B:
F77B 68         PLA
F77C 48         PHA
F77D AA         TAX
F77E BD 00 50   LDA L5000,X
F781 8D 00 52   STA L5200
F784 BD 01 50   LDA L5001,X
F787 8D 01 52   STA L5201
F78A BD 03 50   LDA L5003,X
F78D 8D 04 52   STA L5204
F790 BD 02 50   LDA L5002,X
F793 8D 05 52   STA L5205
F796 A9 00      LDA #$0
F798 8D 02 52   STA L5202
F79B 8D 03 52   STA L5203
F79E 20 BF F7   JSR LF7BF
F7A1 B0 19      BCS LF7BC
F7A3          LF7A3:
F7A3 68         PLA
F7A4 48         PHA
F7A5 AA         TAX
F7A6 AD 02 52   LDA L5202
F7A9 DD 05 50   CMP L5005,X
F7AC D0 0E      BNE LF7BC
F7AE          LF7AE:
F7AE AD 03 52   LDA L5203
F7B1 DD 04 50   CMP L5004,X
F7B4 D0 06      BNE LF7BC
F7B6          LF7B6:
F7B6 68         PLA
F7B7 20 36 F7   JSR LF736
F7BA 18         CLC
F7BB 60         RTS
F7BC          LF7BC:
F7BC 68         PLA
F7BD 38         SEC
F7BE 60         RTS
F7BF          LF7BF:
F7BF 78         SEI
F7C0 AD 00 52   LDA L5200
F7C3 85 6C      STA L6C
F7C5 A9 00      LDA #$0
F7C7 85 6B      STA L6B
F7C9 A2 00      LDX #$0
F7CB AD 05 52   LDA L5205
F7CE 4A         LSR A
F7CF 9D 00 28   STA L2800,X
F7D2 AD 04 52   LDA L5204
F7D5 6A         ROR A
F7D6 9D 01 28   STA L2801,X
F7D9 AD 01 52   LDA L5201
F7DC 4A         LSR A
F7DD 9D A0 28   STA L28A0,X
F7E0 A5 6B      LDA L6B
F7E2 9D 80 28   STA L2880,X
F7E5 A5 6C      LDA L6C
F7E7 9D 60 28   STA L2860,X
F7EA A9 FC      LDA #$FC
F7EC 20 C9 F6   JSR LF6C9
F7EF B0 29      BCS LF81A
F7F1          LF7F1:
F7F1 AE 01 52   LDX L5201
F7F4 A0 00      LDY #$0
F7F6          LF7F6:
F7F6 AD 02 52   LDA L5202
F7F9          LF7F9:
F7F9 18         CLC
F7FA 71 6B      ADC (L6B),Y
F7FC 90 03      BCC LF801
F7FE          LF7FE:
F7FE EE 03 52   INC L5203
F801          LF801:
F801 C8         INY
F802 D0 F5      BNE LF7F9
F804          LF804:
F804 8D 02 52   STA L5202
F807 E6 6C      INC L6C
F809 A5 6C      LDA L6C
F80B C9 C0      CMP #$C0
F80D D0 07      BNE LF816
F80F          LF80F:
F80F A9 40      LDA #$40
F811 85 6C      STA L6C
F813 20 2B F7   JSR LF72B
F816          LF816:
F816 CA         DEX
F817 D0 DD      BNE LF7F6
F819          LF819:
F819 18         CLC
F81A          LF81A:
F81A 60         RTS
F81B          LF81B:
F81B 78         SEI
F81C 20 F9 95   JSR L95F9
F81F A9 10      LDA #$10
F821 8D 00 80   STA VIA1+$00
F824 A9 00      LDA #$0
F826 C5 4B      CMP L4B
F828 F0 09      BEQ LF833
F82A          LF82A:
F82A 85 4B      STA L4B
F82C 58         CLI
F82D 20 15 B6   JSR LB615
F830 20 9B 97   JSR L979B
F833          LF833:
F833 58         CLI
F834 2C 00 80   BIT VIA1+$00
F837 30 05      BMI LF83E
F839          LF839:
F839 2C 01 88   BIT PIO+$01
F83C 10 03      BPL LF841
F83E          LF83E:
F83E 4C 3C FF   JMP LFF3C
F841          LF841:
F841 78         SEI
F842 A0 00      LDY #$0
F844 A2 0E      LDX #$E
F846          LF846:
F846 BD 48 2C   LDA L2C48,X
F849 C9 FF      CMP #$FF
F84B F0 01      BEQ LF84E
F84D          LF84D:
F84D C8         INY
F84E          LF84E:
F84E CA         DEX
F84F 10 F5      BPL LF846
F851          LF851:
F851 A2 1F      LDX #$1F
F853          LF853:
F853 B5 20      LDA L20,X
F855 10 01      BPL LF858
F857          LF857:
F857 C8         INY
F858          LF858:
F858 CA         DEX
F859 10 F8      BPL LF853
F85B          LF85B:
F85B 98         TYA
F85C F0 06      BEQ LF864
F85E          LF85E:
F85E 20 3C EE   JSR LEE3C
F861 4C 67 F8   JMP LF867
F864          LF864:
F864 20 4D EE   JSR LEE4D
F867          LF867:
F867 20 DD F2   JSR LF2DD
F86A 4C 33 F8   JMP LF833
F86D          LF86D:
F86D 48         PHA
F86E 98         TYA
F86F 48         PHA
F870 8A         TXA
F871 48         PHA
F872 AE 0D 80   LDX VIA1+$0D
F875 8A         TXA
F876 29 02      AND #$2
F878 F0 0B      BEQ LF885
F87A          LF87A:
F87A 8D 0D 80   STA VIA1+$0D
F87D A9 40      LDA #$40
F87F 0D D7 2B   ORA L2BD7
F882 8D D7 2B   STA L2BD7
F885          LF885:
F885 8A         TXA
F886 29 04      AND #$4
F888 F0 0F      BEQ LF899
F88A          LF88A:
F88A 8D 0D 80   STA VIA1+$0D
F88D 25 46      AND L46
F88F F0 08      BEQ LF899
F891          LF891:
F891 A9 80      LDA #$80
F893 0D D8 2B   ORA L2BD8
F896 8D D8 2B   STA L2BD8
F899          LF899:
F899 8A         TXA
F89A 29 40      AND #$40
F89C F0 06      BEQ LF8A4
F89E          LF89E:
F89E 8D 0D 80   STA VIA1+$0D
F8A1 20 51 FF   JSR LFF51
F8A4          LF8A4:
F8A4 BA         TSX
F8A5 BD 04 01   LDA L104,X
F8A8 29 10      AND #$10
F8AA F0 03      BEQ LF8AF
F8AC          LF8AC:
F8AC 20 51 FF   JSR LFF51
F8AF          LF8AF:
F8AF 68         PLA
F8B0 AA         TAX
F8B1 68         PLA
F8B2 A8         TAY
F8B3 68         PLA
F8B4 40         RTI
F8B5 00 00 00   .BYTE $0,$0,$0
F8B8 00 00 00   .BYTE $0,$0,$0
F8BB 00 00 00   .BYTE $0,$0,$0
F8BE 00 00 00   .BYTE $0,$0,$0
F8C1 00 00 00   .BYTE $0,$0,$0
F8C4 00 00 00   .BYTE $0,$0,$0
F8C7 00 00 00   .BYTE $0,$0,$0
F8CA 00 00 00   .BYTE $0,$0,$0
F8CD 00 00 00   .BYTE $0,$0,$0
F8D0 00 00 00   .BYTE $0,$0,$0
F8D3 00 00 00   .BYTE $0,$0,$0
F8D6 00 00 00   .BYTE $0,$0,$0
F8D9 00 00 00   .BYTE $0,$0,$0
F8DC 00 00 00   .BYTE $0,$0,$0
F8DF 00 00 00   .BYTE $0,$0,$0
F8E2 00 00 00   .BYTE $0,$0,$0
F8E5 00 00 00   .BYTE $0,$0,$0
F8E8 00 00 00   .BYTE $0,$0,$0
F8EB 00 00 00   .BYTE $0,$0,$0
F8EE 00 00 00   .BYTE $0,$0,$0
F8F1 00 00 00   .BYTE $0,$0,$0
F8F4 00 00 00   .BYTE $0,$0,$0
F8F7 00 00 00   .BYTE $0,$0,$0
F8FA 00 00 00   .BYTE $0,$0,$0
F8FD 00 00 00   .BYTE $0,$0,$0
F900 00 00 00   .BYTE $0,$0,$0
F903 00 00 00   .BYTE $0,$0,$0
F906 00 00 00   .BYTE $0,$0,$0
F909 00 00 00   .BYTE $0,$0,$0
F90C 00 00 00   .BYTE $0,$0,$0
F90F 00 00 00   .BYTE $0,$0,$0
F912 00 00 00   .BYTE $0,$0,$0
F915 00 00 00   .BYTE $0,$0,$0
F918 00 00 00   .BYTE $0,$0,$0
F91B 00 00 00   .BYTE $0,$0,$0
F91E 00 00 00   .BYTE $0,$0,$0
F921 00 00 00   .BYTE $0,$0,$0
F924 00 00 00   .BYTE $0,$0,$0
F927 00 00 00   .BYTE $0,$0,$0
F92A 00 00 00   .BYTE $0,$0,$0
F92D 00 00 00   .BYTE $0,$0,$0
F930 00 00 00   .BYTE $0,$0,$0
F933 00 00 00   .BYTE $0,$0,$0
F936 00 00 00   .BYTE $0,$0,$0
F939 00 00 00   .BYTE $0,$0,$0
F93C 00 00 00   .BYTE $0,$0,$0
F93F 00 00 00   .BYTE $0,$0,$0
F942 00 00 00   .BYTE $0,$0,$0
F945 00 00 00   .BYTE $0,$0,$0
F948 00 00 00   .BYTE $0,$0,$0
F94B 00 00 00   .BYTE $0,$0,$0
F94E 00 00 00   .BYTE $0,$0,$0
F951 00 00 00   .BYTE $0,$0,$0
F954 00 00 00   .BYTE $0,$0,$0
F957 00 00 00   .BYTE $0,$0,$0
F95A 00 00 00   .BYTE $0,$0,$0
F95D 00 00 00   .BYTE $0,$0,$0
F960 00 00 00   .BYTE $0,$0,$0
F963 00 00 00   .BYTE $0,$0,$0
F966 00 00 00   .BYTE $0,$0,$0
F969 00 00 00   .BYTE $0,$0,$0
F96C 00 00 00   .BYTE $0,$0,$0
F96F 00 00 00   .BYTE $0,$0,$0
F972 00 00 00   .BYTE $0,$0,$0
F975 00 00 00   .BYTE $0,$0,$0
F978 00 00 00   .BYTE $0,$0,$0
F97B 00 00 00   .BYTE $0,$0,$0
F97E 00 00 00   .BYTE $0,$0,$0
F981 00 00 00   .BYTE $0,$0,$0
F984 00 00 00   .BYTE $0,$0,$0
F987 00 00 00   .BYTE $0,$0,$0
F98A 00 00 00   .BYTE $0,$0,$0
F98D 00 00 00   .BYTE $0,$0,$0
F990 00 00 00   .BYTE $0,$0,$0
F993 00 00 00   .BYTE $0,$0,$0
F996 00 00 00   .BYTE $0,$0,$0
F999 00 00 00   .BYTE $0,$0,$0
F99C 00 00 00   .BYTE $0,$0,$0
F99F 00 00 00   .BYTE $0,$0,$0
F9A2 00 00 00   .BYTE $0,$0,$0
F9A5 00 00 00   .BYTE $0,$0,$0
F9A8 00 00 00   .BYTE $0,$0,$0
F9AB 00 00 00   .BYTE $0,$0,$0
F9AE 00 00 00   .BYTE $0,$0,$0
F9B1 00 00 00   .BYTE $0,$0,$0
F9B4 00 00 00   .BYTE $0,$0,$0
F9B7 00 00 00   .BYTE $0,$0,$0
F9BA 00 00 00   .BYTE $0,$0,$0
F9BD 00 00 00   .BYTE $0,$0,$0
F9C0 00 00 00   .BYTE $0,$0,$0
F9C3 00 00 00   .BYTE $0,$0,$0
F9C6 00 00 00   .BYTE $0,$0,$0
F9C9 00 00 00   .BYTE $0,$0,$0
F9CC 00 00 00   .BYTE $0,$0,$0
F9CF 00 00 00   .BYTE $0,$0,$0
F9D2 00 00 00   .BYTE $0,$0,$0
F9D5 00 00 00   .BYTE $0,$0,$0
F9D8 00 00 00   .BYTE $0,$0,$0
F9DB 00 00 00   .BYTE $0,$0,$0
F9DE 00 00 00   .BYTE $0,$0,$0
F9E1 00 00 00   .BYTE $0,$0,$0
F9E4 00 00 00   .BYTE $0,$0,$0
F9E7 00 00 00   .BYTE $0,$0,$0
F9EA 00 00 00   .BYTE $0,$0,$0
F9ED 00 00 00   .BYTE $0,$0,$0
F9F0 00 00 00   .BYTE $0,$0,$0
F9F3 00 00 00   .BYTE $0,$0,$0
F9F6 00 00 00   .BYTE $0,$0,$0
F9F9 00 00 00   .BYTE $0,$0,$0
F9FC 00 00 00   .BYTE $0,$0,$0
F9FF 00 00 00   .BYTE $0,$0,$0
FA02 00 00 00   .BYTE $0,$0,$0
FA05 00 00 00   .BYTE $0,$0,$0
FA08 00 00 00   .BYTE $0,$0,$0
FA0B 00 00 00   .BYTE $0,$0,$0
FA0E 00 00 00   .BYTE $0,$0,$0
FA11 00 00 00   .BYTE $0,$0,$0
FA14 00 00 00   .BYTE $0,$0,$0
FA17 00 00 00   .BYTE $0,$0,$0
FA1A 00 00 00   .BYTE $0,$0,$0
FA1D 00 00 00   .BYTE $0,$0,$0
FA20 00 00 00   .BYTE $0,$0,$0
FA23 00 00 00   .BYTE $0,$0,$0
FA26 00 00 00   .BYTE $0,$0,$0
FA29 00 00 00   .BYTE $0,$0,$0
FA2C 00 00 00   .BYTE $0,$0,$0
FA2F 00 00 00   .BYTE $0,$0,$0
FA32 00 00 00   .BYTE $0,$0,$0
FA35 00 00 00   .BYTE $0,$0,$0
FA38 00 00 00   .BYTE $0,$0,$0
FA3B 00 00 00   .BYTE $0,$0,$0
FA3E 00 00 00   .BYTE $0,$0,$0
FA41 00 00 00   .BYTE $0,$0,$0
FA44 00 00 00   .BYTE $0,$0,$0
FA47 00 00 00   .BYTE $0,$0,$0
FA4A 00 00 00   .BYTE $0,$0,$0
FA4D 00 00 00   .BYTE $0,$0,$0
FA50 00 00 00   .BYTE $0,$0,$0
FA53 00 00 00   .BYTE $0,$0,$0
FA56 00 00 00   .BYTE $0,$0,$0
FA59 00 00 00   .BYTE $0,$0,$0
FA5C 00 00 00   .BYTE $0,$0,$0
FA5F 00 00 00   .BYTE $0,$0,$0
FA62 00 00 00   .BYTE $0,$0,$0
FA65 00 00 00   .BYTE $0,$0,$0
FA68 00 00 00   .BYTE $0,$0,$0
FA6B 00 00 00   .BYTE $0,$0,$0
FA6E 00 00 00   .BYTE $0,$0,$0
FA71 00 00 00   .BYTE $0,$0,$0
FA74 00 00 00   .BYTE $0,$0,$0
FA77 00 00 00   .BYTE $0,$0,$0
FA7A 00 00 00   .BYTE $0,$0,$0
FA7D 00 00 00   .BYTE $0,$0,$0
FA80 00 00 00   .BYTE $0,$0,$0
FA83 00 00 00   .BYTE $0,$0,$0
FA86 00 00 00   .BYTE $0,$0,$0
FA89 00 00 00   .BYTE $0,$0,$0
FA8C 00 00 00   .BYTE $0,$0,$0
FA8F 00 00 00   .BYTE $0,$0,$0
FA92 00 00 00   .BYTE $0,$0,$0
FA95 00 00 00   .BYTE $0,$0,$0
FA98 00 00 00   .BYTE $0,$0,$0
FA9B 00 00 00   .BYTE $0,$0,$0
FA9E 00 00 00   .BYTE $0,$0,$0
FAA1 00 00 00   .BYTE $0,$0,$0
FAA4 00 00 00   .BYTE $0,$0,$0
FAA7 00 00 00   .BYTE $0,$0,$0
FAAA 00 00 00   .BYTE $0,$0,$0
FAAD 00 00 00   .BYTE $0,$0,$0
FAB0 00 00 00   .BYTE $0,$0,$0
FAB3 00 00 00   .BYTE $0,$0,$0
FAB6 00 00 00   .BYTE $0,$0,$0
FAB9 00 00 00   .BYTE $0,$0,$0
FABC 00 00 00   .BYTE $0,$0,$0
FABF 00 00 00   .BYTE $0,$0,$0
FAC2 00 00 00   .BYTE $0,$0,$0
FAC5 00 00 00   .BYTE $0,$0,$0
FAC8 00 00 00   .BYTE $0,$0,$0
FACB 00 00 00   .BYTE $0,$0,$0
FACE 00 00 00   .BYTE $0,$0,$0
FAD1 00 00 00   .BYTE $0,$0,$0
FAD4 00 00 00   .BYTE $0,$0,$0
FAD7 00 00 00   .BYTE $0,$0,$0
FADA 00 00 00   .BYTE $0,$0,$0
FADD 00 00 00   .BYTE $0,$0,$0
FAE0 00 00 00   .BYTE $0,$0,$0
FAE3 00 00 00   .BYTE $0,$0,$0
FAE6 00 00 00   .BYTE $0,$0,$0
FAE9 00 00 00   .BYTE $0,$0,$0
FAEC 00 00 00   .BYTE $0,$0,$0
FAEF 00 00 00   .BYTE $0,$0,$0
FAF2 00 00 00   .BYTE $0,$0,$0
FAF5 00 00 00   .BYTE $0,$0,$0
FAF8 00 00 00   .BYTE $0,$0,$0
FAFB 00 00 00   .BYTE $0,$0,$0
FAFE 00 00 00   .BYTE $0,$0,$0
FB01 00 00 00   .BYTE $0,$0,$0
FB04 00 00 00   .BYTE $0,$0,$0
FB07 00 00 00   .BYTE $0,$0,$0
FB0A 00 00 00   .BYTE $0,$0,$0
FB0D 00 00 00   .BYTE $0,$0,$0
FB10 00 00 00   .BYTE $0,$0,$0
FB13 00 00 00   .BYTE $0,$0,$0
FB16 00 00 00   .BYTE $0,$0,$0
FB19 00 00 00   .BYTE $0,$0,$0
FB1C 00 00 00   .BYTE $0,$0,$0
FB1F 00 00 00   .BYTE $0,$0,$0
FB22 00 00 00   .BYTE $0,$0,$0
FB25 00 00 00   .BYTE $0,$0,$0
FB28 00 00 00   .BYTE $0,$0,$0
FB2B 00 00 00   .BYTE $0,$0,$0
FB2E 00 00 00   .BYTE $0,$0,$0
FB31 00 00 00   .BYTE $0,$0,$0
FB34 00 00 00   .BYTE $0,$0,$0
FB37 00 00 00   .BYTE $0,$0,$0
FB3A 00 00 00   .BYTE $0,$0,$0
FB3D 00 00 00   .BYTE $0,$0,$0
FB40 00 00 00   .BYTE $0,$0,$0
FB43 00 00 00   .BYTE $0,$0,$0
FB46 00 00 00   .BYTE $0,$0,$0
FB49 00 00 00   .BYTE $0,$0,$0
FB4C 00 00 00   .BYTE $0,$0,$0
FB4F 00 00 00   .BYTE $0,$0,$0
FB52 00 00 00   .BYTE $0,$0,$0
FB55 00 00 00   .BYTE $0,$0,$0
FB58 00 00 00   .BYTE $0,$0,$0
FB5B 00 00 00   .BYTE $0,$0,$0
FB5E 00 00 00   .BYTE $0,$0,$0
FB61 00 00 00   .BYTE $0,$0,$0
FB64 00 00 00   .BYTE $0,$0,$0
FB67 00 00 00   .BYTE $0,$0,$0
FB6A 00 00 00   .BYTE $0,$0,$0
FB6D 00 00 00   .BYTE $0,$0,$0
FB70 00 00 00   .BYTE $0,$0,$0
FB73 00 00 00   .BYTE $0,$0,$0
FB76 00 00 00   .BYTE $0,$0,$0
FB79 00 00 00   .BYTE $0,$0,$0
FB7C 00 00 00   .BYTE $0,$0,$0
FB7F 00 00 00   .BYTE $0,$0,$0
FB82 00 00 00   .BYTE $0,$0,$0
FB85 00 00 00   .BYTE $0,$0,$0
FB88 00 00 00   .BYTE $0,$0,$0
FB8B 00 00 00   .BYTE $0,$0,$0
FB8E 00 00 00   .BYTE $0,$0,$0
FB91 00 00 00   .BYTE $0,$0,$0
FB94 00 00 00   .BYTE $0,$0,$0
FB97 00 00 00   .BYTE $0,$0,$0
FB9A 00 00 00   .BYTE $0,$0,$0
FB9D 00 00 00   .BYTE $0,$0,$0
FBA0 00 00 00   .BYTE $0,$0,$0
FBA3 00 00 00   .BYTE $0,$0,$0
FBA6 00 00 00   .BYTE $0,$0,$0
FBA9 00 00 00   .BYTE $0,$0,$0
FBAC 00 00 00   .BYTE $0,$0,$0
FBAF 00 00 00   .BYTE $0,$0,$0
FBB2 00 00 00   .BYTE $0,$0,$0
FBB5 00 00 00   .BYTE $0,$0,$0
FBB8 00 00 00   .BYTE $0,$0,$0
FBBB 00 00 00   .BYTE $0,$0,$0
FBBE 00 00 00   .BYTE $0,$0,$0
FBC1 00 00 00   .BYTE $0,$0,$0
FBC4 00 00 00   .BYTE $0,$0,$0
FBC7 00 00 00   .BYTE $0,$0,$0
FBCA 00 00 00   .BYTE $0,$0,$0
FBCD 00 00 00   .BYTE $0,$0,$0
FBD0 00 00 00   .BYTE $0,$0,$0
FBD3 00 00 00   .BYTE $0,$0,$0
FBD6 00 00 00   .BYTE $0,$0,$0
FBD9 00 00 00   .BYTE $0,$0,$0
FBDC 00 00 00   .BYTE $0,$0,$0
FBDF 00 00 00   .BYTE $0,$0,$0
FBE2 00 00 00   .BYTE $0,$0,$0
FBE5 00 00 00   .BYTE $0,$0,$0
FBE8 00 00 00   .BYTE $0,$0,$0
FBEB 00 00 00   .BYTE $0,$0,$0
FBEE 00 00 00   .BYTE $0,$0,$0
FBF1 00 00 00   .BYTE $0,$0,$0
FBF4 00 00 00   .BYTE $0,$0,$0
FBF7 00 00 00   .BYTE $0,$0,$0
FBFA 00 00 00   .BYTE $0,$0,$0
FBFD 00 00 00   .BYTE $0,$0,$0
FC00 00 00 00   .BYTE $0,$0,$0
FC03 00 00 00   .BYTE $0,$0,$0
FC06 00 00 00   .BYTE $0,$0,$0
FC09 00 00 00   .BYTE $0,$0,$0
FC0C 00 00 00   .BYTE $0,$0,$0
FC0F 00 00 00   .BYTE $0,$0,$0
FC12 00 00 00   .BYTE $0,$0,$0
FC15 00 00 00   .BYTE $0,$0,$0
FC18 00 00 00   .BYTE $0,$0,$0
FC1B 00 00 00   .BYTE $0,$0,$0
FC1E 00 00 00   .BYTE $0,$0,$0
FC21 00 00 00   .BYTE $0,$0,$0
FC24 00 00 00   .BYTE $0,$0,$0
FC27 00 00 00   .BYTE $0,$0,$0
FC2A 00 00 00   .BYTE $0,$0,$0
FC2D 00 00 00   .BYTE $0,$0,$0
FC30 00 00 00   .BYTE $0,$0,$0
FC33 00 00 00   .BYTE $0,$0,$0
FC36 00 00 00   .BYTE $0,$0,$0
FC39 00 00 00   .BYTE $0,$0,$0
FC3C 00 00 00   .BYTE $0,$0,$0
FC3F 00 00 00   .BYTE $0,$0,$0
FC42 00 00 00   .BYTE $0,$0,$0
FC45 00 00 00   .BYTE $0,$0,$0
FC48 00 00 00   .BYTE $0,$0,$0
FC4B 00 00 00   .BYTE $0,$0,$0
FC4E 00 00 00   .BYTE $0,$0,$0
FC51 00 00 00   .BYTE $0,$0,$0
FC54 00 00 00   .BYTE $0,$0,$0
FC57 00 00 00   .BYTE $0,$0,$0
FC5A 00 00 00   .BYTE $0,$0,$0
FC5D 00 00 00   .BYTE $0,$0,$0
FC60 00 00 00   .BYTE $0,$0,$0
FC63 00 00 00   .BYTE $0,$0,$0
FC66 00 00 00   .BYTE $0,$0,$0
FC69 00 00 00   .BYTE $0,$0,$0
FC6C 00 00 00   .BYTE $0,$0,$0
FC6F 00 00 00   .BYTE $0,$0,$0
FC72 00 00 00   .BYTE $0,$0,$0
FC75 00 00 00   .BYTE $0,$0,$0
FC78 00 00 00   .BYTE $0,$0,$0
FC7B 00 00 00   .BYTE $0,$0,$0
FC7E 00 00 00   .BYTE $0,$0,$0
FC81 00 00 00   .BYTE $0,$0,$0
FC84 00 00 00   .BYTE $0,$0,$0
FC87 00 00 00   .BYTE $0,$0,$0
FC8A 00 00 00   .BYTE $0,$0,$0
FC8D 00 00 00   .BYTE $0,$0,$0
FC90 00 00 00   .BYTE $0,$0,$0
FC93 00 00 00   .BYTE $0,$0,$0
FC96 00 00 00   .BYTE $0,$0,$0
FC99 00 00 00   .BYTE $0,$0,$0
FC9C 00 00 00   .BYTE $0,$0,$0
FC9F 00 00 00   .BYTE $0,$0,$0
FCA2 00 00 00   .BYTE $0,$0,$0
FCA5 00 00 00   .BYTE $0,$0,$0
FCA8 00 00 00   .BYTE $0,$0,$0
FCAB 00 00 00   .BYTE $0,$0,$0
FCAE 00 00 00   .BYTE $0,$0,$0
FCB1 00 00 00   .BYTE $0,$0,$0
FCB4 00 00 00   .BYTE $0,$0,$0
FCB7 00 00 00   .BYTE $0,$0,$0
FCBA 00 00 00   .BYTE $0,$0,$0
FCBD 00 00 00   .BYTE $0,$0,$0
FCC0 00 00 00   .BYTE $0,$0,$0
FCC3 00 00 00   .BYTE $0,$0,$0
FCC6 00 00 00   .BYTE $0,$0,$0
FCC9 00 00 00   .BYTE $0,$0,$0
FCCC 00 00 00   .BYTE $0,$0,$0
FCCF 00 00 00   .BYTE $0,$0,$0
FCD2 00 00 00   .BYTE $0,$0,$0
FCD5 00 00 00   .BYTE $0,$0,$0
FCD8 00 00 00   .BYTE $0,$0,$0
FCDB 00 00 00   .BYTE $0,$0,$0
FCDE 00 00 00   .BYTE $0,$0,$0
FCE1 00 00 00   .BYTE $0,$0,$0
FCE4 00 00 00   .BYTE $0,$0,$0
FCE7 00 00 00   .BYTE $0,$0,$0
FCEA 00 00 00   .BYTE $0,$0,$0
FCED 00 00 00   .BYTE $0,$0,$0
FCF0 00 00 00   .BYTE $0,$0,$0
FCF3 00 00 00   .BYTE $0,$0,$0
FCF6 00 00 00   .BYTE $0,$0,$0
FCF9 00 00 00   .BYTE $0,$0,$0
FCFC 00 00 00   .BYTE $0,$0,$0
FCFF 00 00 00   .BYTE $0,$0,$0
FD02 00 00 00   .BYTE $0,$0,$0
FD05 00 00 00   .BYTE $0,$0,$0
FD08 00 00 00   .BYTE $0,$0,$0
FD0B 00 00 00   .BYTE $0,$0,$0
FD0E 00 00 00   .BYTE $0,$0,$0
FD11 00 00 00   .BYTE $0,$0,$0
FD14 00 00 00   .BYTE $0,$0,$0
FD17 00 00 00   .BYTE $0,$0,$0
FD1A 00 00 00   .BYTE $0,$0,$0
FD1D 00 00 00   .BYTE $0,$0,$0
FD20 00 00 00   .BYTE $0,$0,$0
FD23 00 00 00   .BYTE $0,$0,$0
FD26 00 00 00   .BYTE $0,$0,$0
FD29 00 00 00   .BYTE $0,$0,$0
FD2C 00 00 00   .BYTE $0,$0,$0
FD2F 00 00 00   .BYTE $0,$0,$0
FD32 00 00 00   .BYTE $0,$0,$0
FD35 00 00 00   .BYTE $0,$0,$0
FD38 00 00 00   .BYTE $0,$0,$0
FD3B 00 00 00   .BYTE $0,$0,$0
FD3E 00 00 00   .BYTE $0,$0,$0
FD41 00 00 00   .BYTE $0,$0,$0
FD44 00 00 00   .BYTE $0,$0,$0
FD47 00 00 00   .BYTE $0,$0,$0
FD4A 00 00 00   .BYTE $0,$0,$0
FD4D 00 00 00   .BYTE $0,$0,$0
FD50 00 00 00   .BYTE $0,$0,$0
FD53 00 00 00   .BYTE $0,$0,$0
FD56 00 00 00   .BYTE $0,$0,$0
FD59 00 00 00   .BYTE $0,$0,$0
FD5C 00 00 00   .BYTE $0,$0,$0
FD5F 00 00 00   .BYTE $0,$0,$0
FD62 00 00 00   .BYTE $0,$0,$0
FD65 00 00 00   .BYTE $0,$0,$0
FD68 00 00 00   .BYTE $0,$0,$0
FD6B 00 00 00   .BYTE $0,$0,$0
FD6E 00 00 00   .BYTE $0,$0,$0
FD71 00 00 00   .BYTE $0,$0,$0
FD74 00 00 00   .BYTE $0,$0,$0
FD77 00 00 00   .BYTE $0,$0,$0
FD7A 00 00 00   .BYTE $0,$0,$0
FD7D 00 00 00   .BYTE $0,$0,$0
FD80 00 00 00   .BYTE $0,$0,$0
FD83 00 00 00   .BYTE $0,$0,$0
FD86 00 00 00   .BYTE $0,$0,$0
FD89 00 00 00   .BYTE $0,$0,$0
FD8C 00 00 00   .BYTE $0,$0,$0
FD8F 00 00 00   .BYTE $0,$0,$0
FD92 00 00 00   .BYTE $0,$0,$0
FD95 00 00 00   .BYTE $0,$0,$0
FD98 00 00 00   .BYTE $0,$0,$0
FD9B 00 00 00   .BYTE $0,$0,$0
FD9E 00 00 00   .BYTE $0,$0,$0
FDA1 00 00 00   .BYTE $0,$0,$0
FDA4 00 00 00   .BYTE $0,$0,$0
FDA7 00 00 00   .BYTE $0,$0,$0
FDAA 00 00 00   .BYTE $0,$0,$0
FDAD 00 00 00   .BYTE $0,$0,$0
FDB0 00 00 00   .BYTE $0,$0,$0
FDB3 00 00 00   .BYTE $0,$0,$0
FDB6 00 00 00   .BYTE $0,$0,$0
FDB9 00 00 00   .BYTE $0,$0,$0
FDBC 00 00 00   .BYTE $0,$0,$0
FDBF 00 00 00   .BYTE $0,$0,$0
FDC2 00 00 00   .BYTE $0,$0,$0
FDC5 00 00 00   .BYTE $0,$0,$0
FDC8 00 00 00   .BYTE $0,$0,$0
FDCB 00 00 00   .BYTE $0,$0,$0
FDCE 00 00 00   .BYTE $0,$0,$0
FDD1 00 00 00   .BYTE $0,$0,$0
FDD4 00 00 00   .BYTE $0,$0,$0
FDD7 00 00 00   .BYTE $0,$0,$0
FDDA 00 00 00   .BYTE $0,$0,$0
FDDD 00 00 00   .BYTE $0,$0,$0
FDE0 00 00 00   .BYTE $0,$0,$0
FDE3 00 00 00   .BYTE $0,$0,$0
FDE6 00 00 00   .BYTE $0,$0,$0
FDE9 00 00 00   .BYTE $0,$0,$0
FDEC 00 00 00   .BYTE $0,$0,$0
FDEF 00 00 00   .BYTE $0,$0,$0
FDF2 00 00 00   .BYTE $0,$0,$0
FDF5 00 00 00   .BYTE $0,$0,$0
FDF8 00 00 00   .BYTE $0,$0,$0
FDFB 00 00 00   .BYTE $0,$0,$0
FDFE 00 00      .BYTE $0,$0
FE00          LFE00:
FE01          LFE01 = * + 1
FE00 B5 A9      .WORD LA9B5
FE02 33 B9      .WORD LB933
FE04 03 BE      .WORD LBE03
FE06 EC AE      .WORD LAEEC
FE08 D0 BC      .WORD LBCD0
FE0A CD A6      .WORD LA6CD
FE0C EB D3      .WORD LD3EB
FE0E AE BD      .WORD LBDAE
FE10 88 AD      .WORD LAD88
FE12 52 B3      .WORD LB352
FE14 36 DD      .WORD LDD36
FE16 88 9C      .WORD L9C88
FE18 38 BB      .WORD LBB38
FE1A 29 DE      .WORD LDE29
FE1C D6 F4      .WORD LF4D6
FE1E EE DE      .WORD LDEEE
FE20 1B F8      .WORD LF81B
FE22 3B DF      .WORD LDF3B
FE24 13 DF      .WORD LDF13
FE26 6D F8      .WORD LF86D
FE28 4A 94      .WORD L944A
FE2A 21 A0      .WORD LA021
FE2C 54 9E      .WORD L9E54
FE2E          LFE2E:
FE2E 3D E4 1B   AND L1BE4,X
FE31 E4 1C      CPX L1C
FE33 E8         INX
FE34 25 E8      AND LE8
FE36 60         RTS
FE37 E8         .BYTE $E8
FE38 C7 E9      .WORD LE9C7
FE3A FB B1      .WORD LB1FB
FE3C 2A B2      .WORD LB22A
FE3E 00 00 00   .BYTE $0,$0,$0
FE41 00 00 00   .BYTE $0,$0,$0
FE44 00 00 00   .BYTE $0,$0,$0
FE47 00 00 00   .BYTE $0,$0,$0
FE4A 00 00 00   .BYTE $0,$0,$0
FE4D 00 00 00   .BYTE $0,$0,$0
FE50 00 00 00   .BYTE $0,$0,$0
FE53 00 00 00   .BYTE $0,$0,$0
FE56 00 00 00   .BYTE $0,$0,$0
FE59 00 00 00   .BYTE $0,$0,$0
FE5C 00 00 00   .BYTE $0,$0,$0
FE5F 00 00 00   .BYTE $0,$0,$0
FE62 00 00 00   .BYTE $0,$0,$0
FE65 00 00 00   .BYTE $0,$0,$0
FE68 00 00 00   .BYTE $0,$0,$0
FE6B 00 00 00   .BYTE $0,$0,$0
FE6E 00 00 00   .BYTE $0,$0,$0
FE71 00 00 00   .BYTE $0,$0,$0
FE74 00 00 00   .BYTE $0,$0,$0
FE77 00 00 00   .BYTE $0,$0,$0
FE7A 00 00 00   .BYTE $0,$0,$0
FE7D 00 00 00   .BYTE $0,$0,$0
FE80 00 00 00   .BYTE $0,$0,$0
FE83 00 00 00   .BYTE $0,$0,$0
FE86 00 00 00   .BYTE $0,$0,$0
FE89 00 00 00   .BYTE $0,$0,$0
FE8C 00 00 00   .BYTE $0,$0,$0
FE8F 00 00 00   .BYTE $0,$0,$0
FE92 00 00 00   .BYTE $0,$0,$0
FE95 00 00 00   .BYTE $0,$0,$0
FE98 00 00 00   .BYTE $0,$0,$0
FE9B 00 00 00   .BYTE $0,$0,$0
FE9E 00 00 43   .BYTE $0,$0,$43
FEA1 4D 44 20   .BYTE $4D,$44,$20
FEA4 48 44 20   .BYTE $48,$44,$20
FEA9          LFEA9 = * + 2
FEA7 44 4F 53   .BYTE $44,$4F,$53
FEAA 20 43 4F   .BYTE $20,$43,$4F
FEAD 50 59 52   .BYTE $50,$59,$52
FEB0 49 47 48   .BYTE $49,$47,$48
FEB3 54 20 31   .BYTE $54,$20,$31
FEB6 39 39 30   .BYTE $39,$39,$30
FEB9 20 43 52   .BYTE $20,$43,$52
FEBC 45 41 54   .BYTE $45,$41,$54
FEBF 49 56 45   .BYTE $49,$56,$45
FEC2 20 4D 49   .BYTE $20,$4D,$49
FEC5 43 52 4F   .BYTE $43,$52,$4F
FEC8 20 44 45   .BYTE $20,$44,$45
FECB 53 49 47   .BYTE $53,$49,$47
FECE 4E 53      .BYTE $4E,$53
FED0          LFED0:
FED0 2C 20 49   BIT L4920
FED3 4E 43 2E   LSR L2E43
FED6 20 41 4C   JSR L4C41
FED9 4C 20 52   JMP L5220
FEDC 49 47 48   .BYTE $49,$47,$48
FEDF 54 53 20   .BYTE $54,$53,$20
FEE2 52 45 53   .BYTE $52,$45,$53
FEE5 45 52 56   .BYTE $45,$52,$56
FEE8 45 44 00   .BYTE $45,$44,$0
FEEB 00 00 00   .BYTE $0,$0,$0
FEEE 00 00 00   .BYTE $0,$0,$0
FEF1 00 00 00   .BYTE $0,$0,$0
FEF4 00 00 00   .BYTE $0,$0,$0
FEF7 00 00 00   .BYTE $0,$0,$0
FEFA 00 00 00   .BYTE $0,$0,$0
FEFD 00 00 00   .BYTE $0,$0,$0
FF00          LFF00:
FF01          LFF01 = * + 1
FF02          LFF02 = * + 2
FF00 4C B5 A9   JMP LA9B5
FF03          LFF03:
FF03 4C 33 B9   JMP LB933
FF06          LFF06:
FF06 4C 03 BE   JMP LBE03
FF09          LFF09:
FF09 4C EC AE   JMP LAEEC
FF0C          LFF0C:
FF0C 4C D0 BC   JMP LBCD0
FF0F          LFF0F:
FF0F 4C CD A6   JMP LA6CD
FF12          LFF12:
FF12 4C EB D3   JMP LD3EB
FF15          LFF15:
FF15 4C AE BD   JMP LBDAE
FF18          LFF18:
FF18 4C 88 AD   JMP LAD88
FF1B          LFF1B:
FF1B 4C 52 B3   JMP LB352
FF1E          LFF1E:
FF1E 4C 36 DD   JMP LDD36
FF21          LFF21:
FF21 4C 88 9C   JMP L9C88
FF24          LFF24:
FF24 4C 38 BB   JMP LBB38
FF27          LFF27:
FF27 4C 29 DE   JMP LDE29
FF2A          LFF2A:
FF2A 4C D6 F4   JMP LF4D6
FF2D          LFF2D:
FF2D 4C EE DE   JMP LDEEE
FF30          LFF30:
FF30 4C 1B F8   JMP LF81B
FF33          LFF33:
FF34          LFF34 = * + 1
              ; Instruction parameter accessed.
FF35          LFF35 = * + 2
              ; Instruction parameter accessed.
FF33 4C 3B DF   JMP LDF3B
FF36          LFF36:
FF37          LFF37 = * + 1
              ; Instruction parameter accessed.
FF38          LFF38 = * + 2
              ; Instruction parameter accessed.
FF36 4C 13 DF   JMP LDF13
FF39          LFF39:
FF39 4C 6D F8   JMP LF86D
FF3C          LFF3C:
FF3C 4C 4A 94   JMP L944A
FF3F          LFF3F:
FF3F 4C 21 A0   JMP LA021
FF42          LFF42:
FF42 4C 54 9E   JMP L9E54
FF45          LFF45:
FF45 4C 3D E4   JMP LE43D
FF48          LFF48:
FF48 4C 1B E4   JMP LE41B
FF4B          LFF4B:
FF4B 4C 1C E8   JMP LE81C
FF4E          LFF4E:
FF4E 4C 25 E8   JMP LE825
FF51          LFF51:
FF51 4C 60 E8   JMP LE860
FF54          LFF54:
FF54 4C C7 E9   JMP LE9C7
FF57          LFF57:
FF57 4C FB B1   JMP LB1FB
FF5A          LFF5A:
FF5A 4C 2A B2   JMP LB22A
FF5D 00 00 00   .BYTE $0,$0,$0
FF60 00 00 00   .BYTE $0,$0,$0
FF63 00 00 00   .BYTE $0,$0,$0
FF66 00 00 00   .BYTE $0,$0,$0
FF69 00 00 00   .BYTE $0,$0,$0
FF6C 00 00 00   .BYTE $0,$0,$0
FF6F 00 00 00   .BYTE $0,$0,$0
FF72 00 00 00   .BYTE $0,$0,$0
FF75 00 00 00   .BYTE $0,$0,$0
FF78 00 00 00   .BYTE $0,$0,$0
FF7B 00 00 00   .BYTE $0,$0,$0
FF7E 00 00 00   .BYTE $0,$0,$0
FF81 00 00 00   .BYTE $0,$0,$0
FF84 00 00 00   .BYTE $0,$0,$0
FF87 00 00 00   .BYTE $0,$0,$0
FF8A 00 00 00   .BYTE $0,$0,$0
FF8D 00 00 00   .BYTE $0,$0,$0
FF90 00 00 00   .BYTE $0,$0,$0
FF93 00 00 00   .BYTE $0,$0,$0
FF96 00 00 00   .BYTE $0,$0,$0
FF99 00 00 00   .BYTE $0,$0,$0
FF9C 00 00 00   .BYTE $0,$0,$0
FF9F 00 00 00   .BYTE $0,$0,$0
FFA2 00 00 00   .BYTE $0,$0,$0
FFA5 00 00 00   .BYTE $0,$0,$0
FFA8 00 00 00   .BYTE $0,$0,$0
FFAB 00 00 00   .BYTE $0,$0,$0
FFAE 00 00 00   .BYTE $0,$0,$0
FFB1 00 00 00   .BYTE $0,$0,$0
FFB4 00 00 00   .BYTE $0,$0,$0
FFB7 00 00 00   .BYTE $0,$0,$0
FFBA 00 00 00   .BYTE $0,$0,$0
FFBD 00 00 00   .BYTE $0,$0,$0
FFC0 00 00 00   .BYTE $0,$0,$0
FFC3 00 00 00   .BYTE $0,$0,$0
FFC6 00 00 00   .BYTE $0,$0,$0
FFC9 00 00 00   .BYTE $0,$0,$0
FFCC 00 00 00   .BYTE $0,$0,$0
FFCF 00 00 00   .BYTE $0,$0,$0
FFD2 00 00 00   .BYTE $0,$0,$0
FFD5 00 00 00   .BYTE $0,$0,$0
FFD8 00 00 00   .BYTE $0,$0,$0
FFDB 00 00 00   .BYTE $0,$0,$0
FFDE 00 00 00   .BYTE $0,$0,$0
FFE1 00 00 00   .BYTE $0,$0,$0
FFE4 00 00 00   .BYTE $0,$0,$0
FFE7 00 00 00   .BYTE $0,$0,$0
FFEA 00 00 00   .BYTE $0,$0,$0
FFED 00 00 00   .BYTE $0,$0,$0
FFF0 00 00 00   .BYTE $0,$0,$0
FFF3 00 00 00   .BYTE $0,$0,$0
FFF6 00 00 00   .BYTE $0,$0,$0
FFF9 00         .BYTE $0
FFFA 7C 9A      .WORD L9A7C
FFFC 37 F4      .WORD LF437
FFFE 39 FF      .WORD LFF39
